; Listing generated by Microsoft (R) Optimizing Compiler Version 15.00.21022.08 

	TITLE	c:\Develop\DScaler423a\DScaler\ParsingCommon.cpp
	.686P
	.XMM
	include listing.inc
	.model	flat

INCLUDELIB OLDNAMES

PUBLIC	??_C@_1CM@NKAGKMMA@?$AAP?$AAH?$AAI?$AAL?$AAI?$AAP?$AAS?$AA_?$AAF?$AAM?$AAD?$AA1?$AA2?$AA1?$AA6?$AAM?$AAE?$AA_?$AAM?$AAK?$AA3?$AA?$AA@ ; `string'
PUBLIC	??_C@_1BK@PEHEKEAO@?$AAT?$AAE?$AAN?$AAA?$AA_?$AA9?$AA5?$AA3?$AA3?$AA_?$AAD?$AAI?$AA?$AA@ ; `string'
PUBLIC	??_C@_1CA@CNOGJENC@?$AAY?$AAM?$AAE?$AAC?$AA_?$AAT?$AAV?$AAF?$AA_?$AA5?$AA5?$AA3?$AA3?$AAM?$AAF?$AA?$AA@ ; `string'
PUBLIC	??_C@_1CA@NIDJODPE@?$AAY?$AAM?$AAE?$AAC?$AA_?$AAT?$AAV?$AAF?$AA_?$AA8?$AA5?$AA3?$AA1?$AAM?$AAF?$AA?$AA@ ; `string'
PUBLIC	??_C@_1CA@PHAKLDDM@?$AAP?$AAH?$AAI?$AAL?$AAI?$AAP?$AAS?$AA_?$AAT?$AAD?$AAA?$AA8?$AA2?$AA7?$AA5?$AA?$AA@ ; `string'
PUBLIC	??_C@_1CI@PFGDHJOM@?$AAP?$AAH?$AAI?$AAL?$AAI?$AAP?$AAS?$AA_?$AAF?$AAQ?$AA1?$AA2?$AA3?$AA6?$AAA?$AA_?$AAM?$AAK?$AA4?$AA?$AA@ ; `string'
PUBLIC	??_C@_1DI@EAGAPDHM@?$AAT?$AAU?$AAN?$AAE?$AAR?$AA_?$AAP?$AAH?$AAI?$AAL?$AAI?$AAP?$AAS?$AA_?$AAF?$AAQ?$AA1?$AA2?$AA1?$AA6?$AAA?$AAM?$AAE?$AA_?$AAM?$AAK?$AA4?$AA?$AA@ ; `string'
PUBLIC	??_C@_1BI@DMIKHBF@?$AAL?$AAG?$AA_?$AAP?$AAA?$AAL?$AA_?$AAT?$AAA?$AAP?$AAE?$AA?$AA@ ; `string'
PUBLIC	??_C@_1BO@PGCKBBBK@?$AAP?$AAH?$AAI?$AAL?$AAI?$AAP?$AAS?$AA_?$AAF?$AAQ?$AA1?$AA2?$AA8?$AA6?$AA?$AA@ ; `string'
PUBLIC	??_C@_1CG@LGMDAEOM@?$AAP?$AAH?$AAI?$AAL?$AAI?$AAP?$AAS?$AA_?$AAF?$AAM?$AA1?$AA2?$AA5?$AA6?$AA_?$AAI?$AAH?$AA3?$AA?$AA@ ; `string'
PUBLIC	??_C@_1BK@CBBAAEDD@?$AAT?$AAN?$AAF?$AA_?$AA8?$AA8?$AA3?$AA1?$AAB?$AAG?$AAF?$AAF?$AA?$AA@ ; `string'
PUBLIC	??_C@_1BK@JHDPBOPP@?$AAL?$AAG?$AA_?$AAN?$AAT?$AAS?$AAC?$AA_?$AAT?$AAA?$AAP?$AAE?$AA?$AA@ ; `string'
PUBLIC	??_C@_1CG@EMNPDDAO@?$AAP?$AAH?$AAI?$AAL?$AAI?$AAP?$AAS?$AA_?$AAF?$AAM?$AA1?$AA2?$AA3?$AA6?$AA_?$AAM?$AAK?$AA3?$AA?$AA@ ; `string'
PUBLIC	??_C@_1BO@OOKBNEEN@?$AAP?$AAH?$AAI?$AAL?$AAI?$AAP?$AAS?$AA_?$AAP?$AAA?$AAL?$AA_?$AAM?$AAK?$AA?$AA@ ; `string'
PUBLIC	??_C@_1BK@CFFBIHHG@?$AAH?$AAI?$AAT?$AAA?$AAC?$AAH?$AAI?$AA_?$AAN?$AAT?$AAS?$AAC?$AA?$AA@ ; `string'
PUBLIC	??_C@_1BE@OEGEIDDF@?$AAT?$AAC?$AAL?$AA_?$AA2?$AA0?$AA0?$AA2?$AAN?$AA?$AA@ ; `string'
PUBLIC	??_C@_1BK@PNPMMDOJ@?$AAP?$AAH?$AAI?$AAL?$AAI?$AAP?$AAS?$AA_?$AA4?$AAI?$AAN?$AA1?$AA?$AA@ ; `string'
PUBLIC	??_C@_1BG@EAALJKKI@?$AAM?$AAT?$AA2?$AA0?$AA5?$AA0?$AA_?$AAP?$AAA?$AAL?$AA?$AA@ ; `string'
PUBLIC	??_C@_1O@KKCNAPCG@?$AAM?$AAT?$AA2?$AA0?$AA5?$AA0?$AA?$AA@ ; `string'
PUBLIC	??_C@_1DA@JEOOMIMC@?$AAP?$AAH?$AAI?$AAL?$AAI?$AAP?$AAS?$AA_?$AAF?$AAI?$AA1?$AA2?$AA8?$AA6?$AA_?$AAN?$AAT?$AAS?$AAC?$AA_?$AAM?$AA_?$AAJ?$AA?$AA@ ; `string'
PUBLIC	??_C@_1BG@FEPCEPIB@?$AAM?$AAT?$AA2?$AA0?$AA3?$AA2?$AA_?$AAP?$AAA?$AAL?$AA?$AA@ ; `string'
PUBLIC	??_C@_1CA@GAGMPGBP@?$AAL?$AAG?$AA_?$AAT?$AAA?$AAP?$AAC?$AAN?$AAE?$AAW?$AA_?$AAN?$AAT?$AAS?$AAC?$AA?$AA@ ; `string'
PUBLIC	??_C@_1CK@CLKCBCPN@?$AAP?$AAH?$AAI?$AAL?$AAI?$AAP?$AAS?$AA_?$AAF?$AAM?$AA1?$AA2?$AA1?$AA6?$AAM?$AAE?$AA_?$AAM?$AAK?$AA3?$AA?$AA@ ; `string'
PUBLIC	??_C@_1BO@EHMDLLBA@?$AAL?$AAG?$AA_?$AAT?$AAA?$AAP?$AAC?$AAN?$AAE?$AAW?$AA_?$AAP?$AAA?$AAL?$AA?$AA@ ; `string'
PUBLIC	??_C@_1BM@JANAKEML@?$AAT?$AAE?$AAM?$AAI?$AAC?$AA_?$AA4?$AA1?$AA3?$AA6?$AAF?$AAY?$AA5?$AA?$AA@ ; `string'
PUBLIC	??_C@_1BM@OIAPHLFI@?$AAT?$AAE?$AAM?$AAI?$AAC?$AA_?$AA4?$AA0?$AA1?$AA2?$AAF?$AAY?$AA5?$AA?$AA@ ; `string'
PUBLIC	??_C@_1BM@CPMEKHAF@?$AAT?$AAE?$AAM?$AAI?$AAC?$AA_?$AA4?$AA1?$AA0?$AA6?$AAF?$AAH?$AA5?$AA?$AA@ ; `string'
PUBLIC	??_C@_1DC@PNFJNOKI@?$AAS?$AAA?$AAM?$AAS?$AAU?$AAN?$AAG?$AA_?$AAP?$AAA?$AAL?$AA_?$AAT?$AAC?$AAP?$AAM?$AA9?$AA0?$AA9?$AA1?$AAP?$AAD?$AA2?$AA7?$AA?$AA@ ; `string'
PUBLIC	??_C@_1CE@CODMLBHG@?$AAL?$AAG?$AA_?$AAT?$AAA?$AAP?$AAC?$AAH?$AA7?$AA0?$AA1?$AAP?$AA_?$AAN?$AAT?$AAS?$AAC?$AA?$AA@ ; `string'
PUBLIC	??_C@_1CK@MHILDIAN@?$AAS?$AAH?$AAA?$AAR?$AAP?$AA_?$AA2?$AAU?$AA5?$AAJ?$AAF?$AA5?$AA5?$AA4?$AA0?$AA_?$AAN?$AAT?$AAS?$AAC?$AA?$AA@ ; `string'
PUBLIC	??_C@_1O@NGHNCELA@?$AAM?$AAT?$AA2?$AA0?$AA3?$AA2?$AA?$AA@ ; `string'
PUBLIC	??_C@_1CE@BCGOJMKC@?$AAT?$AAE?$AAM?$AAI?$AAC?$AA_?$AA4?$AA0?$AA0?$AA9?$AAF?$AAN?$AA5?$AA_?$AAP?$AAA?$AAL?$AA?$AA@ ; `string'
PUBLIC	??_C@_1BI@CKLFPNIN@?$AAL?$AAG?$AA_?$AAB?$AA1?$AA1?$AAD?$AA_?$AAP?$AAA?$AAL?$AA?$AA@ ; `string'
PUBLIC	??_C@_1BI@IENNGMBM@?$AAL?$AAG?$AA_?$AAB?$AA0?$AA1?$AAD?$AA_?$AAP?$AAA?$AAL?$AA?$AA@ ; `string'
PUBLIC	??_C@_1BK@NFMGFCPC@?$AAL?$AAG?$AA_?$AAR?$AA0?$AA1?$AAF?$AA_?$AAN?$AAT?$AAS?$AAC?$AA?$AA@ ; `string'
PUBLIC	??_C@_1BO@FADGBOEK@?$AAL?$AAG?$AA_?$AAI?$AA7?$AA0?$AA1?$AAD?$AA_?$AAP?$AAA?$AAL?$AA_?$AAI?$AA?$AA@ ; `string'
PUBLIC	??_C@_1BO@DFOPCAAK@?$AAL?$AAG?$AA_?$AAI?$AA0?$AA0?$AA1?$AAD?$AA_?$AAP?$AAA?$AAL?$AA_?$AAI?$AA?$AA@ ; `string'
PUBLIC	??_C@_1BM@PFKAHCHD@?$AAP?$AAH?$AAI?$AAL?$AAI?$AAP?$AAS?$AA_?$AAM?$AAU?$AAL?$AAT?$AAI?$AA?$AA@ ; `string'
PUBLIC	??_C@_1BO@MJKOIFIF@?$AAP?$AAH?$AAI?$AAL?$AAI?$AAP?$AAS?$AA_?$AAP?$AAA?$AAL?$AA_?$AAD?$AAK?$AA?$AA@ ; `string'
PUBLIC	??_C@_1CI@IJEHGMNA@?$AAT?$AAE?$AAM?$AAI?$AAC?$AA_?$AA4?$AA0?$AA4?$AA6?$AAF?$AAM?$AA5?$AA_?$AAM?$AAU?$AAL?$AAT?$AAI?$AA?$AA@ ; `string'
PUBLIC	??_C@_1CG@GLOIJKPF@?$AAT?$AAE?$AAM?$AAI?$AAC?$AA_?$AA4?$AA0?$AA3?$AA9?$AAF?$AAR?$AA5?$AA_?$AAN?$AAT?$AAS?$AAC?$AA?$AA@ ; `string'
PUBLIC	??_C@_1CE@FOCJDBOD@?$AAT?$AAE?$AAM?$AAI?$AAC?$AA_?$AA4?$AA0?$AA0?$AA9?$AAF?$AAR?$AA5?$AA_?$AAP?$AAA?$AAL?$AA?$AA@ ; `string'
PUBLIC	??_C@_1CE@OEBBDIMK@?$AAT?$AAE?$AAM?$AAI?$AAC?$AA_?$AA4?$AA0?$AA0?$AA6?$AAF?$AAN?$AA5?$AA_?$AAP?$AAA?$AAL?$AA?$AA@ ; `string'
PUBLIC	??_C@_1CI@KDECBGIC@?$AAT?$AAE?$AAM?$AAI?$AAC?$AA_?$AA4?$AA0?$AA6?$AA6?$AAF?$AAY?$AA5?$AA_?$AAP?$AAA?$AAL?$AA_?$AAI?$AA?$AA@ ; `string'
PUBLIC	??_C@_1CC@FGAIIFMP@?$AAP?$AAH?$AAI?$AAL?$AAI?$AAP?$AAS?$AA_?$AAM?$AAK?$AA2?$AA_?$AAN?$AAT?$AAS?$AAC?$AA?$AA@ ; `string'
PUBLIC	??_C@_1CE@ICAJJFCA@?$AAT?$AAE?$AAM?$AAI?$AAC?$AA_?$AA4?$AA0?$AA1?$AA6?$AAF?$AAY?$AA5?$AA_?$AAP?$AAA?$AAL?$AA?$AA@ ; `string'
PUBLIC	??_C@_1CA@OEJFEMFE@?$AAA?$AAL?$AAP?$AAS?$AA_?$AAT?$AAS?$AAC?$AAH?$AA6?$AA_?$AAN?$AAT?$AAS?$AAC?$AA?$AA@ ; `string'
PUBLIC	??_C@_1DE@MMPEKFHL@?$AAP?$AAH?$AAI?$AAL?$AAI?$AAP?$AAS?$AA_?$AA1?$AA2?$AA3?$AA6?$AAD?$AA_?$AAN?$AAT?$AAS?$AAC?$AA_?$AAI?$AAN?$AAP?$AAU?$AAT?$AA2?$AA?$AA@ ; `string'
PUBLIC	??_C@_1DE@NOEBAKJF@?$AAP?$AAH?$AAI?$AAL?$AAI?$AAP?$AAS?$AA_?$AA1?$AA2?$AA3?$AA6?$AAD?$AA_?$AAN?$AAT?$AAS?$AAC?$AA_?$AAI?$AAN?$AAP?$AAU?$AAT?$AA1?$AA?$AA@ ; `string'
PUBLIC	??_C@_1CE@BMNDHDHM@?$AAT?$AAE?$AAM?$AAI?$AAC?$AA_?$AA4?$AA0?$AA0?$AA6?$AAF?$AAH?$AA5?$AA_?$AAP?$AAA?$AAL?$AA?$AA@ ; `string'
PUBLIC	??_C@_1BO@JIFHKPHC@?$AAA?$AAL?$AAP?$AAS?$AA_?$AAT?$AAS?$AAB?$AAC?$AA5?$AA_?$AAP?$AAA?$AAL?$AA?$AA@ ; `string'
PUBLIC	??_C@_1BO@GAJFOEME@?$AAA?$AAL?$AAP?$AAS?$AA_?$AAT?$AAS?$AAB?$AAE?$AA5?$AA_?$AAP?$AAA?$AAL?$AA?$AA@ ; `string'
PUBLIC	??_C@_1CC@OMKKLJNL@?$AAA?$AAL?$AAP?$AAS?$AA_?$AAT?$AAS?$AAB?$AAB?$AA5?$AA_?$AAP?$AAA?$AAL?$AA_?$AAI?$AA?$AA@ ; `string'
PUBLIC	??_C@_1BO@GDJDNPLL@?$AAA?$AAL?$AAP?$AAS?$AA_?$AAT?$AAS?$AAB?$AAE?$AA1?$AA_?$AAP?$AAA?$AAL?$AA?$AA@ ; `string'
PUBLIC	??_C@_1CA@GOAKFAHF@?$AAA?$AAL?$AAP?$AAS?$AA_?$AAT?$AAS?$AAB?$AAH?$AA1?$AA_?$AAN?$AAT?$AAS?$AAC?$AA?$AA@ ; `string'
PUBLIC	??_C@_1CG@ENKMMBGJ@?$AAT?$AAE?$AAM?$AAI?$AAC?$AA_?$AA4?$AA0?$AA3?$AA6?$AAF?$AAY?$AA5?$AA_?$AAN?$AAT?$AAS?$AAC?$AA?$AA@ ; `string'
PUBLIC	??_C@_1CI@PPODIFIC@?$AAT?$AAE?$AAM?$AAI?$AAC?$AA_?$AA4?$AA0?$AA6?$AA2?$AAF?$AAY?$AA5?$AA_?$AAP?$AAA?$AAL?$AA_?$AAI?$AA?$AA@ ; `string'
PUBLIC	??_C@_1CG@DEBCKDA@?$AAT?$AAE?$AAM?$AAI?$AAC?$AA_?$AA4?$AA0?$AA3?$AA2?$AAF?$AAY?$AA5?$AA_?$AAN?$AAT?$AAS?$AAC?$AA?$AA@ ; `string'
PUBLIC	??_C@_1CE@BHHLKEHK@?$AAT?$AAE?$AAM?$AAI?$AAC?$AA_?$AA4?$AA0?$AA0?$AA2?$AAF?$AAH?$AA5?$AA_?$AAP?$AAA?$AAL?$AA?$AA@ ; `string'
PUBLIC	??_C@_1BI@IKKAFKBC@?$AAP?$AAH?$AAI?$AAL?$AAI?$AAP?$AAS?$AA_?$AAP?$AAA?$AAL?$AA?$AA@ ; `string'
PUBLIC	??_C@_1BM@DCHONLKK@?$AAP?$AAH?$AAI?$AAL?$AAI?$AAP?$AAS?$AA_?$AAS?$AAE?$AAC?$AAA?$AAM?$AA?$AA@ ; `string'
PUBLIC	??_C@_1BK@IFFHILBA@?$AAP?$AAH?$AAI?$AAL?$AAI?$AAP?$AAS?$AA_?$AAN?$AAT?$AAS?$AAC?$AA?$AA@ ; `string'
PUBLIC	??_C@_1BM@CDJFEPDA@?$AAP?$AAH?$AAI?$AAL?$AAI?$AAP?$AAS?$AA_?$AAP?$AAA?$AAL?$AA_?$AAI?$AA?$AA@ ; `string'
PUBLIC	??_C@_1O@GMMJLLPL@?$AAA?$AAB?$AAS?$AAE?$AAN?$AAT?$AA?$AA@ ; `string'
PUBLIC	??_C@_1M@PBHOBGFC@?$AAS?$AAE?$AAT?$AAU?$AAP?$AA?$AA@ ; `string'
PUBLIC	??_C@_19CEKDAEDP@?$AAA?$AAU?$AAT?$AAO?$AA?$AA@	; `string'
PUBLIC	??_C@_1BA@BKMKJFAN@?$AAN?$AAT?$AAS?$AAC?$AA?9?$AAJ?$AAP?$AA?$AA@ ; `string'
PUBLIC	??_C@_1O@LMGGCLHH@?$AAN?$AAT?$AAS?$AAC?$AA?9?$AAM?$AA?$AA@ ; `string'
PUBLIC	??_C@_1BC@PFJOKPCA@?$AAS?$AAE?$AAC?$AAA?$AAM?$AA?9?$AAD?$AAK?$AA?$AA@ ; `string'
PUBLIC	??_C@_1BA@NJCCHOGP@?$AAS?$AAE?$AAC?$AAA?$AAM?$AA?9?$AAL?$AA?$AA@ ; `string'
PUBLIC	??_C@_1O@IMHBBACP@?$AAP?$AAA?$AAL?$AA?9?$AAM?$AAN?$AA?$AA@ ; `string'
PUBLIC	??_C@_1O@JMKALBNF@?$AAP?$AAA?$AAL?$AA?9?$AAD?$AAK?$AA?$AA@ ; `string'
PUBLIC	??_C@_1M@OKDFNJPP@?$AAP?$AAA?$AAL?$AA?9?$AAI?$AA?$AA@ ; `string'
PUBLIC	??_C@_1O@CPONHA@?$AAP?$AAA?$AAL?$AA?9?$AAB?$AAG?$AA?$AA@ ; `string'
PUBLIC	??_C@_1O@COJGIGIJ@?$AAG?$AAL?$AAO?$AAB?$AAA?$AAL?$AA?$AA@ ; `string'
PUBLIC	??_C@_17OBLMBIF@?$AAq?$AAs?$AAs?$AA?$AA@	; `string'
PUBLIC	??_C@_1BK@BJKJAFD@?$AAi?$AAn?$AAt?$AAe?$AAr?$AAc?$AAa?$AAr?$AAr?$AAi?$AAe?$AAr?$AA?$AA@ ; `string'
PUBLIC	??_C@_1BC@DBHEDMBL@?$AAi?$AAn?$AAa?$AAc?$AAt?$AAi?$AAv?$AAe?$AA?$AA@ ; `string'
PUBLIC	??_C@_1O@IBNPCBAA@?$AAa?$AAc?$AAt?$AAi?$AAv?$AAe?$AA?$AA@ ; `string'
PUBLIC	??_C@_1M@HCOOECOK@?$AAF?$AAA?$AAL?$AAS?$AAE?$AA?$AA@ ; `string'
PUBLIC	??_C@_19ELAAHEEL@?$AAT?$AAR?$AAU?$AAE?$AA?$AA@	; `string'
PUBLIC	??_C@_17LMBAMBHA@?$AAm?$AAa?$AAx?$AA?$AA@	; `string'
PUBLIC	??_C@_17CFDBELFO@?$AAm?$AAi?$AAn?$AA?$AA@	; `string'
PUBLIC	??_C@_1BM@DLNBHEGJ@?$AAT?$AAa?$AAk?$AAe?$AAO?$AAv?$AAe?$AAr?$AAP?$AAo?$AAi?$AAn?$AAt?$AA?$AA@ ; `string'
PUBLIC	??_C@_1BI@BPJAFCLP@?$AAO?$AAu?$AAt?$AAp?$AAu?$AAt?$AAP?$AAo?$AAr?$AAt?$AA2?$AA?$AA@ ; `string'
PUBLIC	??_C@_1BI@NCFPNFB@?$AAO?$AAu?$AAt?$AAp?$AAu?$AAt?$AAP?$AAo?$AAr?$AAt?$AA1?$AA?$AA@ ; `string'
PUBLIC	??_C@_1BA@GJEGJPFN@?$AAC?$AAa?$AAr?$AAr?$AAi?$AAe?$AAr?$AA?$AA@ ; `string'
PUBLIC	??_C@_17FAPDAJNL@?$AAQ?$AAS?$AAS?$AA?$AA@	; `string'
PUBLIC	??_C@_1BK@IOEPCAOC@?$AAI?$AAn?$AAt?$AAe?$AAr?$AAc?$AAa?$AAr?$AAr?$AAi?$AAe?$AAr?$AA?$AA@ ; `string'
PUBLIC	??_C@_1O@FDFOMCPN@?$AAF?$AAo?$AAr?$AAm?$AAa?$AAt?$AA?$AA@ ; `string'
PUBLIC	??_C@_1BC@KNKFHLFO@?$AAS?$AAe?$AAt?$AAM?$AAo?$AAd?$AAe?$AAs?$AA?$AA@ ; `string'
PUBLIC	??_C@_17GFFKFGK@?$AAU?$AAs?$AAe?$AA?$AA@	; `string'
PUBLIC	??_C@_0BB@DPAAIHBB@Invalid?5tuner?5Id?$AA@	; `string'
PUBLIC	??_C@_0BP@JMNHPJIF@Invalid?5value?5of?5TakeOverPoint?$AA@ ; `string'
PUBLIC	??_C@_1BA@HANLFFFG@?$AAd?$AAe?$AAf?$AAa?$AAu?$AAl?$AAt?$AA?$AA@ ; `string'
;	COMDAT ??_C@_1BA@HANLFFFG@?$AAd?$AAe?$AAf?$AAa?$AAu?$AAl?$AAt?$AA?$AA@
CONST	SEGMENT
??_C@_1BA@HANLFFFG@?$AAd?$AAe?$AAf?$AAa?$AAu?$AAl?$AAt?$AA?$AA@ DB 'd', 00H
	DB	'e', 00H, 'f', 00H, 'a', 00H, 'u', 00H, 'l', 00H, 't', 00H, 00H
	DB	00H						; `string'
CONST	ENDS
;	COMDAT ??_C@_0BP@JMNHPJIF@Invalid?5value?5of?5TakeOverPoint?$AA@
CONST	SEGMENT
??_C@_0BP@JMNHPJIF@Invalid?5value?5of?5TakeOverPoint?$AA@ DB 'Invalid val'
	DB	'ue of TakeOverPoint', 00H			; `string'
CONST	ENDS
;	COMDAT ??_C@_0BB@DPAAIHBB@Invalid?5tuner?5Id?$AA@
CONST	SEGMENT
??_C@_0BB@DPAAIHBB@Invalid?5tuner?5Id?$AA@ DB 'Invalid tuner Id', 00H ; `string'
CONST	ENDS
;	COMDAT ??_C@_17GFFKFGK@?$AAU?$AAs?$AAe?$AA?$AA@
CONST	SEGMENT
??_C@_17GFFKFGK@?$AAU?$AAs?$AAe?$AA?$AA@ DB 'U', 00H, 's', 00H, 'e', 00H, 00H
	DB	00H						; `string'
CONST	ENDS
;	COMDAT ??_C@_1BC@KNKFHLFO@?$AAS?$AAe?$AAt?$AAM?$AAo?$AAd?$AAe?$AAs?$AA?$AA@
CONST	SEGMENT
??_C@_1BC@KNKFHLFO@?$AAS?$AAe?$AAt?$AAM?$AAo?$AAd?$AAe?$AAs?$AA?$AA@ DB 'S'
	DB	00H, 'e', 00H, 't', 00H, 'M', 00H, 'o', 00H, 'd', 00H, 'e', 00H
	DB	's', 00H, 00H, 00H				; `string'
CONST	ENDS
;	COMDAT ??_C@_1O@FDFOMCPN@?$AAF?$AAo?$AAr?$AAm?$AAa?$AAt?$AA?$AA@
CONST	SEGMENT
??_C@_1O@FDFOMCPN@?$AAF?$AAo?$AAr?$AAm?$AAa?$AAt?$AA?$AA@ DB 'F', 00H, 'o'
	DB	00H, 'r', 00H, 'm', 00H, 'a', 00H, 't', 00H, 00H, 00H ; `string'
CONST	ENDS
;	COMDAT ??_C@_1BK@IOEPCAOC@?$AAI?$AAn?$AAt?$AAe?$AAr?$AAc?$AAa?$AAr?$AAr?$AAi?$AAe?$AAr?$AA?$AA@
CONST	SEGMENT
??_C@_1BK@IOEPCAOC@?$AAI?$AAn?$AAt?$AAe?$AAr?$AAc?$AAa?$AAr?$AAr?$AAi?$AAe?$AAr?$AA?$AA@ DB 'I'
	DB	00H, 'n', 00H, 't', 00H, 'e', 00H, 'r', 00H, 'c', 00H, 'a', 00H
	DB	'r', 00H, 'r', 00H, 'i', 00H, 'e', 00H, 'r', 00H, 00H, 00H ; `string'
CONST	ENDS
;	COMDAT ??_C@_17FAPDAJNL@?$AAQ?$AAS?$AAS?$AA?$AA@
CONST	SEGMENT
??_C@_17FAPDAJNL@?$AAQ?$AAS?$AAS?$AA?$AA@ DB 'Q', 00H, 'S', 00H, 'S', 00H
	DB	00H, 00H					; `string'
CONST	ENDS
;	COMDAT ??_C@_1BA@GJEGJPFN@?$AAC?$AAa?$AAr?$AAr?$AAi?$AAe?$AAr?$AA?$AA@
CONST	SEGMENT
??_C@_1BA@GJEGJPFN@?$AAC?$AAa?$AAr?$AAr?$AAi?$AAe?$AAr?$AA?$AA@ DB 'C', 00H
	DB	'a', 00H, 'r', 00H, 'r', 00H, 'i', 00H, 'e', 00H, 'r', 00H, 00H
	DB	00H						; `string'
CONST	ENDS
;	COMDAT ??_C@_1BI@NCFPNFB@?$AAO?$AAu?$AAt?$AAp?$AAu?$AAt?$AAP?$AAo?$AAr?$AAt?$AA1?$AA?$AA@
CONST	SEGMENT
??_C@_1BI@NCFPNFB@?$AAO?$AAu?$AAt?$AAp?$AAu?$AAt?$AAP?$AAo?$AAr?$AAt?$AA1?$AA?$AA@ DB 'O'
	DB	00H, 'u', 00H, 't', 00H, 'p', 00H, 'u', 00H, 't', 00H, 'P', 00H
	DB	'o', 00H, 'r', 00H, 't', 00H, '1', 00H, 00H, 00H ; `string'
CONST	ENDS
;	COMDAT ??_C@_1BI@BPJAFCLP@?$AAO?$AAu?$AAt?$AAp?$AAu?$AAt?$AAP?$AAo?$AAr?$AAt?$AA2?$AA?$AA@
CONST	SEGMENT
??_C@_1BI@BPJAFCLP@?$AAO?$AAu?$AAt?$AAp?$AAu?$AAt?$AAP?$AAo?$AAr?$AAt?$AA2?$AA?$AA@ DB 'O'
	DB	00H, 'u', 00H, 't', 00H, 'p', 00H, 'u', 00H, 't', 00H, 'P', 00H
	DB	'o', 00H, 'r', 00H, 't', 00H, '2', 00H, 00H, 00H ; `string'
CONST	ENDS
;	COMDAT ??_C@_1BM@DLNBHEGJ@?$AAT?$AAa?$AAk?$AAe?$AAO?$AAv?$AAe?$AAr?$AAP?$AAo?$AAi?$AAn?$AAt?$AA?$AA@
CONST	SEGMENT
??_C@_1BM@DLNBHEGJ@?$AAT?$AAa?$AAk?$AAe?$AAO?$AAv?$AAe?$AAr?$AAP?$AAo?$AAi?$AAn?$AAt?$AA?$AA@ DB 'T'
	DB	00H, 'a', 00H, 'k', 00H, 'e', 00H, 'O', 00H, 'v', 00H, 'e', 00H
	DB	'r', 00H, 'P', 00H, 'o', 00H, 'i', 00H, 'n', 00H, 't', 00H, 00H
	DB	00H						; `string'
CONST	ENDS
;	COMDAT ??_C@_17CFDBELFO@?$AAm?$AAi?$AAn?$AA?$AA@
CONST	SEGMENT
??_C@_17CFDBELFO@?$AAm?$AAi?$AAn?$AA?$AA@ DB 'm', 00H, 'i', 00H, 'n', 00H
	DB	00H, 00H					; `string'
CONST	ENDS
;	COMDAT ??_C@_17LMBAMBHA@?$AAm?$AAa?$AAx?$AA?$AA@
CONST	SEGMENT
??_C@_17LMBAMBHA@?$AAm?$AAa?$AAx?$AA?$AA@ DB 'm', 00H, 'a', 00H, 'x', 00H
	DB	00H, 00H					; `string'
CONST	ENDS
;	COMDAT ??_C@_19ELAAHEEL@?$AAT?$AAR?$AAU?$AAE?$AA?$AA@
CONST	SEGMENT
??_C@_19ELAAHEEL@?$AAT?$AAR?$AAU?$AAE?$AA?$AA@ DB 'T', 00H, 'R', 00H, 'U', 00H
	DB	'E', 00H, 00H, 00H				; `string'
CONST	ENDS
;	COMDAT ??_C@_1M@HCOOECOK@?$AAF?$AAA?$AAL?$AAS?$AAE?$AA?$AA@
CONST	SEGMENT
??_C@_1M@HCOOECOK@?$AAF?$AAA?$AAL?$AAS?$AAE?$AA?$AA@ DB 'F', 00H, 'A', 00H
	DB	'L', 00H, 'S', 00H, 'E', 00H, 00H, 00H	; `string'
CONST	ENDS
;	COMDAT ??_C@_1O@IBNPCBAA@?$AAa?$AAc?$AAt?$AAi?$AAv?$AAe?$AA?$AA@
CONST	SEGMENT
??_C@_1O@IBNPCBAA@?$AAa?$AAc?$AAt?$AAi?$AAv?$AAe?$AA?$AA@ DB 'a', 00H, 'c'
	DB	00H, 't', 00H, 'i', 00H, 'v', 00H, 'e', 00H, 00H, 00H ; `string'
CONST	ENDS
;	COMDAT ??_C@_1BC@DBHEDMBL@?$AAi?$AAn?$AAa?$AAc?$AAt?$AAi?$AAv?$AAe?$AA?$AA@
CONST	SEGMENT
??_C@_1BC@DBHEDMBL@?$AAi?$AAn?$AAa?$AAc?$AAt?$AAi?$AAv?$AAe?$AA?$AA@ DB 'i'
	DB	00H, 'n', 00H, 'a', 00H, 'c', 00H, 't', 00H, 'i', 00H, 'v', 00H
	DB	'e', 00H, 00H, 00H				; `string'
CONST	ENDS
;	COMDAT ??_C@_1BK@BJKJAFD@?$AAi?$AAn?$AAt?$AAe?$AAr?$AAc?$AAa?$AAr?$AAr?$AAi?$AAe?$AAr?$AA?$AA@
CONST	SEGMENT
??_C@_1BK@BJKJAFD@?$AAi?$AAn?$AAt?$AAe?$AAr?$AAc?$AAa?$AAr?$AAr?$AAi?$AAe?$AAr?$AA?$AA@ DB 'i'
	DB	00H, 'n', 00H, 't', 00H, 'e', 00H, 'r', 00H, 'c', 00H, 'a', 00H
	DB	'r', 00H, 'r', 00H, 'i', 00H, 'e', 00H, 'r', 00H, 00H, 00H ; `string'
CONST	ENDS
;	COMDAT ??_C@_17OBLMBIF@?$AAq?$AAs?$AAs?$AA?$AA@
CONST	SEGMENT
??_C@_17OBLMBIF@?$AAq?$AAs?$AAs?$AA?$AA@ DB 'q', 00H, 's', 00H, 's', 00H, 00H
	DB	00H						; `string'
CONST	ENDS
;	COMDAT ??_C@_1O@COJGIGIJ@?$AAG?$AAL?$AAO?$AAB?$AAA?$AAL?$AA?$AA@
CONST	SEGMENT
??_C@_1O@COJGIGIJ@?$AAG?$AAL?$AAO?$AAB?$AAA?$AAL?$AA?$AA@ DB 'G', 00H, 'L'
	DB	00H, 'O', 00H, 'B', 00H, 'A', 00H, 'L', 00H, 00H, 00H ; `string'
CONST	ENDS
;	COMDAT ??_C@_1O@CPONHA@?$AAP?$AAA?$AAL?$AA?9?$AAB?$AAG?$AA?$AA@
CONST	SEGMENT
??_C@_1O@CPONHA@?$AAP?$AAA?$AAL?$AA?9?$AAB?$AAG?$AA?$AA@ DB 'P', 00H, 'A', 00H
	DB	'L', 00H, '-', 00H, 'B', 00H, 'G', 00H, 00H, 00H ; `string'
CONST	ENDS
;	COMDAT ??_C@_1M@OKDFNJPP@?$AAP?$AAA?$AAL?$AA?9?$AAI?$AA?$AA@
CONST	SEGMENT
??_C@_1M@OKDFNJPP@?$AAP?$AAA?$AAL?$AA?9?$AAI?$AA?$AA@ DB 'P', 00H, 'A', 00H
	DB	'L', 00H, '-', 00H, 'I', 00H, 00H, 00H	; `string'
CONST	ENDS
;	COMDAT ??_C@_1O@JMKALBNF@?$AAP?$AAA?$AAL?$AA?9?$AAD?$AAK?$AA?$AA@
CONST	SEGMENT
??_C@_1O@JMKALBNF@?$AAP?$AAA?$AAL?$AA?9?$AAD?$AAK?$AA?$AA@ DB 'P', 00H, 'A'
	DB	00H, 'L', 00H, '-', 00H, 'D', 00H, 'K', 00H, 00H, 00H ; `string'
CONST	ENDS
;	COMDAT ??_C@_1O@IMHBBACP@?$AAP?$AAA?$AAL?$AA?9?$AAM?$AAN?$AA?$AA@
CONST	SEGMENT
??_C@_1O@IMHBBACP@?$AAP?$AAA?$AAL?$AA?9?$AAM?$AAN?$AA?$AA@ DB 'P', 00H, 'A'
	DB	00H, 'L', 00H, '-', 00H, 'M', 00H, 'N', 00H, 00H, 00H ; `string'
CONST	ENDS
;	COMDAT ??_C@_1BA@NJCCHOGP@?$AAS?$AAE?$AAC?$AAA?$AAM?$AA?9?$AAL?$AA?$AA@
CONST	SEGMENT
??_C@_1BA@NJCCHOGP@?$AAS?$AAE?$AAC?$AAA?$AAM?$AA?9?$AAL?$AA?$AA@ DB 'S', 00H
	DB	'E', 00H, 'C', 00H, 'A', 00H, 'M', 00H, '-', 00H, 'L', 00H, 00H
	DB	00H						; `string'
CONST	ENDS
;	COMDAT ??_C@_1BC@PFJOKPCA@?$AAS?$AAE?$AAC?$AAA?$AAM?$AA?9?$AAD?$AAK?$AA?$AA@
CONST	SEGMENT
??_C@_1BC@PFJOKPCA@?$AAS?$AAE?$AAC?$AAA?$AAM?$AA?9?$AAD?$AAK?$AA?$AA@ DB 'S'
	DB	00H, 'E', 00H, 'C', 00H, 'A', 00H, 'M', 00H, '-', 00H, 'D', 00H
	DB	'K', 00H, 00H, 00H				; `string'
CONST	ENDS
;	COMDAT ??_C@_1O@LMGGCLHH@?$AAN?$AAT?$AAS?$AAC?$AA?9?$AAM?$AA?$AA@
CONST	SEGMENT
??_C@_1O@LMGGCLHH@?$AAN?$AAT?$AAS?$AAC?$AA?9?$AAM?$AA?$AA@ DB 'N', 00H, 'T'
	DB	00H, 'S', 00H, 'C', 00H, '-', 00H, 'M', 00H, 00H, 00H ; `string'
CONST	ENDS
;	COMDAT ??_C@_1BA@BKMKJFAN@?$AAN?$AAT?$AAS?$AAC?$AA?9?$AAJ?$AAP?$AA?$AA@
CONST	SEGMENT
??_C@_1BA@BKMKJFAN@?$AAN?$AAT?$AAS?$AAC?$AA?9?$AAJ?$AAP?$AA?$AA@ DB 'N', 00H
	DB	'T', 00H, 'S', 00H, 'C', 00H, '-', 00H, 'J', 00H, 'P', 00H, 00H
	DB	00H						; `string'
CONST	ENDS
;	COMDAT ??_C@_19CEKDAEDP@?$AAA?$AAU?$AAT?$AAO?$AA?$AA@
CONST	SEGMENT
??_C@_19CEKDAEDP@?$AAA?$AAU?$AAT?$AAO?$AA?$AA@ DB 'A', 00H, 'U', 00H, 'T', 00H
	DB	'O', 00H, 00H, 00H				; `string'
CONST	ENDS
;	COMDAT ??_C@_1M@PBHOBGFC@?$AAS?$AAE?$AAT?$AAU?$AAP?$AA?$AA@
CONST	SEGMENT
??_C@_1M@PBHOBGFC@?$AAS?$AAE?$AAT?$AAU?$AAP?$AA?$AA@ DB 'S', 00H, 'E', 00H
	DB	'T', 00H, 'U', 00H, 'P', 00H, 00H, 00H	; `string'
CONST	ENDS
;	COMDAT ??_C@_1O@GMMJLLPL@?$AAA?$AAB?$AAS?$AAE?$AAN?$AAT?$AA?$AA@
CONST	SEGMENT
??_C@_1O@GMMJLLPL@?$AAA?$AAB?$AAS?$AAE?$AAN?$AAT?$AA?$AA@ DB 'A', 00H, 'B'
	DB	00H, 'S', 00H, 'E', 00H, 'N', 00H, 'T', 00H, 00H, 00H ; `string'
CONST	ENDS
;	COMDAT ??_C@_1BM@CDJFEPDA@?$AAP?$AAH?$AAI?$AAL?$AAI?$AAP?$AAS?$AA_?$AAP?$AAA?$AAL?$AA_?$AAI?$AA?$AA@
CONST	SEGMENT
??_C@_1BM@CDJFEPDA@?$AAP?$AAH?$AAI?$AAL?$AAI?$AAP?$AAS?$AA_?$AAP?$AAA?$AAL?$AA_?$AAI?$AA?$AA@ DB 'P'
	DB	00H, 'H', 00H, 'I', 00H, 'L', 00H, 'I', 00H, 'P', 00H, 'S', 00H
	DB	'_', 00H, 'P', 00H, 'A', 00H, 'L', 00H, '_', 00H, 'I', 00H, 00H
	DB	00H						; `string'
CONST	ENDS
;	COMDAT ??_C@_1BK@IFFHILBA@?$AAP?$AAH?$AAI?$AAL?$AAI?$AAP?$AAS?$AA_?$AAN?$AAT?$AAS?$AAC?$AA?$AA@
CONST	SEGMENT
??_C@_1BK@IFFHILBA@?$AAP?$AAH?$AAI?$AAL?$AAI?$AAP?$AAS?$AA_?$AAN?$AAT?$AAS?$AAC?$AA?$AA@ DB 'P'
	DB	00H, 'H', 00H, 'I', 00H, 'L', 00H, 'I', 00H, 'P', 00H, 'S', 00H
	DB	'_', 00H, 'N', 00H, 'T', 00H, 'S', 00H, 'C', 00H, 00H, 00H ; `string'
CONST	ENDS
;	COMDAT ??_C@_1BM@DCHONLKK@?$AAP?$AAH?$AAI?$AAL?$AAI?$AAP?$AAS?$AA_?$AAS?$AAE?$AAC?$AAA?$AAM?$AA?$AA@
CONST	SEGMENT
??_C@_1BM@DCHONLKK@?$AAP?$AAH?$AAI?$AAL?$AAI?$AAP?$AAS?$AA_?$AAS?$AAE?$AAC?$AAA?$AAM?$AA?$AA@ DB 'P'
	DB	00H, 'H', 00H, 'I', 00H, 'L', 00H, 'I', 00H, 'P', 00H, 'S', 00H
	DB	'_', 00H, 'S', 00H, 'E', 00H, 'C', 00H, 'A', 00H, 'M', 00H, 00H
	DB	00H						; `string'
CONST	ENDS
;	COMDAT ??_C@_1BI@IKKAFKBC@?$AAP?$AAH?$AAI?$AAL?$AAI?$AAP?$AAS?$AA_?$AAP?$AAA?$AAL?$AA?$AA@
CONST	SEGMENT
??_C@_1BI@IKKAFKBC@?$AAP?$AAH?$AAI?$AAL?$AAI?$AAP?$AAS?$AA_?$AAP?$AAA?$AAL?$AA?$AA@ DB 'P'
	DB	00H, 'H', 00H, 'I', 00H, 'L', 00H, 'I', 00H, 'P', 00H, 'S', 00H
	DB	'_', 00H, 'P', 00H, 'A', 00H, 'L', 00H, 00H, 00H ; `string'
CONST	ENDS
;	COMDAT ??_C@_1CE@BHHLKEHK@?$AAT?$AAE?$AAM?$AAI?$AAC?$AA_?$AA4?$AA0?$AA0?$AA2?$AAF?$AAH?$AA5?$AA_?$AAP?$AAA?$AAL?$AA?$AA@
CONST	SEGMENT
??_C@_1CE@BHHLKEHK@?$AAT?$AAE?$AAM?$AAI?$AAC?$AA_?$AA4?$AA0?$AA0?$AA2?$AAF?$AAH?$AA5?$AA_?$AAP?$AAA?$AAL?$AA?$AA@ DB 'T'
	DB	00H, 'E', 00H, 'M', 00H, 'I', 00H, 'C', 00H, '_', 00H, '4', 00H
	DB	'0', 00H, '0', 00H, '2', 00H, 'F', 00H, 'H', 00H, '5', 00H, '_'
	DB	00H, 'P', 00H, 'A', 00H, 'L', 00H, 00H, 00H	; `string'
CONST	ENDS
;	COMDAT ??_C@_1CG@DEBCKDA@?$AAT?$AAE?$AAM?$AAI?$AAC?$AA_?$AA4?$AA0?$AA3?$AA2?$AAF?$AAY?$AA5?$AA_?$AAN?$AAT?$AAS?$AAC?$AA?$AA@
CONST	SEGMENT
??_C@_1CG@DEBCKDA@?$AAT?$AAE?$AAM?$AAI?$AAC?$AA_?$AA4?$AA0?$AA3?$AA2?$AAF?$AAY?$AA5?$AA_?$AAN?$AAT?$AAS?$AAC?$AA?$AA@ DB 'T'
	DB	00H, 'E', 00H, 'M', 00H, 'I', 00H, 'C', 00H, '_', 00H, '4', 00H
	DB	'0', 00H, '3', 00H, '2', 00H, 'F', 00H, 'Y', 00H, '5', 00H, '_'
	DB	00H, 'N', 00H, 'T', 00H, 'S', 00H, 'C', 00H, 00H, 00H ; `string'
CONST	ENDS
;	COMDAT ??_C@_1CI@PPODIFIC@?$AAT?$AAE?$AAM?$AAI?$AAC?$AA_?$AA4?$AA0?$AA6?$AA2?$AAF?$AAY?$AA5?$AA_?$AAP?$AAA?$AAL?$AA_?$AAI?$AA?$AA@
CONST	SEGMENT
??_C@_1CI@PPODIFIC@?$AAT?$AAE?$AAM?$AAI?$AAC?$AA_?$AA4?$AA0?$AA6?$AA2?$AAF?$AAY?$AA5?$AA_?$AAP?$AAA?$AAL?$AA_?$AAI?$AA?$AA@ DB 'T'
	DB	00H, 'E', 00H, 'M', 00H, 'I', 00H, 'C', 00H, '_', 00H, '4', 00H
	DB	'0', 00H, '6', 00H, '2', 00H, 'F', 00H, 'Y', 00H, '5', 00H, '_'
	DB	00H, 'P', 00H, 'A', 00H, 'L', 00H, '_', 00H, 'I', 00H, 00H, 00H ; `string'
CONST	ENDS
;	COMDAT ??_C@_1CG@ENKMMBGJ@?$AAT?$AAE?$AAM?$AAI?$AAC?$AA_?$AA4?$AA0?$AA3?$AA6?$AAF?$AAY?$AA5?$AA_?$AAN?$AAT?$AAS?$AAC?$AA?$AA@
CONST	SEGMENT
??_C@_1CG@ENKMMBGJ@?$AAT?$AAE?$AAM?$AAI?$AAC?$AA_?$AA4?$AA0?$AA3?$AA6?$AAF?$AAY?$AA5?$AA_?$AAN?$AAT?$AAS?$AAC?$AA?$AA@ DB 'T'
	DB	00H, 'E', 00H, 'M', 00H, 'I', 00H, 'C', 00H, '_', 00H, '4', 00H
	DB	'0', 00H, '3', 00H, '6', 00H, 'F', 00H, 'Y', 00H, '5', 00H, '_'
	DB	00H, 'N', 00H, 'T', 00H, 'S', 00H, 'C', 00H, 00H, 00H ; `string'
CONST	ENDS
;	COMDAT ??_C@_1CA@GOAKFAHF@?$AAA?$AAL?$AAP?$AAS?$AA_?$AAT?$AAS?$AAB?$AAH?$AA1?$AA_?$AAN?$AAT?$AAS?$AAC?$AA?$AA@
CONST	SEGMENT
??_C@_1CA@GOAKFAHF@?$AAA?$AAL?$AAP?$AAS?$AA_?$AAT?$AAS?$AAB?$AAH?$AA1?$AA_?$AAN?$AAT?$AAS?$AAC?$AA?$AA@ DB 'A'
	DB	00H, 'L', 00H, 'P', 00H, 'S', 00H, '_', 00H, 'T', 00H, 'S', 00H
	DB	'B', 00H, 'H', 00H, '1', 00H, '_', 00H, 'N', 00H, 'T', 00H, 'S'
	DB	00H, 'C', 00H, 00H, 00H			; `string'
CONST	ENDS
;	COMDAT ??_C@_1BO@GDJDNPLL@?$AAA?$AAL?$AAP?$AAS?$AA_?$AAT?$AAS?$AAB?$AAE?$AA1?$AA_?$AAP?$AAA?$AAL?$AA?$AA@
CONST	SEGMENT
??_C@_1BO@GDJDNPLL@?$AAA?$AAL?$AAP?$AAS?$AA_?$AAT?$AAS?$AAB?$AAE?$AA1?$AA_?$AAP?$AAA?$AAL?$AA?$AA@ DB 'A'
	DB	00H, 'L', 00H, 'P', 00H, 'S', 00H, '_', 00H, 'T', 00H, 'S', 00H
	DB	'B', 00H, 'E', 00H, '1', 00H, '_', 00H, 'P', 00H, 'A', 00H, 'L'
	DB	00H, 00H, 00H				; `string'
CONST	ENDS
;	COMDAT ??_C@_1CC@OMKKLJNL@?$AAA?$AAL?$AAP?$AAS?$AA_?$AAT?$AAS?$AAB?$AAB?$AA5?$AA_?$AAP?$AAA?$AAL?$AA_?$AAI?$AA?$AA@
CONST	SEGMENT
??_C@_1CC@OMKKLJNL@?$AAA?$AAL?$AAP?$AAS?$AA_?$AAT?$AAS?$AAB?$AAB?$AA5?$AA_?$AAP?$AAA?$AAL?$AA_?$AAI?$AA?$AA@ DB 'A'
	DB	00H, 'L', 00H, 'P', 00H, 'S', 00H, '_', 00H, 'T', 00H, 'S', 00H
	DB	'B', 00H, 'B', 00H, '5', 00H, '_', 00H, 'P', 00H, 'A', 00H, 'L'
	DB	00H, '_', 00H, 'I', 00H, 00H, 00H		; `string'
CONST	ENDS
;	COMDAT ??_C@_1BO@GAJFOEME@?$AAA?$AAL?$AAP?$AAS?$AA_?$AAT?$AAS?$AAB?$AAE?$AA5?$AA_?$AAP?$AAA?$AAL?$AA?$AA@
CONST	SEGMENT
??_C@_1BO@GAJFOEME@?$AAA?$AAL?$AAP?$AAS?$AA_?$AAT?$AAS?$AAB?$AAE?$AA5?$AA_?$AAP?$AAA?$AAL?$AA?$AA@ DB 'A'
	DB	00H, 'L', 00H, 'P', 00H, 'S', 00H, '_', 00H, 'T', 00H, 'S', 00H
	DB	'B', 00H, 'E', 00H, '5', 00H, '_', 00H, 'P', 00H, 'A', 00H, 'L'
	DB	00H, 00H, 00H				; `string'
CONST	ENDS
;	COMDAT ??_C@_1BO@JIFHKPHC@?$AAA?$AAL?$AAP?$AAS?$AA_?$AAT?$AAS?$AAB?$AAC?$AA5?$AA_?$AAP?$AAA?$AAL?$AA?$AA@
CONST	SEGMENT
??_C@_1BO@JIFHKPHC@?$AAA?$AAL?$AAP?$AAS?$AA_?$AAT?$AAS?$AAB?$AAC?$AA5?$AA_?$AAP?$AAA?$AAL?$AA?$AA@ DB 'A'
	DB	00H, 'L', 00H, 'P', 00H, 'S', 00H, '_', 00H, 'T', 00H, 'S', 00H
	DB	'B', 00H, 'C', 00H, '5', 00H, '_', 00H, 'P', 00H, 'A', 00H, 'L'
	DB	00H, 00H, 00H				; `string'
CONST	ENDS
;	COMDAT ??_C@_1CE@BMNDHDHM@?$AAT?$AAE?$AAM?$AAI?$AAC?$AA_?$AA4?$AA0?$AA0?$AA6?$AAF?$AAH?$AA5?$AA_?$AAP?$AAA?$AAL?$AA?$AA@
CONST	SEGMENT
??_C@_1CE@BMNDHDHM@?$AAT?$AAE?$AAM?$AAI?$AAC?$AA_?$AA4?$AA0?$AA0?$AA6?$AAF?$AAH?$AA5?$AA_?$AAP?$AAA?$AAL?$AA?$AA@ DB 'T'
	DB	00H, 'E', 00H, 'M', 00H, 'I', 00H, 'C', 00H, '_', 00H, '4', 00H
	DB	'0', 00H, '0', 00H, '6', 00H, 'F', 00H, 'H', 00H, '5', 00H, '_'
	DB	00H, 'P', 00H, 'A', 00H, 'L', 00H, 00H, 00H	; `string'
CONST	ENDS
;	COMDAT ??_C@_1DE@NOEBAKJF@?$AAP?$AAH?$AAI?$AAL?$AAI?$AAP?$AAS?$AA_?$AA1?$AA2?$AA3?$AA6?$AAD?$AA_?$AAN?$AAT?$AAS?$AAC?$AA_?$AAI?$AAN?$AAP?$AAU?$AAT?$AA1?$AA?$AA@
CONST	SEGMENT
??_C@_1DE@NOEBAKJF@?$AAP?$AAH?$AAI?$AAL?$AAI?$AAP?$AAS?$AA_?$AA1?$AA2?$AA3?$AA6?$AAD?$AA_?$AAN?$AAT?$AAS?$AAC?$AA_?$AAI?$AAN?$AAP?$AAU?$AAT?$AA1?$AA?$AA@ DB 'P'
	DB	00H, 'H', 00H, 'I', 00H, 'L', 00H, 'I', 00H, 'P', 00H, 'S', 00H
	DB	'_', 00H, '1', 00H, '2', 00H, '3', 00H, '6', 00H, 'D', 00H, '_'
	DB	00H, 'N', 00H, 'T', 00H, 'S', 00H, 'C', 00H, '_', 00H, 'I', 00H
	DB	'N', 00H, 'P', 00H, 'U', 00H, 'T', 00H, '1', 00H, 00H, 00H ; `string'
CONST	ENDS
;	COMDAT ??_C@_1DE@MMPEKFHL@?$AAP?$AAH?$AAI?$AAL?$AAI?$AAP?$AAS?$AA_?$AA1?$AA2?$AA3?$AA6?$AAD?$AA_?$AAN?$AAT?$AAS?$AAC?$AA_?$AAI?$AAN?$AAP?$AAU?$AAT?$AA2?$AA?$AA@
CONST	SEGMENT
??_C@_1DE@MMPEKFHL@?$AAP?$AAH?$AAI?$AAL?$AAI?$AAP?$AAS?$AA_?$AA1?$AA2?$AA3?$AA6?$AAD?$AA_?$AAN?$AAT?$AAS?$AAC?$AA_?$AAI?$AAN?$AAP?$AAU?$AAT?$AA2?$AA?$AA@ DB 'P'
	DB	00H, 'H', 00H, 'I', 00H, 'L', 00H, 'I', 00H, 'P', 00H, 'S', 00H
	DB	'_', 00H, '1', 00H, '2', 00H, '3', 00H, '6', 00H, 'D', 00H, '_'
	DB	00H, 'N', 00H, 'T', 00H, 'S', 00H, 'C', 00H, '_', 00H, 'I', 00H
	DB	'N', 00H, 'P', 00H, 'U', 00H, 'T', 00H, '2', 00H, 00H, 00H ; `string'
CONST	ENDS
;	COMDAT ??_C@_1CA@OEJFEMFE@?$AAA?$AAL?$AAP?$AAS?$AA_?$AAT?$AAS?$AAC?$AAH?$AA6?$AA_?$AAN?$AAT?$AAS?$AAC?$AA?$AA@
CONST	SEGMENT
??_C@_1CA@OEJFEMFE@?$AAA?$AAL?$AAP?$AAS?$AA_?$AAT?$AAS?$AAC?$AAH?$AA6?$AA_?$AAN?$AAT?$AAS?$AAC?$AA?$AA@ DB 'A'
	DB	00H, 'L', 00H, 'P', 00H, 'S', 00H, '_', 00H, 'T', 00H, 'S', 00H
	DB	'C', 00H, 'H', 00H, '6', 00H, '_', 00H, 'N', 00H, 'T', 00H, 'S'
	DB	00H, 'C', 00H, 00H, 00H			; `string'
CONST	ENDS
;	COMDAT ??_C@_1CE@ICAJJFCA@?$AAT?$AAE?$AAM?$AAI?$AAC?$AA_?$AA4?$AA0?$AA1?$AA6?$AAF?$AAY?$AA5?$AA_?$AAP?$AAA?$AAL?$AA?$AA@
CONST	SEGMENT
??_C@_1CE@ICAJJFCA@?$AAT?$AAE?$AAM?$AAI?$AAC?$AA_?$AA4?$AA0?$AA1?$AA6?$AAF?$AAY?$AA5?$AA_?$AAP?$AAA?$AAL?$AA?$AA@ DB 'T'
	DB	00H, 'E', 00H, 'M', 00H, 'I', 00H, 'C', 00H, '_', 00H, '4', 00H
	DB	'0', 00H, '1', 00H, '6', 00H, 'F', 00H, 'Y', 00H, '5', 00H, '_'
	DB	00H, 'P', 00H, 'A', 00H, 'L', 00H, 00H, 00H	; `string'
CONST	ENDS
;	COMDAT ??_C@_1CC@FGAIIFMP@?$AAP?$AAH?$AAI?$AAL?$AAI?$AAP?$AAS?$AA_?$AAM?$AAK?$AA2?$AA_?$AAN?$AAT?$AAS?$AAC?$AA?$AA@
CONST	SEGMENT
??_C@_1CC@FGAIIFMP@?$AAP?$AAH?$AAI?$AAL?$AAI?$AAP?$AAS?$AA_?$AAM?$AAK?$AA2?$AA_?$AAN?$AAT?$AAS?$AAC?$AA?$AA@ DB 'P'
	DB	00H, 'H', 00H, 'I', 00H, 'L', 00H, 'I', 00H, 'P', 00H, 'S', 00H
	DB	'_', 00H, 'M', 00H, 'K', 00H, '2', 00H, '_', 00H, 'N', 00H, 'T'
	DB	00H, 'S', 00H, 'C', 00H, 00H, 00H		; `string'
CONST	ENDS
;	COMDAT ??_C@_1CI@KDECBGIC@?$AAT?$AAE?$AAM?$AAI?$AAC?$AA_?$AA4?$AA0?$AA6?$AA6?$AAF?$AAY?$AA5?$AA_?$AAP?$AAA?$AAL?$AA_?$AAI?$AA?$AA@
CONST	SEGMENT
??_C@_1CI@KDECBGIC@?$AAT?$AAE?$AAM?$AAI?$AAC?$AA_?$AA4?$AA0?$AA6?$AA6?$AAF?$AAY?$AA5?$AA_?$AAP?$AAA?$AAL?$AA_?$AAI?$AA?$AA@ DB 'T'
	DB	00H, 'E', 00H, 'M', 00H, 'I', 00H, 'C', 00H, '_', 00H, '4', 00H
	DB	'0', 00H, '6', 00H, '6', 00H, 'F', 00H, 'Y', 00H, '5', 00H, '_'
	DB	00H, 'P', 00H, 'A', 00H, 'L', 00H, '_', 00H, 'I', 00H, 00H, 00H ; `string'
CONST	ENDS
;	COMDAT ??_C@_1CE@OEBBDIMK@?$AAT?$AAE?$AAM?$AAI?$AAC?$AA_?$AA4?$AA0?$AA0?$AA6?$AAF?$AAN?$AA5?$AA_?$AAP?$AAA?$AAL?$AA?$AA@
CONST	SEGMENT
??_C@_1CE@OEBBDIMK@?$AAT?$AAE?$AAM?$AAI?$AAC?$AA_?$AA4?$AA0?$AA0?$AA6?$AAF?$AAN?$AA5?$AA_?$AAP?$AAA?$AAL?$AA?$AA@ DB 'T'
	DB	00H, 'E', 00H, 'M', 00H, 'I', 00H, 'C', 00H, '_', 00H, '4', 00H
	DB	'0', 00H, '0', 00H, '6', 00H, 'F', 00H, 'N', 00H, '5', 00H, '_'
	DB	00H, 'P', 00H, 'A', 00H, 'L', 00H, 00H, 00H	; `string'
CONST	ENDS
;	COMDAT ??_C@_1CE@FOCJDBOD@?$AAT?$AAE?$AAM?$AAI?$AAC?$AA_?$AA4?$AA0?$AA0?$AA9?$AAF?$AAR?$AA5?$AA_?$AAP?$AAA?$AAL?$AA?$AA@
CONST	SEGMENT
??_C@_1CE@FOCJDBOD@?$AAT?$AAE?$AAM?$AAI?$AAC?$AA_?$AA4?$AA0?$AA0?$AA9?$AAF?$AAR?$AA5?$AA_?$AAP?$AAA?$AAL?$AA?$AA@ DB 'T'
	DB	00H, 'E', 00H, 'M', 00H, 'I', 00H, 'C', 00H, '_', 00H, '4', 00H
	DB	'0', 00H, '0', 00H, '9', 00H, 'F', 00H, 'R', 00H, '5', 00H, '_'
	DB	00H, 'P', 00H, 'A', 00H, 'L', 00H, 00H, 00H	; `string'
CONST	ENDS
;	COMDAT ??_C@_1CG@GLOIJKPF@?$AAT?$AAE?$AAM?$AAI?$AAC?$AA_?$AA4?$AA0?$AA3?$AA9?$AAF?$AAR?$AA5?$AA_?$AAN?$AAT?$AAS?$AAC?$AA?$AA@
CONST	SEGMENT
??_C@_1CG@GLOIJKPF@?$AAT?$AAE?$AAM?$AAI?$AAC?$AA_?$AA4?$AA0?$AA3?$AA9?$AAF?$AAR?$AA5?$AA_?$AAN?$AAT?$AAS?$AAC?$AA?$AA@ DB 'T'
	DB	00H, 'E', 00H, 'M', 00H, 'I', 00H, 'C', 00H, '_', 00H, '4', 00H
	DB	'0', 00H, '3', 00H, '9', 00H, 'F', 00H, 'R', 00H, '5', 00H, '_'
	DB	00H, 'N', 00H, 'T', 00H, 'S', 00H, 'C', 00H, 00H, 00H ; `string'
CONST	ENDS
;	COMDAT ??_C@_1CI@IJEHGMNA@?$AAT?$AAE?$AAM?$AAI?$AAC?$AA_?$AA4?$AA0?$AA4?$AA6?$AAF?$AAM?$AA5?$AA_?$AAM?$AAU?$AAL?$AAT?$AAI?$AA?$AA@
CONST	SEGMENT
??_C@_1CI@IJEHGMNA@?$AAT?$AAE?$AAM?$AAI?$AAC?$AA_?$AA4?$AA0?$AA4?$AA6?$AAF?$AAM?$AA5?$AA_?$AAM?$AAU?$AAL?$AAT?$AAI?$AA?$AA@ DB 'T'
	DB	00H, 'E', 00H, 'M', 00H, 'I', 00H, 'C', 00H, '_', 00H, '4', 00H
	DB	'0', 00H, '4', 00H, '6', 00H, 'F', 00H, 'M', 00H, '5', 00H, '_'
	DB	00H, 'M', 00H, 'U', 00H, 'L', 00H, 'T', 00H, 'I', 00H, 00H, 00H ; `string'
CONST	ENDS
;	COMDAT ??_C@_1BO@MJKOIFIF@?$AAP?$AAH?$AAI?$AAL?$AAI?$AAP?$AAS?$AA_?$AAP?$AAA?$AAL?$AA_?$AAD?$AAK?$AA?$AA@
CONST	SEGMENT
??_C@_1BO@MJKOIFIF@?$AAP?$AAH?$AAI?$AAL?$AAI?$AAP?$AAS?$AA_?$AAP?$AAA?$AAL?$AA_?$AAD?$AAK?$AA?$AA@ DB 'P'
	DB	00H, 'H', 00H, 'I', 00H, 'L', 00H, 'I', 00H, 'P', 00H, 'S', 00H
	DB	'_', 00H, 'P', 00H, 'A', 00H, 'L', 00H, '_', 00H, 'D', 00H, 'K'
	DB	00H, 00H, 00H				; `string'
CONST	ENDS
;	COMDAT ??_C@_1BM@PFKAHCHD@?$AAP?$AAH?$AAI?$AAL?$AAI?$AAP?$AAS?$AA_?$AAM?$AAU?$AAL?$AAT?$AAI?$AA?$AA@
CONST	SEGMENT
??_C@_1BM@PFKAHCHD@?$AAP?$AAH?$AAI?$AAL?$AAI?$AAP?$AAS?$AA_?$AAM?$AAU?$AAL?$AAT?$AAI?$AA?$AA@ DB 'P'
	DB	00H, 'H', 00H, 'I', 00H, 'L', 00H, 'I', 00H, 'P', 00H, 'S', 00H
	DB	'_', 00H, 'M', 00H, 'U', 00H, 'L', 00H, 'T', 00H, 'I', 00H, 00H
	DB	00H						; `string'
CONST	ENDS
;	COMDAT ??_C@_1BO@DFOPCAAK@?$AAL?$AAG?$AA_?$AAI?$AA0?$AA0?$AA1?$AAD?$AA_?$AAP?$AAA?$AAL?$AA_?$AAI?$AA?$AA@
CONST	SEGMENT
??_C@_1BO@DFOPCAAK@?$AAL?$AAG?$AA_?$AAI?$AA0?$AA0?$AA1?$AAD?$AA_?$AAP?$AAA?$AAL?$AA_?$AAI?$AA?$AA@ DB 'L'
	DB	00H, 'G', 00H, '_', 00H, 'I', 00H, '0', 00H, '0', 00H, '1', 00H
	DB	'D', 00H, '_', 00H, 'P', 00H, 'A', 00H, 'L', 00H, '_', 00H, 'I'
	DB	00H, 00H, 00H				; `string'
CONST	ENDS
;	COMDAT ??_C@_1BO@FADGBOEK@?$AAL?$AAG?$AA_?$AAI?$AA7?$AA0?$AA1?$AAD?$AA_?$AAP?$AAA?$AAL?$AA_?$AAI?$AA?$AA@
CONST	SEGMENT
??_C@_1BO@FADGBOEK@?$AAL?$AAG?$AA_?$AAI?$AA7?$AA0?$AA1?$AAD?$AA_?$AAP?$AAA?$AAL?$AA_?$AAI?$AA?$AA@ DB 'L'
	DB	00H, 'G', 00H, '_', 00H, 'I', 00H, '7', 00H, '0', 00H, '1', 00H
	DB	'D', 00H, '_', 00H, 'P', 00H, 'A', 00H, 'L', 00H, '_', 00H, 'I'
	DB	00H, 00H, 00H				; `string'
CONST	ENDS
;	COMDAT ??_C@_1BK@NFMGFCPC@?$AAL?$AAG?$AA_?$AAR?$AA0?$AA1?$AAF?$AA_?$AAN?$AAT?$AAS?$AAC?$AA?$AA@
CONST	SEGMENT
??_C@_1BK@NFMGFCPC@?$AAL?$AAG?$AA_?$AAR?$AA0?$AA1?$AAF?$AA_?$AAN?$AAT?$AAS?$AAC?$AA?$AA@ DB 'L'
	DB	00H, 'G', 00H, '_', 00H, 'R', 00H, '0', 00H, '1', 00H, 'F', 00H
	DB	'_', 00H, 'N', 00H, 'T', 00H, 'S', 00H, 'C', 00H, 00H, 00H ; `string'
CONST	ENDS
;	COMDAT ??_C@_1BI@IENNGMBM@?$AAL?$AAG?$AA_?$AAB?$AA0?$AA1?$AAD?$AA_?$AAP?$AAA?$AAL?$AA?$AA@
CONST	SEGMENT
??_C@_1BI@IENNGMBM@?$AAL?$AAG?$AA_?$AAB?$AA0?$AA1?$AAD?$AA_?$AAP?$AAA?$AAL?$AA?$AA@ DB 'L'
	DB	00H, 'G', 00H, '_', 00H, 'B', 00H, '0', 00H, '1', 00H, 'D', 00H
	DB	'_', 00H, 'P', 00H, 'A', 00H, 'L', 00H, 00H, 00H ; `string'
CONST	ENDS
;	COMDAT ??_C@_1BI@CKLFPNIN@?$AAL?$AAG?$AA_?$AAB?$AA1?$AA1?$AAD?$AA_?$AAP?$AAA?$AAL?$AA?$AA@
CONST	SEGMENT
??_C@_1BI@CKLFPNIN@?$AAL?$AAG?$AA_?$AAB?$AA1?$AA1?$AAD?$AA_?$AAP?$AAA?$AAL?$AA?$AA@ DB 'L'
	DB	00H, 'G', 00H, '_', 00H, 'B', 00H, '1', 00H, '1', 00H, 'D', 00H
	DB	'_', 00H, 'P', 00H, 'A', 00H, 'L', 00H, 00H, 00H ; `string'
CONST	ENDS
;	COMDAT ??_C@_1CE@BCGOJMKC@?$AAT?$AAE?$AAM?$AAI?$AAC?$AA_?$AA4?$AA0?$AA0?$AA9?$AAF?$AAN?$AA5?$AA_?$AAP?$AAA?$AAL?$AA?$AA@
CONST	SEGMENT
??_C@_1CE@BCGOJMKC@?$AAT?$AAE?$AAM?$AAI?$AAC?$AA_?$AA4?$AA0?$AA0?$AA9?$AAF?$AAN?$AA5?$AA_?$AAP?$AAA?$AAL?$AA?$AA@ DB 'T'
	DB	00H, 'E', 00H, 'M', 00H, 'I', 00H, 'C', 00H, '_', 00H, '4', 00H
	DB	'0', 00H, '0', 00H, '9', 00H, 'F', 00H, 'N', 00H, '5', 00H, '_'
	DB	00H, 'P', 00H, 'A', 00H, 'L', 00H, 00H, 00H	; `string'
CONST	ENDS
;	COMDAT ??_C@_1O@NGHNCELA@?$AAM?$AAT?$AA2?$AA0?$AA3?$AA2?$AA?$AA@
CONST	SEGMENT
??_C@_1O@NGHNCELA@?$AAM?$AAT?$AA2?$AA0?$AA3?$AA2?$AA?$AA@ DB 'M', 00H, 'T'
	DB	00H, '2', 00H, '0', 00H, '3', 00H, '2', 00H, 00H, 00H ; `string'
CONST	ENDS
;	COMDAT ??_C@_1CK@MHILDIAN@?$AAS?$AAH?$AAA?$AAR?$AAP?$AA_?$AA2?$AAU?$AA5?$AAJ?$AAF?$AA5?$AA5?$AA4?$AA0?$AA_?$AAN?$AAT?$AAS?$AAC?$AA?$AA@
CONST	SEGMENT
??_C@_1CK@MHILDIAN@?$AAS?$AAH?$AAA?$AAR?$AAP?$AA_?$AA2?$AAU?$AA5?$AAJ?$AAF?$AA5?$AA5?$AA4?$AA0?$AA_?$AAN?$AAT?$AAS?$AAC?$AA?$AA@ DB 'S'
	DB	00H, 'H', 00H, 'A', 00H, 'R', 00H, 'P', 00H, '_', 00H, '2', 00H
	DB	'U', 00H, '5', 00H, 'J', 00H, 'F', 00H, '5', 00H, '5', 00H, '4'
	DB	00H, '0', 00H, '_', 00H, 'N', 00H, 'T', 00H, 'S', 00H, 'C', 00H
	DB	00H, 00H					; `string'
CONST	ENDS
;	COMDAT ??_C@_1CE@CODMLBHG@?$AAL?$AAG?$AA_?$AAT?$AAA?$AAP?$AAC?$AAH?$AA7?$AA0?$AA1?$AAP?$AA_?$AAN?$AAT?$AAS?$AAC?$AA?$AA@
CONST	SEGMENT
??_C@_1CE@CODMLBHG@?$AAL?$AAG?$AA_?$AAT?$AAA?$AAP?$AAC?$AAH?$AA7?$AA0?$AA1?$AAP?$AA_?$AAN?$AAT?$AAS?$AAC?$AA?$AA@ DB 'L'
	DB	00H, 'G', 00H, '_', 00H, 'T', 00H, 'A', 00H, 'P', 00H, 'C', 00H
	DB	'H', 00H, '7', 00H, '0', 00H, '1', 00H, 'P', 00H, '_', 00H, 'N'
	DB	00H, 'T', 00H, 'S', 00H, 'C', 00H, 00H, 00H	; `string'
CONST	ENDS
;	COMDAT ??_C@_1DC@PNFJNOKI@?$AAS?$AAA?$AAM?$AAS?$AAU?$AAN?$AAG?$AA_?$AAP?$AAA?$AAL?$AA_?$AAT?$AAC?$AAP?$AAM?$AA9?$AA0?$AA9?$AA1?$AAP?$AAD?$AA2?$AA7?$AA?$AA@
CONST	SEGMENT
??_C@_1DC@PNFJNOKI@?$AAS?$AAA?$AAM?$AAS?$AAU?$AAN?$AAG?$AA_?$AAP?$AAA?$AAL?$AA_?$AAT?$AAC?$AAP?$AAM?$AA9?$AA0?$AA9?$AA1?$AAP?$AAD?$AA2?$AA7?$AA?$AA@ DB 'S'
	DB	00H, 'A', 00H, 'M', 00H, 'S', 00H, 'U', 00H, 'N', 00H, 'G', 00H
	DB	'_', 00H, 'P', 00H, 'A', 00H, 'L', 00H, '_', 00H, 'T', 00H, 'C'
	DB	00H, 'P', 00H, 'M', 00H, '9', 00H, '0', 00H, '9', 00H, '1', 00H
	DB	'P', 00H, 'D', 00H, '2', 00H, '7', 00H, 00H, 00H ; `string'
CONST	ENDS
;	COMDAT ??_C@_1BM@CPMEKHAF@?$AAT?$AAE?$AAM?$AAI?$AAC?$AA_?$AA4?$AA1?$AA0?$AA6?$AAF?$AAH?$AA5?$AA?$AA@
CONST	SEGMENT
??_C@_1BM@CPMEKHAF@?$AAT?$AAE?$AAM?$AAI?$AAC?$AA_?$AA4?$AA1?$AA0?$AA6?$AAF?$AAH?$AA5?$AA?$AA@ DB 'T'
	DB	00H, 'E', 00H, 'M', 00H, 'I', 00H, 'C', 00H, '_', 00H, '4', 00H
	DB	'1', 00H, '0', 00H, '6', 00H, 'F', 00H, 'H', 00H, '5', 00H, 00H
	DB	00H						; `string'
CONST	ENDS
;	COMDAT ??_C@_1BM@OIAPHLFI@?$AAT?$AAE?$AAM?$AAI?$AAC?$AA_?$AA4?$AA0?$AA1?$AA2?$AAF?$AAY?$AA5?$AA?$AA@
CONST	SEGMENT
??_C@_1BM@OIAPHLFI@?$AAT?$AAE?$AAM?$AAI?$AAC?$AA_?$AA4?$AA0?$AA1?$AA2?$AAF?$AAY?$AA5?$AA?$AA@ DB 'T'
	DB	00H, 'E', 00H, 'M', 00H, 'I', 00H, 'C', 00H, '_', 00H, '4', 00H
	DB	'0', 00H, '1', 00H, '2', 00H, 'F', 00H, 'Y', 00H, '5', 00H, 00H
	DB	00H						; `string'
CONST	ENDS
;	COMDAT ??_C@_1BM@JANAKEML@?$AAT?$AAE?$AAM?$AAI?$AAC?$AA_?$AA4?$AA1?$AA3?$AA6?$AAF?$AAY?$AA5?$AA?$AA@
CONST	SEGMENT
??_C@_1BM@JANAKEML@?$AAT?$AAE?$AAM?$AAI?$AAC?$AA_?$AA4?$AA1?$AA3?$AA6?$AAF?$AAY?$AA5?$AA?$AA@ DB 'T'
	DB	00H, 'E', 00H, 'M', 00H, 'I', 00H, 'C', 00H, '_', 00H, '4', 00H
	DB	'1', 00H, '3', 00H, '6', 00H, 'F', 00H, 'Y', 00H, '5', 00H, 00H
	DB	00H						; `string'
CONST	ENDS
;	COMDAT ??_C@_1BO@EHMDLLBA@?$AAL?$AAG?$AA_?$AAT?$AAA?$AAP?$AAC?$AAN?$AAE?$AAW?$AA_?$AAP?$AAA?$AAL?$AA?$AA@
CONST	SEGMENT
??_C@_1BO@EHMDLLBA@?$AAL?$AAG?$AA_?$AAT?$AAA?$AAP?$AAC?$AAN?$AAE?$AAW?$AA_?$AAP?$AAA?$AAL?$AA?$AA@ DB 'L'
	DB	00H, 'G', 00H, '_', 00H, 'T', 00H, 'A', 00H, 'P', 00H, 'C', 00H
	DB	'N', 00H, 'E', 00H, 'W', 00H, '_', 00H, 'P', 00H, 'A', 00H, 'L'
	DB	00H, 00H, 00H				; `string'
CONST	ENDS
;	COMDAT ??_C@_1CK@CLKCBCPN@?$AAP?$AAH?$AAI?$AAL?$AAI?$AAP?$AAS?$AA_?$AAF?$AAM?$AA1?$AA2?$AA1?$AA6?$AAM?$AAE?$AA_?$AAM?$AAK?$AA3?$AA?$AA@
CONST	SEGMENT
??_C@_1CK@CLKCBCPN@?$AAP?$AAH?$AAI?$AAL?$AAI?$AAP?$AAS?$AA_?$AAF?$AAM?$AA1?$AA2?$AA1?$AA6?$AAM?$AAE?$AA_?$AAM?$AAK?$AA3?$AA?$AA@ DB 'P'
	DB	00H, 'H', 00H, 'I', 00H, 'L', 00H, 'I', 00H, 'P', 00H, 'S', 00H
	DB	'_', 00H, 'F', 00H, 'M', 00H, '1', 00H, '2', 00H, '1', 00H, '6'
	DB	00H, 'M', 00H, 'E', 00H, '_', 00H, 'M', 00H, 'K', 00H, '3', 00H
	DB	00H, 00H					; `string'
CONST	ENDS
;	COMDAT ??_C@_1CA@GAGMPGBP@?$AAL?$AAG?$AA_?$AAT?$AAA?$AAP?$AAC?$AAN?$AAE?$AAW?$AA_?$AAN?$AAT?$AAS?$AAC?$AA?$AA@
CONST	SEGMENT
??_C@_1CA@GAGMPGBP@?$AAL?$AAG?$AA_?$AAT?$AAA?$AAP?$AAC?$AAN?$AAE?$AAW?$AA_?$AAN?$AAT?$AAS?$AAC?$AA?$AA@ DB 'L'
	DB	00H, 'G', 00H, '_', 00H, 'T', 00H, 'A', 00H, 'P', 00H, 'C', 00H
	DB	'N', 00H, 'E', 00H, 'W', 00H, '_', 00H, 'N', 00H, 'T', 00H, 'S'
	DB	00H, 'C', 00H, 00H, 00H			; `string'
CONST	ENDS
;	COMDAT ??_C@_1BG@FEPCEPIB@?$AAM?$AAT?$AA2?$AA0?$AA3?$AA2?$AA_?$AAP?$AAA?$AAL?$AA?$AA@
CONST	SEGMENT
??_C@_1BG@FEPCEPIB@?$AAM?$AAT?$AA2?$AA0?$AA3?$AA2?$AA_?$AAP?$AAA?$AAL?$AA?$AA@ DB 'M'
	DB	00H, 'T', 00H, '2', 00H, '0', 00H, '3', 00H, '2', 00H, '_', 00H
	DB	'P', 00H, 'A', 00H, 'L', 00H, 00H, 00H	; `string'
CONST	ENDS
;	COMDAT ??_C@_1DA@JEOOMIMC@?$AAP?$AAH?$AAI?$AAL?$AAI?$AAP?$AAS?$AA_?$AAF?$AAI?$AA1?$AA2?$AA8?$AA6?$AA_?$AAN?$AAT?$AAS?$AAC?$AA_?$AAM?$AA_?$AAJ?$AA?$AA@
CONST	SEGMENT
??_C@_1DA@JEOOMIMC@?$AAP?$AAH?$AAI?$AAL?$AAI?$AAP?$AAS?$AA_?$AAF?$AAI?$AA1?$AA2?$AA8?$AA6?$AA_?$AAN?$AAT?$AAS?$AAC?$AA_?$AAM?$AA_?$AAJ?$AA?$AA@ DB 'P'
	DB	00H, 'H', 00H, 'I', 00H, 'L', 00H, 'I', 00H, 'P', 00H, 'S', 00H
	DB	'_', 00H, 'F', 00H, 'I', 00H, '1', 00H, '2', 00H, '8', 00H, '6'
	DB	00H, '_', 00H, 'N', 00H, 'T', 00H, 'S', 00H, 'C', 00H, '_', 00H
	DB	'M', 00H, '_', 00H, 'J', 00H, 00H, 00H	; `string'
CONST	ENDS
;	COMDAT ??_C@_1O@KKCNAPCG@?$AAM?$AAT?$AA2?$AA0?$AA5?$AA0?$AA?$AA@
CONST	SEGMENT
??_C@_1O@KKCNAPCG@?$AAM?$AAT?$AA2?$AA0?$AA5?$AA0?$AA?$AA@ DB 'M', 00H, 'T'
	DB	00H, '2', 00H, '0', 00H, '5', 00H, '0', 00H, 00H, 00H ; `string'
CONST	ENDS
;	COMDAT ??_C@_1BG@EAALJKKI@?$AAM?$AAT?$AA2?$AA0?$AA5?$AA0?$AA_?$AAP?$AAA?$AAL?$AA?$AA@
CONST	SEGMENT
??_C@_1BG@EAALJKKI@?$AAM?$AAT?$AA2?$AA0?$AA5?$AA0?$AA_?$AAP?$AAA?$AAL?$AA?$AA@ DB 'M'
	DB	00H, 'T', 00H, '2', 00H, '0', 00H, '5', 00H, '0', 00H, '_', 00H
	DB	'P', 00H, 'A', 00H, 'L', 00H, 00H, 00H	; `string'
CONST	ENDS
;	COMDAT ??_C@_1BK@PNPMMDOJ@?$AAP?$AAH?$AAI?$AAL?$AAI?$AAP?$AAS?$AA_?$AA4?$AAI?$AAN?$AA1?$AA?$AA@
CONST	SEGMENT
??_C@_1BK@PNPMMDOJ@?$AAP?$AAH?$AAI?$AAL?$AAI?$AAP?$AAS?$AA_?$AA4?$AAI?$AAN?$AA1?$AA?$AA@ DB 'P'
	DB	00H, 'H', 00H, 'I', 00H, 'L', 00H, 'I', 00H, 'P', 00H, 'S', 00H
	DB	'_', 00H, '4', 00H, 'I', 00H, 'N', 00H, '1', 00H, 00H, 00H ; `string'
CONST	ENDS
;	COMDAT ??_C@_1BE@OEGEIDDF@?$AAT?$AAC?$AAL?$AA_?$AA2?$AA0?$AA0?$AA2?$AAN?$AA?$AA@
CONST	SEGMENT
??_C@_1BE@OEGEIDDF@?$AAT?$AAC?$AAL?$AA_?$AA2?$AA0?$AA0?$AA2?$AAN?$AA?$AA@ DB 'T'
	DB	00H, 'C', 00H, 'L', 00H, '_', 00H, '2', 00H, '0', 00H, '0', 00H
	DB	'2', 00H, 'N', 00H, 00H, 00H			; `string'
CONST	ENDS
;	COMDAT ??_C@_1BK@CFFBIHHG@?$AAH?$AAI?$AAT?$AAA?$AAC?$AAH?$AAI?$AA_?$AAN?$AAT?$AAS?$AAC?$AA?$AA@
CONST	SEGMENT
??_C@_1BK@CFFBIHHG@?$AAH?$AAI?$AAT?$AAA?$AAC?$AAH?$AAI?$AA_?$AAN?$AAT?$AAS?$AAC?$AA?$AA@ DB 'H'
	DB	00H, 'I', 00H, 'T', 00H, 'A', 00H, 'C', 00H, 'H', 00H, 'I', 00H
	DB	'_', 00H, 'N', 00H, 'T', 00H, 'S', 00H, 'C', 00H, 00H, 00H ; `string'
CONST	ENDS
;	COMDAT ??_C@_1BO@OOKBNEEN@?$AAP?$AAH?$AAI?$AAL?$AAI?$AAP?$AAS?$AA_?$AAP?$AAA?$AAL?$AA_?$AAM?$AAK?$AA?$AA@
CONST	SEGMENT
??_C@_1BO@OOKBNEEN@?$AAP?$AAH?$AAI?$AAL?$AAI?$AAP?$AAS?$AA_?$AAP?$AAA?$AAL?$AA_?$AAM?$AAK?$AA?$AA@ DB 'P'
	DB	00H, 'H', 00H, 'I', 00H, 'L', 00H, 'I', 00H, 'P', 00H, 'S', 00H
	DB	'_', 00H, 'P', 00H, 'A', 00H, 'L', 00H, '_', 00H, 'M', 00H, 'K'
	DB	00H, 00H, 00H				; `string'
CONST	ENDS
;	COMDAT ??_C@_1CG@EMNPDDAO@?$AAP?$AAH?$AAI?$AAL?$AAI?$AAP?$AAS?$AA_?$AAF?$AAM?$AA1?$AA2?$AA3?$AA6?$AA_?$AAM?$AAK?$AA3?$AA?$AA@
CONST	SEGMENT
??_C@_1CG@EMNPDDAO@?$AAP?$AAH?$AAI?$AAL?$AAI?$AAP?$AAS?$AA_?$AAF?$AAM?$AA1?$AA2?$AA3?$AA6?$AA_?$AAM?$AAK?$AA3?$AA?$AA@ DB 'P'
	DB	00H, 'H', 00H, 'I', 00H, 'L', 00H, 'I', 00H, 'P', 00H, 'S', 00H
	DB	'_', 00H, 'F', 00H, 'M', 00H, '1', 00H, '2', 00H, '3', 00H, '6'
	DB	00H, '_', 00H, 'M', 00H, 'K', 00H, '3', 00H, 00H, 00H ; `string'
CONST	ENDS
;	COMDAT ??_C@_1BK@JHDPBOPP@?$AAL?$AAG?$AA_?$AAN?$AAT?$AAS?$AAC?$AA_?$AAT?$AAA?$AAP?$AAE?$AA?$AA@
CONST	SEGMENT
??_C@_1BK@JHDPBOPP@?$AAL?$AAG?$AA_?$AAN?$AAT?$AAS?$AAC?$AA_?$AAT?$AAA?$AAP?$AAE?$AA?$AA@ DB 'L'
	DB	00H, 'G', 00H, '_', 00H, 'N', 00H, 'T', 00H, 'S', 00H, 'C', 00H
	DB	'_', 00H, 'T', 00H, 'A', 00H, 'P', 00H, 'E', 00H, 00H, 00H ; `string'
CONST	ENDS
;	COMDAT ??_C@_1BK@CBBAAEDD@?$AAT?$AAN?$AAF?$AA_?$AA8?$AA8?$AA3?$AA1?$AAB?$AAG?$AAF?$AAF?$AA?$AA@
CONST	SEGMENT
??_C@_1BK@CBBAAEDD@?$AAT?$AAN?$AAF?$AA_?$AA8?$AA8?$AA3?$AA1?$AAB?$AAG?$AAF?$AAF?$AA?$AA@ DB 'T'
	DB	00H, 'N', 00H, 'F', 00H, '_', 00H, '8', 00H, '8', 00H, '3', 00H
	DB	'1', 00H, 'B', 00H, 'G', 00H, 'F', 00H, 'F', 00H, 00H, 00H ; `string'
CONST	ENDS
;	COMDAT ??_C@_1CG@LGMDAEOM@?$AAP?$AAH?$AAI?$AAL?$AAI?$AAP?$AAS?$AA_?$AAF?$AAM?$AA1?$AA2?$AA5?$AA6?$AA_?$AAI?$AAH?$AA3?$AA?$AA@
CONST	SEGMENT
??_C@_1CG@LGMDAEOM@?$AAP?$AAH?$AAI?$AAL?$AAI?$AAP?$AAS?$AA_?$AAF?$AAM?$AA1?$AA2?$AA5?$AA6?$AA_?$AAI?$AAH?$AA3?$AA?$AA@ DB 'P'
	DB	00H, 'H', 00H, 'I', 00H, 'L', 00H, 'I', 00H, 'P', 00H, 'S', 00H
	DB	'_', 00H, 'F', 00H, 'M', 00H, '1', 00H, '2', 00H, '5', 00H, '6'
	DB	00H, '_', 00H, 'I', 00H, 'H', 00H, '3', 00H, 00H, 00H ; `string'
CONST	ENDS
;	COMDAT ??_C@_1BO@PGCKBBBK@?$AAP?$AAH?$AAI?$AAL?$AAI?$AAP?$AAS?$AA_?$AAF?$AAQ?$AA1?$AA2?$AA8?$AA6?$AA?$AA@
CONST	SEGMENT
??_C@_1BO@PGCKBBBK@?$AAP?$AAH?$AAI?$AAL?$AAI?$AAP?$AAS?$AA_?$AAF?$AAQ?$AA1?$AA2?$AA8?$AA6?$AA?$AA@ DB 'P'
	DB	00H, 'H', 00H, 'I', 00H, 'L', 00H, 'I', 00H, 'P', 00H, 'S', 00H
	DB	'_', 00H, 'F', 00H, 'Q', 00H, '1', 00H, '2', 00H, '8', 00H, '6'
	DB	00H, 00H, 00H				; `string'
CONST	ENDS
;	COMDAT ??_C@_1BI@DMIKHBF@?$AAL?$AAG?$AA_?$AAP?$AAA?$AAL?$AA_?$AAT?$AAA?$AAP?$AAE?$AA?$AA@
CONST	SEGMENT
??_C@_1BI@DMIKHBF@?$AAL?$AAG?$AA_?$AAP?$AAA?$AAL?$AA_?$AAT?$AAA?$AAP?$AAE?$AA?$AA@ DB 'L'
	DB	00H, 'G', 00H, '_', 00H, 'P', 00H, 'A', 00H, 'L', 00H, '_', 00H
	DB	'T', 00H, 'A', 00H, 'P', 00H, 'E', 00H, 00H, 00H ; `string'
CONST	ENDS
;	COMDAT ??_C@_1DI@EAGAPDHM@?$AAT?$AAU?$AAN?$AAE?$AAR?$AA_?$AAP?$AAH?$AAI?$AAL?$AAI?$AAP?$AAS?$AA_?$AAF?$AAQ?$AA1?$AA2?$AA1?$AA6?$AAA?$AAM?$AAE?$AA_?$AAM?$AAK?$AA4?$AA?$AA@
CONST	SEGMENT
??_C@_1DI@EAGAPDHM@?$AAT?$AAU?$AAN?$AAE?$AAR?$AA_?$AAP?$AAH?$AAI?$AAL?$AAI?$AAP?$AAS?$AA_?$AAF?$AAQ?$AA1?$AA2?$AA1?$AA6?$AAA?$AAM?$AAE?$AA_?$AAM?$AAK?$AA4?$AA?$AA@ DB 'T'
	DB	00H, 'U', 00H, 'N', 00H, 'E', 00H, 'R', 00H, '_', 00H, 'P', 00H
	DB	'H', 00H, 'I', 00H, 'L', 00H, 'I', 00H, 'P', 00H, 'S', 00H, '_'
	DB	00H, 'F', 00H, 'Q', 00H, '1', 00H, '2', 00H, '1', 00H, '6', 00H
	DB	'A', 00H, 'M', 00H, 'E', 00H, '_', 00H, 'M', 00H, 'K', 00H, '4'
	DB	00H, 00H, 00H				; `string'
CONST	ENDS
;	COMDAT ??_C@_1CI@PFGDHJOM@?$AAP?$AAH?$AAI?$AAL?$AAI?$AAP?$AAS?$AA_?$AAF?$AAQ?$AA1?$AA2?$AA3?$AA6?$AAA?$AA_?$AAM?$AAK?$AA4?$AA?$AA@
CONST	SEGMENT
??_C@_1CI@PFGDHJOM@?$AAP?$AAH?$AAI?$AAL?$AAI?$AAP?$AAS?$AA_?$AAF?$AAQ?$AA1?$AA2?$AA3?$AA6?$AAA?$AA_?$AAM?$AAK?$AA4?$AA?$AA@ DB 'P'
	DB	00H, 'H', 00H, 'I', 00H, 'L', 00H, 'I', 00H, 'P', 00H, 'S', 00H
	DB	'_', 00H, 'F', 00H, 'Q', 00H, '1', 00H, '2', 00H, '3', 00H, '6'
	DB	00H, 'A', 00H, '_', 00H, 'M', 00H, 'K', 00H, '4', 00H, 00H, 00H ; `string'
CONST	ENDS
;	COMDAT ??_C@_1CA@PHAKLDDM@?$AAP?$AAH?$AAI?$AAL?$AAI?$AAP?$AAS?$AA_?$AAT?$AAD?$AAA?$AA8?$AA2?$AA7?$AA5?$AA?$AA@
CONST	SEGMENT
??_C@_1CA@PHAKLDDM@?$AAP?$AAH?$AAI?$AAL?$AAI?$AAP?$AAS?$AA_?$AAT?$AAD?$AAA?$AA8?$AA2?$AA7?$AA5?$AA?$AA@ DB 'P'
	DB	00H, 'H', 00H, 'I', 00H, 'L', 00H, 'I', 00H, 'P', 00H, 'S', 00H
	DB	'_', 00H, 'T', 00H, 'D', 00H, 'A', 00H, '8', 00H, '2', 00H, '7'
	DB	00H, '5', 00H, 00H, 00H			; `string'
CONST	ENDS
;	COMDAT ??_C@_1CA@NIDJODPE@?$AAY?$AAM?$AAE?$AAC?$AA_?$AAT?$AAV?$AAF?$AA_?$AA8?$AA5?$AA3?$AA1?$AAM?$AAF?$AA?$AA@
CONST	SEGMENT
??_C@_1CA@NIDJODPE@?$AAY?$AAM?$AAE?$AAC?$AA_?$AAT?$AAV?$AAF?$AA_?$AA8?$AA5?$AA3?$AA1?$AAM?$AAF?$AA?$AA@ DB 'Y'
	DB	00H, 'M', 00H, 'E', 00H, 'C', 00H, '_', 00H, 'T', 00H, 'V', 00H
	DB	'F', 00H, '_', 00H, '8', 00H, '5', 00H, '3', 00H, '1', 00H, 'M'
	DB	00H, 'F', 00H, 00H, 00H			; `string'
CONST	ENDS
;	COMDAT ??_C@_1CA@CNOGJENC@?$AAY?$AAM?$AAE?$AAC?$AA_?$AAT?$AAV?$AAF?$AA_?$AA5?$AA5?$AA3?$AA3?$AAM?$AAF?$AA?$AA@
CONST	SEGMENT
??_C@_1CA@CNOGJENC@?$AAY?$AAM?$AAE?$AAC?$AA_?$AAT?$AAV?$AAF?$AA_?$AA5?$AA5?$AA3?$AA3?$AAM?$AAF?$AA?$AA@ DB 'Y'
	DB	00H, 'M', 00H, 'E', 00H, 'C', 00H, '_', 00H, 'T', 00H, 'V', 00H
	DB	'F', 00H, '_', 00H, '5', 00H, '5', 00H, '3', 00H, '3', 00H, 'M'
	DB	00H, 'F', 00H, 00H, 00H			; `string'
CONST	ENDS
;	COMDAT ??_C@_1BK@PEHEKEAO@?$AAT?$AAE?$AAN?$AAA?$AA_?$AA9?$AA5?$AA3?$AA3?$AA_?$AAD?$AAI?$AA?$AA@
CONST	SEGMENT
??_C@_1BK@PEHEKEAO@?$AAT?$AAE?$AAN?$AAA?$AA_?$AA9?$AA5?$AA3?$AA3?$AA_?$AAD?$AAI?$AA?$AA@ DB 'T'
	DB	00H, 'E', 00H, 'N', 00H, 'A', 00H, '_', 00H, '9', 00H, '5', 00H
	DB	'3', 00H, '3', 00H, '_', 00H, 'D', 00H, 'I', 00H, 00H, 00H ; `string'
CONST	ENDS
;	COMDAT ??_C@_1CM@NKAGKMMA@?$AAP?$AAH?$AAI?$AAL?$AAI?$AAP?$AAS?$AA_?$AAF?$AAM?$AAD?$AA1?$AA2?$AA1?$AA6?$AAM?$AAE?$AA_?$AAM?$AAK?$AA3?$AA?$AA@
CONST	SEGMENT
??_C@_1CM@NKAGKMMA@?$AAP?$AAH?$AAI?$AAL?$AAI?$AAP?$AAS?$AA_?$AAF?$AAM?$AAD?$AA1?$AA2?$AA1?$AA6?$AAM?$AAE?$AA_?$AAM?$AAK?$AA3?$AA?$AA@ DB 'P'
	DB	00H, 'H', 00H, 'I', 00H, 'L', 00H, 'I', 00H, 'P', 00H, 'S', 00H
	DB	'_', 00H, 'F', 00H, 'M', 00H, 'D', 00H, '1', 00H, '2', 00H, '1'
	DB	00H, '6', 00H, 'M', 00H, 'E', 00H, '_', 00H, 'M', 00H, 'K', 00H
	DB	'3', 00H, 00H, 00H				; `string'
; Function compile flags: /Odtp
; File c:\develop\dscaler423a\dscaler\parsingcommon.cpp
;	COMDAT ?SetTDA9887ModeMaskAndBits@@YAXAAUTTDA9887Modes@@EH@Z
_TEXT	SEGMENT
_specifics$ = 8						; size = 4
_bit$ = 12						; size = 1
_set$ = 16						; size = 4
?SetTDA9887ModeMaskAndBits@@YAXAAUTTDA9887Modes@@EH@Z PROC ; SetTDA9887ModeMaskAndBits, COMDAT

; 343  : {

  00000	55		 push	 ebp
  00001	8b ec		 mov	 ebp, esp

; 344  :     specifics.mask |= bit;

  00003	0f b6 45 0c	 movzx	 eax, BYTE PTR _bit$[ebp]
  00007	8b 4d 08	 mov	 ecx, DWORD PTR _specifics$[ebp]
  0000a	0f b6 11	 movzx	 edx, BYTE PTR [ecx]
  0000d	0b d0		 or	 edx, eax
  0000f	8b 45 08	 mov	 eax, DWORD PTR _specifics$[ebp]
  00012	88 10		 mov	 BYTE PTR [eax], dl

; 345  :     if (set)

  00014	83 7d 10 00	 cmp	 DWORD PTR _set$[ebp], 0
  00018	74 15		 je	 SHORT $LN2@SetTDA9887

; 346  :     {
; 347  :         specifics.bits |= bit;

  0001a	0f b6 4d 0c	 movzx	 ecx, BYTE PTR _bit$[ebp]
  0001e	8b 55 08	 mov	 edx, DWORD PTR _specifics$[ebp]
  00021	0f b6 42 01	 movzx	 eax, BYTE PTR [edx+1]
  00025	0b c1		 or	 eax, ecx
  00027	8b 4d 08	 mov	 ecx, DWORD PTR _specifics$[ebp]
  0002a	88 41 01	 mov	 BYTE PTR [ecx+1], al

; 348  :     }
; 349  :     else

  0002d	eb 15		 jmp	 SHORT $LN3@SetTDA9887
$LN2@SetTDA9887:

; 350  :     {
; 351  :         specifics.bits &= ~bit;

  0002f	0f b6 55 0c	 movzx	 edx, BYTE PTR _bit$[ebp]
  00033	f7 d2		 not	 edx
  00035	8b 45 08	 mov	 eax, DWORD PTR _specifics$[ebp]
  00038	0f b6 48 01	 movzx	 ecx, BYTE PTR [eax+1]
  0003c	23 ca		 and	 ecx, edx
  0003e	8b 55 08	 mov	 edx, DWORD PTR _specifics$[ebp]
  00041	88 4a 01	 mov	 BYTE PTR [edx+1], cl
$LN3@SetTDA9887:

; 352  :     }
; 353  : }

  00044	5d		 pop	 ebp
  00045	c3		 ret	 0
?SetTDA9887ModeMaskAndBits@@YAXAAUTTDA9887Modes@@EH@Z ENDP ; SetTDA9887ModeMaskAndBits
_TEXT	ENDS
PUBLIC	?ReadUseTDA9887Proc@@YAHHPBVCParseTag@HCParser@@EPBVCParseValue@2@PAU_ParseUseTDA9887Info@@@Z ; ReadUseTDA9887Proc
; Function compile flags: /Odtp
;	COMDAT ?ReadUseTDA9887Proc@@YAHHPBVCParseTag@HCParser@@EPBVCParseValue@2@PAU_ParseUseTDA9887Info@@@Z
_TEXT	SEGMENT
$T294754 = -28						; size = 4
$T294753 = -24						; size = 12
_point$141584 = -9					; size = 1
_i$141561 = -8						; size = 4
_i$141556 = -4						; size = 4
_report$ = 8						; size = 4
_tag$ = 12						; size = 4
_type$ = 16						; size = 1
_value$ = 20						; size = 4
_useTDA9887Info$ = 24					; size = 4
?ReadUseTDA9887Proc@@YAHHPBVCParseTag@HCParser@@EPBVCParseValue@2@PAU_ParseUseTDA9887Info@@@Z PROC ; ReadUseTDA9887Proc, COMDAT

; 205  : {

  00000	55		 push	 ebp
  00001	8b ec		 mov	 ebp, esp
  00003	83 ec 1c	 sub	 esp, 28			; 0000001cH

; 206  :     // Use
; 207  :     if (tag == k_parseUseTDA9887 + 0)

  00006	81 7d 0c 00 00
	00 00		 cmp	 DWORD PTR _tag$[ebp], OFFSET ?k_parseUseTDA9887@@3QBVCParseTag@HCParser@@B
  0000d	75 23		 jne	 SHORT $LN39@ReadUseTDA

; 208  :     {
; 209  :         if (report == REPORT_VALUE)

  0000f	83 7d 08 03	 cmp	 DWORD PTR _report$[ebp], 3
  00013	75 18		 jne	 SHORT $LN38@ReadUseTDA

; 210  :         {
; 211  :             useTDA9887Info->useTDA9887 = value->GetNumber() != 0;

  00015	8b 45 14	 mov	 eax, DWORD PTR _value$[ebp]
  00018	8b 10		 mov	 edx, DWORD PTR [eax]
  0001a	8b 4d 14	 mov	 ecx, DWORD PTR _value$[ebp]
  0001d	8b 42 08	 mov	 eax, DWORD PTR [edx+8]
  00020	ff d0		 call	 eax
  00022	f7 d8		 neg	 eax
  00024	1b c0		 sbb	 eax, eax
  00026	f7 d8		 neg	 eax
  00028	8b 4d 18	 mov	 ecx, DWORD PTR _useTDA9887Info$[ebp]
  0002b	89 01		 mov	 DWORD PTR [ecx], eax
$LN38@ReadUseTDA:

; 212  :         }
; 213  :     }

  0002d	e9 08 03 00 00	 jmp	 $LN37@ReadUseTDA
$LN39@ReadUseTDA:

; 214  :     // SetOverride
; 215  :     else if (tag == k_parseUseTDA9887 + 1)

  00032	81 7d 0c 1c 00
	00 00		 cmp	 DWORD PTR _tag$[ebp], OFFSET ?k_parseUseTDA9887@@3QBVCParseTag@HCParser@@B+28
  00039	0f 85 27 01 00
	00		 jne	 $LN36@ReadUseTDA

; 216  :     {
; 217  :         if (report == REPORT_OPEN)

  0003f	83 7d 08 01	 cmp	 DWORD PTR _report$[ebp], 1
  00043	75 1d		 jne	 SHORT $LN35@ReadUseTDA

; 218  :         {
; 219  :             useTDA9887Info->_readingFormat = TDA9887_FORMAT_NONE;

  00045	8b 55 18	 mov	 edx, DWORD PTR _useTDA9887Info$[ebp]
  00048	c7 42 18 ff ff
	ff ff		 mov	 DWORD PTR [edx+24], -1

; 220  :             useTDA9887Info->_readingModes.mask = 0;

  0004f	8b 45 18	 mov	 eax, DWORD PTR _useTDA9887Info$[ebp]
  00052	c6 40 1c 00	 mov	 BYTE PTR [eax+28], 0

; 221  :             useTDA9887Info->_readingModes.bits = 0;

  00056	8b 4d 18	 mov	 ecx, DWORD PTR _useTDA9887Info$[ebp]
  00059	c6 41 1d 00	 mov	 BYTE PTR [ecx+29], 0
  0005d	e9 ff 00 00 00	 jmp	 $LN34@ReadUseTDA
$LN35@ReadUseTDA:

; 222  :         }
; 223  :         else if (report == REPORT_CLOSE)

  00062	83 7d 08 02	 cmp	 DWORD PTR _report$[ebp], 2
  00066	0f 85 f5 00 00
	00		 jne	 $LN34@ReadUseTDA

; 224  :         {
; 225  :             // This should not fail because constants only provide 0 .. TDA9887_LASTFORMAT.
; 226  :             _ASSERTE(useTDA9887Info->_readingFormat == TDA9887_FORMAT_NONE ||
; 227  :                 (useTDA9887Info->_readingFormat >= 0 &&
; 228  :                 useTDA9887Info->_readingFormat < TDA9887_FORMAT_LASTONE));
; 229  : 
; 230  :             // It is pointless copying if mask is zero.
; 231  :             if (useTDA9887Info->_readingModes.mask != 0)

  0006c	8b 55 18	 mov	 edx, DWORD PTR _useTDA9887Info$[ebp]
  0006f	0f b6 42 1c	 movzx	 eax, BYTE PTR [edx+28]
  00073	85 c0		 test	 eax, eax
  00075	0f 84 e6 00 00
	00		 je	 $LN34@ReadUseTDA

; 232  :             {
; 233  :                 if (useTDA9887Info->_readingFormat == TDA9887_FORMAT_NONE)

  0007b	8b 4d 18	 mov	 ecx, DWORD PTR _useTDA9887Info$[ebp]
  0007e	83 79 18 ff	 cmp	 DWORD PTR [ecx+24], -1
  00082	75 78		 jne	 SHORT $LN31@ReadUseTDA

; 234  :                 {
; 235  :                     // Copy for all formats.
; 236  :                     for (int i = 0; i < TDA9887_FORMAT_LASTONE; i++)

  00084	c7 45 fc 00 00
	00 00		 mov	 DWORD PTR _i$141556[ebp], 0
  0008b	eb 09		 jmp	 SHORT $LN30@ReadUseTDA
$LN29@ReadUseTDA:
  0008d	8b 55 fc	 mov	 edx, DWORD PTR _i$141556[ebp]
  00090	83 c2 01	 add	 edx, 1
  00093	89 55 fc	 mov	 DWORD PTR _i$141556[ebp], edx
$LN30@ReadUseTDA:
  00096	83 7d fc 09	 cmp	 DWORD PTR _i$141556[ebp], 9
  0009a	7d 5e		 jge	 SHORT $LN28@ReadUseTDA

; 237  :                     {
; 238  :                         useTDA9887Info->tdaModes[i].bits &= ~useTDA9887Info->_readingModes.mask;

  0009c	8b 45 18	 mov	 eax, DWORD PTR _useTDA9887Info$[ebp]
  0009f	0f b6 48 1c	 movzx	 ecx, BYTE PTR [eax+28]
  000a3	f7 d1		 not	 ecx
  000a5	8b 55 fc	 mov	 edx, DWORD PTR _i$141556[ebp]
  000a8	8b 45 18	 mov	 eax, DWORD PTR _useTDA9887Info$[ebp]
  000ab	0f b6 54 50 05	 movzx	 edx, BYTE PTR [eax+edx*2+5]
  000b0	23 d1		 and	 edx, ecx
  000b2	8b 45 fc	 mov	 eax, DWORD PTR _i$141556[ebp]
  000b5	8b 4d 18	 mov	 ecx, DWORD PTR _useTDA9887Info$[ebp]
  000b8	88 54 41 05	 mov	 BYTE PTR [ecx+eax*2+5], dl

; 239  :                         useTDA9887Info->tdaModes[i].bits |= useTDA9887Info->_readingModes.bits;

  000bc	8b 55 18	 mov	 edx, DWORD PTR _useTDA9887Info$[ebp]
  000bf	0f b6 42 1d	 movzx	 eax, BYTE PTR [edx+29]
  000c3	8b 4d fc	 mov	 ecx, DWORD PTR _i$141556[ebp]
  000c6	8b 55 18	 mov	 edx, DWORD PTR _useTDA9887Info$[ebp]
  000c9	0f b6 4c 4a 05	 movzx	 ecx, BYTE PTR [edx+ecx*2+5]
  000ce	0b c8		 or	 ecx, eax
  000d0	8b 55 fc	 mov	 edx, DWORD PTR _i$141556[ebp]
  000d3	8b 45 18	 mov	 eax, DWORD PTR _useTDA9887Info$[ebp]
  000d6	88 4c 50 05	 mov	 BYTE PTR [eax+edx*2+5], cl

; 240  :                         useTDA9887Info->tdaModes[i].mask |= useTDA9887Info->_readingModes.mask;

  000da	8b 4d 18	 mov	 ecx, DWORD PTR _useTDA9887Info$[ebp]
  000dd	0f b6 51 1c	 movzx	 edx, BYTE PTR [ecx+28]
  000e1	8b 45 fc	 mov	 eax, DWORD PTR _i$141556[ebp]
  000e4	8b 4d 18	 mov	 ecx, DWORD PTR _useTDA9887Info$[ebp]
  000e7	0f b6 44 41 04	 movzx	 eax, BYTE PTR [ecx+eax*2+4]
  000ec	0b c2		 or	 eax, edx
  000ee	8b 4d fc	 mov	 ecx, DWORD PTR _i$141556[ebp]
  000f1	8b 55 18	 mov	 edx, DWORD PTR _useTDA9887Info$[ebp]
  000f4	88 44 4a 04	 mov	 BYTE PTR [edx+ecx*2+4], al

; 241  :                     }

  000f8	eb 93		 jmp	 SHORT $LN29@ReadUseTDA
$LN28@ReadUseTDA:

; 242  :                 }
; 243  :                 else

  000fa	eb 65		 jmp	 SHORT $LN34@ReadUseTDA
$LN31@ReadUseTDA:

; 244  :                 {
; 245  :                     int i = useTDA9887Info->_readingFormat;

  000fc	8b 45 18	 mov	 eax, DWORD PTR _useTDA9887Info$[ebp]
  000ff	8b 48 18	 mov	 ecx, DWORD PTR [eax+24]
  00102	89 4d f8	 mov	 DWORD PTR _i$141561[ebp], ecx

; 246  :                     useTDA9887Info->tdaModes[i].bits &= ~useTDA9887Info->_readingModes.mask;

  00105	8b 55 18	 mov	 edx, DWORD PTR _useTDA9887Info$[ebp]
  00108	0f b6 42 1c	 movzx	 eax, BYTE PTR [edx+28]
  0010c	f7 d0		 not	 eax
  0010e	8b 4d f8	 mov	 ecx, DWORD PTR _i$141561[ebp]
  00111	8b 55 18	 mov	 edx, DWORD PTR _useTDA9887Info$[ebp]
  00114	0f b6 4c 4a 05	 movzx	 ecx, BYTE PTR [edx+ecx*2+5]
  00119	23 c8		 and	 ecx, eax
  0011b	8b 55 f8	 mov	 edx, DWORD PTR _i$141561[ebp]
  0011e	8b 45 18	 mov	 eax, DWORD PTR _useTDA9887Info$[ebp]
  00121	88 4c 50 05	 mov	 BYTE PTR [eax+edx*2+5], cl

; 247  :                     useTDA9887Info->tdaModes[i].bits |= useTDA9887Info->_readingModes.bits;

  00125	8b 4d 18	 mov	 ecx, DWORD PTR _useTDA9887Info$[ebp]
  00128	0f b6 51 1d	 movzx	 edx, BYTE PTR [ecx+29]
  0012c	8b 45 f8	 mov	 eax, DWORD PTR _i$141561[ebp]
  0012f	8b 4d 18	 mov	 ecx, DWORD PTR _useTDA9887Info$[ebp]
  00132	0f b6 44 41 05	 movzx	 eax, BYTE PTR [ecx+eax*2+5]
  00137	0b c2		 or	 eax, edx
  00139	8b 4d f8	 mov	 ecx, DWORD PTR _i$141561[ebp]
  0013c	8b 55 18	 mov	 edx, DWORD PTR _useTDA9887Info$[ebp]
  0013f	88 44 4a 05	 mov	 BYTE PTR [edx+ecx*2+5], al

; 248  :                     useTDA9887Info->tdaModes[i].mask |= useTDA9887Info->_readingModes.mask;

  00143	8b 45 18	 mov	 eax, DWORD PTR _useTDA9887Info$[ebp]
  00146	0f b6 48 1c	 movzx	 ecx, BYTE PTR [eax+28]
  0014a	8b 55 f8	 mov	 edx, DWORD PTR _i$141561[ebp]
  0014d	8b 45 18	 mov	 eax, DWORD PTR _useTDA9887Info$[ebp]
  00150	0f b6 54 50 04	 movzx	 edx, BYTE PTR [eax+edx*2+4]
  00155	0b d1		 or	 edx, ecx
  00157	8b 45 f8	 mov	 eax, DWORD PTR _i$141561[ebp]
  0015a	8b 4d 18	 mov	 ecx, DWORD PTR _useTDA9887Info$[ebp]
  0015d	88 54 41 04	 mov	 BYTE PTR [ecx+eax*2+4], dl
$LN34@ReadUseTDA:

; 249  :                 }
; 250  :             }
; 251  :         }
; 252  :     }

  00161	e9 d4 01 00 00	 jmp	 $LN37@ReadUseTDA
$LN36@ReadUseTDA:

; 253  :     // Format
; 254  :     else if (tag == k_parseUseTDA9887SetOverride + 0)

  00166	81 7d 0c 00 00
	00 00		 cmp	 DWORD PTR _tag$[ebp], OFFSET _k_parseUseTDA9887SetOverride
  0016d	75 1e		 jne	 SHORT $LN25@ReadUseTDA

; 255  :     {
; 256  :         if (report == REPORT_VALUE)

  0016f	83 7d 08 03	 cmp	 DWORD PTR _report$[ebp], 3
  00173	75 13		 jne	 SHORT $LN24@ReadUseTDA

; 257  :         {
; 258  :             useTDA9887Info->_readingFormat = static_cast<eTDA9887Format>(value->GetNumber());

  00175	8b 55 14	 mov	 edx, DWORD PTR _value$[ebp]
  00178	8b 02		 mov	 eax, DWORD PTR [edx]
  0017a	8b 4d 14	 mov	 ecx, DWORD PTR _value$[ebp]
  0017d	8b 50 08	 mov	 edx, DWORD PTR [eax+8]
  00180	ff d2		 call	 edx
  00182	8b 4d 18	 mov	 ecx, DWORD PTR _useTDA9887Info$[ebp]
  00185	89 41 18	 mov	 DWORD PTR [ecx+24], eax
$LN24@ReadUseTDA:

; 259  :         }
; 260  :     }

  00188	e9 ad 01 00 00	 jmp	 $LN37@ReadUseTDA
$LN25@ReadUseTDA:

; 261  :     // Intercarrier
; 262  :     else if (tag == k_parseUseTDA9887SetOverride + 1)

  0018d	81 7d 0c 1c 00
	00 00		 cmp	 DWORD PTR _tag$[ebp], OFFSET _k_parseUseTDA9887SetOverride+28
  00194	75 1e		 jne	 SHORT $LN22@ReadUseTDA

; 263  :     {
; 264  :         if (report == REPORT_TAG)

  00196	83 7d 08 00	 cmp	 DWORD PTR _report$[ebp], 0
  0019a	75 13		 jne	 SHORT $LN21@ReadUseTDA

; 265  :         {
; 266  :             SetTDA9887ModeMaskAndBits(useTDA9887Info->_readingModes,
; 267  :                 TDA9887_SM_CARRIER_QSS, FALSE);

  0019c	6a 00		 push	 0
  0019e	6a 20		 push	 32			; 00000020H
  001a0	8b 55 18	 mov	 edx, DWORD PTR _useTDA9887Info$[ebp]
  001a3	83 c2 1c	 add	 edx, 28			; 0000001cH
  001a6	52		 push	 edx
  001a7	e8 00 00 00 00	 call	 ?SetTDA9887ModeMaskAndBits@@YAXAAUTTDA9887Modes@@EH@Z ; SetTDA9887ModeMaskAndBits
  001ac	83 c4 0c	 add	 esp, 12			; 0000000cH
$LN21@ReadUseTDA:

; 268  :         }
; 269  :     }

  001af	e9 86 01 00 00	 jmp	 $LN37@ReadUseTDA
$LN22@ReadUseTDA:

; 270  :     // QSS
; 271  :     else if (tag == k_parseUseTDA9887SetOverride + 2)

  001b4	81 7d 0c 38 00
	00 00		 cmp	 DWORD PTR _tag$[ebp], OFFSET _k_parseUseTDA9887SetOverride+56
  001bb	75 1e		 jne	 SHORT $LN19@ReadUseTDA

; 272  :     {
; 273  :         if (report == REPORT_TAG)

  001bd	83 7d 08 00	 cmp	 DWORD PTR _report$[ebp], 0
  001c1	75 13		 jne	 SHORT $LN18@ReadUseTDA

; 274  :         {
; 275  :             SetTDA9887ModeMaskAndBits(useTDA9887Info->_readingModes,
; 276  :                 TDA9887_SM_CARRIER_QSS, TRUE);

  001c3	6a 01		 push	 1
  001c5	6a 20		 push	 32			; 00000020H
  001c7	8b 45 18	 mov	 eax, DWORD PTR _useTDA9887Info$[ebp]
  001ca	83 c0 1c	 add	 eax, 28			; 0000001cH
  001cd	50		 push	 eax
  001ce	e8 00 00 00 00	 call	 ?SetTDA9887ModeMaskAndBits@@YAXAAUTTDA9887Modes@@EH@Z ; SetTDA9887ModeMaskAndBits
  001d3	83 c4 0c	 add	 esp, 12			; 0000000cH
$LN18@ReadUseTDA:

; 277  :         }
; 278  :     }

  001d6	e9 5f 01 00 00	 jmp	 $LN37@ReadUseTDA
$LN19@ReadUseTDA:

; 279  :     // Carrier
; 280  :     else if (tag == k_parseUseTDA9887SetOverride + 3)

  001db	81 7d 0c 54 00
	00 00		 cmp	 DWORD PTR _tag$[ebp], OFFSET _k_parseUseTDA9887SetOverride+84
  001e2	75 30		 jne	 SHORT $LN16@ReadUseTDA

; 281  :     {
; 282  :         if (report == REPORT_VALUE)

  001e4	83 7d 08 03	 cmp	 DWORD PTR _report$[ebp], 3
  001e8	75 25		 jne	 SHORT $LN15@ReadUseTDA

; 283  :         {
; 284  :             SetTDA9887ModeMaskAndBits(useTDA9887Info->_readingModes,
; 285  :                 TDA9887_SM_CARRIER_QSS, value->GetNumber() != 0);

  001ea	8b 4d 14	 mov	 ecx, DWORD PTR _value$[ebp]
  001ed	8b 11		 mov	 edx, DWORD PTR [ecx]
  001ef	8b 4d 14	 mov	 ecx, DWORD PTR _value$[ebp]
  001f2	8b 42 08	 mov	 eax, DWORD PTR [edx+8]
  001f5	ff d0		 call	 eax
  001f7	f7 d8		 neg	 eax
  001f9	1b c0		 sbb	 eax, eax
  001fb	f7 d8		 neg	 eax
  001fd	50		 push	 eax
  001fe	6a 20		 push	 32			; 00000020H
  00200	8b 4d 18	 mov	 ecx, DWORD PTR _useTDA9887Info$[ebp]
  00203	83 c1 1c	 add	 ecx, 28			; 0000001cH
  00206	51		 push	 ecx
  00207	e8 00 00 00 00	 call	 ?SetTDA9887ModeMaskAndBits@@YAXAAUTTDA9887Modes@@EH@Z ; SetTDA9887ModeMaskAndBits
  0020c	83 c4 0c	 add	 esp, 12			; 0000000cH
$LN15@ReadUseTDA:

; 286  :         }
; 287  :     }

  0020f	e9 26 01 00 00	 jmp	 $LN37@ReadUseTDA
$LN16@ReadUseTDA:

; 288  :     // OutputPort1
; 289  :     else if (tag == k_parseUseTDA9887SetOverride + 4)

  00214	81 7d 0c 70 00
	00 00		 cmp	 DWORD PTR _tag$[ebp], OFFSET _k_parseUseTDA9887SetOverride+112
  0021b	75 31		 jne	 SHORT $LN13@ReadUseTDA

; 290  :     {
; 291  :         if (report == REPORT_VALUE)

  0021d	83 7d 08 03	 cmp	 DWORD PTR _report$[ebp], 3
  00221	75 26		 jne	 SHORT $LN12@ReadUseTDA

; 292  :         {
; 293  :             SetTDA9887ModeMaskAndBits(useTDA9887Info->_readingModes,
; 294  :                 TDA9887_SM_OUTPUTPORT1_INACTIVE, value->GetNumber() == 0);

  00223	8b 55 14	 mov	 edx, DWORD PTR _value$[ebp]
  00226	8b 02		 mov	 eax, DWORD PTR [edx]
  00228	8b 4d 14	 mov	 ecx, DWORD PTR _value$[ebp]
  0022b	8b 50 08	 mov	 edx, DWORD PTR [eax+8]
  0022e	ff d2		 call	 edx
  00230	f7 d8		 neg	 eax
  00232	1b c0		 sbb	 eax, eax
  00234	83 c0 01	 add	 eax, 1
  00237	50		 push	 eax
  00238	6a 40		 push	 64			; 00000040H
  0023a	8b 45 18	 mov	 eax, DWORD PTR _useTDA9887Info$[ebp]
  0023d	83 c0 1c	 add	 eax, 28			; 0000001cH
  00240	50		 push	 eax
  00241	e8 00 00 00 00	 call	 ?SetTDA9887ModeMaskAndBits@@YAXAAUTTDA9887Modes@@EH@Z ; SetTDA9887ModeMaskAndBits
  00246	83 c4 0c	 add	 esp, 12			; 0000000cH
$LN12@ReadUseTDA:

; 295  :         }
; 296  :     }

  00249	e9 ec 00 00 00	 jmp	 $LN37@ReadUseTDA
$LN13@ReadUseTDA:

; 297  :     // OutputPort2
; 298  :     else if (tag == k_parseUseTDA9887SetOverride + 5)

  0024e	81 7d 0c 8c 00
	00 00		 cmp	 DWORD PTR _tag$[ebp], OFFSET _k_parseUseTDA9887SetOverride+140
  00255	75 34		 jne	 SHORT $LN10@ReadUseTDA

; 299  :     {
; 300  :         if (report == REPORT_VALUE)

  00257	83 7d 08 03	 cmp	 DWORD PTR _report$[ebp], 3
  0025b	75 29		 jne	 SHORT $LN9@ReadUseTDA

; 301  :         {
; 302  :             SetTDA9887ModeMaskAndBits(useTDA9887Info->_readingModes,
; 303  :                 TDA9887_SM_OUTPUTPORT2_INACTIVE, value->GetNumber() == 0);

  0025d	8b 4d 14	 mov	 ecx, DWORD PTR _value$[ebp]
  00260	8b 11		 mov	 edx, DWORD PTR [ecx]
  00262	8b 4d 14	 mov	 ecx, DWORD PTR _value$[ebp]
  00265	8b 42 08	 mov	 eax, DWORD PTR [edx+8]
  00268	ff d0		 call	 eax
  0026a	f7 d8		 neg	 eax
  0026c	1b c0		 sbb	 eax, eax
  0026e	83 c0 01	 add	 eax, 1
  00271	50		 push	 eax
  00272	68 80 00 00 00	 push	 128			; 00000080H
  00277	8b 4d 18	 mov	 ecx, DWORD PTR _useTDA9887Info$[ebp]
  0027a	83 c1 1c	 add	 ecx, 28			; 0000001cH
  0027d	51		 push	 ecx
  0027e	e8 00 00 00 00	 call	 ?SetTDA9887ModeMaskAndBits@@YAXAAUTTDA9887Modes@@EH@Z ; SetTDA9887ModeMaskAndBits
  00283	83 c4 0c	 add	 esp, 12			; 0000000cH
$LN9@ReadUseTDA:

; 304  :         }
; 305  :     }

  00286	e9 af 00 00 00	 jmp	 $LN37@ReadUseTDA
$LN10@ReadUseTDA:

; 306  :     // TakeOverPoint
; 307  :     else if (tag == k_parseUseTDA9887SetOverride + 6)

  0028b	81 7d 0c a8 00
	00 00		 cmp	 DWORD PTR _tag$[ebp], OFFSET _k_parseUseTDA9887SetOverride+168
  00292	75 75		 jne	 SHORT $LN7@ReadUseTDA

; 308  :     {
; 309  :         if (report == REPORT_VALUE)

  00294	83 7d 08 03	 cmp	 DWORD PTR _report$[ebp], 3
  00298	75 6d		 jne	 SHORT $LN6@ReadUseTDA

; 310  :         {
; 311  :             BYTE point = static_cast<BYTE>(value->GetNumber());

  0029a	8b 55 14	 mov	 edx, DWORD PTR _value$[ebp]
  0029d	8b 02		 mov	 eax, DWORD PTR [edx]
  0029f	8b 4d 14	 mov	 ecx, DWORD PTR _value$[ebp]
  002a2	8b 50 08	 mov	 edx, DWORD PTR [eax+8]
  002a5	ff d2		 call	 edx
  002a7	88 45 f7	 mov	 BYTE PTR _point$141584[ebp], al

; 312  :             if (point & ~TDA9887_SM_TAKEOVERPOINT_MASK)

  002aa	0f b6 45 f7	 movzx	 eax, BYTE PTR _point$141584[ebp]
  002ae	83 e0 e0	 and	 eax, -32		; ffffffe0H
  002b1	74 21		 je	 SHORT $LN5@ReadUseTDA

; 313  :             {
; 314  :                 throw std::exception("Invalid value of TakeOverPoint");

  002b3	c7 45 e4 00 00
	00 00		 mov	 DWORD PTR $T294754[ebp], OFFSET ??_C@_0BP@JMNHPJIF@Invalid?5value?5of?5TakeOverPoint?$AA@
  002ba	8d 4d e4	 lea	 ecx, DWORD PTR $T294754[ebp]
  002bd	51		 push	 ecx
  002be	8d 4d e8	 lea	 ecx, DWORD PTR $T294753[ebp]
  002c1	e8 00 00 00 00	 call	 ??0exception@std@@QAE@ABQBD@Z ; std::exception::exception
  002c6	68 00 00 00 00	 push	 OFFSET __TI1?AVexception@std@@
  002cb	8d 55 e8	 lea	 edx, DWORD PTR $T294753[ebp]
  002ce	52		 push	 edx
  002cf	e8 00 00 00 00	 call	 __CxxThrowException@8
$LN5@ReadUseTDA:

; 315  :             }
; 316  : 
; 317  :             useTDA9887Info->_readingModes.mask |= TDA9887_SM_TAKEOVERPOINT_MASK;

  002d4	8b 45 18	 mov	 eax, DWORD PTR _useTDA9887Info$[ebp]
  002d7	0f b6 48 1c	 movzx	 ecx, BYTE PTR [eax+28]
  002db	83 c9 1f	 or	 ecx, 31			; 0000001fH
  002de	8b 55 18	 mov	 edx, DWORD PTR _useTDA9887Info$[ebp]
  002e1	88 4a 1c	 mov	 BYTE PTR [edx+28], cl

; 318  :             useTDA9887Info->_readingModes.bits &= ~TDA9887_SM_TAKEOVERPOINT_MASK;

  002e4	8b 45 18	 mov	 eax, DWORD PTR _useTDA9887Info$[ebp]
  002e7	0f b6 48 1d	 movzx	 ecx, BYTE PTR [eax+29]
  002eb	83 e1 e0	 and	 ecx, -32		; ffffffe0H
  002ee	8b 55 18	 mov	 edx, DWORD PTR _useTDA9887Info$[ebp]
  002f1	88 4a 1d	 mov	 BYTE PTR [edx+29], cl

; 319  :             useTDA9887Info->_readingModes.bits |= (point << TDA9887_SM_TAKEOVERPOINT_OFFSET);

  002f4	0f b6 45 f7	 movzx	 eax, BYTE PTR _point$141584[ebp]
  002f8	8b 4d 18	 mov	 ecx, DWORD PTR _useTDA9887Info$[ebp]
  002fb	0f b6 51 1d	 movzx	 edx, BYTE PTR [ecx+29]
  002ff	0b d0		 or	 edx, eax
  00301	8b 45 18	 mov	 eax, DWORD PTR _useTDA9887Info$[ebp]
  00304	88 50 1d	 mov	 BYTE PTR [eax+29], dl
$LN6@ReadUseTDA:

; 320  :         }
; 321  :     }
; 322  :     // This unknown tag is hopefully the parent tag.  There's no other way of
; 323  :     // checking.  An incorrect tag here can only result from incorrect setup
; 324  :     // outside ParsingCommon's control.
; 325  :     else

  00307	eb 31		 jmp	 SHORT $LN37@ReadUseTDA
$LN7@ReadUseTDA:

; 326  :     {
; 327  :         if (report == REPORT_OPEN)

  00309	83 7d 08 01	 cmp	 DWORD PTR _report$[ebp], 1
  0030d	75 1e		 jne	 SHORT $LN3@ReadUseTDA

; 328  :         {
; 329  :             useTDA9887Info->useTDA9887 = TRUE;

  0030f	8b 4d 18	 mov	 ecx, DWORD PTR _useTDA9887Info$[ebp]
  00312	c7 01 01 00 00
	00		 mov	 DWORD PTR [ecx], 1

; 330  :             ZeroMemory(useTDA9887Info->tdaModes, sizeof(useTDA9887Info->tdaModes));

  00318	6a 12		 push	 18			; 00000012H
  0031a	6a 00		 push	 0
  0031c	8b 55 18	 mov	 edx, DWORD PTR _useTDA9887Info$[ebp]
  0031f	83 c2 04	 add	 edx, 4
  00322	52		 push	 edx
  00323	e8 00 00 00 00	 call	 _memset
  00328	83 c4 0c	 add	 esp, 12			; 0000000cH
  0032b	eb 0d		 jmp	 SHORT $LN37@ReadUseTDA
$LN3@ReadUseTDA:

; 331  :         }
; 332  :         else if (report == REPORT_CLOSE)

  0032d	83 7d 08 02	 cmp	 DWORD PTR _report$[ebp], 2
  00331	75 07		 jne	 SHORT $LN37@ReadUseTDA

; 333  :         {
; 334  :             // Everything about the UseTDA9887 tag is considered read and
; 335  :             // ParseUseTDA9887Info considered fill at this point.
; 336  :             return TRUE;

  00333	b8 01 00 00 00	 mov	 eax, 1
  00338	eb 02		 jmp	 SHORT $LN41@ReadUseTDA
$LN37@ReadUseTDA:

; 337  :         }
; 338  :     }
; 339  :     return FALSE;

  0033a	33 c0		 xor	 eax, eax
$LN41@ReadUseTDA:

; 340  : }

  0033c	8b e5		 mov	 esp, ebp
  0033e	5d		 pop	 ebp
  0033f	c3		 ret	 0
?ReadUseTDA9887Proc@@YAHHPBVCParseTag@HCParser@@EPBVCParseValue@2@PAU_ParseUseTDA9887Info@@@Z ENDP ; ReadUseTDA9887Proc
_TEXT	ENDS
PUBLIC	?ReadTunerProc@@YAHHPBVCParseTag@HCParser@@EPBVCParseValue@2@PAU_ParseTunerInfo@@@Z ; ReadTunerProc
; Function compile flags: /Odtp
;	COMDAT ?ReadTunerProc@@YAHHPBVCParseTag@HCParser@@EPBVCParseValue@2@PAU_ParseTunerInfo@@@Z
_TEXT	SEGMENT
$T294758 = -20						; size = 4
$T294757 = -16						; size = 12
_n$141527 = -4						; size = 4
_report$ = 8						; size = 4
_tag$ = 12						; size = 4
_type$ = 16						; size = 1
_value$ = 20						; size = 4
_tunerInfo$ = 24					; size = 4
?ReadTunerProc@@YAHHPBVCParseTag@HCParser@@EPBVCParseValue@2@PAU_ParseTunerInfo@@@Z PROC ; ReadTunerProc, COMDAT

; 178  : {

  00000	55		 push	 ebp
  00001	8b ec		 mov	 ebp, esp
  00003	83 ec 14	 sub	 esp, 20			; 00000014H

; 179  :     if (report == REPORT_OPEN)

  00006	83 7d 08 01	 cmp	 DWORD PTR _report$[ebp], 1
  0000a	75 0b		 jne	 SHORT $LN7@ReadTunerP

; 180  :     {
; 181  :         // Set the default tuner id for if there is no value.
; 182  :         tunerInfo->tunerId = TUNER_ABSENT;

  0000c	8b 45 18	 mov	 eax, DWORD PTR _tunerInfo$[ebp]
  0000f	c7 00 00 00 00
	00		 mov	 DWORD PTR [eax], 0
  00015	eb 5a		 jmp	 SHORT $LN6@ReadTunerP
$LN7@ReadTunerP:

; 183  :     }
; 184  :     else if (report == REPORT_VALUE)

  00017	83 7d 08 03	 cmp	 DWORD PTR _report$[ebp], 3
  0001b	75 47		 jne	 SHORT $LN5@ReadTunerP

; 185  :     {
; 186  :         int n = value->GetNumber();

  0001d	8b 4d 14	 mov	 ecx, DWORD PTR _value$[ebp]
  00020	8b 11		 mov	 edx, DWORD PTR [ecx]
  00022	8b 4d 14	 mov	 ecx, DWORD PTR _value$[ebp]
  00025	8b 42 08	 mov	 eax, DWORD PTR [edx+8]
  00028	ff d0		 call	 eax
  0002a	89 45 fc	 mov	 DWORD PTR _n$141527[ebp], eax

; 187  :         if (n < TUNER_AUTODETECT || n >= TUNER_LASTONE)

  0002d	83 7d fc fe	 cmp	 DWORD PTR _n$141527[ebp], -2 ; fffffffeH
  00031	7c 06		 jl	 SHORT $LN3@ReadTunerP
  00033	83 7d fc 40	 cmp	 DWORD PTR _n$141527[ebp], 64 ; 00000040H
  00037	7c 21		 jl	 SHORT $LN4@ReadTunerP
$LN3@ReadTunerP:

; 188  :         {
; 189  :             throw std::exception("Invalid tuner Id");

  00039	c7 45 ec 00 00
	00 00		 mov	 DWORD PTR $T294758[ebp], OFFSET ??_C@_0BB@DPAAIHBB@Invalid?5tuner?5Id?$AA@
  00040	8d 4d ec	 lea	 ecx, DWORD PTR $T294758[ebp]
  00043	51		 push	 ecx
  00044	8d 4d f0	 lea	 ecx, DWORD PTR $T294757[ebp]
  00047	e8 00 00 00 00	 call	 ??0exception@std@@QAE@ABQBD@Z ; std::exception::exception
  0004c	68 00 00 00 00	 push	 OFFSET __TI1?AVexception@std@@
  00051	8d 55 f0	 lea	 edx, DWORD PTR $T294757[ebp]
  00054	52		 push	 edx
  00055	e8 00 00 00 00	 call	 __CxxThrowException@8
$LN4@ReadTunerP:

; 190  :         }
; 191  :         tunerInfo->tunerId = static_cast<eTunerId>(n);

  0005a	8b 45 18	 mov	 eax, DWORD PTR _tunerInfo$[ebp]
  0005d	8b 4d fc	 mov	 ecx, DWORD PTR _n$141527[ebp]
  00060	89 08		 mov	 DWORD PTR [eax], ecx
  00062	eb 0d		 jmp	 SHORT $LN6@ReadTunerP
$LN5@ReadTunerP:

; 192  :     }
; 193  :     else if (report == REPORT_CLOSE)

  00064	83 7d 08 02	 cmp	 DWORD PTR _report$[ebp], 2
  00068	75 07		 jne	 SHORT $LN6@ReadTunerP

; 194  :     {
; 195  :         // The value could be considered read at the end of REPORT_VALUE
; 196  :         // but putting the 'return TRUE' here is also good.
; 197  :         return TRUE;

  0006a	b8 01 00 00 00	 mov	 eax, 1
  0006f	eb 02		 jmp	 SHORT $LN9@ReadTunerP
$LN6@ReadTunerP:

; 198  :     }
; 199  :     return FALSE;

  00071	33 c0		 xor	 eax, eax
$LN9@ReadTunerP:

; 200  : }

  00073	8b e5		 mov	 esp, ebp
  00075	5d		 pop	 ebp
  00076	c3		 ret	 0
?ReadTunerProc@@YAHHPBVCParseTag@HCParser@@EPBVCParseValue@2@PAU_ParseTunerInfo@@@Z ENDP ; ReadTunerProc
;	COMDAT xdata$x
xdata$x	SEGMENT
__unwindtable$??__Ek_parseTunerConstants@@YAXXZ DD 0ffffffffH
	DD	FLAT:__unwindfunclet$??__Ek_parseTunerConstants@@YAXXZ$0
	DD	0ffffffffH
	DD	FLAT:__unwindfunclet$??__Ek_parseTunerConstants@@YAXXZ$1
	DD	01H
	DD	FLAT:__unwindfunclet$??__Ek_parseTunerConstants@@YAXXZ$2
	DD	0ffffffffH
	DD	FLAT:__unwindfunclet$??__Ek_parseTunerConstants@@YAXXZ$2
	DD	03H
	DD	FLAT:__unwindfunclet$??__Ek_parseTunerConstants@@YAXXZ$3
	DD	03H
	DD	FLAT:__unwindfunclet$??__Ek_parseTunerConstants@@YAXXZ$4
	DD	05H
	DD	FLAT:__unwindfunclet$??__Ek_parseTunerConstants@@YAXXZ$5
	DD	03H
	DD	FLAT:__unwindfunclet$??__Ek_parseTunerConstants@@YAXXZ$5
	DD	07H
	DD	FLAT:__unwindfunclet$??__Ek_parseTunerConstants@@YAXXZ$6
	DD	07H
	DD	FLAT:__unwindfunclet$??__Ek_parseTunerConstants@@YAXXZ$7
	DD	09H
	DD	FLAT:__unwindfunclet$??__Ek_parseTunerConstants@@YAXXZ$8
	DD	07H
	DD	FLAT:__unwindfunclet$??__Ek_parseTunerConstants@@YAXXZ$8
	DD	0bH
	DD	FLAT:__unwindfunclet$??__Ek_parseTunerConstants@@YAXXZ$9
	DD	0bH
	DD	FLAT:__unwindfunclet$??__Ek_parseTunerConstants@@YAXXZ$10
	DD	0dH
	DD	FLAT:__unwindfunclet$??__Ek_parseTunerConstants@@YAXXZ$11
	DD	0bH
	DD	FLAT:__unwindfunclet$??__Ek_parseTunerConstants@@YAXXZ$11
	DD	0fH
	DD	FLAT:__unwindfunclet$??__Ek_parseTunerConstants@@YAXXZ$12
	DD	0fH
	DD	FLAT:__unwindfunclet$??__Ek_parseTunerConstants@@YAXXZ$13
	DD	011H
	DD	FLAT:__unwindfunclet$??__Ek_parseTunerConstants@@YAXXZ$14
	DD	0fH
	DD	FLAT:__unwindfunclet$??__Ek_parseTunerConstants@@YAXXZ$14
	DD	013H
	DD	FLAT:__unwindfunclet$??__Ek_parseTunerConstants@@YAXXZ$15
	DD	013H
	DD	FLAT:__unwindfunclet$??__Ek_parseTunerConstants@@YAXXZ$16
	DD	015H
	DD	FLAT:__unwindfunclet$??__Ek_parseTunerConstants@@YAXXZ$17
	DD	013H
	DD	FLAT:__unwindfunclet$??__Ek_parseTunerConstants@@YAXXZ$17
	DD	017H
	DD	FLAT:__unwindfunclet$??__Ek_parseTunerConstants@@YAXXZ$18
	DD	017H
	DD	FLAT:__unwindfunclet$??__Ek_parseTunerConstants@@YAXXZ$19
	DD	019H
	DD	FLAT:__unwindfunclet$??__Ek_parseTunerConstants@@YAXXZ$20
	DD	017H
	DD	FLAT:__unwindfunclet$??__Ek_parseTunerConstants@@YAXXZ$20
	DD	01bH
	DD	FLAT:__unwindfunclet$??__Ek_parseTunerConstants@@YAXXZ$21
	DD	01bH
	DD	FLAT:__unwindfunclet$??__Ek_parseTunerConstants@@YAXXZ$22
	DD	01dH
	DD	FLAT:__unwindfunclet$??__Ek_parseTunerConstants@@YAXXZ$23
	DD	01bH
	DD	FLAT:__unwindfunclet$??__Ek_parseTunerConstants@@YAXXZ$23
	DD	01fH
	DD	FLAT:__unwindfunclet$??__Ek_parseTunerConstants@@YAXXZ$24
	DD	01fH
	DD	FLAT:__unwindfunclet$??__Ek_parseTunerConstants@@YAXXZ$25
	DD	021H
	DD	FLAT:__unwindfunclet$??__Ek_parseTunerConstants@@YAXXZ$26
	DD	01fH
	DD	FLAT:__unwindfunclet$??__Ek_parseTunerConstants@@YAXXZ$26
	DD	023H
	DD	FLAT:__unwindfunclet$??__Ek_parseTunerConstants@@YAXXZ$27
	DD	023H
	DD	FLAT:__unwindfunclet$??__Ek_parseTunerConstants@@YAXXZ$28
	DD	025H
	DD	FLAT:__unwindfunclet$??__Ek_parseTunerConstants@@YAXXZ$29
	DD	023H
	DD	FLAT:__unwindfunclet$??__Ek_parseTunerConstants@@YAXXZ$29
	DD	027H
	DD	FLAT:__unwindfunclet$??__Ek_parseTunerConstants@@YAXXZ$30
	DD	027H
	DD	FLAT:__unwindfunclet$??__Ek_parseTunerConstants@@YAXXZ$31
	DD	029H
	DD	FLAT:__unwindfunclet$??__Ek_parseTunerConstants@@YAXXZ$32
	DD	027H
	DD	FLAT:__unwindfunclet$??__Ek_parseTunerConstants@@YAXXZ$32
	DD	02bH
	DD	FLAT:__unwindfunclet$??__Ek_parseTunerConstants@@YAXXZ$33
	DD	02bH
	DD	FLAT:__unwindfunclet$??__Ek_parseTunerConstants@@YAXXZ$34
	DD	02dH
	DD	FLAT:__unwindfunclet$??__Ek_parseTunerConstants@@YAXXZ$35
	DD	02bH
	DD	FLAT:__unwindfunclet$??__Ek_parseTunerConstants@@YAXXZ$35
	DD	02fH
	DD	FLAT:__unwindfunclet$??__Ek_parseTunerConstants@@YAXXZ$36
	DD	02fH
	DD	FLAT:__unwindfunclet$??__Ek_parseTunerConstants@@YAXXZ$37
	DD	031H
	DD	FLAT:__unwindfunclet$??__Ek_parseTunerConstants@@YAXXZ$38
	DD	02fH
	DD	FLAT:__unwindfunclet$??__Ek_parseTunerConstants@@YAXXZ$38
	DD	033H
	DD	FLAT:__unwindfunclet$??__Ek_parseTunerConstants@@YAXXZ$39
	DD	033H
	DD	FLAT:__unwindfunclet$??__Ek_parseTunerConstants@@YAXXZ$40
	DD	035H
	DD	FLAT:__unwindfunclet$??__Ek_parseTunerConstants@@YAXXZ$41
	DD	033H
	DD	FLAT:__unwindfunclet$??__Ek_parseTunerConstants@@YAXXZ$41
	DD	037H
	DD	FLAT:__unwindfunclet$??__Ek_parseTunerConstants@@YAXXZ$42
	DD	037H
	DD	FLAT:__unwindfunclet$??__Ek_parseTunerConstants@@YAXXZ$43
	DD	039H
	DD	FLAT:__unwindfunclet$??__Ek_parseTunerConstants@@YAXXZ$44
	DD	037H
	DD	FLAT:__unwindfunclet$??__Ek_parseTunerConstants@@YAXXZ$44
	DD	03bH
	DD	FLAT:__unwindfunclet$??__Ek_parseTunerConstants@@YAXXZ$45
	DD	03bH
	DD	FLAT:__unwindfunclet$??__Ek_parseTunerConstants@@YAXXZ$46
	DD	03dH
	DD	FLAT:__unwindfunclet$??__Ek_parseTunerConstants@@YAXXZ$47
	DD	03bH
	DD	FLAT:__unwindfunclet$??__Ek_parseTunerConstants@@YAXXZ$47
	DD	03fH
	DD	FLAT:__unwindfunclet$??__Ek_parseTunerConstants@@YAXXZ$48
	DD	03fH
	DD	FLAT:__unwindfunclet$??__Ek_parseTunerConstants@@YAXXZ$49
	DD	041H
	DD	FLAT:__unwindfunclet$??__Ek_parseTunerConstants@@YAXXZ$50
	DD	03fH
	DD	FLAT:__unwindfunclet$??__Ek_parseTunerConstants@@YAXXZ$50
	DD	043H
	DD	FLAT:__unwindfunclet$??__Ek_parseTunerConstants@@YAXXZ$51
	DD	043H
	DD	FLAT:__unwindfunclet$??__Ek_parseTunerConstants@@YAXXZ$52
	DD	045H
	DD	FLAT:__unwindfunclet$??__Ek_parseTunerConstants@@YAXXZ$53
	DD	043H
	DD	FLAT:__unwindfunclet$??__Ek_parseTunerConstants@@YAXXZ$53
	DD	047H
	DD	FLAT:__unwindfunclet$??__Ek_parseTunerConstants@@YAXXZ$54
	DD	047H
	DD	FLAT:__unwindfunclet$??__Ek_parseTunerConstants@@YAXXZ$55
	DD	049H
	DD	FLAT:__unwindfunclet$??__Ek_parseTunerConstants@@YAXXZ$56
	DD	047H
	DD	FLAT:__unwindfunclet$??__Ek_parseTunerConstants@@YAXXZ$56
	DD	04bH
	DD	FLAT:__unwindfunclet$??__Ek_parseTunerConstants@@YAXXZ$57
	DD	04bH
	DD	FLAT:__unwindfunclet$??__Ek_parseTunerConstants@@YAXXZ$58
	DD	04dH
	DD	FLAT:__unwindfunclet$??__Ek_parseTunerConstants@@YAXXZ$59
	DD	04bH
	DD	FLAT:__unwindfunclet$??__Ek_parseTunerConstants@@YAXXZ$59
	DD	04fH
	DD	FLAT:__unwindfunclet$??__Ek_parseTunerConstants@@YAXXZ$60
	DD	04fH
	DD	FLAT:__unwindfunclet$??__Ek_parseTunerConstants@@YAXXZ$61
	DD	051H
	DD	FLAT:__unwindfunclet$??__Ek_parseTunerConstants@@YAXXZ$62
	DD	04fH
	DD	FLAT:__unwindfunclet$??__Ek_parseTunerConstants@@YAXXZ$62
	DD	053H
	DD	FLAT:__unwindfunclet$??__Ek_parseTunerConstants@@YAXXZ$63
	DD	053H
	DD	FLAT:__unwindfunclet$??__Ek_parseTunerConstants@@YAXXZ$64
	DD	055H
	DD	FLAT:__unwindfunclet$??__Ek_parseTunerConstants@@YAXXZ$65
	DD	053H
	DD	FLAT:__unwindfunclet$??__Ek_parseTunerConstants@@YAXXZ$65
	DD	057H
	DD	FLAT:__unwindfunclet$??__Ek_parseTunerConstants@@YAXXZ$66
	DD	057H
	DD	FLAT:__unwindfunclet$??__Ek_parseTunerConstants@@YAXXZ$67
	DD	059H
	DD	FLAT:__unwindfunclet$??__Ek_parseTunerConstants@@YAXXZ$68
	DD	057H
	DD	FLAT:__unwindfunclet$??__Ek_parseTunerConstants@@YAXXZ$68
	DD	05bH
	DD	FLAT:__unwindfunclet$??__Ek_parseTunerConstants@@YAXXZ$69
	DD	05bH
	DD	FLAT:__unwindfunclet$??__Ek_parseTunerConstants@@YAXXZ$70
	DD	05dH
	DD	FLAT:__unwindfunclet$??__Ek_parseTunerConstants@@YAXXZ$71
	DD	05bH
	DD	FLAT:__unwindfunclet$??__Ek_parseTunerConstants@@YAXXZ$71
	DD	05fH
	DD	FLAT:__unwindfunclet$??__Ek_parseTunerConstants@@YAXXZ$72
	DD	05fH
	DD	FLAT:__unwindfunclet$??__Ek_parseTunerConstants@@YAXXZ$73
	DD	061H
	DD	FLAT:__unwindfunclet$??__Ek_parseTunerConstants@@YAXXZ$74
	DD	05fH
	DD	FLAT:__unwindfunclet$??__Ek_parseTunerConstants@@YAXXZ$74
	DD	063H
	DD	FLAT:__unwindfunclet$??__Ek_parseTunerConstants@@YAXXZ$75
	DD	063H
	DD	FLAT:__unwindfunclet$??__Ek_parseTunerConstants@@YAXXZ$76
	DD	065H
	DD	FLAT:__unwindfunclet$??__Ek_parseTunerConstants@@YAXXZ$77
	DD	063H
	DD	FLAT:__unwindfunclet$??__Ek_parseTunerConstants@@YAXXZ$77
	DD	067H
	DD	FLAT:__unwindfunclet$??__Ek_parseTunerConstants@@YAXXZ$78
	DD	067H
	DD	FLAT:__unwindfunclet$??__Ek_parseTunerConstants@@YAXXZ$79
	DD	069H
	DD	FLAT:__unwindfunclet$??__Ek_parseTunerConstants@@YAXXZ$80
	DD	067H
	DD	FLAT:__unwindfunclet$??__Ek_parseTunerConstants@@YAXXZ$80
	DD	06bH
	DD	FLAT:__unwindfunclet$??__Ek_parseTunerConstants@@YAXXZ$81
	DD	06bH
	DD	FLAT:__unwindfunclet$??__Ek_parseTunerConstants@@YAXXZ$82
	DD	06dH
	DD	FLAT:__unwindfunclet$??__Ek_parseTunerConstants@@YAXXZ$83
	DD	06bH
	DD	FLAT:__unwindfunclet$??__Ek_parseTunerConstants@@YAXXZ$83
	DD	06fH
	DD	FLAT:__unwindfunclet$??__Ek_parseTunerConstants@@YAXXZ$84
	DD	06fH
	DD	FLAT:__unwindfunclet$??__Ek_parseTunerConstants@@YAXXZ$85
	DD	071H
	DD	FLAT:__unwindfunclet$??__Ek_parseTunerConstants@@YAXXZ$86
	DD	06fH
	DD	FLAT:__unwindfunclet$??__Ek_parseTunerConstants@@YAXXZ$86
	DD	073H
	DD	FLAT:__unwindfunclet$??__Ek_parseTunerConstants@@YAXXZ$87
	DD	073H
	DD	FLAT:__unwindfunclet$??__Ek_parseTunerConstants@@YAXXZ$88
	DD	075H
	DD	FLAT:__unwindfunclet$??__Ek_parseTunerConstants@@YAXXZ$89
	DD	073H
	DD	FLAT:__unwindfunclet$??__Ek_parseTunerConstants@@YAXXZ$89
	DD	077H
	DD	FLAT:__unwindfunclet$??__Ek_parseTunerConstants@@YAXXZ$90
	DD	077H
	DD	FLAT:__unwindfunclet$??__Ek_parseTunerConstants@@YAXXZ$91
	DD	079H
	DD	FLAT:__unwindfunclet$??__Ek_parseTunerConstants@@YAXXZ$92
	DD	077H
	DD	FLAT:__unwindfunclet$??__Ek_parseTunerConstants@@YAXXZ$92
	DD	07bH
	DD	FLAT:__unwindfunclet$??__Ek_parseTunerConstants@@YAXXZ$93
	DD	07bH
	DD	FLAT:__unwindfunclet$??__Ek_parseTunerConstants@@YAXXZ$94
	DD	07dH
	DD	FLAT:__unwindfunclet$??__Ek_parseTunerConstants@@YAXXZ$95
	DD	07bH
	DD	FLAT:__unwindfunclet$??__Ek_parseTunerConstants@@YAXXZ$95
	DD	07fH
	DD	FLAT:__unwindfunclet$??__Ek_parseTunerConstants@@YAXXZ$96
	DD	07fH
	DD	FLAT:__unwindfunclet$??__Ek_parseTunerConstants@@YAXXZ$97
	DD	081H
	DD	FLAT:__unwindfunclet$??__Ek_parseTunerConstants@@YAXXZ$98
	DD	07fH
	DD	FLAT:__unwindfunclet$??__Ek_parseTunerConstants@@YAXXZ$98
	DD	083H
	DD	FLAT:__unwindfunclet$??__Ek_parseTunerConstants@@YAXXZ$99
	DD	083H
	DD	FLAT:__unwindfunclet$??__Ek_parseTunerConstants@@YAXXZ$100
	DD	085H
	DD	FLAT:__unwindfunclet$??__Ek_parseTunerConstants@@YAXXZ$101
	DD	083H
	DD	FLAT:__unwindfunclet$??__Ek_parseTunerConstants@@YAXXZ$101
	DD	087H
	DD	FLAT:__unwindfunclet$??__Ek_parseTunerConstants@@YAXXZ$102
	DD	087H
	DD	FLAT:__unwindfunclet$??__Ek_parseTunerConstants@@YAXXZ$103
	DD	089H
	DD	FLAT:__unwindfunclet$??__Ek_parseTunerConstants@@YAXXZ$104
	DD	087H
	DD	FLAT:__unwindfunclet$??__Ek_parseTunerConstants@@YAXXZ$104
	DD	08bH
	DD	FLAT:__unwindfunclet$??__Ek_parseTunerConstants@@YAXXZ$105
	DD	08bH
	DD	FLAT:__unwindfunclet$??__Ek_parseTunerConstants@@YAXXZ$106
	DD	08dH
	DD	FLAT:__unwindfunclet$??__Ek_parseTunerConstants@@YAXXZ$107
	DD	08bH
	DD	FLAT:__unwindfunclet$??__Ek_parseTunerConstants@@YAXXZ$107
	DD	08fH
	DD	FLAT:__unwindfunclet$??__Ek_parseTunerConstants@@YAXXZ$108
	DD	08fH
	DD	FLAT:__unwindfunclet$??__Ek_parseTunerConstants@@YAXXZ$109
	DD	091H
	DD	FLAT:__unwindfunclet$??__Ek_parseTunerConstants@@YAXXZ$110
	DD	08fH
	DD	FLAT:__unwindfunclet$??__Ek_parseTunerConstants@@YAXXZ$110
	DD	093H
	DD	FLAT:__unwindfunclet$??__Ek_parseTunerConstants@@YAXXZ$111
	DD	093H
	DD	FLAT:__unwindfunclet$??__Ek_parseTunerConstants@@YAXXZ$112
	DD	095H
	DD	FLAT:__unwindfunclet$??__Ek_parseTunerConstants@@YAXXZ$113
	DD	093H
	DD	FLAT:__unwindfunclet$??__Ek_parseTunerConstants@@YAXXZ$113
	DD	097H
	DD	FLAT:__unwindfunclet$??__Ek_parseTunerConstants@@YAXXZ$114
	DD	097H
	DD	FLAT:__unwindfunclet$??__Ek_parseTunerConstants@@YAXXZ$115
	DD	099H
	DD	FLAT:__unwindfunclet$??__Ek_parseTunerConstants@@YAXXZ$116
	DD	097H
	DD	FLAT:__unwindfunclet$??__Ek_parseTunerConstants@@YAXXZ$116
	DD	09bH
	DD	FLAT:__unwindfunclet$??__Ek_parseTunerConstants@@YAXXZ$117
	DD	09bH
	DD	FLAT:__unwindfunclet$??__Ek_parseTunerConstants@@YAXXZ$118
	DD	09dH
	DD	FLAT:__unwindfunclet$??__Ek_parseTunerConstants@@YAXXZ$119
	DD	09bH
	DD	FLAT:__unwindfunclet$??__Ek_parseTunerConstants@@YAXXZ$119
	DD	09fH
	DD	FLAT:__unwindfunclet$??__Ek_parseTunerConstants@@YAXXZ$120
	DD	09fH
	DD	FLAT:__unwindfunclet$??__Ek_parseTunerConstants@@YAXXZ$121
	DD	0a1H
	DD	FLAT:__unwindfunclet$??__Ek_parseTunerConstants@@YAXXZ$122
	DD	09fH
	DD	FLAT:__unwindfunclet$??__Ek_parseTunerConstants@@YAXXZ$122
	DD	0a3H
	DD	FLAT:__unwindfunclet$??__Ek_parseTunerConstants@@YAXXZ$123
	DD	0a3H
	DD	FLAT:__unwindfunclet$??__Ek_parseTunerConstants@@YAXXZ$124
	DD	0a5H
	DD	FLAT:__unwindfunclet$??__Ek_parseTunerConstants@@YAXXZ$125
	DD	0a3H
	DD	FLAT:__unwindfunclet$??__Ek_parseTunerConstants@@YAXXZ$125
	DD	0a7H
	DD	FLAT:__unwindfunclet$??__Ek_parseTunerConstants@@YAXXZ$126
	DD	0a7H
	DD	FLAT:__unwindfunclet$??__Ek_parseTunerConstants@@YAXXZ$127
	DD	0a9H
	DD	FLAT:__unwindfunclet$??__Ek_parseTunerConstants@@YAXXZ$128
	DD	0a7H
	DD	FLAT:__unwindfunclet$??__Ek_parseTunerConstants@@YAXXZ$128
	DD	0abH
	DD	FLAT:__unwindfunclet$??__Ek_parseTunerConstants@@YAXXZ$129
	DD	0abH
	DD	FLAT:__unwindfunclet$??__Ek_parseTunerConstants@@YAXXZ$130
	DD	0adH
	DD	FLAT:__unwindfunclet$??__Ek_parseTunerConstants@@YAXXZ$131
	DD	0abH
	DD	FLAT:__unwindfunclet$??__Ek_parseTunerConstants@@YAXXZ$131
	DD	0afH
	DD	FLAT:__unwindfunclet$??__Ek_parseTunerConstants@@YAXXZ$132
	DD	0afH
	DD	FLAT:__unwindfunclet$??__Ek_parseTunerConstants@@YAXXZ$133
	DD	0b1H
	DD	FLAT:__unwindfunclet$??__Ek_parseTunerConstants@@YAXXZ$134
	DD	0afH
	DD	FLAT:__unwindfunclet$??__Ek_parseTunerConstants@@YAXXZ$134
	DD	0b3H
	DD	FLAT:__unwindfunclet$??__Ek_parseTunerConstants@@YAXXZ$135
	DD	0b3H
	DD	FLAT:__unwindfunclet$??__Ek_parseTunerConstants@@YAXXZ$136
	DD	0b5H
	DD	FLAT:__unwindfunclet$??__Ek_parseTunerConstants@@YAXXZ$137
	DD	0b3H
	DD	FLAT:__unwindfunclet$??__Ek_parseTunerConstants@@YAXXZ$137
	DD	0b7H
	DD	FLAT:__unwindfunclet$??__Ek_parseTunerConstants@@YAXXZ$138
	DD	0b7H
	DD	FLAT:__unwindfunclet$??__Ek_parseTunerConstants@@YAXXZ$139
	DD	0b9H
	DD	FLAT:__unwindfunclet$??__Ek_parseTunerConstants@@YAXXZ$140
	DD	0b7H
	DD	FLAT:__unwindfunclet$??__Ek_parseTunerConstants@@YAXXZ$140
	DD	0bbH
	DD	FLAT:__unwindfunclet$??__Ek_parseTunerConstants@@YAXXZ$141
	DD	0bbH
	DD	FLAT:__unwindfunclet$??__Ek_parseTunerConstants@@YAXXZ$142
	DD	0bdH
	DD	FLAT:__unwindfunclet$??__Ek_parseTunerConstants@@YAXXZ$143
	DD	0bbH
	DD	FLAT:__unwindfunclet$??__Ek_parseTunerConstants@@YAXXZ$143
	DD	0bfH
	DD	FLAT:__unwindfunclet$??__Ek_parseTunerConstants@@YAXXZ$144
	DD	0bfH
	DD	FLAT:__unwindfunclet$??__Ek_parseTunerConstants@@YAXXZ$145
	DD	0c1H
	DD	FLAT:__unwindfunclet$??__Ek_parseTunerConstants@@YAXXZ$146
	DD	0bfH
	DD	FLAT:__unwindfunclet$??__Ek_parseTunerConstants@@YAXXZ$146
	DD	0c3H
	DD	FLAT:__unwindfunclet$??__Ek_parseTunerConstants@@YAXXZ$147
	DD	0c3H
	DD	FLAT:__unwindfunclet$??__Ek_parseTunerConstants@@YAXXZ$148
	DD	0c5H
	DD	FLAT:__unwindfunclet$??__Ek_parseTunerConstants@@YAXXZ$149
	DD	0c3H
	DD	FLAT:__unwindfunclet$??__Ek_parseTunerConstants@@YAXXZ$149
	DD	0c7H
	DD	FLAT:__unwindfunclet$??__Ek_parseTunerConstants@@YAXXZ$150
	DD	0c7H
	DD	FLAT:__unwindfunclet$??__Ek_parseTunerConstants@@YAXXZ$151
	DD	0c9H
	DD	FLAT:__unwindfunclet$??__Ek_parseTunerConstants@@YAXXZ$152
	DD	0c7H
	DD	FLAT:__unwindfunclet$??__Ek_parseTunerConstants@@YAXXZ$152
	DD	0cbH
	DD	FLAT:__unwindfunclet$??__Ek_parseTunerConstants@@YAXXZ$153
	DD	0cbH
	DD	FLAT:__unwindfunclet$??__Ek_parseTunerConstants@@YAXXZ$154
	DD	0cdH
	DD	FLAT:__unwindfunclet$??__Ek_parseTunerConstants@@YAXXZ$155
	DD	0cbH
	DD	FLAT:__unwindfunclet$??__Ek_parseTunerConstants@@YAXXZ$155
	DD	0cfH
	DD	FLAT:__unwindfunclet$??__Ek_parseTunerConstants@@YAXXZ$156
	DD	0cfH
	DD	FLAT:__unwindfunclet$??__Ek_parseTunerConstants@@YAXXZ$157
	DD	0d1H
	DD	FLAT:__unwindfunclet$??__Ek_parseTunerConstants@@YAXXZ$158
	DD	0cfH
	DD	FLAT:__unwindfunclet$??__Ek_parseTunerConstants@@YAXXZ$158
	DD	0d3H
	DD	FLAT:__unwindfunclet$??__Ek_parseTunerConstants@@YAXXZ$159
	DD	0d3H
	DD	FLAT:__unwindfunclet$??__Ek_parseTunerConstants@@YAXXZ$160
	DD	0d5H
	DD	FLAT:__unwindfunclet$??__Ek_parseTunerConstants@@YAXXZ$161
	DD	0d3H
	DD	FLAT:__unwindfunclet$??__Ek_parseTunerConstants@@YAXXZ$161
	DD	0d7H
	DD	FLAT:__unwindfunclet$??__Ek_parseTunerConstants@@YAXXZ$162
	DD	0d7H
	DD	FLAT:__unwindfunclet$??__Ek_parseTunerConstants@@YAXXZ$163
	DD	0d9H
	DD	FLAT:__unwindfunclet$??__Ek_parseTunerConstants@@YAXXZ$164
	DD	0d7H
	DD	FLAT:__unwindfunclet$??__Ek_parseTunerConstants@@YAXXZ$164
	DD	0dbH
	DD	FLAT:__unwindfunclet$??__Ek_parseTunerConstants@@YAXXZ$165
	DD	0dbH
	DD	FLAT:__unwindfunclet$??__Ek_parseTunerConstants@@YAXXZ$166
	DD	0ddH
	DD	FLAT:__unwindfunclet$??__Ek_parseTunerConstants@@YAXXZ$167
	DD	0dbH
	DD	FLAT:__unwindfunclet$??__Ek_parseTunerConstants@@YAXXZ$167
	DD	0dfH
	DD	FLAT:__unwindfunclet$??__Ek_parseTunerConstants@@YAXXZ$168
	DD	0dfH
	DD	FLAT:__unwindfunclet$??__Ek_parseTunerConstants@@YAXXZ$169
	DD	0e1H
	DD	FLAT:__unwindfunclet$??__Ek_parseTunerConstants@@YAXXZ$170
	DD	0dfH
	DD	FLAT:__unwindfunclet$??__Ek_parseTunerConstants@@YAXXZ$170
	DD	0e3H
	DD	FLAT:__unwindfunclet$??__Ek_parseTunerConstants@@YAXXZ$171
	DD	0e3H
	DD	FLAT:__unwindfunclet$??__Ek_parseTunerConstants@@YAXXZ$172
	DD	0e5H
	DD	FLAT:__unwindfunclet$??__Ek_parseTunerConstants@@YAXXZ$173
	DD	0e3H
	DD	FLAT:__unwindfunclet$??__Ek_parseTunerConstants@@YAXXZ$173
	DD	0e7H
	DD	FLAT:__unwindfunclet$??__Ek_parseTunerConstants@@YAXXZ$174
	DD	0e7H
	DD	FLAT:__unwindfunclet$??__Ek_parseTunerConstants@@YAXXZ$175
	DD	0e9H
	DD	FLAT:__unwindfunclet$??__Ek_parseTunerConstants@@YAXXZ$176
	DD	0e7H
	DD	FLAT:__unwindfunclet$??__Ek_parseTunerConstants@@YAXXZ$176
	DD	0ebH
	DD	FLAT:__unwindfunclet$??__Ek_parseTunerConstants@@YAXXZ$177
	DD	0ebH
	DD	FLAT:__unwindfunclet$??__Ek_parseTunerConstants@@YAXXZ$178
	DD	0edH
	DD	FLAT:__unwindfunclet$??__Ek_parseTunerConstants@@YAXXZ$179
	DD	0ebH
	DD	FLAT:__unwindfunclet$??__Ek_parseTunerConstants@@YAXXZ$179
	DD	0efH
	DD	FLAT:__unwindfunclet$??__Ek_parseTunerConstants@@YAXXZ$180
	DD	0efH
	DD	FLAT:__unwindfunclet$??__Ek_parseTunerConstants@@YAXXZ$181
	DD	0f1H
	DD	FLAT:__unwindfunclet$??__Ek_parseTunerConstants@@YAXXZ$182
	DD	0efH
	DD	FLAT:__unwindfunclet$??__Ek_parseTunerConstants@@YAXXZ$182
	DD	0f3H
	DD	FLAT:__unwindfunclet$??__Ek_parseTunerConstants@@YAXXZ$183
	DD	0f3H
	DD	FLAT:__unwindfunclet$??__Ek_parseTunerConstants@@YAXXZ$184
	DD	0f5H
	DD	FLAT:__unwindfunclet$??__Ek_parseTunerConstants@@YAXXZ$185
	DD	0f3H
	DD	FLAT:__unwindfunclet$??__Ek_parseTunerConstants@@YAXXZ$185
	DD	0f7H
	DD	FLAT:__unwindfunclet$??__Ek_parseTunerConstants@@YAXXZ$186
	DD	0f7H
	DD	FLAT:__unwindfunclet$??__Ek_parseTunerConstants@@YAXXZ$187
	DD	0f9H
	DD	FLAT:__unwindfunclet$??__Ek_parseTunerConstants@@YAXXZ$188
	DD	0f7H
	DD	FLAT:__unwindfunclet$??__Ek_parseTunerConstants@@YAXXZ$188
	DD	0fbH
	DD	FLAT:__unwindfunclet$??__Ek_parseTunerConstants@@YAXXZ$189
	DD	0fbH
	DD	FLAT:__unwindfunclet$??__Ek_parseTunerConstants@@YAXXZ$190
	DD	0fdH
	DD	FLAT:__unwindfunclet$??__Ek_parseTunerConstants@@YAXXZ$191
	DD	0fbH
	DD	FLAT:__unwindfunclet$??__Ek_parseTunerConstants@@YAXXZ$191
	DD	0ffH
	DD	FLAT:__unwindfunclet$??__Ek_parseTunerConstants@@YAXXZ$192
	DD	0ffH
	DD	FLAT:__unwindfunclet$??__Ek_parseTunerConstants@@YAXXZ$193
	DD	0101H
	DD	FLAT:__unwindfunclet$??__Ek_parseTunerConstants@@YAXXZ$194
	DD	0ffH
	DD	FLAT:__unwindfunclet$??__Ek_parseTunerConstants@@YAXXZ$194
	DD	0103H
	DD	FLAT:__unwindfunclet$??__Ek_parseTunerConstants@@YAXXZ$195
	DD	0103H
	DD	FLAT:__unwindfunclet$??__Ek_parseTunerConstants@@YAXXZ$196
	DD	0105H
	DD	FLAT:__unwindfunclet$??__Ek_parseTunerConstants@@YAXXZ$197
	DD	0103H
	DD	FLAT:__unwindfunclet$??__Ek_parseTunerConstants@@YAXXZ$197
	DD	0107H
	DD	FLAT:__unwindfunclet$??__Ek_parseTunerConstants@@YAXXZ$198
	DD	0107H
	DD	FLAT:__unwindfunclet$??__Ek_parseTunerConstants@@YAXXZ$199
	DD	0109H
	DD	FLAT:__unwindfunclet$??__Ek_parseTunerConstants@@YAXXZ$200
	DD	0107H
	DD	FLAT:__unwindfunclet$??__Ek_parseTunerConstants@@YAXXZ$200
__ehfuncinfo$??__Ek_parseTunerConstants@@YAXXZ DD 019930522H
	DD	010cH
	DD	FLAT:__unwindtable$??__Ek_parseTunerConstants@@YAXXZ
	DD	2 DUP(00H)
	DD	2 DUP(00H)
	DD	00H
	DD	00H
; Function compile flags: /Odtp
xdata$x	ENDS
;	COMDAT ??__Ek_parseTunerConstants@@YAXXZ
text$yc	SEGMENT
tv2293 = -2424						; size = 4
tv2291 = -2420						; size = 4
tv2290 = -2416						; size = 4
tv1816 = -2412						; size = 4
tv2287 = -2408						; size = 4
tv2285 = -2404						; size = 4
tv2284 = -2400						; size = 4
tv1793 = -2396						; size = 4
tv2281 = -2392						; size = 4
tv2279 = -2388						; size = 4
tv2278 = -2384						; size = 4
tv1738 = -2380						; size = 4
tv2275 = -2376						; size = 4
tv2273 = -2372						; size = 4
tv2272 = -2368						; size = 4
tv1715 = -2364						; size = 4
tv2269 = -2360						; size = 4
tv2267 = -2356						; size = 4
tv2266 = -2352						; size = 4
tv1692 = -2348						; size = 4
tv2263 = -2344						; size = 4
tv2261 = -2340						; size = 4
tv2260 = -2336						; size = 4
tv1669 = -2332						; size = 4
tv2257 = -2328						; size = 4
tv2255 = -2324						; size = 4
tv2254 = -2320						; size = 4
tv1646 = -2316						; size = 4
tv2251 = -2312						; size = 4
tv2249 = -2308						; size = 4
tv2248 = -2304						; size = 4
tv1623 = -2300						; size = 4
tv2245 = -2296						; size = 4
tv2243 = -2292						; size = 4
tv2242 = -2288						; size = 4
tv1600 = -2284						; size = 4
tv2239 = -2280						; size = 4
tv2237 = -2276						; size = 4
tv2236 = -2272						; size = 4
tv1577 = -2268						; size = 4
tv2233 = -2264						; size = 4
tv2231 = -2260						; size = 4
tv2230 = -2256						; size = 4
tv1554 = -2252						; size = 4
tv2227 = -2248						; size = 4
tv2225 = -2244						; size = 4
tv2224 = -2240						; size = 4
tv1531 = -2236						; size = 4
tv2221 = -2232						; size = 4
tv2219 = -2228						; size = 4
tv2218 = -2224						; size = 4
tv1508 = -2220						; size = 4
tv2215 = -2216						; size = 4
tv2213 = -2212						; size = 4
tv2212 = -2208						; size = 4
tv1485 = -2204						; size = 4
tv2209 = -2200						; size = 4
tv2207 = -2196						; size = 4
tv2206 = -2192						; size = 4
tv1462 = -2188						; size = 4
tv2203 = -2184						; size = 4
tv2201 = -2180						; size = 4
tv2200 = -2176						; size = 4
tv1439 = -2172						; size = 4
tv2197 = -2168						; size = 4
tv2195 = -2164						; size = 4
tv2194 = -2160						; size = 4
tv1416 = -2156						; size = 4
tv2191 = -2152						; size = 4
tv2189 = -2148						; size = 4
tv2188 = -2144						; size = 4
tv1361 = -2140						; size = 4
tv2185 = -2136						; size = 4
tv2183 = -2132						; size = 4
tv2182 = -2128						; size = 4
tv1306 = -2124						; size = 4
tv2179 = -2120						; size = 4
tv2177 = -2116						; size = 4
tv2176 = -2112						; size = 4
tv1283 = -2108						; size = 4
tv2173 = -2104						; size = 4
tv2171 = -2100						; size = 4
tv2170 = -2096						; size = 4
tv1260 = -2092						; size = 4
tv2167 = -2088						; size = 4
tv2165 = -2084						; size = 4
tv2164 = -2080						; size = 4
tv1237 = -2076						; size = 4
tv2161 = -2072						; size = 4
tv2159 = -2068						; size = 4
tv2158 = -2064						; size = 4
tv1214 = -2060						; size = 4
tv2155 = -2056						; size = 4
tv2153 = -2052						; size = 4
tv2152 = -2048						; size = 4
tv1191 = -2044						; size = 4
tv2149 = -2040						; size = 4
tv2147 = -2036						; size = 4
tv2146 = -2032						; size = 4
tv1168 = -2028						; size = 4
tv2143 = -2024						; size = 4
tv2141 = -2020						; size = 4
tv2140 = -2016						; size = 4
tv1145 = -2012						; size = 4
tv2137 = -2008						; size = 4
tv2135 = -2004						; size = 4
tv2134 = -2000						; size = 4
tv1122 = -1996						; size = 4
tv2131 = -1992						; size = 4
tv2129 = -1988						; size = 4
tv2128 = -1984						; size = 4
tv1099 = -1980						; size = 4
tv2125 = -1976						; size = 4
tv2123 = -1972						; size = 4
tv2122 = -1968						; size = 4
tv1076 = -1964						; size = 4
tv2119 = -1960						; size = 4
tv2117 = -1956						; size = 4
tv2116 = -1952						; size = 4
tv1053 = -1948						; size = 4
tv2113 = -1944						; size = 4
tv2111 = -1940						; size = 4
tv2110 = -1936						; size = 4
tv1030 = -1932						; size = 4
tv2107 = -1928						; size = 4
tv2105 = -1924						; size = 4
tv2104 = -1920						; size = 4
tv1007 = -1916						; size = 4
tv2101 = -1912						; size = 4
tv2099 = -1908						; size = 4
tv2098 = -1904						; size = 4
tv952 = -1900						; size = 4
tv2095 = -1896						; size = 4
tv2093 = -1892						; size = 4
tv2092 = -1888						; size = 4
tv929 = -1884						; size = 4
tv2089 = -1880						; size = 4
tv2087 = -1876						; size = 4
tv2086 = -1872						; size = 4
tv874 = -1868						; size = 4
tv2083 = -1864						; size = 4
tv2081 = -1860						; size = 4
tv2080 = -1856						; size = 4
tv851 = -1852						; size = 4
tv2077 = -1848						; size = 4
tv2075 = -1844						; size = 4
tv2074 = -1840						; size = 4
tv828 = -1836						; size = 4
tv2071 = -1832						; size = 4
tv2069 = -1828						; size = 4
tv2068 = -1824						; size = 4
tv805 = -1820						; size = 4
tv2065 = -1816						; size = 4
tv2063 = -1812						; size = 4
tv2062 = -1808						; size = 4
tv782 = -1804						; size = 4
tv2059 = -1800						; size = 4
tv2057 = -1796						; size = 4
tv2056 = -1792						; size = 4
tv759 = -1788						; size = 4
tv2053 = -1784						; size = 4
tv2051 = -1780						; size = 4
tv2050 = -1776						; size = 4
tv736 = -1772						; size = 4
tv2047 = -1768						; size = 4
tv2045 = -1764						; size = 4
tv2044 = -1760						; size = 4
tv713 = -1756						; size = 4
tv2041 = -1752						; size = 4
tv2039 = -1748						; size = 4
tv2038 = -1744						; size = 4
tv690 = -1740						; size = 4
tv2035 = -1736						; size = 4
tv2033 = -1732						; size = 4
tv2032 = -1728						; size = 4
tv667 = -1724						; size = 4
tv2029 = -1720						; size = 4
tv2027 = -1716						; size = 4
tv2026 = -1712						; size = 4
tv644 = -1708						; size = 4
tv2023 = -1704						; size = 4
tv2021 = -1700						; size = 4
tv2020 = -1696						; size = 4
tv621 = -1692						; size = 4
tv2017 = -1688						; size = 4
tv2015 = -1684						; size = 4
tv2014 = -1680						; size = 4
tv598 = -1676						; size = 4
tv2011 = -1672						; size = 4
tv2009 = -1668						; size = 4
tv2008 = -1664						; size = 4
tv575 = -1660						; size = 4
tv2005 = -1656						; size = 4
tv2003 = -1652						; size = 4
tv2002 = -1648						; size = 4
tv552 = -1644						; size = 4
tv1999 = -1640						; size = 4
tv1997 = -1636						; size = 4
tv1996 = -1632						; size = 4
tv497 = -1628						; size = 4
tv1993 = -1624						; size = 4
tv1991 = -1620						; size = 4
tv1990 = -1616						; size = 4
tv442 = -1612						; size = 4
tv1987 = -1608						; size = 4
tv1985 = -1604						; size = 4
tv1984 = -1600						; size = 4
tv419 = -1596						; size = 4
tv1981 = -1592						; size = 4
tv1979 = -1588						; size = 4
tv1978 = -1584						; size = 4
tv396 = -1580						; size = 4
tv1975 = -1576						; size = 4
tv1973 = -1572						; size = 4
tv1972 = -1568						; size = 4
tv373 = -1564						; size = 4
tv1969 = -1560						; size = 4
tv1967 = -1556						; size = 4
tv1966 = -1552						; size = 4
tv350 = -1548						; size = 4
tv1963 = -1544						; size = 4
tv1961 = -1540						; size = 4
tv1960 = -1536						; size = 4
tv327 = -1532						; size = 4
tv1957 = -1528						; size = 4
tv1955 = -1524						; size = 4
tv1954 = -1520						; size = 4
tv304 = -1516						; size = 4
tv1951 = -1512						; size = 4
tv1949 = -1508						; size = 4
tv1948 = -1504						; size = 4
tv281 = -1500						; size = 4
tv1945 = -1496						; size = 4
tv1943 = -1492						; size = 4
tv1942 = -1488						; size = 4
tv258 = -1484						; size = 4
tv1939 = -1480						; size = 4
tv1937 = -1476						; size = 4
tv1936 = -1472						; size = 4
tv235 = -1468						; size = 4
tv1933 = -1464						; size = 4
tv1931 = -1460						; size = 4
tv1930 = -1456						; size = 4
tv212 = -1452						; size = 4
tv1927 = -1448						; size = 4
tv1925 = -1444						; size = 4
tv1924 = -1440						; size = 4
tv189 = -1436						; size = 4
tv1921 = -1432						; size = 4
tv1919 = -1428						; size = 4
tv1918 = -1424						; size = 4
tv166 = -1420						; size = 4
tv1915 = -1416						; size = 4
tv1913 = -1412						; size = 4
tv1912 = -1408						; size = 4
tv143 = -1404						; size = 4
tv1909 = -1400						; size = 4
tv1907 = -1396						; size = 4
tv1906 = -1392						; size = 4
tv88 = -1388						; size = 4
tv1903 = -1384						; size = 4
tv1901 = -1380						; size = 4
tv1900 = -1376						; size = 4
tv65 = -1372						; size = 4
tv1897 = -1368						; size = 4
tv1895 = -1364						; size = 4
tv1894 = -1360						; size = 4
tv2295 = -1356						; size = 4
$T362700 = -1352					; size = 4
$T362699 = -1348					; size = 16
$T362698 = -1332					; size = 4
$T362697 = -1328					; size = 16
$T362696 = -1312					; size = 4
$T362695 = -1308					; size = 16
$T362694 = -1292					; size = 4
$T362693 = -1288					; size = 16
$T362692 = -1272					; size = 4
$T362691 = -1268					; size = 16
$T362690 = -1252					; size = 4
$T362689 = -1248					; size = 16
$T362688 = -1232					; size = 4
$T362687 = -1228					; size = 16
$T362686 = -1212					; size = 4
$T362685 = -1208					; size = 16
$T362684 = -1192					; size = 4
$T362683 = -1188					; size = 16
$T362682 = -1172					; size = 4
$T362681 = -1168					; size = 16
$T362680 = -1152					; size = 4
$T362679 = -1148					; size = 16
$T362678 = -1132					; size = 4
$T362677 = -1128					; size = 16
$T362676 = -1112					; size = 4
$T362675 = -1108					; size = 16
$T362674 = -1092					; size = 4
$T362673 = -1088					; size = 16
$T362672 = -1072					; size = 4
$T362671 = -1068					; size = 16
$T362670 = -1052					; size = 4
$T362669 = -1048					; size = 16
$T362668 = -1032					; size = 4
$T362667 = -1028					; size = 16
$T362666 = -1012					; size = 4
$T362665 = -1008					; size = 16
$T362664 = -992						; size = 4
$T362663 = -988						; size = 16
$T362662 = -972						; size = 4
$T362661 = -968						; size = 16
$T362660 = -952						; size = 4
$T362659 = -948						; size = 16
$T362658 = -932						; size = 4
$T362657 = -928						; size = 16
$T362656 = -912						; size = 4
$T362655 = -908						; size = 16
$T362654 = -892						; size = 4
$T362653 = -888						; size = 16
$T362652 = -872						; size = 4
$T362651 = -868						; size = 16
$T362650 = -852						; size = 4
$T362649 = -848						; size = 16
$T362648 = -832						; size = 4
$T362647 = -828						; size = 16
$T362646 = -812						; size = 4
$T362645 = -808						; size = 16
$T362644 = -792						; size = 4
$T362643 = -788						; size = 16
$T362642 = -772						; size = 4
$T362641 = -768						; size = 16
$T362640 = -752						; size = 4
$T362639 = -748						; size = 16
$T362638 = -732						; size = 4
$T362637 = -728						; size = 16
$T362636 = -712						; size = 4
$T362635 = -708						; size = 16
$T362634 = -692						; size = 4
$T362633 = -688						; size = 16
$T362632 = -672						; size = 4
$T362631 = -668						; size = 16
$T362630 = -652						; size = 4
$T362629 = -648						; size = 16
$T362628 = -632						; size = 4
$T362627 = -628						; size = 16
$T362626 = -612						; size = 4
$T362625 = -608						; size = 16
$T362624 = -592						; size = 4
$T362623 = -588						; size = 16
$T362622 = -572						; size = 4
$T362621 = -568						; size = 16
$T362620 = -552						; size = 4
$T362619 = -548						; size = 16
$T362618 = -532						; size = 4
$T362617 = -528						; size = 16
$T362616 = -512						; size = 4
$T362615 = -508						; size = 16
$T362614 = -492						; size = 4
$T362613 = -488						; size = 16
$T362612 = -472						; size = 4
$T362611 = -468						; size = 16
$T362610 = -452						; size = 4
$T362609 = -448						; size = 16
$T362608 = -432						; size = 4
$T362607 = -428						; size = 16
$T362606 = -412						; size = 4
$T362605 = -408						; size = 16
$T362604 = -392						; size = 4
$T362603 = -388						; size = 16
$T362602 = -372						; size = 4
$T362601 = -368						; size = 16
$T362600 = -352						; size = 4
$T362599 = -348						; size = 16
$T362598 = -332						; size = 4
$T362597 = -328						; size = 16
$T362596 = -312						; size = 4
$T362595 = -308						; size = 16
$T362594 = -292						; size = 4
$T362593 = -288						; size = 16
$T362592 = -272						; size = 4
$T362591 = -268						; size = 16
$T362590 = -252						; size = 4
$T362589 = -248						; size = 16
$T362588 = -232						; size = 4
$T362587 = -228						; size = 16
$T362586 = -212						; size = 4
$T362585 = -208						; size = 16
$T362584 = -192						; size = 4
$T362583 = -188						; size = 16
$T362582 = -172						; size = 4
$T362581 = -168						; size = 16
$T362580 = -152						; size = 4
$T362579 = -148						; size = 16
$T362578 = -132						; size = 4
$T362577 = -128						; size = 16
$T362576 = -112						; size = 4
$T362575 = -108						; size = 16
$T362574 = -92						; size = 4
$T362573 = -88						; size = 16
$T362572 = -72						; size = 4
$T362571 = -68						; size = 16
$T362570 = -52						; size = 4
$T362569 = -48						; size = 16
$T362568 = -32						; size = 4
$T362567 = -28						; size = 16
__$EHRec$ = -12						; size = 12
??__Ek_parseTunerConstants@@YAXXZ PROC			; `dynamic initializer for 'k_parseTunerConstants'', COMDAT

; 39   : {

  00000	55		 push	 ebp
  00001	8b ec		 mov	 ebp, esp
  00003	6a ff		 push	 -1
  00005	68 00 00 00 00	 push	 __ehhandler$??__Ek_parseTunerConstants@@YAXXZ
  0000a	64 a1 00 00 00
	00		 mov	 eax, DWORD PTR fs:0
  00010	50		 push	 eax
  00011	81 ec 6c 09 00
	00		 sub	 esp, 2412		; 0000096cH
  00017	a1 00 00 00 00	 mov	 eax, DWORD PTR ___security_cookie
  0001c	33 c5		 xor	 eax, ebp
  0001e	50		 push	 eax
  0001f	8d 45 f4	 lea	 eax, DWORD PTR __$EHRec$[ebp]
  00022	64 a3 00 00 00
	00		 mov	 DWORD PTR fs:0, eax

; 40   :     PC( _T("AUTO"),                            TUNER_AUTODETECT                ),

  00028	83 ec 0c	 sub	 esp, 12			; 0000000cH
  0002b	8b cc		 mov	 ecx, esp
  0002d	89 65 e0	 mov	 DWORD PTR $T362568[ebp], esp
  00030	6a fe		 push	 -2			; fffffffeH
  00032	e8 00 00 00 00	 call	 ??0CParseValue@HCParser@@QAE@H@Z ; HCParser::CParseValue::CParseValue
  00037	89 85 b4 fa ff
	ff		 mov	 DWORD PTR tv2295[ebp], eax
  0003d	8b 85 b4 fa ff
	ff		 mov	 eax, DWORD PTR tv2295[ebp]
  00043	89 85 b0 fa ff
	ff		 mov	 DWORD PTR tv1894[ebp], eax
  00049	c7 45 fc 00 00
	00 00		 mov	 DWORD PTR __$EHRec$[ebp+8], 0
  00050	68 00 00 00 00	 push	 OFFSET ??_C@_19CEKDAEDP@?$AAA?$AAU?$AAT?$AAO?$AA?$AA@
  00055	c7 45 fc ff ff
	ff ff		 mov	 DWORD PTR __$EHRec$[ebp+8], -1
  0005c	8d 4d e4	 lea	 ecx, DWORD PTR $T362567[ebp]
  0005f	e8 00 00 00 00	 call	 ??0CParseConstant@HCParser@@QAE@PB_WVCParseValue@1@@Z ; HCParser::CParseConstant::CParseConstant
  00064	89 85 ac fa ff
	ff		 mov	 DWORD PTR tv1895[ebp], eax
  0006a	8b 8d ac fa ff
	ff		 mov	 ecx, DWORD PTR tv1895[ebp]
  00070	89 8d a8 fa ff
	ff		 mov	 DWORD PTR tv1897[ebp], ecx
  00076	c7 45 fc 01 00
	00 00		 mov	 DWORD PTR __$EHRec$[ebp+8], 1
  0007d	8b 95 a8 fa ff
	ff		 mov	 edx, DWORD PTR tv1897[ebp]
  00083	52		 push	 edx
  00084	b9 00 00 00 00	 mov	 ecx, OFFSET ?k_parseTunerConstants@@3QBVCParseConstant@HCParser@@B ; k_parseTunerConstants
  00089	e8 00 00 00 00	 call	 ??0CParseConstant@HCParser@@QAE@ABV01@@Z
  0008e	c6 45 fc 03	 mov	 BYTE PTR __$EHRec$[ebp+8], 3
  00092	8d 4d e4	 lea	 ecx, DWORD PTR $T362567[ebp]
  00095	e8 00 00 00 00	 call	 ??1CParseConstant@HCParser@@QAE@XZ

; 41   :     PC( _T("SETUP"),                        TUNER_USER_SETUP                ),

  0009a	83 ec 0c	 sub	 esp, 12			; 0000000cH
  0009d	8b cc		 mov	 ecx, esp
  0009f	89 65 cc	 mov	 DWORD PTR $T362570[ebp], esp
  000a2	6a ff		 push	 -1
  000a4	e8 00 00 00 00	 call	 ??0CParseValue@HCParser@@QAE@H@Z ; HCParser::CParseValue::CParseValue
  000a9	89 85 a4 fa ff
	ff		 mov	 DWORD PTR tv65[ebp], eax
  000af	8b 85 a4 fa ff
	ff		 mov	 eax, DWORD PTR tv65[ebp]
  000b5	89 85 a0 fa ff
	ff		 mov	 DWORD PTR tv1900[ebp], eax
  000bb	c6 45 fc 04	 mov	 BYTE PTR __$EHRec$[ebp+8], 4
  000bf	68 00 00 00 00	 push	 OFFSET ??_C@_1M@PBHOBGFC@?$AAS?$AAE?$AAT?$AAU?$AAP?$AA?$AA@
  000c4	c6 45 fc 03	 mov	 BYTE PTR __$EHRec$[ebp+8], 3
  000c8	8d 4d d0	 lea	 ecx, DWORD PTR $T362569[ebp]
  000cb	e8 00 00 00 00	 call	 ??0CParseConstant@HCParser@@QAE@PB_WVCParseValue@1@@Z ; HCParser::CParseConstant::CParseConstant
  000d0	89 85 9c fa ff
	ff		 mov	 DWORD PTR tv1901[ebp], eax
  000d6	8b 8d 9c fa ff
	ff		 mov	 ecx, DWORD PTR tv1901[ebp]
  000dc	89 8d 98 fa ff
	ff		 mov	 DWORD PTR tv1903[ebp], ecx
  000e2	c6 45 fc 05	 mov	 BYTE PTR __$EHRec$[ebp+8], 5
  000e6	8b 95 98 fa ff
	ff		 mov	 edx, DWORD PTR tv1903[ebp]
  000ec	52		 push	 edx
  000ed	b9 10 00 00 00	 mov	 ecx, OFFSET ?k_parseTunerConstants@@3QBVCParseConstant@HCParser@@B+16
  000f2	e8 00 00 00 00	 call	 ??0CParseConstant@HCParser@@QAE@ABV01@@Z
  000f7	c6 45 fc 07	 mov	 BYTE PTR __$EHRec$[ebp+8], 7
  000fb	8d 4d d0	 lea	 ecx, DWORD PTR $T362569[ebp]
  000fe	e8 00 00 00 00	 call	 ??1CParseConstant@HCParser@@QAE@XZ

; 42   :     PC( _T("ABSENT"),                        TUNER_ABSENT                    ),

  00103	83 ec 0c	 sub	 esp, 12			; 0000000cH
  00106	8b cc		 mov	 ecx, esp
  00108	89 65 b8	 mov	 DWORD PTR $T362572[ebp], esp
  0010b	6a 00		 push	 0
  0010d	e8 00 00 00 00	 call	 ??0CParseValue@HCParser@@QAE@H@Z ; HCParser::CParseValue::CParseValue
  00112	89 85 94 fa ff
	ff		 mov	 DWORD PTR tv88[ebp], eax
  00118	8b 85 94 fa ff
	ff		 mov	 eax, DWORD PTR tv88[ebp]
  0011e	89 85 90 fa ff
	ff		 mov	 DWORD PTR tv1906[ebp], eax
  00124	c6 45 fc 08	 mov	 BYTE PTR __$EHRec$[ebp+8], 8
  00128	68 00 00 00 00	 push	 OFFSET ??_C@_1O@GMMJLLPL@?$AAA?$AAB?$AAS?$AAE?$AAN?$AAT?$AA?$AA@
  0012d	c6 45 fc 07	 mov	 BYTE PTR __$EHRec$[ebp+8], 7
  00131	8d 4d bc	 lea	 ecx, DWORD PTR $T362571[ebp]
  00134	e8 00 00 00 00	 call	 ??0CParseConstant@HCParser@@QAE@PB_WVCParseValue@1@@Z ; HCParser::CParseConstant::CParseConstant
  00139	89 85 8c fa ff
	ff		 mov	 DWORD PTR tv1907[ebp], eax
  0013f	8b 8d 8c fa ff
	ff		 mov	 ecx, DWORD PTR tv1907[ebp]
  00145	89 8d 88 fa ff
	ff		 mov	 DWORD PTR tv1909[ebp], ecx
  0014b	c6 45 fc 09	 mov	 BYTE PTR __$EHRec$[ebp+8], 9
  0014f	8b 95 88 fa ff
	ff		 mov	 edx, DWORD PTR tv1909[ebp]
  00155	52		 push	 edx
  00156	b9 20 00 00 00	 mov	 ecx, OFFSET ?k_parseTunerConstants@@3QBVCParseConstant@HCParser@@B+32
  0015b	e8 00 00 00 00	 call	 ??0CParseConstant@HCParser@@QAE@ABV01@@Z
  00160	c6 45 fc 0b	 mov	 BYTE PTR __$EHRec$[ebp+8], 11 ; 0000000bH
  00164	8d 4d bc	 lea	 ecx, DWORD PTR $T362571[ebp]
  00167	e8 00 00 00 00	 call	 ??1CParseConstant@HCParser@@QAE@XZ

; 43   :     PC( _T("PHILIPS_PAL_I"),                TUNER_PHILIPS_PAL_I                ),

  0016c	83 ec 0c	 sub	 esp, 12			; 0000000cH
  0016f	8b cc		 mov	 ecx, esp
  00171	89 65 a4	 mov	 DWORD PTR $T362574[ebp], esp
  00174	6a 01		 push	 1
  00176	e8 00 00 00 00	 call	 ??0CParseValue@HCParser@@QAE@H@Z ; HCParser::CParseValue::CParseValue
  0017b	89 85 84 fa ff
	ff		 mov	 DWORD PTR tv143[ebp], eax
  00181	8b 85 84 fa ff
	ff		 mov	 eax, DWORD PTR tv143[ebp]
  00187	89 85 80 fa ff
	ff		 mov	 DWORD PTR tv1912[ebp], eax
  0018d	c6 45 fc 0c	 mov	 BYTE PTR __$EHRec$[ebp+8], 12 ; 0000000cH
  00191	68 00 00 00 00	 push	 OFFSET ??_C@_1BM@CDJFEPDA@?$AAP?$AAH?$AAI?$AAL?$AAI?$AAP?$AAS?$AA_?$AAP?$AAA?$AAL?$AA_?$AAI?$AA?$AA@
  00196	c6 45 fc 0b	 mov	 BYTE PTR __$EHRec$[ebp+8], 11 ; 0000000bH
  0019a	8d 4d a8	 lea	 ecx, DWORD PTR $T362573[ebp]
  0019d	e8 00 00 00 00	 call	 ??0CParseConstant@HCParser@@QAE@PB_WVCParseValue@1@@Z ; HCParser::CParseConstant::CParseConstant
  001a2	89 85 7c fa ff
	ff		 mov	 DWORD PTR tv1913[ebp], eax
  001a8	8b 8d 7c fa ff
	ff		 mov	 ecx, DWORD PTR tv1913[ebp]
  001ae	89 8d 78 fa ff
	ff		 mov	 DWORD PTR tv1915[ebp], ecx
  001b4	c6 45 fc 0d	 mov	 BYTE PTR __$EHRec$[ebp+8], 13 ; 0000000dH
  001b8	8b 95 78 fa ff
	ff		 mov	 edx, DWORD PTR tv1915[ebp]
  001be	52		 push	 edx
  001bf	b9 30 00 00 00	 mov	 ecx, OFFSET ?k_parseTunerConstants@@3QBVCParseConstant@HCParser@@B+48
  001c4	e8 00 00 00 00	 call	 ??0CParseConstant@HCParser@@QAE@ABV01@@Z
  001c9	c6 45 fc 0f	 mov	 BYTE PTR __$EHRec$[ebp+8], 15 ; 0000000fH
  001cd	8d 4d a8	 lea	 ecx, DWORD PTR $T362573[ebp]
  001d0	e8 00 00 00 00	 call	 ??1CParseConstant@HCParser@@QAE@XZ

; 44   :     PC( _T("PHILIPS_NTSC"),                    TUNER_PHILIPS_NTSC                ),

  001d5	83 ec 0c	 sub	 esp, 12			; 0000000cH
  001d8	8b cc		 mov	 ecx, esp
  001da	89 65 90	 mov	 DWORD PTR $T362576[ebp], esp
  001dd	6a 02		 push	 2
  001df	e8 00 00 00 00	 call	 ??0CParseValue@HCParser@@QAE@H@Z ; HCParser::CParseValue::CParseValue
  001e4	89 85 74 fa ff
	ff		 mov	 DWORD PTR tv166[ebp], eax
  001ea	8b 85 74 fa ff
	ff		 mov	 eax, DWORD PTR tv166[ebp]
  001f0	89 85 70 fa ff
	ff		 mov	 DWORD PTR tv1918[ebp], eax
  001f6	c6 45 fc 10	 mov	 BYTE PTR __$EHRec$[ebp+8], 16 ; 00000010H
  001fa	68 00 00 00 00	 push	 OFFSET ??_C@_1BK@IFFHILBA@?$AAP?$AAH?$AAI?$AAL?$AAI?$AAP?$AAS?$AA_?$AAN?$AAT?$AAS?$AAC?$AA?$AA@
  001ff	c6 45 fc 0f	 mov	 BYTE PTR __$EHRec$[ebp+8], 15 ; 0000000fH
  00203	8d 4d 94	 lea	 ecx, DWORD PTR $T362575[ebp]
  00206	e8 00 00 00 00	 call	 ??0CParseConstant@HCParser@@QAE@PB_WVCParseValue@1@@Z ; HCParser::CParseConstant::CParseConstant
  0020b	89 85 6c fa ff
	ff		 mov	 DWORD PTR tv1919[ebp], eax
  00211	8b 8d 6c fa ff
	ff		 mov	 ecx, DWORD PTR tv1919[ebp]
  00217	89 8d 68 fa ff
	ff		 mov	 DWORD PTR tv1921[ebp], ecx
  0021d	c6 45 fc 11	 mov	 BYTE PTR __$EHRec$[ebp+8], 17 ; 00000011H
  00221	8b 95 68 fa ff
	ff		 mov	 edx, DWORD PTR tv1921[ebp]
  00227	52		 push	 edx
  00228	b9 40 00 00 00	 mov	 ecx, OFFSET ?k_parseTunerConstants@@3QBVCParseConstant@HCParser@@B+64
  0022d	e8 00 00 00 00	 call	 ??0CParseConstant@HCParser@@QAE@ABV01@@Z
  00232	c6 45 fc 13	 mov	 BYTE PTR __$EHRec$[ebp+8], 19 ; 00000013H
  00236	8d 4d 94	 lea	 ecx, DWORD PTR $T362575[ebp]
  00239	e8 00 00 00 00	 call	 ??1CParseConstant@HCParser@@QAE@XZ

; 45   :     PC( _T("PHILIPS_SECAM"),                TUNER_PHILIPS_SECAM                ),

  0023e	83 ec 0c	 sub	 esp, 12			; 0000000cH
  00241	8b cc		 mov	 ecx, esp
  00243	89 a5 7c ff ff
	ff		 mov	 DWORD PTR $T362578[ebp], esp
  00249	6a 03		 push	 3
  0024b	e8 00 00 00 00	 call	 ??0CParseValue@HCParser@@QAE@H@Z ; HCParser::CParseValue::CParseValue
  00250	89 85 64 fa ff
	ff		 mov	 DWORD PTR tv189[ebp], eax
  00256	8b 85 64 fa ff
	ff		 mov	 eax, DWORD PTR tv189[ebp]
  0025c	89 85 60 fa ff
	ff		 mov	 DWORD PTR tv1924[ebp], eax
  00262	c6 45 fc 14	 mov	 BYTE PTR __$EHRec$[ebp+8], 20 ; 00000014H
  00266	68 00 00 00 00	 push	 OFFSET ??_C@_1BM@DCHONLKK@?$AAP?$AAH?$AAI?$AAL?$AAI?$AAP?$AAS?$AA_?$AAS?$AAE?$AAC?$AAA?$AAM?$AA?$AA@
  0026b	c6 45 fc 13	 mov	 BYTE PTR __$EHRec$[ebp+8], 19 ; 00000013H
  0026f	8d 4d 80	 lea	 ecx, DWORD PTR $T362577[ebp]
  00272	e8 00 00 00 00	 call	 ??0CParseConstant@HCParser@@QAE@PB_WVCParseValue@1@@Z ; HCParser::CParseConstant::CParseConstant
  00277	89 85 5c fa ff
	ff		 mov	 DWORD PTR tv1925[ebp], eax
  0027d	8b 8d 5c fa ff
	ff		 mov	 ecx, DWORD PTR tv1925[ebp]
  00283	89 8d 58 fa ff
	ff		 mov	 DWORD PTR tv1927[ebp], ecx
  00289	c6 45 fc 15	 mov	 BYTE PTR __$EHRec$[ebp+8], 21 ; 00000015H
  0028d	8b 95 58 fa ff
	ff		 mov	 edx, DWORD PTR tv1927[ebp]
  00293	52		 push	 edx
  00294	b9 50 00 00 00	 mov	 ecx, OFFSET ?k_parseTunerConstants@@3QBVCParseConstant@HCParser@@B+80
  00299	e8 00 00 00 00	 call	 ??0CParseConstant@HCParser@@QAE@ABV01@@Z
  0029e	c6 45 fc 17	 mov	 BYTE PTR __$EHRec$[ebp+8], 23 ; 00000017H
  002a2	8d 4d 80	 lea	 ecx, DWORD PTR $T362577[ebp]
  002a5	e8 00 00 00 00	 call	 ??1CParseConstant@HCParser@@QAE@XZ

; 46   :     PC( _T("PHILIPS_PAL"),                    TUNER_PHILIPS_PAL                ),

  002aa	83 ec 0c	 sub	 esp, 12			; 0000000cH
  002ad	8b cc		 mov	 ecx, esp
  002af	89 a5 68 ff ff
	ff		 mov	 DWORD PTR $T362580[ebp], esp
  002b5	6a 04		 push	 4
  002b7	e8 00 00 00 00	 call	 ??0CParseValue@HCParser@@QAE@H@Z ; HCParser::CParseValue::CParseValue
  002bc	89 85 54 fa ff
	ff		 mov	 DWORD PTR tv212[ebp], eax
  002c2	8b 85 54 fa ff
	ff		 mov	 eax, DWORD PTR tv212[ebp]
  002c8	89 85 50 fa ff
	ff		 mov	 DWORD PTR tv1930[ebp], eax
  002ce	c6 45 fc 18	 mov	 BYTE PTR __$EHRec$[ebp+8], 24 ; 00000018H
  002d2	68 00 00 00 00	 push	 OFFSET ??_C@_1BI@IKKAFKBC@?$AAP?$AAH?$AAI?$AAL?$AAI?$AAP?$AAS?$AA_?$AAP?$AAA?$AAL?$AA?$AA@
  002d7	c6 45 fc 17	 mov	 BYTE PTR __$EHRec$[ebp+8], 23 ; 00000017H
  002db	8d 8d 6c ff ff
	ff		 lea	 ecx, DWORD PTR $T362579[ebp]
  002e1	e8 00 00 00 00	 call	 ??0CParseConstant@HCParser@@QAE@PB_WVCParseValue@1@@Z ; HCParser::CParseConstant::CParseConstant
  002e6	89 85 4c fa ff
	ff		 mov	 DWORD PTR tv1931[ebp], eax
  002ec	8b 8d 4c fa ff
	ff		 mov	 ecx, DWORD PTR tv1931[ebp]
  002f2	89 8d 48 fa ff
	ff		 mov	 DWORD PTR tv1933[ebp], ecx
  002f8	c6 45 fc 19	 mov	 BYTE PTR __$EHRec$[ebp+8], 25 ; 00000019H
  002fc	8b 95 48 fa ff
	ff		 mov	 edx, DWORD PTR tv1933[ebp]
  00302	52		 push	 edx
  00303	b9 60 00 00 00	 mov	 ecx, OFFSET ?k_parseTunerConstants@@3QBVCParseConstant@HCParser@@B+96
  00308	e8 00 00 00 00	 call	 ??0CParseConstant@HCParser@@QAE@ABV01@@Z
  0030d	c6 45 fc 1b	 mov	 BYTE PTR __$EHRec$[ebp+8], 27 ; 0000001bH
  00311	8d 8d 6c ff ff
	ff		 lea	 ecx, DWORD PTR $T362579[ebp]
  00317	e8 00 00 00 00	 call	 ??1CParseConstant@HCParser@@QAE@XZ

; 47   :     PC( _T("TEMIC_4002FH5_PAL"),            TUNER_TEMIC_4002FH5_PAL            ),

  0031c	83 ec 0c	 sub	 esp, 12			; 0000000cH
  0031f	8b cc		 mov	 ecx, esp
  00321	89 a5 54 ff ff
	ff		 mov	 DWORD PTR $T362582[ebp], esp
  00327	6a 05		 push	 5
  00329	e8 00 00 00 00	 call	 ??0CParseValue@HCParser@@QAE@H@Z ; HCParser::CParseValue::CParseValue
  0032e	89 85 44 fa ff
	ff		 mov	 DWORD PTR tv235[ebp], eax
  00334	8b 85 44 fa ff
	ff		 mov	 eax, DWORD PTR tv235[ebp]
  0033a	89 85 40 fa ff
	ff		 mov	 DWORD PTR tv1936[ebp], eax
  00340	c6 45 fc 1c	 mov	 BYTE PTR __$EHRec$[ebp+8], 28 ; 0000001cH
  00344	68 00 00 00 00	 push	 OFFSET ??_C@_1CE@BHHLKEHK@?$AAT?$AAE?$AAM?$AAI?$AAC?$AA_?$AA4?$AA0?$AA0?$AA2?$AAF?$AAH?$AA5?$AA_?$AAP?$AAA?$AAL?$AA?$AA@
  00349	c6 45 fc 1b	 mov	 BYTE PTR __$EHRec$[ebp+8], 27 ; 0000001bH
  0034d	8d 8d 58 ff ff
	ff		 lea	 ecx, DWORD PTR $T362581[ebp]
  00353	e8 00 00 00 00	 call	 ??0CParseConstant@HCParser@@QAE@PB_WVCParseValue@1@@Z ; HCParser::CParseConstant::CParseConstant
  00358	89 85 3c fa ff
	ff		 mov	 DWORD PTR tv1937[ebp], eax
  0035e	8b 8d 3c fa ff
	ff		 mov	 ecx, DWORD PTR tv1937[ebp]
  00364	89 8d 38 fa ff
	ff		 mov	 DWORD PTR tv1939[ebp], ecx
  0036a	c6 45 fc 1d	 mov	 BYTE PTR __$EHRec$[ebp+8], 29 ; 0000001dH
  0036e	8b 95 38 fa ff
	ff		 mov	 edx, DWORD PTR tv1939[ebp]
  00374	52		 push	 edx
  00375	b9 70 00 00 00	 mov	 ecx, OFFSET ?k_parseTunerConstants@@3QBVCParseConstant@HCParser@@B+112
  0037a	e8 00 00 00 00	 call	 ??0CParseConstant@HCParser@@QAE@ABV01@@Z
  0037f	c6 45 fc 1f	 mov	 BYTE PTR __$EHRec$[ebp+8], 31 ; 0000001fH
  00383	8d 8d 58 ff ff
	ff		 lea	 ecx, DWORD PTR $T362581[ebp]
  00389	e8 00 00 00 00	 call	 ??1CParseConstant@HCParser@@QAE@XZ

; 48   :     PC( _T("TEMIC_4032FY5_NTSC"),            TUNER_TEMIC_4032FY5_NTSC        ),

  0038e	83 ec 0c	 sub	 esp, 12			; 0000000cH
  00391	8b cc		 mov	 ecx, esp
  00393	89 a5 40 ff ff
	ff		 mov	 DWORD PTR $T362584[ebp], esp
  00399	6a 06		 push	 6
  0039b	e8 00 00 00 00	 call	 ??0CParseValue@HCParser@@QAE@H@Z ; HCParser::CParseValue::CParseValue
  003a0	89 85 34 fa ff
	ff		 mov	 DWORD PTR tv258[ebp], eax
  003a6	8b 85 34 fa ff
	ff		 mov	 eax, DWORD PTR tv258[ebp]
  003ac	89 85 30 fa ff
	ff		 mov	 DWORD PTR tv1942[ebp], eax
  003b2	c6 45 fc 20	 mov	 BYTE PTR __$EHRec$[ebp+8], 32 ; 00000020H
  003b6	68 00 00 00 00	 push	 OFFSET ??_C@_1CG@DEBCKDA@?$AAT?$AAE?$AAM?$AAI?$AAC?$AA_?$AA4?$AA0?$AA3?$AA2?$AAF?$AAY?$AA5?$AA_?$AAN?$AAT?$AAS?$AAC?$AA?$AA@
  003bb	c6 45 fc 1f	 mov	 BYTE PTR __$EHRec$[ebp+8], 31 ; 0000001fH
  003bf	8d 8d 44 ff ff
	ff		 lea	 ecx, DWORD PTR $T362583[ebp]
  003c5	e8 00 00 00 00	 call	 ??0CParseConstant@HCParser@@QAE@PB_WVCParseValue@1@@Z ; HCParser::CParseConstant::CParseConstant
  003ca	89 85 2c fa ff
	ff		 mov	 DWORD PTR tv1943[ebp], eax
  003d0	8b 8d 2c fa ff
	ff		 mov	 ecx, DWORD PTR tv1943[ebp]
  003d6	89 8d 28 fa ff
	ff		 mov	 DWORD PTR tv1945[ebp], ecx
  003dc	c6 45 fc 21	 mov	 BYTE PTR __$EHRec$[ebp+8], 33 ; 00000021H
  003e0	8b 95 28 fa ff
	ff		 mov	 edx, DWORD PTR tv1945[ebp]
  003e6	52		 push	 edx
  003e7	b9 80 00 00 00	 mov	 ecx, OFFSET ?k_parseTunerConstants@@3QBVCParseConstant@HCParser@@B+128
  003ec	e8 00 00 00 00	 call	 ??0CParseConstant@HCParser@@QAE@ABV01@@Z
  003f1	c6 45 fc 23	 mov	 BYTE PTR __$EHRec$[ebp+8], 35 ; 00000023H
  003f5	8d 8d 44 ff ff
	ff		 lea	 ecx, DWORD PTR $T362583[ebp]
  003fb	e8 00 00 00 00	 call	 ??1CParseConstant@HCParser@@QAE@XZ

; 49   :     PC( _T("TEMIC_4062FY5_PAL_I"),            TUNER_TEMIC_4062FY5_PAL_I        ),

  00400	83 ec 0c	 sub	 esp, 12			; 0000000cH
  00403	8b cc		 mov	 ecx, esp
  00405	89 a5 2c ff ff
	ff		 mov	 DWORD PTR $T362586[ebp], esp
  0040b	6a 07		 push	 7
  0040d	e8 00 00 00 00	 call	 ??0CParseValue@HCParser@@QAE@H@Z ; HCParser::CParseValue::CParseValue
  00412	89 85 24 fa ff
	ff		 mov	 DWORD PTR tv281[ebp], eax
  00418	8b 85 24 fa ff
	ff		 mov	 eax, DWORD PTR tv281[ebp]
  0041e	89 85 20 fa ff
	ff		 mov	 DWORD PTR tv1948[ebp], eax
  00424	c6 45 fc 24	 mov	 BYTE PTR __$EHRec$[ebp+8], 36 ; 00000024H
  00428	68 00 00 00 00	 push	 OFFSET ??_C@_1CI@PPODIFIC@?$AAT?$AAE?$AAM?$AAI?$AAC?$AA_?$AA4?$AA0?$AA6?$AA2?$AAF?$AAY?$AA5?$AA_?$AAP?$AAA?$AAL?$AA_?$AAI?$AA?$AA@
  0042d	c6 45 fc 23	 mov	 BYTE PTR __$EHRec$[ebp+8], 35 ; 00000023H
  00431	8d 8d 30 ff ff
	ff		 lea	 ecx, DWORD PTR $T362585[ebp]
  00437	e8 00 00 00 00	 call	 ??0CParseConstant@HCParser@@QAE@PB_WVCParseValue@1@@Z ; HCParser::CParseConstant::CParseConstant
  0043c	89 85 1c fa ff
	ff		 mov	 DWORD PTR tv1949[ebp], eax
  00442	8b 8d 1c fa ff
	ff		 mov	 ecx, DWORD PTR tv1949[ebp]
  00448	89 8d 18 fa ff
	ff		 mov	 DWORD PTR tv1951[ebp], ecx
  0044e	c6 45 fc 25	 mov	 BYTE PTR __$EHRec$[ebp+8], 37 ; 00000025H
  00452	8b 95 18 fa ff
	ff		 mov	 edx, DWORD PTR tv1951[ebp]
  00458	52		 push	 edx
  00459	b9 90 00 00 00	 mov	 ecx, OFFSET ?k_parseTunerConstants@@3QBVCParseConstant@HCParser@@B+144
  0045e	e8 00 00 00 00	 call	 ??0CParseConstant@HCParser@@QAE@ABV01@@Z
  00463	c6 45 fc 27	 mov	 BYTE PTR __$EHRec$[ebp+8], 39 ; 00000027H
  00467	8d 8d 30 ff ff
	ff		 lea	 ecx, DWORD PTR $T362585[ebp]
  0046d	e8 00 00 00 00	 call	 ??1CParseConstant@HCParser@@QAE@XZ

; 50   :     PC( _T("TEMIC_4036FY5_NTSC"),            TUNER_TEMIC_4036FY5_NTSC        ),

  00472	83 ec 0c	 sub	 esp, 12			; 0000000cH
  00475	8b cc		 mov	 ecx, esp
  00477	89 a5 18 ff ff
	ff		 mov	 DWORD PTR $T362588[ebp], esp
  0047d	6a 08		 push	 8
  0047f	e8 00 00 00 00	 call	 ??0CParseValue@HCParser@@QAE@H@Z ; HCParser::CParseValue::CParseValue
  00484	89 85 14 fa ff
	ff		 mov	 DWORD PTR tv304[ebp], eax
  0048a	8b 85 14 fa ff
	ff		 mov	 eax, DWORD PTR tv304[ebp]
  00490	89 85 10 fa ff
	ff		 mov	 DWORD PTR tv1954[ebp], eax
  00496	c6 45 fc 28	 mov	 BYTE PTR __$EHRec$[ebp+8], 40 ; 00000028H
  0049a	68 00 00 00 00	 push	 OFFSET ??_C@_1CG@ENKMMBGJ@?$AAT?$AAE?$AAM?$AAI?$AAC?$AA_?$AA4?$AA0?$AA3?$AA6?$AAF?$AAY?$AA5?$AA_?$AAN?$AAT?$AAS?$AAC?$AA?$AA@
  0049f	c6 45 fc 27	 mov	 BYTE PTR __$EHRec$[ebp+8], 39 ; 00000027H
  004a3	8d 8d 1c ff ff
	ff		 lea	 ecx, DWORD PTR $T362587[ebp]
  004a9	e8 00 00 00 00	 call	 ??0CParseConstant@HCParser@@QAE@PB_WVCParseValue@1@@Z ; HCParser::CParseConstant::CParseConstant
  004ae	89 85 0c fa ff
	ff		 mov	 DWORD PTR tv1955[ebp], eax
  004b4	8b 8d 0c fa ff
	ff		 mov	 ecx, DWORD PTR tv1955[ebp]
  004ba	89 8d 08 fa ff
	ff		 mov	 DWORD PTR tv1957[ebp], ecx
  004c0	c6 45 fc 29	 mov	 BYTE PTR __$EHRec$[ebp+8], 41 ; 00000029H
  004c4	8b 95 08 fa ff
	ff		 mov	 edx, DWORD PTR tv1957[ebp]
  004ca	52		 push	 edx
  004cb	b9 a0 00 00 00	 mov	 ecx, OFFSET ?k_parseTunerConstants@@3QBVCParseConstant@HCParser@@B+160
  004d0	e8 00 00 00 00	 call	 ??0CParseConstant@HCParser@@QAE@ABV01@@Z
  004d5	c6 45 fc 2b	 mov	 BYTE PTR __$EHRec$[ebp+8], 43 ; 0000002bH
  004d9	8d 8d 1c ff ff
	ff		 lea	 ecx, DWORD PTR $T362587[ebp]
  004df	e8 00 00 00 00	 call	 ??1CParseConstant@HCParser@@QAE@XZ

; 51   :     PC( _T("ALPS_TSBH1_NTSC"),                TUNER_ALPS_TSBH1_NTSC            ),

  004e4	83 ec 0c	 sub	 esp, 12			; 0000000cH
  004e7	8b cc		 mov	 ecx, esp
  004e9	89 a5 04 ff ff
	ff		 mov	 DWORD PTR $T362590[ebp], esp
  004ef	6a 09		 push	 9
  004f1	e8 00 00 00 00	 call	 ??0CParseValue@HCParser@@QAE@H@Z ; HCParser::CParseValue::CParseValue
  004f6	89 85 04 fa ff
	ff		 mov	 DWORD PTR tv327[ebp], eax
  004fc	8b 85 04 fa ff
	ff		 mov	 eax, DWORD PTR tv327[ebp]
  00502	89 85 00 fa ff
	ff		 mov	 DWORD PTR tv1960[ebp], eax
  00508	c6 45 fc 2c	 mov	 BYTE PTR __$EHRec$[ebp+8], 44 ; 0000002cH
  0050c	68 00 00 00 00	 push	 OFFSET ??_C@_1CA@GOAKFAHF@?$AAA?$AAL?$AAP?$AAS?$AA_?$AAT?$AAS?$AAB?$AAH?$AA1?$AA_?$AAN?$AAT?$AAS?$AAC?$AA?$AA@
  00511	c6 45 fc 2b	 mov	 BYTE PTR __$EHRec$[ebp+8], 43 ; 0000002bH
  00515	8d 8d 08 ff ff
	ff		 lea	 ecx, DWORD PTR $T362589[ebp]
  0051b	e8 00 00 00 00	 call	 ??0CParseConstant@HCParser@@QAE@PB_WVCParseValue@1@@Z ; HCParser::CParseConstant::CParseConstant
  00520	89 85 fc f9 ff
	ff		 mov	 DWORD PTR tv1961[ebp], eax
  00526	8b 8d fc f9 ff
	ff		 mov	 ecx, DWORD PTR tv1961[ebp]
  0052c	89 8d f8 f9 ff
	ff		 mov	 DWORD PTR tv1963[ebp], ecx
  00532	c6 45 fc 2d	 mov	 BYTE PTR __$EHRec$[ebp+8], 45 ; 0000002dH
  00536	8b 95 f8 f9 ff
	ff		 mov	 edx, DWORD PTR tv1963[ebp]
  0053c	52		 push	 edx
  0053d	b9 b0 00 00 00	 mov	 ecx, OFFSET ?k_parseTunerConstants@@3QBVCParseConstant@HCParser@@B+176
  00542	e8 00 00 00 00	 call	 ??0CParseConstant@HCParser@@QAE@ABV01@@Z
  00547	c6 45 fc 2f	 mov	 BYTE PTR __$EHRec$[ebp+8], 47 ; 0000002fH
  0054b	8d 8d 08 ff ff
	ff		 lea	 ecx, DWORD PTR $T362589[ebp]
  00551	e8 00 00 00 00	 call	 ??1CParseConstant@HCParser@@QAE@XZ

; 52   :     PC( _T("ALPS_TSBE1_PAL"),                TUNER_ALPS_TSBE1_PAL            ),

  00556	83 ec 0c	 sub	 esp, 12			; 0000000cH
  00559	8b cc		 mov	 ecx, esp
  0055b	89 a5 f0 fe ff
	ff		 mov	 DWORD PTR $T362592[ebp], esp
  00561	6a 0a		 push	 10			; 0000000aH
  00563	e8 00 00 00 00	 call	 ??0CParseValue@HCParser@@QAE@H@Z ; HCParser::CParseValue::CParseValue
  00568	89 85 f4 f9 ff
	ff		 mov	 DWORD PTR tv350[ebp], eax
  0056e	8b 85 f4 f9 ff
	ff		 mov	 eax, DWORD PTR tv350[ebp]
  00574	89 85 f0 f9 ff
	ff		 mov	 DWORD PTR tv1966[ebp], eax
  0057a	c6 45 fc 30	 mov	 BYTE PTR __$EHRec$[ebp+8], 48 ; 00000030H
  0057e	68 00 00 00 00	 push	 OFFSET ??_C@_1BO@GDJDNPLL@?$AAA?$AAL?$AAP?$AAS?$AA_?$AAT?$AAS?$AAB?$AAE?$AA1?$AA_?$AAP?$AAA?$AAL?$AA?$AA@
  00583	c6 45 fc 2f	 mov	 BYTE PTR __$EHRec$[ebp+8], 47 ; 0000002fH
  00587	8d 8d f4 fe ff
	ff		 lea	 ecx, DWORD PTR $T362591[ebp]
  0058d	e8 00 00 00 00	 call	 ??0CParseConstant@HCParser@@QAE@PB_WVCParseValue@1@@Z ; HCParser::CParseConstant::CParseConstant
  00592	89 85 ec f9 ff
	ff		 mov	 DWORD PTR tv1967[ebp], eax
  00598	8b 8d ec f9 ff
	ff		 mov	 ecx, DWORD PTR tv1967[ebp]
  0059e	89 8d e8 f9 ff
	ff		 mov	 DWORD PTR tv1969[ebp], ecx
  005a4	c6 45 fc 31	 mov	 BYTE PTR __$EHRec$[ebp+8], 49 ; 00000031H
  005a8	8b 95 e8 f9 ff
	ff		 mov	 edx, DWORD PTR tv1969[ebp]
  005ae	52		 push	 edx
  005af	b9 c0 00 00 00	 mov	 ecx, OFFSET ?k_parseTunerConstants@@3QBVCParseConstant@HCParser@@B+192
  005b4	e8 00 00 00 00	 call	 ??0CParseConstant@HCParser@@QAE@ABV01@@Z
  005b9	c6 45 fc 33	 mov	 BYTE PTR __$EHRec$[ebp+8], 51 ; 00000033H
  005bd	8d 8d f4 fe ff
	ff		 lea	 ecx, DWORD PTR $T362591[ebp]
  005c3	e8 00 00 00 00	 call	 ??1CParseConstant@HCParser@@QAE@XZ

; 53   :     PC( _T("ALPS_TSBB5_PAL_I"),                TUNER_ALPS_TSBB5_PAL_I            ),

  005c8	83 ec 0c	 sub	 esp, 12			; 0000000cH
  005cb	8b cc		 mov	 ecx, esp
  005cd	89 a5 dc fe ff
	ff		 mov	 DWORD PTR $T362594[ebp], esp
  005d3	6a 0b		 push	 11			; 0000000bH
  005d5	e8 00 00 00 00	 call	 ??0CParseValue@HCParser@@QAE@H@Z ; HCParser::CParseValue::CParseValue
  005da	89 85 e4 f9 ff
	ff		 mov	 DWORD PTR tv373[ebp], eax
  005e0	8b 85 e4 f9 ff
	ff		 mov	 eax, DWORD PTR tv373[ebp]
  005e6	89 85 e0 f9 ff
	ff		 mov	 DWORD PTR tv1972[ebp], eax
  005ec	c6 45 fc 34	 mov	 BYTE PTR __$EHRec$[ebp+8], 52 ; 00000034H
  005f0	68 00 00 00 00	 push	 OFFSET ??_C@_1CC@OMKKLJNL@?$AAA?$AAL?$AAP?$AAS?$AA_?$AAT?$AAS?$AAB?$AAB?$AA5?$AA_?$AAP?$AAA?$AAL?$AA_?$AAI?$AA?$AA@
  005f5	c6 45 fc 33	 mov	 BYTE PTR __$EHRec$[ebp+8], 51 ; 00000033H
  005f9	8d 8d e0 fe ff
	ff		 lea	 ecx, DWORD PTR $T362593[ebp]
  005ff	e8 00 00 00 00	 call	 ??0CParseConstant@HCParser@@QAE@PB_WVCParseValue@1@@Z ; HCParser::CParseConstant::CParseConstant
  00604	89 85 dc f9 ff
	ff		 mov	 DWORD PTR tv1973[ebp], eax
  0060a	8b 8d dc f9 ff
	ff		 mov	 ecx, DWORD PTR tv1973[ebp]
  00610	89 8d d8 f9 ff
	ff		 mov	 DWORD PTR tv1975[ebp], ecx
  00616	c6 45 fc 35	 mov	 BYTE PTR __$EHRec$[ebp+8], 53 ; 00000035H
  0061a	8b 95 d8 f9 ff
	ff		 mov	 edx, DWORD PTR tv1975[ebp]
  00620	52		 push	 edx
  00621	b9 d0 00 00 00	 mov	 ecx, OFFSET ?k_parseTunerConstants@@3QBVCParseConstant@HCParser@@B+208
  00626	e8 00 00 00 00	 call	 ??0CParseConstant@HCParser@@QAE@ABV01@@Z
  0062b	c6 45 fc 37	 mov	 BYTE PTR __$EHRec$[ebp+8], 55 ; 00000037H
  0062f	8d 8d e0 fe ff
	ff		 lea	 ecx, DWORD PTR $T362593[ebp]
  00635	e8 00 00 00 00	 call	 ??1CParseConstant@HCParser@@QAE@XZ

; 54   :     PC( _T("ALPS_TSBE5_PAL"),                TUNER_ALPS_TSBE5_PAL            ),

  0063a	83 ec 0c	 sub	 esp, 12			; 0000000cH
  0063d	8b cc		 mov	 ecx, esp
  0063f	89 a5 c8 fe ff
	ff		 mov	 DWORD PTR $T362596[ebp], esp
  00645	6a 0c		 push	 12			; 0000000cH
  00647	e8 00 00 00 00	 call	 ??0CParseValue@HCParser@@QAE@H@Z ; HCParser::CParseValue::CParseValue
  0064c	89 85 d4 f9 ff
	ff		 mov	 DWORD PTR tv396[ebp], eax
  00652	8b 85 d4 f9 ff
	ff		 mov	 eax, DWORD PTR tv396[ebp]
  00658	89 85 d0 f9 ff
	ff		 mov	 DWORD PTR tv1978[ebp], eax
  0065e	c6 45 fc 38	 mov	 BYTE PTR __$EHRec$[ebp+8], 56 ; 00000038H
  00662	68 00 00 00 00	 push	 OFFSET ??_C@_1BO@GAJFOEME@?$AAA?$AAL?$AAP?$AAS?$AA_?$AAT?$AAS?$AAB?$AAE?$AA5?$AA_?$AAP?$AAA?$AAL?$AA?$AA@
  00667	c6 45 fc 37	 mov	 BYTE PTR __$EHRec$[ebp+8], 55 ; 00000037H
  0066b	8d 8d cc fe ff
	ff		 lea	 ecx, DWORD PTR $T362595[ebp]
  00671	e8 00 00 00 00	 call	 ??0CParseConstant@HCParser@@QAE@PB_WVCParseValue@1@@Z ; HCParser::CParseConstant::CParseConstant
  00676	89 85 cc f9 ff
	ff		 mov	 DWORD PTR tv1979[ebp], eax
  0067c	8b 8d cc f9 ff
	ff		 mov	 ecx, DWORD PTR tv1979[ebp]
  00682	89 8d c8 f9 ff
	ff		 mov	 DWORD PTR tv1981[ebp], ecx
  00688	c6 45 fc 39	 mov	 BYTE PTR __$EHRec$[ebp+8], 57 ; 00000039H
  0068c	8b 95 c8 f9 ff
	ff		 mov	 edx, DWORD PTR tv1981[ebp]
  00692	52		 push	 edx
  00693	b9 e0 00 00 00	 mov	 ecx, OFFSET ?k_parseTunerConstants@@3QBVCParseConstant@HCParser@@B+224
  00698	e8 00 00 00 00	 call	 ??0CParseConstant@HCParser@@QAE@ABV01@@Z
  0069d	c6 45 fc 3b	 mov	 BYTE PTR __$EHRec$[ebp+8], 59 ; 0000003bH
  006a1	8d 8d cc fe ff
	ff		 lea	 ecx, DWORD PTR $T362595[ebp]
  006a7	e8 00 00 00 00	 call	 ??1CParseConstant@HCParser@@QAE@XZ

; 55   :     PC( _T("ALPS_TSBC5_PAL"),                TUNER_ALPS_TSBC5_PAL            ),

  006ac	83 ec 0c	 sub	 esp, 12			; 0000000cH
  006af	8b cc		 mov	 ecx, esp
  006b1	89 a5 b4 fe ff
	ff		 mov	 DWORD PTR $T362598[ebp], esp
  006b7	6a 0d		 push	 13			; 0000000dH
  006b9	e8 00 00 00 00	 call	 ??0CParseValue@HCParser@@QAE@H@Z ; HCParser::CParseValue::CParseValue
  006be	89 85 c4 f9 ff
	ff		 mov	 DWORD PTR tv419[ebp], eax
  006c4	8b 85 c4 f9 ff
	ff		 mov	 eax, DWORD PTR tv419[ebp]
  006ca	89 85 c0 f9 ff
	ff		 mov	 DWORD PTR tv1984[ebp], eax
  006d0	c6 45 fc 3c	 mov	 BYTE PTR __$EHRec$[ebp+8], 60 ; 0000003cH
  006d4	68 00 00 00 00	 push	 OFFSET ??_C@_1BO@JIFHKPHC@?$AAA?$AAL?$AAP?$AAS?$AA_?$AAT?$AAS?$AAB?$AAC?$AA5?$AA_?$AAP?$AAA?$AAL?$AA?$AA@
  006d9	c6 45 fc 3b	 mov	 BYTE PTR __$EHRec$[ebp+8], 59 ; 0000003bH
  006dd	8d 8d b8 fe ff
	ff		 lea	 ecx, DWORD PTR $T362597[ebp]
  006e3	e8 00 00 00 00	 call	 ??0CParseConstant@HCParser@@QAE@PB_WVCParseValue@1@@Z ; HCParser::CParseConstant::CParseConstant
  006e8	89 85 bc f9 ff
	ff		 mov	 DWORD PTR tv1985[ebp], eax
  006ee	8b 8d bc f9 ff
	ff		 mov	 ecx, DWORD PTR tv1985[ebp]
  006f4	89 8d b8 f9 ff
	ff		 mov	 DWORD PTR tv1987[ebp], ecx
  006fa	c6 45 fc 3d	 mov	 BYTE PTR __$EHRec$[ebp+8], 61 ; 0000003dH
  006fe	8b 95 b8 f9 ff
	ff		 mov	 edx, DWORD PTR tv1987[ebp]
  00704	52		 push	 edx
  00705	b9 f0 00 00 00	 mov	 ecx, OFFSET ?k_parseTunerConstants@@3QBVCParseConstant@HCParser@@B+240
  0070a	e8 00 00 00 00	 call	 ??0CParseConstant@HCParser@@QAE@ABV01@@Z
  0070f	c6 45 fc 3f	 mov	 BYTE PTR __$EHRec$[ebp+8], 63 ; 0000003fH
  00713	8d 8d b8 fe ff
	ff		 lea	 ecx, DWORD PTR $T362597[ebp]
  00719	e8 00 00 00 00	 call	 ??1CParseConstant@HCParser@@QAE@XZ

; 56   :     PC( _T("TEMIC_4006FH5_PAL"),            TUNER_TEMIC_4006FH5_PAL            ),

  0071e	83 ec 0c	 sub	 esp, 12			; 0000000cH
  00721	8b cc		 mov	 ecx, esp
  00723	89 a5 a0 fe ff
	ff		 mov	 DWORD PTR $T362600[ebp], esp
  00729	6a 0e		 push	 14			; 0000000eH
  0072b	e8 00 00 00 00	 call	 ??0CParseValue@HCParser@@QAE@H@Z ; HCParser::CParseValue::CParseValue
  00730	89 85 b4 f9 ff
	ff		 mov	 DWORD PTR tv442[ebp], eax
  00736	8b 85 b4 f9 ff
	ff		 mov	 eax, DWORD PTR tv442[ebp]
  0073c	89 85 b0 f9 ff
	ff		 mov	 DWORD PTR tv1990[ebp], eax
  00742	c6 45 fc 40	 mov	 BYTE PTR __$EHRec$[ebp+8], 64 ; 00000040H
  00746	68 00 00 00 00	 push	 OFFSET ??_C@_1CE@BMNDHDHM@?$AAT?$AAE?$AAM?$AAI?$AAC?$AA_?$AA4?$AA0?$AA0?$AA6?$AAF?$AAH?$AA5?$AA_?$AAP?$AAA?$AAL?$AA?$AA@
  0074b	c6 45 fc 3f	 mov	 BYTE PTR __$EHRec$[ebp+8], 63 ; 0000003fH
  0074f	8d 8d a4 fe ff
	ff		 lea	 ecx, DWORD PTR $T362599[ebp]
  00755	e8 00 00 00 00	 call	 ??0CParseConstant@HCParser@@QAE@PB_WVCParseValue@1@@Z ; HCParser::CParseConstant::CParseConstant
  0075a	89 85 ac f9 ff
	ff		 mov	 DWORD PTR tv1991[ebp], eax
  00760	8b 8d ac f9 ff
	ff		 mov	 ecx, DWORD PTR tv1991[ebp]
  00766	89 8d a8 f9 ff
	ff		 mov	 DWORD PTR tv1993[ebp], ecx
  0076c	c6 45 fc 41	 mov	 BYTE PTR __$EHRec$[ebp+8], 65 ; 00000041H
  00770	8b 95 a8 f9 ff
	ff		 mov	 edx, DWORD PTR tv1993[ebp]
  00776	52		 push	 edx
  00777	b9 00 01 00 00	 mov	 ecx, OFFSET ?k_parseTunerConstants@@3QBVCParseConstant@HCParser@@B+256
  0077c	e8 00 00 00 00	 call	 ??0CParseConstant@HCParser@@QAE@ABV01@@Z
  00781	c6 45 fc 43	 mov	 BYTE PTR __$EHRec$[ebp+8], 67 ; 00000043H
  00785	8d 8d a4 fe ff
	ff		 lea	 ecx, DWORD PTR $T362599[ebp]
  0078b	e8 00 00 00 00	 call	 ??1CParseConstant@HCParser@@QAE@XZ

; 57   :     PC( _T("PHILIPS_1236D_NTSC_INPUT1"),    TUNER_PHILIPS_1236D_NTSC_INPUT1    ),

  00790	83 ec 0c	 sub	 esp, 12			; 0000000cH
  00793	8b cc		 mov	 ecx, esp
  00795	89 a5 8c fe ff
	ff		 mov	 DWORD PTR $T362602[ebp], esp
  0079b	6a 0f		 push	 15			; 0000000fH
  0079d	e8 00 00 00 00	 call	 ??0CParseValue@HCParser@@QAE@H@Z ; HCParser::CParseValue::CParseValue
  007a2	89 85 a4 f9 ff
	ff		 mov	 DWORD PTR tv497[ebp], eax
  007a8	8b 85 a4 f9 ff
	ff		 mov	 eax, DWORD PTR tv497[ebp]
  007ae	89 85 a0 f9 ff
	ff		 mov	 DWORD PTR tv1996[ebp], eax
  007b4	c6 45 fc 44	 mov	 BYTE PTR __$EHRec$[ebp+8], 68 ; 00000044H
  007b8	68 00 00 00 00	 push	 OFFSET ??_C@_1DE@NOEBAKJF@?$AAP?$AAH?$AAI?$AAL?$AAI?$AAP?$AAS?$AA_?$AA1?$AA2?$AA3?$AA6?$AAD?$AA_?$AAN?$AAT?$AAS?$AAC?$AA_?$AAI?$AAN?$AAP?$AAU?$AAT?$AA1?$AA?$AA@
  007bd	c6 45 fc 43	 mov	 BYTE PTR __$EHRec$[ebp+8], 67 ; 00000043H
  007c1	8d 8d 90 fe ff
	ff		 lea	 ecx, DWORD PTR $T362601[ebp]
  007c7	e8 00 00 00 00	 call	 ??0CParseConstant@HCParser@@QAE@PB_WVCParseValue@1@@Z ; HCParser::CParseConstant::CParseConstant
  007cc	89 85 9c f9 ff
	ff		 mov	 DWORD PTR tv1997[ebp], eax
  007d2	8b 8d 9c f9 ff
	ff		 mov	 ecx, DWORD PTR tv1997[ebp]
  007d8	89 8d 98 f9 ff
	ff		 mov	 DWORD PTR tv1999[ebp], ecx
  007de	c6 45 fc 45	 mov	 BYTE PTR __$EHRec$[ebp+8], 69 ; 00000045H
  007e2	8b 95 98 f9 ff
	ff		 mov	 edx, DWORD PTR tv1999[ebp]
  007e8	52		 push	 edx
  007e9	b9 10 01 00 00	 mov	 ecx, OFFSET ?k_parseTunerConstants@@3QBVCParseConstant@HCParser@@B+272
  007ee	e8 00 00 00 00	 call	 ??0CParseConstant@HCParser@@QAE@ABV01@@Z
  007f3	c6 45 fc 47	 mov	 BYTE PTR __$EHRec$[ebp+8], 71 ; 00000047H
  007f7	8d 8d 90 fe ff
	ff		 lea	 ecx, DWORD PTR $T362601[ebp]
  007fd	e8 00 00 00 00	 call	 ??1CParseConstant@HCParser@@QAE@XZ

; 58   :     PC( _T("PHILIPS_1236D_NTSC_INPUT2"),    TUNER_PHILIPS_1236D_NTSC_INPUT2    ),

  00802	83 ec 0c	 sub	 esp, 12			; 0000000cH
  00805	8b cc		 mov	 ecx, esp
  00807	89 a5 78 fe ff
	ff		 mov	 DWORD PTR $T362604[ebp], esp
  0080d	6a 10		 push	 16			; 00000010H
  0080f	e8 00 00 00 00	 call	 ??0CParseValue@HCParser@@QAE@H@Z ; HCParser::CParseValue::CParseValue
  00814	89 85 94 f9 ff
	ff		 mov	 DWORD PTR tv552[ebp], eax
  0081a	8b 85 94 f9 ff
	ff		 mov	 eax, DWORD PTR tv552[ebp]
  00820	89 85 90 f9 ff
	ff		 mov	 DWORD PTR tv2002[ebp], eax
  00826	c6 45 fc 48	 mov	 BYTE PTR __$EHRec$[ebp+8], 72 ; 00000048H
  0082a	68 00 00 00 00	 push	 OFFSET ??_C@_1DE@MMPEKFHL@?$AAP?$AAH?$AAI?$AAL?$AAI?$AAP?$AAS?$AA_?$AA1?$AA2?$AA3?$AA6?$AAD?$AA_?$AAN?$AAT?$AAS?$AAC?$AA_?$AAI?$AAN?$AAP?$AAU?$AAT?$AA2?$AA?$AA@
  0082f	c6 45 fc 47	 mov	 BYTE PTR __$EHRec$[ebp+8], 71 ; 00000047H
  00833	8d 8d 7c fe ff
	ff		 lea	 ecx, DWORD PTR $T362603[ebp]
  00839	e8 00 00 00 00	 call	 ??0CParseConstant@HCParser@@QAE@PB_WVCParseValue@1@@Z ; HCParser::CParseConstant::CParseConstant
  0083e	89 85 8c f9 ff
	ff		 mov	 DWORD PTR tv2003[ebp], eax
  00844	8b 8d 8c f9 ff
	ff		 mov	 ecx, DWORD PTR tv2003[ebp]
  0084a	89 8d 88 f9 ff
	ff		 mov	 DWORD PTR tv2005[ebp], ecx
  00850	c6 45 fc 49	 mov	 BYTE PTR __$EHRec$[ebp+8], 73 ; 00000049H
  00854	8b 95 88 f9 ff
	ff		 mov	 edx, DWORD PTR tv2005[ebp]
  0085a	52		 push	 edx
  0085b	b9 20 01 00 00	 mov	 ecx, OFFSET ?k_parseTunerConstants@@3QBVCParseConstant@HCParser@@B+288
  00860	e8 00 00 00 00	 call	 ??0CParseConstant@HCParser@@QAE@ABV01@@Z
  00865	c6 45 fc 4b	 mov	 BYTE PTR __$EHRec$[ebp+8], 75 ; 0000004bH
  00869	8d 8d 7c fe ff
	ff		 lea	 ecx, DWORD PTR $T362603[ebp]
  0086f	e8 00 00 00 00	 call	 ??1CParseConstant@HCParser@@QAE@XZ

; 59   :     PC( _T("ALPS_TSCH6_NTSC"),                TUNER_ALPS_TSCH6_NTSC            ),

  00874	83 ec 0c	 sub	 esp, 12			; 0000000cH
  00877	8b cc		 mov	 ecx, esp
  00879	89 a5 64 fe ff
	ff		 mov	 DWORD PTR $T362606[ebp], esp
  0087f	6a 11		 push	 17			; 00000011H
  00881	e8 00 00 00 00	 call	 ??0CParseValue@HCParser@@QAE@H@Z ; HCParser::CParseValue::CParseValue
  00886	89 85 84 f9 ff
	ff		 mov	 DWORD PTR tv575[ebp], eax
  0088c	8b 85 84 f9 ff
	ff		 mov	 eax, DWORD PTR tv575[ebp]
  00892	89 85 80 f9 ff
	ff		 mov	 DWORD PTR tv2008[ebp], eax
  00898	c6 45 fc 4c	 mov	 BYTE PTR __$EHRec$[ebp+8], 76 ; 0000004cH
  0089c	68 00 00 00 00	 push	 OFFSET ??_C@_1CA@OEJFEMFE@?$AAA?$AAL?$AAP?$AAS?$AA_?$AAT?$AAS?$AAC?$AAH?$AA6?$AA_?$AAN?$AAT?$AAS?$AAC?$AA?$AA@
  008a1	c6 45 fc 4b	 mov	 BYTE PTR __$EHRec$[ebp+8], 75 ; 0000004bH
  008a5	8d 8d 68 fe ff
	ff		 lea	 ecx, DWORD PTR $T362605[ebp]
  008ab	e8 00 00 00 00	 call	 ??0CParseConstant@HCParser@@QAE@PB_WVCParseValue@1@@Z ; HCParser::CParseConstant::CParseConstant
  008b0	89 85 7c f9 ff
	ff		 mov	 DWORD PTR tv2009[ebp], eax
  008b6	8b 8d 7c f9 ff
	ff		 mov	 ecx, DWORD PTR tv2009[ebp]
  008bc	89 8d 78 f9 ff
	ff		 mov	 DWORD PTR tv2011[ebp], ecx
  008c2	c6 45 fc 4d	 mov	 BYTE PTR __$EHRec$[ebp+8], 77 ; 0000004dH
  008c6	8b 95 78 f9 ff
	ff		 mov	 edx, DWORD PTR tv2011[ebp]
  008cc	52		 push	 edx
  008cd	b9 30 01 00 00	 mov	 ecx, OFFSET ?k_parseTunerConstants@@3QBVCParseConstant@HCParser@@B+304
  008d2	e8 00 00 00 00	 call	 ??0CParseConstant@HCParser@@QAE@ABV01@@Z
  008d7	c6 45 fc 4f	 mov	 BYTE PTR __$EHRec$[ebp+8], 79 ; 0000004fH
  008db	8d 8d 68 fe ff
	ff		 lea	 ecx, DWORD PTR $T362605[ebp]
  008e1	e8 00 00 00 00	 call	 ??1CParseConstant@HCParser@@QAE@XZ

; 60   :     PC( _T("TEMIC_4016FY5_PAL"),            TUNER_TEMIC_4016FY5_PAL            ),

  008e6	83 ec 0c	 sub	 esp, 12			; 0000000cH
  008e9	8b cc		 mov	 ecx, esp
  008eb	89 a5 50 fe ff
	ff		 mov	 DWORD PTR $T362608[ebp], esp
  008f1	6a 12		 push	 18			; 00000012H
  008f3	e8 00 00 00 00	 call	 ??0CParseValue@HCParser@@QAE@H@Z ; HCParser::CParseValue::CParseValue
  008f8	89 85 74 f9 ff
	ff		 mov	 DWORD PTR tv598[ebp], eax
  008fe	8b 85 74 f9 ff
	ff		 mov	 eax, DWORD PTR tv598[ebp]
  00904	89 85 70 f9 ff
	ff		 mov	 DWORD PTR tv2014[ebp], eax
  0090a	c6 45 fc 50	 mov	 BYTE PTR __$EHRec$[ebp+8], 80 ; 00000050H
  0090e	68 00 00 00 00	 push	 OFFSET ??_C@_1CE@ICAJJFCA@?$AAT?$AAE?$AAM?$AAI?$AAC?$AA_?$AA4?$AA0?$AA1?$AA6?$AAF?$AAY?$AA5?$AA_?$AAP?$AAA?$AAL?$AA?$AA@
  00913	c6 45 fc 4f	 mov	 BYTE PTR __$EHRec$[ebp+8], 79 ; 0000004fH
  00917	8d 8d 54 fe ff
	ff		 lea	 ecx, DWORD PTR $T362607[ebp]
  0091d	e8 00 00 00 00	 call	 ??0CParseConstant@HCParser@@QAE@PB_WVCParseValue@1@@Z ; HCParser::CParseConstant::CParseConstant
  00922	89 85 6c f9 ff
	ff		 mov	 DWORD PTR tv2015[ebp], eax
  00928	8b 8d 6c f9 ff
	ff		 mov	 ecx, DWORD PTR tv2015[ebp]
  0092e	89 8d 68 f9 ff
	ff		 mov	 DWORD PTR tv2017[ebp], ecx
  00934	c6 45 fc 51	 mov	 BYTE PTR __$EHRec$[ebp+8], 81 ; 00000051H
  00938	8b 95 68 f9 ff
	ff		 mov	 edx, DWORD PTR tv2017[ebp]
  0093e	52		 push	 edx
  0093f	b9 40 01 00 00	 mov	 ecx, OFFSET ?k_parseTunerConstants@@3QBVCParseConstant@HCParser@@B+320
  00944	e8 00 00 00 00	 call	 ??0CParseConstant@HCParser@@QAE@ABV01@@Z
  00949	c6 45 fc 53	 mov	 BYTE PTR __$EHRec$[ebp+8], 83 ; 00000053H
  0094d	8d 8d 54 fe ff
	ff		 lea	 ecx, DWORD PTR $T362607[ebp]
  00953	e8 00 00 00 00	 call	 ??1CParseConstant@HCParser@@QAE@XZ

; 61   :     PC( _T("PHILIPS_MK2_NTSC"),                TUNER_PHILIPS_MK2_NTSC            ),

  00958	83 ec 0c	 sub	 esp, 12			; 0000000cH
  0095b	8b cc		 mov	 ecx, esp
  0095d	89 a5 3c fe ff
	ff		 mov	 DWORD PTR $T362610[ebp], esp
  00963	6a 13		 push	 19			; 00000013H
  00965	e8 00 00 00 00	 call	 ??0CParseValue@HCParser@@QAE@H@Z ; HCParser::CParseValue::CParseValue
  0096a	89 85 64 f9 ff
	ff		 mov	 DWORD PTR tv621[ebp], eax
  00970	8b 85 64 f9 ff
	ff		 mov	 eax, DWORD PTR tv621[ebp]
  00976	89 85 60 f9 ff
	ff		 mov	 DWORD PTR tv2020[ebp], eax
  0097c	c6 45 fc 54	 mov	 BYTE PTR __$EHRec$[ebp+8], 84 ; 00000054H
  00980	68 00 00 00 00	 push	 OFFSET ??_C@_1CC@FGAIIFMP@?$AAP?$AAH?$AAI?$AAL?$AAI?$AAP?$AAS?$AA_?$AAM?$AAK?$AA2?$AA_?$AAN?$AAT?$AAS?$AAC?$AA?$AA@
  00985	c6 45 fc 53	 mov	 BYTE PTR __$EHRec$[ebp+8], 83 ; 00000053H
  00989	8d 8d 40 fe ff
	ff		 lea	 ecx, DWORD PTR $T362609[ebp]
  0098f	e8 00 00 00 00	 call	 ??0CParseConstant@HCParser@@QAE@PB_WVCParseValue@1@@Z ; HCParser::CParseConstant::CParseConstant
  00994	89 85 5c f9 ff
	ff		 mov	 DWORD PTR tv2021[ebp], eax
  0099a	8b 8d 5c f9 ff
	ff		 mov	 ecx, DWORD PTR tv2021[ebp]
  009a0	89 8d 58 f9 ff
	ff		 mov	 DWORD PTR tv2023[ebp], ecx
  009a6	c6 45 fc 55	 mov	 BYTE PTR __$EHRec$[ebp+8], 85 ; 00000055H
  009aa	8b 95 58 f9 ff
	ff		 mov	 edx, DWORD PTR tv2023[ebp]
  009b0	52		 push	 edx
  009b1	b9 50 01 00 00	 mov	 ecx, OFFSET ?k_parseTunerConstants@@3QBVCParseConstant@HCParser@@B+336
  009b6	e8 00 00 00 00	 call	 ??0CParseConstant@HCParser@@QAE@ABV01@@Z
  009bb	c6 45 fc 57	 mov	 BYTE PTR __$EHRec$[ebp+8], 87 ; 00000057H
  009bf	8d 8d 40 fe ff
	ff		 lea	 ecx, DWORD PTR $T362609[ebp]
  009c5	e8 00 00 00 00	 call	 ??1CParseConstant@HCParser@@QAE@XZ

; 62   :     PC( _T("TEMIC_4066FY5_PAL_I"),            TUNER_TEMIC_4066FY5_PAL_I        ),

  009ca	83 ec 0c	 sub	 esp, 12			; 0000000cH
  009cd	8b cc		 mov	 ecx, esp
  009cf	89 a5 28 fe ff
	ff		 mov	 DWORD PTR $T362612[ebp], esp
  009d5	6a 14		 push	 20			; 00000014H
  009d7	e8 00 00 00 00	 call	 ??0CParseValue@HCParser@@QAE@H@Z ; HCParser::CParseValue::CParseValue
  009dc	89 85 54 f9 ff
	ff		 mov	 DWORD PTR tv644[ebp], eax
  009e2	8b 85 54 f9 ff
	ff		 mov	 eax, DWORD PTR tv644[ebp]
  009e8	89 85 50 f9 ff
	ff		 mov	 DWORD PTR tv2026[ebp], eax
  009ee	c6 45 fc 58	 mov	 BYTE PTR __$EHRec$[ebp+8], 88 ; 00000058H
  009f2	68 00 00 00 00	 push	 OFFSET ??_C@_1CI@KDECBGIC@?$AAT?$AAE?$AAM?$AAI?$AAC?$AA_?$AA4?$AA0?$AA6?$AA6?$AAF?$AAY?$AA5?$AA_?$AAP?$AAA?$AAL?$AA_?$AAI?$AA?$AA@
  009f7	c6 45 fc 57	 mov	 BYTE PTR __$EHRec$[ebp+8], 87 ; 00000057H
  009fb	8d 8d 2c fe ff
	ff		 lea	 ecx, DWORD PTR $T362611[ebp]
  00a01	e8 00 00 00 00	 call	 ??0CParseConstant@HCParser@@QAE@PB_WVCParseValue@1@@Z ; HCParser::CParseConstant::CParseConstant
  00a06	89 85 4c f9 ff
	ff		 mov	 DWORD PTR tv2027[ebp], eax
  00a0c	8b 8d 4c f9 ff
	ff		 mov	 ecx, DWORD PTR tv2027[ebp]
  00a12	89 8d 48 f9 ff
	ff		 mov	 DWORD PTR tv2029[ebp], ecx
  00a18	c6 45 fc 59	 mov	 BYTE PTR __$EHRec$[ebp+8], 89 ; 00000059H
  00a1c	8b 95 48 f9 ff
	ff		 mov	 edx, DWORD PTR tv2029[ebp]
  00a22	52		 push	 edx
  00a23	b9 60 01 00 00	 mov	 ecx, OFFSET ?k_parseTunerConstants@@3QBVCParseConstant@HCParser@@B+352
  00a28	e8 00 00 00 00	 call	 ??0CParseConstant@HCParser@@QAE@ABV01@@Z
  00a2d	c6 45 fc 5b	 mov	 BYTE PTR __$EHRec$[ebp+8], 91 ; 0000005bH
  00a31	8d 8d 2c fe ff
	ff		 lea	 ecx, DWORD PTR $T362611[ebp]
  00a37	e8 00 00 00 00	 call	 ??1CParseConstant@HCParser@@QAE@XZ

; 63   :     PC( _T("TEMIC_4006FN5_PAL"),            TUNER_TEMIC_4006FN5_PAL            ),

  00a3c	83 ec 0c	 sub	 esp, 12			; 0000000cH
  00a3f	8b cc		 mov	 ecx, esp
  00a41	89 a5 14 fe ff
	ff		 mov	 DWORD PTR $T362614[ebp], esp
  00a47	6a 15		 push	 21			; 00000015H
  00a49	e8 00 00 00 00	 call	 ??0CParseValue@HCParser@@QAE@H@Z ; HCParser::CParseValue::CParseValue
  00a4e	89 85 44 f9 ff
	ff		 mov	 DWORD PTR tv667[ebp], eax
  00a54	8b 85 44 f9 ff
	ff		 mov	 eax, DWORD PTR tv667[ebp]
  00a5a	89 85 40 f9 ff
	ff		 mov	 DWORD PTR tv2032[ebp], eax
  00a60	c6 45 fc 5c	 mov	 BYTE PTR __$EHRec$[ebp+8], 92 ; 0000005cH
  00a64	68 00 00 00 00	 push	 OFFSET ??_C@_1CE@OEBBDIMK@?$AAT?$AAE?$AAM?$AAI?$AAC?$AA_?$AA4?$AA0?$AA0?$AA6?$AAF?$AAN?$AA5?$AA_?$AAP?$AAA?$AAL?$AA?$AA@
  00a69	c6 45 fc 5b	 mov	 BYTE PTR __$EHRec$[ebp+8], 91 ; 0000005bH
  00a6d	8d 8d 18 fe ff
	ff		 lea	 ecx, DWORD PTR $T362613[ebp]
  00a73	e8 00 00 00 00	 call	 ??0CParseConstant@HCParser@@QAE@PB_WVCParseValue@1@@Z ; HCParser::CParseConstant::CParseConstant
  00a78	89 85 3c f9 ff
	ff		 mov	 DWORD PTR tv2033[ebp], eax
  00a7e	8b 8d 3c f9 ff
	ff		 mov	 ecx, DWORD PTR tv2033[ebp]
  00a84	89 8d 38 f9 ff
	ff		 mov	 DWORD PTR tv2035[ebp], ecx
  00a8a	c6 45 fc 5d	 mov	 BYTE PTR __$EHRec$[ebp+8], 93 ; 0000005dH
  00a8e	8b 95 38 f9 ff
	ff		 mov	 edx, DWORD PTR tv2035[ebp]
  00a94	52		 push	 edx
  00a95	b9 70 01 00 00	 mov	 ecx, OFFSET ?k_parseTunerConstants@@3QBVCParseConstant@HCParser@@B+368
  00a9a	e8 00 00 00 00	 call	 ??0CParseConstant@HCParser@@QAE@ABV01@@Z
  00a9f	c6 45 fc 5f	 mov	 BYTE PTR __$EHRec$[ebp+8], 95 ; 0000005fH
  00aa3	8d 8d 18 fe ff
	ff		 lea	 ecx, DWORD PTR $T362613[ebp]
  00aa9	e8 00 00 00 00	 call	 ??1CParseConstant@HCParser@@QAE@XZ

; 64   :     PC( _T("TEMIC_4009FR5_PAL"),            TUNER_TEMIC_4009FR5_PAL            ),

  00aae	83 ec 0c	 sub	 esp, 12			; 0000000cH
  00ab1	8b cc		 mov	 ecx, esp
  00ab3	89 a5 00 fe ff
	ff		 mov	 DWORD PTR $T362616[ebp], esp
  00ab9	6a 16		 push	 22			; 00000016H
  00abb	e8 00 00 00 00	 call	 ??0CParseValue@HCParser@@QAE@H@Z ; HCParser::CParseValue::CParseValue
  00ac0	89 85 34 f9 ff
	ff		 mov	 DWORD PTR tv690[ebp], eax
  00ac6	8b 85 34 f9 ff
	ff		 mov	 eax, DWORD PTR tv690[ebp]
  00acc	89 85 30 f9 ff
	ff		 mov	 DWORD PTR tv2038[ebp], eax
  00ad2	c6 45 fc 60	 mov	 BYTE PTR __$EHRec$[ebp+8], 96 ; 00000060H
  00ad6	68 00 00 00 00	 push	 OFFSET ??_C@_1CE@FOCJDBOD@?$AAT?$AAE?$AAM?$AAI?$AAC?$AA_?$AA4?$AA0?$AA0?$AA9?$AAF?$AAR?$AA5?$AA_?$AAP?$AAA?$AAL?$AA?$AA@
  00adb	c6 45 fc 5f	 mov	 BYTE PTR __$EHRec$[ebp+8], 95 ; 0000005fH
  00adf	8d 8d 04 fe ff
	ff		 lea	 ecx, DWORD PTR $T362615[ebp]
  00ae5	e8 00 00 00 00	 call	 ??0CParseConstant@HCParser@@QAE@PB_WVCParseValue@1@@Z ; HCParser::CParseConstant::CParseConstant
  00aea	89 85 2c f9 ff
	ff		 mov	 DWORD PTR tv2039[ebp], eax
  00af0	8b 8d 2c f9 ff
	ff		 mov	 ecx, DWORD PTR tv2039[ebp]
  00af6	89 8d 28 f9 ff
	ff		 mov	 DWORD PTR tv2041[ebp], ecx
  00afc	c6 45 fc 61	 mov	 BYTE PTR __$EHRec$[ebp+8], 97 ; 00000061H
  00b00	8b 95 28 f9 ff
	ff		 mov	 edx, DWORD PTR tv2041[ebp]
  00b06	52		 push	 edx
  00b07	b9 80 01 00 00	 mov	 ecx, OFFSET ?k_parseTunerConstants@@3QBVCParseConstant@HCParser@@B+384
  00b0c	e8 00 00 00 00	 call	 ??0CParseConstant@HCParser@@QAE@ABV01@@Z
  00b11	c6 45 fc 63	 mov	 BYTE PTR __$EHRec$[ebp+8], 99 ; 00000063H
  00b15	8d 8d 04 fe ff
	ff		 lea	 ecx, DWORD PTR $T362615[ebp]
  00b1b	e8 00 00 00 00	 call	 ??1CParseConstant@HCParser@@QAE@XZ

; 65   :     PC( _T("TEMIC_4039FR5_NTSC"),            TUNER_TEMIC_4039FR5_NTSC        ),

  00b20	83 ec 0c	 sub	 esp, 12			; 0000000cH
  00b23	8b cc		 mov	 ecx, esp
  00b25	89 a5 ec fd ff
	ff		 mov	 DWORD PTR $T362618[ebp], esp
  00b2b	6a 17		 push	 23			; 00000017H
  00b2d	e8 00 00 00 00	 call	 ??0CParseValue@HCParser@@QAE@H@Z ; HCParser::CParseValue::CParseValue
  00b32	89 85 24 f9 ff
	ff		 mov	 DWORD PTR tv713[ebp], eax
  00b38	8b 85 24 f9 ff
	ff		 mov	 eax, DWORD PTR tv713[ebp]
  00b3e	89 85 20 f9 ff
	ff		 mov	 DWORD PTR tv2044[ebp], eax
  00b44	c6 45 fc 64	 mov	 BYTE PTR __$EHRec$[ebp+8], 100 ; 00000064H
  00b48	68 00 00 00 00	 push	 OFFSET ??_C@_1CG@GLOIJKPF@?$AAT?$AAE?$AAM?$AAI?$AAC?$AA_?$AA4?$AA0?$AA3?$AA9?$AAF?$AAR?$AA5?$AA_?$AAN?$AAT?$AAS?$AAC?$AA?$AA@
  00b4d	c6 45 fc 63	 mov	 BYTE PTR __$EHRec$[ebp+8], 99 ; 00000063H
  00b51	8d 8d f0 fd ff
	ff		 lea	 ecx, DWORD PTR $T362617[ebp]
  00b57	e8 00 00 00 00	 call	 ??0CParseConstant@HCParser@@QAE@PB_WVCParseValue@1@@Z ; HCParser::CParseConstant::CParseConstant
  00b5c	89 85 1c f9 ff
	ff		 mov	 DWORD PTR tv2045[ebp], eax
  00b62	8b 8d 1c f9 ff
	ff		 mov	 ecx, DWORD PTR tv2045[ebp]
  00b68	89 8d 18 f9 ff
	ff		 mov	 DWORD PTR tv2047[ebp], ecx
  00b6e	c6 45 fc 65	 mov	 BYTE PTR __$EHRec$[ebp+8], 101 ; 00000065H
  00b72	8b 95 18 f9 ff
	ff		 mov	 edx, DWORD PTR tv2047[ebp]
  00b78	52		 push	 edx
  00b79	b9 90 01 00 00	 mov	 ecx, OFFSET ?k_parseTunerConstants@@3QBVCParseConstant@HCParser@@B+400
  00b7e	e8 00 00 00 00	 call	 ??0CParseConstant@HCParser@@QAE@ABV01@@Z
  00b83	c6 45 fc 67	 mov	 BYTE PTR __$EHRec$[ebp+8], 103 ; 00000067H
  00b87	8d 8d f0 fd ff
	ff		 lea	 ecx, DWORD PTR $T362617[ebp]
  00b8d	e8 00 00 00 00	 call	 ??1CParseConstant@HCParser@@QAE@XZ

; 66   :     PC( _T("TEMIC_4046FM5_MULTI"),            TUNER_TEMIC_4046FM5_MULTI        ),

  00b92	83 ec 0c	 sub	 esp, 12			; 0000000cH
  00b95	8b cc		 mov	 ecx, esp
  00b97	89 a5 d8 fd ff
	ff		 mov	 DWORD PTR $T362620[ebp], esp
  00b9d	6a 18		 push	 24			; 00000018H
  00b9f	e8 00 00 00 00	 call	 ??0CParseValue@HCParser@@QAE@H@Z ; HCParser::CParseValue::CParseValue
  00ba4	89 85 14 f9 ff
	ff		 mov	 DWORD PTR tv736[ebp], eax
  00baa	8b 85 14 f9 ff
	ff		 mov	 eax, DWORD PTR tv736[ebp]
  00bb0	89 85 10 f9 ff
	ff		 mov	 DWORD PTR tv2050[ebp], eax
  00bb6	c6 45 fc 68	 mov	 BYTE PTR __$EHRec$[ebp+8], 104 ; 00000068H
  00bba	68 00 00 00 00	 push	 OFFSET ??_C@_1CI@IJEHGMNA@?$AAT?$AAE?$AAM?$AAI?$AAC?$AA_?$AA4?$AA0?$AA4?$AA6?$AAF?$AAM?$AA5?$AA_?$AAM?$AAU?$AAL?$AAT?$AAI?$AA?$AA@
  00bbf	c6 45 fc 67	 mov	 BYTE PTR __$EHRec$[ebp+8], 103 ; 00000067H
  00bc3	8d 8d dc fd ff
	ff		 lea	 ecx, DWORD PTR $T362619[ebp]
  00bc9	e8 00 00 00 00	 call	 ??0CParseConstant@HCParser@@QAE@PB_WVCParseValue@1@@Z ; HCParser::CParseConstant::CParseConstant
  00bce	89 85 0c f9 ff
	ff		 mov	 DWORD PTR tv2051[ebp], eax
  00bd4	8b 8d 0c f9 ff
	ff		 mov	 ecx, DWORD PTR tv2051[ebp]
  00bda	89 8d 08 f9 ff
	ff		 mov	 DWORD PTR tv2053[ebp], ecx
  00be0	c6 45 fc 69	 mov	 BYTE PTR __$EHRec$[ebp+8], 105 ; 00000069H
  00be4	8b 95 08 f9 ff
	ff		 mov	 edx, DWORD PTR tv2053[ebp]
  00bea	52		 push	 edx
  00beb	b9 a0 01 00 00	 mov	 ecx, OFFSET ?k_parseTunerConstants@@3QBVCParseConstant@HCParser@@B+416
  00bf0	e8 00 00 00 00	 call	 ??0CParseConstant@HCParser@@QAE@ABV01@@Z
  00bf5	c6 45 fc 6b	 mov	 BYTE PTR __$EHRec$[ebp+8], 107 ; 0000006bH
  00bf9	8d 8d dc fd ff
	ff		 lea	 ecx, DWORD PTR $T362619[ebp]
  00bff	e8 00 00 00 00	 call	 ??1CParseConstant@HCParser@@QAE@XZ

; 67   :     PC( _T("PHILIPS_PAL_DK"),                TUNER_PHILIPS_PAL_DK            ),

  00c04	83 ec 0c	 sub	 esp, 12			; 0000000cH
  00c07	8b cc		 mov	 ecx, esp
  00c09	89 a5 c4 fd ff
	ff		 mov	 DWORD PTR $T362622[ebp], esp
  00c0f	6a 19		 push	 25			; 00000019H
  00c11	e8 00 00 00 00	 call	 ??0CParseValue@HCParser@@QAE@H@Z ; HCParser::CParseValue::CParseValue
  00c16	89 85 04 f9 ff
	ff		 mov	 DWORD PTR tv759[ebp], eax
  00c1c	8b 85 04 f9 ff
	ff		 mov	 eax, DWORD PTR tv759[ebp]
  00c22	89 85 00 f9 ff
	ff		 mov	 DWORD PTR tv2056[ebp], eax
  00c28	c6 45 fc 6c	 mov	 BYTE PTR __$EHRec$[ebp+8], 108 ; 0000006cH
  00c2c	68 00 00 00 00	 push	 OFFSET ??_C@_1BO@MJKOIFIF@?$AAP?$AAH?$AAI?$AAL?$AAI?$AAP?$AAS?$AA_?$AAP?$AAA?$AAL?$AA_?$AAD?$AAK?$AA?$AA@
  00c31	c6 45 fc 6b	 mov	 BYTE PTR __$EHRec$[ebp+8], 107 ; 0000006bH
  00c35	8d 8d c8 fd ff
	ff		 lea	 ecx, DWORD PTR $T362621[ebp]
  00c3b	e8 00 00 00 00	 call	 ??0CParseConstant@HCParser@@QAE@PB_WVCParseValue@1@@Z ; HCParser::CParseConstant::CParseConstant
  00c40	89 85 fc f8 ff
	ff		 mov	 DWORD PTR tv2057[ebp], eax
  00c46	8b 8d fc f8 ff
	ff		 mov	 ecx, DWORD PTR tv2057[ebp]
  00c4c	89 8d f8 f8 ff
	ff		 mov	 DWORD PTR tv2059[ebp], ecx
  00c52	c6 45 fc 6d	 mov	 BYTE PTR __$EHRec$[ebp+8], 109 ; 0000006dH
  00c56	8b 95 f8 f8 ff
	ff		 mov	 edx, DWORD PTR tv2059[ebp]
  00c5c	52		 push	 edx
  00c5d	b9 b0 01 00 00	 mov	 ecx, OFFSET ?k_parseTunerConstants@@3QBVCParseConstant@HCParser@@B+432
  00c62	e8 00 00 00 00	 call	 ??0CParseConstant@HCParser@@QAE@ABV01@@Z
  00c67	c6 45 fc 6f	 mov	 BYTE PTR __$EHRec$[ebp+8], 111 ; 0000006fH
  00c6b	8d 8d c8 fd ff
	ff		 lea	 ecx, DWORD PTR $T362621[ebp]
  00c71	e8 00 00 00 00	 call	 ??1CParseConstant@HCParser@@QAE@XZ

; 68   :     PC( _T("PHILIPS_MULTI"),                TUNER_PHILIPS_MULTI                ),

  00c76	83 ec 0c	 sub	 esp, 12			; 0000000cH
  00c79	8b cc		 mov	 ecx, esp
  00c7b	89 a5 b0 fd ff
	ff		 mov	 DWORD PTR $T362624[ebp], esp
  00c81	6a 1a		 push	 26			; 0000001aH
  00c83	e8 00 00 00 00	 call	 ??0CParseValue@HCParser@@QAE@H@Z ; HCParser::CParseValue::CParseValue
  00c88	89 85 f4 f8 ff
	ff		 mov	 DWORD PTR tv782[ebp], eax
  00c8e	8b 85 f4 f8 ff
	ff		 mov	 eax, DWORD PTR tv782[ebp]
  00c94	89 85 f0 f8 ff
	ff		 mov	 DWORD PTR tv2062[ebp], eax
  00c9a	c6 45 fc 70	 mov	 BYTE PTR __$EHRec$[ebp+8], 112 ; 00000070H
  00c9e	68 00 00 00 00	 push	 OFFSET ??_C@_1BM@PFKAHCHD@?$AAP?$AAH?$AAI?$AAL?$AAI?$AAP?$AAS?$AA_?$AAM?$AAU?$AAL?$AAT?$AAI?$AA?$AA@
  00ca3	c6 45 fc 6f	 mov	 BYTE PTR __$EHRec$[ebp+8], 111 ; 0000006fH
  00ca7	8d 8d b4 fd ff
	ff		 lea	 ecx, DWORD PTR $T362623[ebp]
  00cad	e8 00 00 00 00	 call	 ??0CParseConstant@HCParser@@QAE@PB_WVCParseValue@1@@Z ; HCParser::CParseConstant::CParseConstant
  00cb2	89 85 ec f8 ff
	ff		 mov	 DWORD PTR tv2063[ebp], eax
  00cb8	8b 8d ec f8 ff
	ff		 mov	 ecx, DWORD PTR tv2063[ebp]
  00cbe	89 8d e8 f8 ff
	ff		 mov	 DWORD PTR tv2065[ebp], ecx
  00cc4	c6 45 fc 71	 mov	 BYTE PTR __$EHRec$[ebp+8], 113 ; 00000071H
  00cc8	8b 95 e8 f8 ff
	ff		 mov	 edx, DWORD PTR tv2065[ebp]
  00cce	52		 push	 edx
  00ccf	b9 c0 01 00 00	 mov	 ecx, OFFSET ?k_parseTunerConstants@@3QBVCParseConstant@HCParser@@B+448
  00cd4	e8 00 00 00 00	 call	 ??0CParseConstant@HCParser@@QAE@ABV01@@Z
  00cd9	c6 45 fc 73	 mov	 BYTE PTR __$EHRec$[ebp+8], 115 ; 00000073H
  00cdd	8d 8d b4 fd ff
	ff		 lea	 ecx, DWORD PTR $T362623[ebp]
  00ce3	e8 00 00 00 00	 call	 ??1CParseConstant@HCParser@@QAE@XZ

; 69   :     PC( _T("LG_I001D_PAL_I"),                TUNER_LG_I001D_PAL_I            ),

  00ce8	83 ec 0c	 sub	 esp, 12			; 0000000cH
  00ceb	8b cc		 mov	 ecx, esp
  00ced	89 a5 9c fd ff
	ff		 mov	 DWORD PTR $T362626[ebp], esp
  00cf3	6a 1b		 push	 27			; 0000001bH
  00cf5	e8 00 00 00 00	 call	 ??0CParseValue@HCParser@@QAE@H@Z ; HCParser::CParseValue::CParseValue
  00cfa	89 85 e4 f8 ff
	ff		 mov	 DWORD PTR tv805[ebp], eax
  00d00	8b 85 e4 f8 ff
	ff		 mov	 eax, DWORD PTR tv805[ebp]
  00d06	89 85 e0 f8 ff
	ff		 mov	 DWORD PTR tv2068[ebp], eax
  00d0c	c6 45 fc 74	 mov	 BYTE PTR __$EHRec$[ebp+8], 116 ; 00000074H
  00d10	68 00 00 00 00	 push	 OFFSET ??_C@_1BO@DFOPCAAK@?$AAL?$AAG?$AA_?$AAI?$AA0?$AA0?$AA1?$AAD?$AA_?$AAP?$AAA?$AAL?$AA_?$AAI?$AA?$AA@
  00d15	c6 45 fc 73	 mov	 BYTE PTR __$EHRec$[ebp+8], 115 ; 00000073H
  00d19	8d 8d a0 fd ff
	ff		 lea	 ecx, DWORD PTR $T362625[ebp]
  00d1f	e8 00 00 00 00	 call	 ??0CParseConstant@HCParser@@QAE@PB_WVCParseValue@1@@Z ; HCParser::CParseConstant::CParseConstant
  00d24	89 85 dc f8 ff
	ff		 mov	 DWORD PTR tv2069[ebp], eax
  00d2a	8b 8d dc f8 ff
	ff		 mov	 ecx, DWORD PTR tv2069[ebp]
  00d30	89 8d d8 f8 ff
	ff		 mov	 DWORD PTR tv2071[ebp], ecx
  00d36	c6 45 fc 75	 mov	 BYTE PTR __$EHRec$[ebp+8], 117 ; 00000075H
  00d3a	8b 95 d8 f8 ff
	ff		 mov	 edx, DWORD PTR tv2071[ebp]
  00d40	52		 push	 edx
  00d41	b9 d0 01 00 00	 mov	 ecx, OFFSET ?k_parseTunerConstants@@3QBVCParseConstant@HCParser@@B+464
  00d46	e8 00 00 00 00	 call	 ??0CParseConstant@HCParser@@QAE@ABV01@@Z
  00d4b	c6 45 fc 77	 mov	 BYTE PTR __$EHRec$[ebp+8], 119 ; 00000077H
  00d4f	8d 8d a0 fd ff
	ff		 lea	 ecx, DWORD PTR $T362625[ebp]
  00d55	e8 00 00 00 00	 call	 ??1CParseConstant@HCParser@@QAE@XZ

; 70   :     PC( _T("LG_I701D_PAL_I"),                TUNER_LG_I701D_PAL_I            ),

  00d5a	83 ec 0c	 sub	 esp, 12			; 0000000cH
  00d5d	8b cc		 mov	 ecx, esp
  00d5f	89 a5 88 fd ff
	ff		 mov	 DWORD PTR $T362628[ebp], esp
  00d65	6a 1c		 push	 28			; 0000001cH
  00d67	e8 00 00 00 00	 call	 ??0CParseValue@HCParser@@QAE@H@Z ; HCParser::CParseValue::CParseValue
  00d6c	89 85 d4 f8 ff
	ff		 mov	 DWORD PTR tv828[ebp], eax
  00d72	8b 85 d4 f8 ff
	ff		 mov	 eax, DWORD PTR tv828[ebp]
  00d78	89 85 d0 f8 ff
	ff		 mov	 DWORD PTR tv2074[ebp], eax
  00d7e	c6 45 fc 78	 mov	 BYTE PTR __$EHRec$[ebp+8], 120 ; 00000078H
  00d82	68 00 00 00 00	 push	 OFFSET ??_C@_1BO@FADGBOEK@?$AAL?$AAG?$AA_?$AAI?$AA7?$AA0?$AA1?$AAD?$AA_?$AAP?$AAA?$AAL?$AA_?$AAI?$AA?$AA@
  00d87	c6 45 fc 77	 mov	 BYTE PTR __$EHRec$[ebp+8], 119 ; 00000077H
  00d8b	8d 8d 8c fd ff
	ff		 lea	 ecx, DWORD PTR $T362627[ebp]
  00d91	e8 00 00 00 00	 call	 ??0CParseConstant@HCParser@@QAE@PB_WVCParseValue@1@@Z ; HCParser::CParseConstant::CParseConstant
  00d96	89 85 cc f8 ff
	ff		 mov	 DWORD PTR tv2075[ebp], eax
  00d9c	8b 8d cc f8 ff
	ff		 mov	 ecx, DWORD PTR tv2075[ebp]
  00da2	89 8d c8 f8 ff
	ff		 mov	 DWORD PTR tv2077[ebp], ecx
  00da8	c6 45 fc 79	 mov	 BYTE PTR __$EHRec$[ebp+8], 121 ; 00000079H
  00dac	8b 95 c8 f8 ff
	ff		 mov	 edx, DWORD PTR tv2077[ebp]
  00db2	52		 push	 edx
  00db3	b9 e0 01 00 00	 mov	 ecx, OFFSET ?k_parseTunerConstants@@3QBVCParseConstant@HCParser@@B+480
  00db8	e8 00 00 00 00	 call	 ??0CParseConstant@HCParser@@QAE@ABV01@@Z
  00dbd	c6 45 fc 7b	 mov	 BYTE PTR __$EHRec$[ebp+8], 123 ; 0000007bH
  00dc1	8d 8d 8c fd ff
	ff		 lea	 ecx, DWORD PTR $T362627[ebp]
  00dc7	e8 00 00 00 00	 call	 ??1CParseConstant@HCParser@@QAE@XZ

; 71   :     PC( _T("LG_R01F_NTSC"),                    TUNER_LG_R01F_NTSC                ),

  00dcc	83 ec 0c	 sub	 esp, 12			; 0000000cH
  00dcf	8b cc		 mov	 ecx, esp
  00dd1	89 a5 74 fd ff
	ff		 mov	 DWORD PTR $T362630[ebp], esp
  00dd7	6a 1d		 push	 29			; 0000001dH
  00dd9	e8 00 00 00 00	 call	 ??0CParseValue@HCParser@@QAE@H@Z ; HCParser::CParseValue::CParseValue
  00dde	89 85 c4 f8 ff
	ff		 mov	 DWORD PTR tv851[ebp], eax
  00de4	8b 85 c4 f8 ff
	ff		 mov	 eax, DWORD PTR tv851[ebp]
  00dea	89 85 c0 f8 ff
	ff		 mov	 DWORD PTR tv2080[ebp], eax
  00df0	c6 45 fc 7c	 mov	 BYTE PTR __$EHRec$[ebp+8], 124 ; 0000007cH
  00df4	68 00 00 00 00	 push	 OFFSET ??_C@_1BK@NFMGFCPC@?$AAL?$AAG?$AA_?$AAR?$AA0?$AA1?$AAF?$AA_?$AAN?$AAT?$AAS?$AAC?$AA?$AA@
  00df9	c6 45 fc 7b	 mov	 BYTE PTR __$EHRec$[ebp+8], 123 ; 0000007bH
  00dfd	8d 8d 78 fd ff
	ff		 lea	 ecx, DWORD PTR $T362629[ebp]
  00e03	e8 00 00 00 00	 call	 ??0CParseConstant@HCParser@@QAE@PB_WVCParseValue@1@@Z ; HCParser::CParseConstant::CParseConstant
  00e08	89 85 bc f8 ff
	ff		 mov	 DWORD PTR tv2081[ebp], eax
  00e0e	8b 8d bc f8 ff
	ff		 mov	 ecx, DWORD PTR tv2081[ebp]
  00e14	89 8d b8 f8 ff
	ff		 mov	 DWORD PTR tv2083[ebp], ecx
  00e1a	c6 45 fc 7d	 mov	 BYTE PTR __$EHRec$[ebp+8], 125 ; 0000007dH
  00e1e	8b 95 b8 f8 ff
	ff		 mov	 edx, DWORD PTR tv2083[ebp]
  00e24	52		 push	 edx
  00e25	b9 f0 01 00 00	 mov	 ecx, OFFSET ?k_parseTunerConstants@@3QBVCParseConstant@HCParser@@B+496
  00e2a	e8 00 00 00 00	 call	 ??0CParseConstant@HCParser@@QAE@ABV01@@Z
  00e2f	c6 45 fc 7f	 mov	 BYTE PTR __$EHRec$[ebp+8], 127 ; 0000007fH
  00e33	8d 8d 78 fd ff
	ff		 lea	 ecx, DWORD PTR $T362629[ebp]
  00e39	e8 00 00 00 00	 call	 ??1CParseConstant@HCParser@@QAE@XZ

; 72   :     PC( _T("LG_B01D_PAL"),                    TUNER_LG_B01D_PAL                ),

  00e3e	83 ec 0c	 sub	 esp, 12			; 0000000cH
  00e41	8b cc		 mov	 ecx, esp
  00e43	89 a5 60 fd ff
	ff		 mov	 DWORD PTR $T362632[ebp], esp
  00e49	6a 1e		 push	 30			; 0000001eH
  00e4b	e8 00 00 00 00	 call	 ??0CParseValue@HCParser@@QAE@H@Z ; HCParser::CParseValue::CParseValue
  00e50	89 85 b4 f8 ff
	ff		 mov	 DWORD PTR tv874[ebp], eax
  00e56	8b 85 b4 f8 ff
	ff		 mov	 eax, DWORD PTR tv874[ebp]
  00e5c	89 85 b0 f8 ff
	ff		 mov	 DWORD PTR tv2086[ebp], eax
  00e62	c6 45 fc 80	 mov	 BYTE PTR __$EHRec$[ebp+8], 128 ; 00000080H
  00e66	68 00 00 00 00	 push	 OFFSET ??_C@_1BI@IENNGMBM@?$AAL?$AAG?$AA_?$AAB?$AA0?$AA1?$AAD?$AA_?$AAP?$AAA?$AAL?$AA?$AA@
  00e6b	c6 45 fc 7f	 mov	 BYTE PTR __$EHRec$[ebp+8], 127 ; 0000007fH
  00e6f	8d 8d 64 fd ff
	ff		 lea	 ecx, DWORD PTR $T362631[ebp]
  00e75	e8 00 00 00 00	 call	 ??0CParseConstant@HCParser@@QAE@PB_WVCParseValue@1@@Z ; HCParser::CParseConstant::CParseConstant
  00e7a	89 85 ac f8 ff
	ff		 mov	 DWORD PTR tv2087[ebp], eax
  00e80	8b 8d ac f8 ff
	ff		 mov	 ecx, DWORD PTR tv2087[ebp]
  00e86	89 8d a8 f8 ff
	ff		 mov	 DWORD PTR tv2089[ebp], ecx
  00e8c	c6 45 fc 81	 mov	 BYTE PTR __$EHRec$[ebp+8], 129 ; 00000081H
  00e90	8b 95 a8 f8 ff
	ff		 mov	 edx, DWORD PTR tv2089[ebp]
  00e96	52		 push	 edx
  00e97	b9 00 02 00 00	 mov	 ecx, OFFSET ?k_parseTunerConstants@@3QBVCParseConstant@HCParser@@B+512
  00e9c	e8 00 00 00 00	 call	 ??0CParseConstant@HCParser@@QAE@ABV01@@Z
  00ea1	c6 45 fc 83	 mov	 BYTE PTR __$EHRec$[ebp+8], 131 ; 00000083H
  00ea5	8d 8d 64 fd ff
	ff		 lea	 ecx, DWORD PTR $T362631[ebp]
  00eab	e8 00 00 00 00	 call	 ??1CParseConstant@HCParser@@QAE@XZ

; 73   :     PC( _T("LG_B11D_PAL"),                    TUNER_LG_B11D_PAL                ),

  00eb0	83 ec 0c	 sub	 esp, 12			; 0000000cH
  00eb3	8b cc		 mov	 ecx, esp
  00eb5	89 a5 4c fd ff
	ff		 mov	 DWORD PTR $T362634[ebp], esp
  00ebb	6a 1f		 push	 31			; 0000001fH
  00ebd	e8 00 00 00 00	 call	 ??0CParseValue@HCParser@@QAE@H@Z ; HCParser::CParseValue::CParseValue
  00ec2	89 85 a4 f8 ff
	ff		 mov	 DWORD PTR tv929[ebp], eax
  00ec8	8b 85 a4 f8 ff
	ff		 mov	 eax, DWORD PTR tv929[ebp]
  00ece	89 85 a0 f8 ff
	ff		 mov	 DWORD PTR tv2092[ebp], eax
  00ed4	c6 45 fc 84	 mov	 BYTE PTR __$EHRec$[ebp+8], 132 ; 00000084H
  00ed8	68 00 00 00 00	 push	 OFFSET ??_C@_1BI@CKLFPNIN@?$AAL?$AAG?$AA_?$AAB?$AA1?$AA1?$AAD?$AA_?$AAP?$AAA?$AAL?$AA?$AA@
  00edd	c6 45 fc 83	 mov	 BYTE PTR __$EHRec$[ebp+8], 131 ; 00000083H
  00ee1	8d 8d 50 fd ff
	ff		 lea	 ecx, DWORD PTR $T362633[ebp]
  00ee7	e8 00 00 00 00	 call	 ??0CParseConstant@HCParser@@QAE@PB_WVCParseValue@1@@Z ; HCParser::CParseConstant::CParseConstant
  00eec	89 85 9c f8 ff
	ff		 mov	 DWORD PTR tv2093[ebp], eax
  00ef2	8b 8d 9c f8 ff
	ff		 mov	 ecx, DWORD PTR tv2093[ebp]
  00ef8	89 8d 98 f8 ff
	ff		 mov	 DWORD PTR tv2095[ebp], ecx
  00efe	c6 45 fc 85	 mov	 BYTE PTR __$EHRec$[ebp+8], 133 ; 00000085H
  00f02	8b 95 98 f8 ff
	ff		 mov	 edx, DWORD PTR tv2095[ebp]
  00f08	52		 push	 edx
  00f09	b9 10 02 00 00	 mov	 ecx, OFFSET ?k_parseTunerConstants@@3QBVCParseConstant@HCParser@@B+528
  00f0e	e8 00 00 00 00	 call	 ??0CParseConstant@HCParser@@QAE@ABV01@@Z
  00f13	c6 45 fc 87	 mov	 BYTE PTR __$EHRec$[ebp+8], 135 ; 00000087H
  00f17	8d 8d 50 fd ff
	ff		 lea	 ecx, DWORD PTR $T362633[ebp]
  00f1d	e8 00 00 00 00	 call	 ??1CParseConstant@HCParser@@QAE@XZ

; 74   :     PC( _T("TEMIC_4009FN5_PAL"),            TUNER_TEMIC_4009FN5_PAL            ),

  00f22	83 ec 0c	 sub	 esp, 12			; 0000000cH
  00f25	8b cc		 mov	 ecx, esp
  00f27	89 a5 38 fd ff
	ff		 mov	 DWORD PTR $T362636[ebp], esp
  00f2d	6a 20		 push	 32			; 00000020H
  00f2f	e8 00 00 00 00	 call	 ??0CParseValue@HCParser@@QAE@H@Z ; HCParser::CParseValue::CParseValue
  00f34	89 85 94 f8 ff
	ff		 mov	 DWORD PTR tv952[ebp], eax
  00f3a	8b 85 94 f8 ff
	ff		 mov	 eax, DWORD PTR tv952[ebp]
  00f40	89 85 90 f8 ff
	ff		 mov	 DWORD PTR tv2098[ebp], eax
  00f46	c6 45 fc 88	 mov	 BYTE PTR __$EHRec$[ebp+8], 136 ; 00000088H
  00f4a	68 00 00 00 00	 push	 OFFSET ??_C@_1CE@BCGOJMKC@?$AAT?$AAE?$AAM?$AAI?$AAC?$AA_?$AA4?$AA0?$AA0?$AA9?$AAF?$AAN?$AA5?$AA_?$AAP?$AAA?$AAL?$AA?$AA@
  00f4f	c6 45 fc 87	 mov	 BYTE PTR __$EHRec$[ebp+8], 135 ; 00000087H
  00f53	8d 8d 3c fd ff
	ff		 lea	 ecx, DWORD PTR $T362635[ebp]
  00f59	e8 00 00 00 00	 call	 ??0CParseConstant@HCParser@@QAE@PB_WVCParseValue@1@@Z ; HCParser::CParseConstant::CParseConstant
  00f5e	89 85 8c f8 ff
	ff		 mov	 DWORD PTR tv2099[ebp], eax
  00f64	8b 8d 8c f8 ff
	ff		 mov	 ecx, DWORD PTR tv2099[ebp]
  00f6a	89 8d 88 f8 ff
	ff		 mov	 DWORD PTR tv2101[ebp], ecx
  00f70	c6 45 fc 89	 mov	 BYTE PTR __$EHRec$[ebp+8], 137 ; 00000089H
  00f74	8b 95 88 f8 ff
	ff		 mov	 edx, DWORD PTR tv2101[ebp]
  00f7a	52		 push	 edx
  00f7b	b9 20 02 00 00	 mov	 ecx, OFFSET ?k_parseTunerConstants@@3QBVCParseConstant@HCParser@@B+544
  00f80	e8 00 00 00 00	 call	 ??0CParseConstant@HCParser@@QAE@ABV01@@Z
  00f85	c6 45 fc 8b	 mov	 BYTE PTR __$EHRec$[ebp+8], 139 ; 0000008bH
  00f89	8d 8d 3c fd ff
	ff		 lea	 ecx, DWORD PTR $T362635[ebp]
  00f8f	e8 00 00 00 00	 call	 ??1CParseConstant@HCParser@@QAE@XZ

; 75   :     PC( _T("MT2032"),                        TUNER_MT2032                    ),

  00f94	83 ec 0c	 sub	 esp, 12			; 0000000cH
  00f97	8b cc		 mov	 ecx, esp
  00f99	89 a5 24 fd ff
	ff		 mov	 DWORD PTR $T362638[ebp], esp
  00f9f	6a 21		 push	 33			; 00000021H
  00fa1	e8 00 00 00 00	 call	 ??0CParseValue@HCParser@@QAE@H@Z ; HCParser::CParseValue::CParseValue
  00fa6	89 85 84 f8 ff
	ff		 mov	 DWORD PTR tv1007[ebp], eax
  00fac	8b 85 84 f8 ff
	ff		 mov	 eax, DWORD PTR tv1007[ebp]
  00fb2	89 85 80 f8 ff
	ff		 mov	 DWORD PTR tv2104[ebp], eax
  00fb8	c6 45 fc 8c	 mov	 BYTE PTR __$EHRec$[ebp+8], 140 ; 0000008cH
  00fbc	68 00 00 00 00	 push	 OFFSET ??_C@_1O@NGHNCELA@?$AAM?$AAT?$AA2?$AA0?$AA3?$AA2?$AA?$AA@
  00fc1	c6 45 fc 8b	 mov	 BYTE PTR __$EHRec$[ebp+8], 139 ; 0000008bH
  00fc5	8d 8d 28 fd ff
	ff		 lea	 ecx, DWORD PTR $T362637[ebp]
  00fcb	e8 00 00 00 00	 call	 ??0CParseConstant@HCParser@@QAE@PB_WVCParseValue@1@@Z ; HCParser::CParseConstant::CParseConstant
  00fd0	89 85 7c f8 ff
	ff		 mov	 DWORD PTR tv2105[ebp], eax
  00fd6	8b 8d 7c f8 ff
	ff		 mov	 ecx, DWORD PTR tv2105[ebp]
  00fdc	89 8d 78 f8 ff
	ff		 mov	 DWORD PTR tv2107[ebp], ecx
  00fe2	c6 45 fc 8d	 mov	 BYTE PTR __$EHRec$[ebp+8], 141 ; 0000008dH
  00fe6	8b 95 78 f8 ff
	ff		 mov	 edx, DWORD PTR tv2107[ebp]
  00fec	52		 push	 edx
  00fed	b9 30 02 00 00	 mov	 ecx, OFFSET ?k_parseTunerConstants@@3QBVCParseConstant@HCParser@@B+560
  00ff2	e8 00 00 00 00	 call	 ??0CParseConstant@HCParser@@QAE@ABV01@@Z
  00ff7	c6 45 fc 8f	 mov	 BYTE PTR __$EHRec$[ebp+8], 143 ; 0000008fH
  00ffb	8d 8d 28 fd ff
	ff		 lea	 ecx, DWORD PTR $T362637[ebp]
  01001	e8 00 00 00 00	 call	 ??1CParseConstant@HCParser@@QAE@XZ

; 76   :     PC( _T("SHARP_2U5JF5540_NTSC"),            TUNER_SHARP_2U5JF5540_NTSC        ),

  01006	83 ec 0c	 sub	 esp, 12			; 0000000cH
  01009	8b cc		 mov	 ecx, esp
  0100b	89 a5 10 fd ff
	ff		 mov	 DWORD PTR $T362640[ebp], esp
  01011	6a 22		 push	 34			; 00000022H
  01013	e8 00 00 00 00	 call	 ??0CParseValue@HCParser@@QAE@H@Z ; HCParser::CParseValue::CParseValue
  01018	89 85 74 f8 ff
	ff		 mov	 DWORD PTR tv1030[ebp], eax
  0101e	8b 85 74 f8 ff
	ff		 mov	 eax, DWORD PTR tv1030[ebp]
  01024	89 85 70 f8 ff
	ff		 mov	 DWORD PTR tv2110[ebp], eax
  0102a	c6 45 fc 90	 mov	 BYTE PTR __$EHRec$[ebp+8], 144 ; 00000090H
  0102e	68 00 00 00 00	 push	 OFFSET ??_C@_1CK@MHILDIAN@?$AAS?$AAH?$AAA?$AAR?$AAP?$AA_?$AA2?$AAU?$AA5?$AAJ?$AAF?$AA5?$AA5?$AA4?$AA0?$AA_?$AAN?$AAT?$AAS?$AAC?$AA?$AA@
  01033	c6 45 fc 8f	 mov	 BYTE PTR __$EHRec$[ebp+8], 143 ; 0000008fH
  01037	8d 8d 14 fd ff
	ff		 lea	 ecx, DWORD PTR $T362639[ebp]
  0103d	e8 00 00 00 00	 call	 ??0CParseConstant@HCParser@@QAE@PB_WVCParseValue@1@@Z ; HCParser::CParseConstant::CParseConstant
  01042	89 85 6c f8 ff
	ff		 mov	 DWORD PTR tv2111[ebp], eax
  01048	8b 8d 6c f8 ff
	ff		 mov	 ecx, DWORD PTR tv2111[ebp]
  0104e	89 8d 68 f8 ff
	ff		 mov	 DWORD PTR tv2113[ebp], ecx
  01054	c6 45 fc 91	 mov	 BYTE PTR __$EHRec$[ebp+8], 145 ; 00000091H
  01058	8b 95 68 f8 ff
	ff		 mov	 edx, DWORD PTR tv2113[ebp]
  0105e	52		 push	 edx
  0105f	b9 40 02 00 00	 mov	 ecx, OFFSET ?k_parseTunerConstants@@3QBVCParseConstant@HCParser@@B+576
  01064	e8 00 00 00 00	 call	 ??0CParseConstant@HCParser@@QAE@ABV01@@Z
  01069	c6 45 fc 93	 mov	 BYTE PTR __$EHRec$[ebp+8], 147 ; 00000093H
  0106d	8d 8d 14 fd ff
	ff		 lea	 ecx, DWORD PTR $T362639[ebp]
  01073	e8 00 00 00 00	 call	 ??1CParseConstant@HCParser@@QAE@XZ

; 77   :     PC( _T("LG_TAPCH701P_NTSC"),            TUNER_LG_TAPCH701P_NTSC            ),

  01078	83 ec 0c	 sub	 esp, 12			; 0000000cH
  0107b	8b cc		 mov	 ecx, esp
  0107d	89 a5 fc fc ff
	ff		 mov	 DWORD PTR $T362642[ebp], esp
  01083	6a 23		 push	 35			; 00000023H
  01085	e8 00 00 00 00	 call	 ??0CParseValue@HCParser@@QAE@H@Z ; HCParser::CParseValue::CParseValue
  0108a	89 85 64 f8 ff
	ff		 mov	 DWORD PTR tv1053[ebp], eax
  01090	8b 85 64 f8 ff
	ff		 mov	 eax, DWORD PTR tv1053[ebp]
  01096	89 85 60 f8 ff
	ff		 mov	 DWORD PTR tv2116[ebp], eax
  0109c	c6 45 fc 94	 mov	 BYTE PTR __$EHRec$[ebp+8], 148 ; 00000094H
  010a0	68 00 00 00 00	 push	 OFFSET ??_C@_1CE@CODMLBHG@?$AAL?$AAG?$AA_?$AAT?$AAA?$AAP?$AAC?$AAH?$AA7?$AA0?$AA1?$AAP?$AA_?$AAN?$AAT?$AAS?$AAC?$AA?$AA@
  010a5	c6 45 fc 93	 mov	 BYTE PTR __$EHRec$[ebp+8], 147 ; 00000093H
  010a9	8d 8d 00 fd ff
	ff		 lea	 ecx, DWORD PTR $T362641[ebp]
  010af	e8 00 00 00 00	 call	 ??0CParseConstant@HCParser@@QAE@PB_WVCParseValue@1@@Z ; HCParser::CParseConstant::CParseConstant
  010b4	89 85 5c f8 ff
	ff		 mov	 DWORD PTR tv2117[ebp], eax
  010ba	8b 8d 5c f8 ff
	ff		 mov	 ecx, DWORD PTR tv2117[ebp]
  010c0	89 8d 58 f8 ff
	ff		 mov	 DWORD PTR tv2119[ebp], ecx
  010c6	c6 45 fc 95	 mov	 BYTE PTR __$EHRec$[ebp+8], 149 ; 00000095H
  010ca	8b 95 58 f8 ff
	ff		 mov	 edx, DWORD PTR tv2119[ebp]
  010d0	52		 push	 edx
  010d1	b9 50 02 00 00	 mov	 ecx, OFFSET ?k_parseTunerConstants@@3QBVCParseConstant@HCParser@@B+592
  010d6	e8 00 00 00 00	 call	 ??0CParseConstant@HCParser@@QAE@ABV01@@Z
  010db	c6 45 fc 97	 mov	 BYTE PTR __$EHRec$[ebp+8], 151 ; 00000097H
  010df	8d 8d 00 fd ff
	ff		 lea	 ecx, DWORD PTR $T362641[ebp]
  010e5	e8 00 00 00 00	 call	 ??1CParseConstant@HCParser@@QAE@XZ

; 78   :     PC( _T("SAMSUNG_PAL_TCPM9091PD27"),        TUNER_SAMSUNG_PAL_TCPM9091PD27    ),

  010ea	83 ec 0c	 sub	 esp, 12			; 0000000cH
  010ed	8b cc		 mov	 ecx, esp
  010ef	89 a5 e8 fc ff
	ff		 mov	 DWORD PTR $T362644[ebp], esp
  010f5	6a 24		 push	 36			; 00000024H
  010f7	e8 00 00 00 00	 call	 ??0CParseValue@HCParser@@QAE@H@Z ; HCParser::CParseValue::CParseValue
  010fc	89 85 54 f8 ff
	ff		 mov	 DWORD PTR tv1076[ebp], eax
  01102	8b 85 54 f8 ff
	ff		 mov	 eax, DWORD PTR tv1076[ebp]
  01108	89 85 50 f8 ff
	ff		 mov	 DWORD PTR tv2122[ebp], eax
  0110e	c6 45 fc 98	 mov	 BYTE PTR __$EHRec$[ebp+8], 152 ; 00000098H
  01112	68 00 00 00 00	 push	 OFFSET ??_C@_1DC@PNFJNOKI@?$AAS?$AAA?$AAM?$AAS?$AAU?$AAN?$AAG?$AA_?$AAP?$AAA?$AAL?$AA_?$AAT?$AAC?$AAP?$AAM?$AA9?$AA0?$AA9?$AA1?$AAP?$AAD?$AA2?$AA7?$AA?$AA@
  01117	c6 45 fc 97	 mov	 BYTE PTR __$EHRec$[ebp+8], 151 ; 00000097H
  0111b	8d 8d ec fc ff
	ff		 lea	 ecx, DWORD PTR $T362643[ebp]
  01121	e8 00 00 00 00	 call	 ??0CParseConstant@HCParser@@QAE@PB_WVCParseValue@1@@Z ; HCParser::CParseConstant::CParseConstant
  01126	89 85 4c f8 ff
	ff		 mov	 DWORD PTR tv2123[ebp], eax
  0112c	8b 8d 4c f8 ff
	ff		 mov	 ecx, DWORD PTR tv2123[ebp]
  01132	89 8d 48 f8 ff
	ff		 mov	 DWORD PTR tv2125[ebp], ecx
  01138	c6 45 fc 99	 mov	 BYTE PTR __$EHRec$[ebp+8], 153 ; 00000099H
  0113c	8b 95 48 f8 ff
	ff		 mov	 edx, DWORD PTR tv2125[ebp]
  01142	52		 push	 edx
  01143	b9 60 02 00 00	 mov	 ecx, OFFSET ?k_parseTunerConstants@@3QBVCParseConstant@HCParser@@B+608
  01148	e8 00 00 00 00	 call	 ??0CParseConstant@HCParser@@QAE@ABV01@@Z
  0114d	c6 45 fc 9b	 mov	 BYTE PTR __$EHRec$[ebp+8], 155 ; 0000009bH
  01151	8d 8d ec fc ff
	ff		 lea	 ecx, DWORD PTR $T362643[ebp]
  01157	e8 00 00 00 00	 call	 ??1CParseConstant@HCParser@@QAE@XZ

; 79   :     PC( _T("TEMIC_4106FH5"),                TUNER_TEMIC_4106FH5                ),

  0115c	83 ec 0c	 sub	 esp, 12			; 0000000cH
  0115f	8b cc		 mov	 ecx, esp
  01161	89 a5 d4 fc ff
	ff		 mov	 DWORD PTR $T362646[ebp], esp
  01167	6a 25		 push	 37			; 00000025H
  01169	e8 00 00 00 00	 call	 ??0CParseValue@HCParser@@QAE@H@Z ; HCParser::CParseValue::CParseValue
  0116e	89 85 44 f8 ff
	ff		 mov	 DWORD PTR tv1099[ebp], eax
  01174	8b 85 44 f8 ff
	ff		 mov	 eax, DWORD PTR tv1099[ebp]
  0117a	89 85 40 f8 ff
	ff		 mov	 DWORD PTR tv2128[ebp], eax
  01180	c6 45 fc 9c	 mov	 BYTE PTR __$EHRec$[ebp+8], 156 ; 0000009cH
  01184	68 00 00 00 00	 push	 OFFSET ??_C@_1BM@CPMEKHAF@?$AAT?$AAE?$AAM?$AAI?$AAC?$AA_?$AA4?$AA1?$AA0?$AA6?$AAF?$AAH?$AA5?$AA?$AA@
  01189	c6 45 fc 9b	 mov	 BYTE PTR __$EHRec$[ebp+8], 155 ; 0000009bH
  0118d	8d 8d d8 fc ff
	ff		 lea	 ecx, DWORD PTR $T362645[ebp]
  01193	e8 00 00 00 00	 call	 ??0CParseConstant@HCParser@@QAE@PB_WVCParseValue@1@@Z ; HCParser::CParseConstant::CParseConstant
  01198	89 85 3c f8 ff
	ff		 mov	 DWORD PTR tv2129[ebp], eax
  0119e	8b 8d 3c f8 ff
	ff		 mov	 ecx, DWORD PTR tv2129[ebp]
  011a4	89 8d 38 f8 ff
	ff		 mov	 DWORD PTR tv2131[ebp], ecx
  011aa	c6 45 fc 9d	 mov	 BYTE PTR __$EHRec$[ebp+8], 157 ; 0000009dH
  011ae	8b 95 38 f8 ff
	ff		 mov	 edx, DWORD PTR tv2131[ebp]
  011b4	52		 push	 edx
  011b5	b9 70 02 00 00	 mov	 ecx, OFFSET ?k_parseTunerConstants@@3QBVCParseConstant@HCParser@@B+624
  011ba	e8 00 00 00 00	 call	 ??0CParseConstant@HCParser@@QAE@ABV01@@Z
  011bf	c6 45 fc 9f	 mov	 BYTE PTR __$EHRec$[ebp+8], 159 ; 0000009fH
  011c3	8d 8d d8 fc ff
	ff		 lea	 ecx, DWORD PTR $T362645[ebp]
  011c9	e8 00 00 00 00	 call	 ??1CParseConstant@HCParser@@QAE@XZ

; 80   :     PC( _T("TEMIC_4012FY5"),                TUNER_TEMIC_4012FY5                ),

  011ce	83 ec 0c	 sub	 esp, 12			; 0000000cH
  011d1	8b cc		 mov	 ecx, esp
  011d3	89 a5 c0 fc ff
	ff		 mov	 DWORD PTR $T362648[ebp], esp
  011d9	6a 26		 push	 38			; 00000026H
  011db	e8 00 00 00 00	 call	 ??0CParseValue@HCParser@@QAE@H@Z ; HCParser::CParseValue::CParseValue
  011e0	89 85 34 f8 ff
	ff		 mov	 DWORD PTR tv1122[ebp], eax
  011e6	8b 85 34 f8 ff
	ff		 mov	 eax, DWORD PTR tv1122[ebp]
  011ec	89 85 30 f8 ff
	ff		 mov	 DWORD PTR tv2134[ebp], eax
  011f2	c6 45 fc a0	 mov	 BYTE PTR __$EHRec$[ebp+8], 160 ; 000000a0H
  011f6	68 00 00 00 00	 push	 OFFSET ??_C@_1BM@OIAPHLFI@?$AAT?$AAE?$AAM?$AAI?$AAC?$AA_?$AA4?$AA0?$AA1?$AA2?$AAF?$AAY?$AA5?$AA?$AA@
  011fb	c6 45 fc 9f	 mov	 BYTE PTR __$EHRec$[ebp+8], 159 ; 0000009fH
  011ff	8d 8d c4 fc ff
	ff		 lea	 ecx, DWORD PTR $T362647[ebp]
  01205	e8 00 00 00 00	 call	 ??0CParseConstant@HCParser@@QAE@PB_WVCParseValue@1@@Z ; HCParser::CParseConstant::CParseConstant
  0120a	89 85 2c f8 ff
	ff		 mov	 DWORD PTR tv2135[ebp], eax
  01210	8b 8d 2c f8 ff
	ff		 mov	 ecx, DWORD PTR tv2135[ebp]
  01216	89 8d 28 f8 ff
	ff		 mov	 DWORD PTR tv2137[ebp], ecx
  0121c	c6 45 fc a1	 mov	 BYTE PTR __$EHRec$[ebp+8], 161 ; 000000a1H
  01220	8b 95 28 f8 ff
	ff		 mov	 edx, DWORD PTR tv2137[ebp]
  01226	52		 push	 edx
  01227	b9 80 02 00 00	 mov	 ecx, OFFSET ?k_parseTunerConstants@@3QBVCParseConstant@HCParser@@B+640
  0122c	e8 00 00 00 00	 call	 ??0CParseConstant@HCParser@@QAE@ABV01@@Z
  01231	c6 45 fc a3	 mov	 BYTE PTR __$EHRec$[ebp+8], 163 ; 000000a3H
  01235	8d 8d c4 fc ff
	ff		 lea	 ecx, DWORD PTR $T362647[ebp]
  0123b	e8 00 00 00 00	 call	 ??1CParseConstant@HCParser@@QAE@XZ

; 81   :     PC( _T("TEMIC_4136FY5"),                TUNER_TEMIC_4136FY5                ),

  01240	83 ec 0c	 sub	 esp, 12			; 0000000cH
  01243	8b cc		 mov	 ecx, esp
  01245	89 a5 ac fc ff
	ff		 mov	 DWORD PTR $T362650[ebp], esp
  0124b	6a 27		 push	 39			; 00000027H
  0124d	e8 00 00 00 00	 call	 ??0CParseValue@HCParser@@QAE@H@Z ; HCParser::CParseValue::CParseValue
  01252	89 85 24 f8 ff
	ff		 mov	 DWORD PTR tv1145[ebp], eax
  01258	8b 85 24 f8 ff
	ff		 mov	 eax, DWORD PTR tv1145[ebp]
  0125e	89 85 20 f8 ff
	ff		 mov	 DWORD PTR tv2140[ebp], eax
  01264	c6 45 fc a4	 mov	 BYTE PTR __$EHRec$[ebp+8], 164 ; 000000a4H
  01268	68 00 00 00 00	 push	 OFFSET ??_C@_1BM@JANAKEML@?$AAT?$AAE?$AAM?$AAI?$AAC?$AA_?$AA4?$AA1?$AA3?$AA6?$AAF?$AAY?$AA5?$AA?$AA@
  0126d	c6 45 fc a3	 mov	 BYTE PTR __$EHRec$[ebp+8], 163 ; 000000a3H
  01271	8d 8d b0 fc ff
	ff		 lea	 ecx, DWORD PTR $T362649[ebp]
  01277	e8 00 00 00 00	 call	 ??0CParseConstant@HCParser@@QAE@PB_WVCParseValue@1@@Z ; HCParser::CParseConstant::CParseConstant
  0127c	89 85 1c f8 ff
	ff		 mov	 DWORD PTR tv2141[ebp], eax
  01282	8b 8d 1c f8 ff
	ff		 mov	 ecx, DWORD PTR tv2141[ebp]
  01288	89 8d 18 f8 ff
	ff		 mov	 DWORD PTR tv2143[ebp], ecx
  0128e	c6 45 fc a5	 mov	 BYTE PTR __$EHRec$[ebp+8], 165 ; 000000a5H
  01292	8b 95 18 f8 ff
	ff		 mov	 edx, DWORD PTR tv2143[ebp]
  01298	52		 push	 edx
  01299	b9 90 02 00 00	 mov	 ecx, OFFSET ?k_parseTunerConstants@@3QBVCParseConstant@HCParser@@B+656
  0129e	e8 00 00 00 00	 call	 ??0CParseConstant@HCParser@@QAE@ABV01@@Z
  012a3	c6 45 fc a7	 mov	 BYTE PTR __$EHRec$[ebp+8], 167 ; 000000a7H
  012a7	8d 8d b0 fc ff
	ff		 lea	 ecx, DWORD PTR $T362649[ebp]
  012ad	e8 00 00 00 00	 call	 ??1CParseConstant@HCParser@@QAE@XZ

; 82   :     PC( _T("LG_TAPCNEW_PAL"),                TUNER_LG_TAPCNEW_PAL            ),

  012b2	83 ec 0c	 sub	 esp, 12			; 0000000cH
  012b5	8b cc		 mov	 ecx, esp
  012b7	89 a5 98 fc ff
	ff		 mov	 DWORD PTR $T362652[ebp], esp
  012bd	6a 28		 push	 40			; 00000028H
  012bf	e8 00 00 00 00	 call	 ??0CParseValue@HCParser@@QAE@H@Z ; HCParser::CParseValue::CParseValue
  012c4	89 85 14 f8 ff
	ff		 mov	 DWORD PTR tv1168[ebp], eax
  012ca	8b 85 14 f8 ff
	ff		 mov	 eax, DWORD PTR tv1168[ebp]
  012d0	89 85 10 f8 ff
	ff		 mov	 DWORD PTR tv2146[ebp], eax
  012d6	c6 45 fc a8	 mov	 BYTE PTR __$EHRec$[ebp+8], 168 ; 000000a8H
  012da	68 00 00 00 00	 push	 OFFSET ??_C@_1BO@EHMDLLBA@?$AAL?$AAG?$AA_?$AAT?$AAA?$AAP?$AAC?$AAN?$AAE?$AAW?$AA_?$AAP?$AAA?$AAL?$AA?$AA@
  012df	c6 45 fc a7	 mov	 BYTE PTR __$EHRec$[ebp+8], 167 ; 000000a7H
  012e3	8d 8d 9c fc ff
	ff		 lea	 ecx, DWORD PTR $T362651[ebp]
  012e9	e8 00 00 00 00	 call	 ??0CParseConstant@HCParser@@QAE@PB_WVCParseValue@1@@Z ; HCParser::CParseConstant::CParseConstant
  012ee	89 85 0c f8 ff
	ff		 mov	 DWORD PTR tv2147[ebp], eax
  012f4	8b 8d 0c f8 ff
	ff		 mov	 ecx, DWORD PTR tv2147[ebp]
  012fa	89 8d 08 f8 ff
	ff		 mov	 DWORD PTR tv2149[ebp], ecx
  01300	c6 45 fc a9	 mov	 BYTE PTR __$EHRec$[ebp+8], 169 ; 000000a9H
  01304	8b 95 08 f8 ff
	ff		 mov	 edx, DWORD PTR tv2149[ebp]
  0130a	52		 push	 edx
  0130b	b9 a0 02 00 00	 mov	 ecx, OFFSET ?k_parseTunerConstants@@3QBVCParseConstant@HCParser@@B+672
  01310	e8 00 00 00 00	 call	 ??0CParseConstant@HCParser@@QAE@ABV01@@Z
  01315	c6 45 fc ab	 mov	 BYTE PTR __$EHRec$[ebp+8], 171 ; 000000abH
  01319	8d 8d 9c fc ff
	ff		 lea	 ecx, DWORD PTR $T362651[ebp]
  0131f	e8 00 00 00 00	 call	 ??1CParseConstant@HCParser@@QAE@XZ

; 83   :     PC( _T("PHILIPS_FM1216ME_MK3"),            TUNER_PHILIPS_FM1216ME_MK3        ),

  01324	83 ec 0c	 sub	 esp, 12			; 0000000cH
  01327	8b cc		 mov	 ecx, esp
  01329	89 a5 84 fc ff
	ff		 mov	 DWORD PTR $T362654[ebp], esp
  0132f	6a 29		 push	 41			; 00000029H
  01331	e8 00 00 00 00	 call	 ??0CParseValue@HCParser@@QAE@H@Z ; HCParser::CParseValue::CParseValue
  01336	89 85 04 f8 ff
	ff		 mov	 DWORD PTR tv1191[ebp], eax
  0133c	8b 85 04 f8 ff
	ff		 mov	 eax, DWORD PTR tv1191[ebp]
  01342	89 85 00 f8 ff
	ff		 mov	 DWORD PTR tv2152[ebp], eax
  01348	c6 45 fc ac	 mov	 BYTE PTR __$EHRec$[ebp+8], 172 ; 000000acH
  0134c	68 00 00 00 00	 push	 OFFSET ??_C@_1CK@CLKCBCPN@?$AAP?$AAH?$AAI?$AAL?$AAI?$AAP?$AAS?$AA_?$AAF?$AAM?$AA1?$AA2?$AA1?$AA6?$AAM?$AAE?$AA_?$AAM?$AAK?$AA3?$AA?$AA@
  01351	c6 45 fc ab	 mov	 BYTE PTR __$EHRec$[ebp+8], 171 ; 000000abH
  01355	8d 8d 88 fc ff
	ff		 lea	 ecx, DWORD PTR $T362653[ebp]
  0135b	e8 00 00 00 00	 call	 ??0CParseConstant@HCParser@@QAE@PB_WVCParseValue@1@@Z ; HCParser::CParseConstant::CParseConstant
  01360	89 85 fc f7 ff
	ff		 mov	 DWORD PTR tv2153[ebp], eax
  01366	8b 8d fc f7 ff
	ff		 mov	 ecx, DWORD PTR tv2153[ebp]
  0136c	89 8d f8 f7 ff
	ff		 mov	 DWORD PTR tv2155[ebp], ecx
  01372	c6 45 fc ad	 mov	 BYTE PTR __$EHRec$[ebp+8], 173 ; 000000adH
  01376	8b 95 f8 f7 ff
	ff		 mov	 edx, DWORD PTR tv2155[ebp]
  0137c	52		 push	 edx
  0137d	b9 b0 02 00 00	 mov	 ecx, OFFSET ?k_parseTunerConstants@@3QBVCParseConstant@HCParser@@B+688
  01382	e8 00 00 00 00	 call	 ??0CParseConstant@HCParser@@QAE@ABV01@@Z
  01387	c6 45 fc af	 mov	 BYTE PTR __$EHRec$[ebp+8], 175 ; 000000afH
  0138b	8d 8d 88 fc ff
	ff		 lea	 ecx, DWORD PTR $T362653[ebp]
  01391	e8 00 00 00 00	 call	 ??1CParseConstant@HCParser@@QAE@XZ

; 84   :     PC( _T("LG_TAPCNEW_NTSC"),                TUNER_LG_TAPCNEW_NTSC            ),

  01396	83 ec 0c	 sub	 esp, 12			; 0000000cH
  01399	8b cc		 mov	 ecx, esp
  0139b	89 a5 70 fc ff
	ff		 mov	 DWORD PTR $T362656[ebp], esp
  013a1	6a 2a		 push	 42			; 0000002aH
  013a3	e8 00 00 00 00	 call	 ??0CParseValue@HCParser@@QAE@H@Z ; HCParser::CParseValue::CParseValue
  013a8	89 85 f4 f7 ff
	ff		 mov	 DWORD PTR tv1214[ebp], eax
  013ae	8b 85 f4 f7 ff
	ff		 mov	 eax, DWORD PTR tv1214[ebp]
  013b4	89 85 f0 f7 ff
	ff		 mov	 DWORD PTR tv2158[ebp], eax
  013ba	c6 45 fc b0	 mov	 BYTE PTR __$EHRec$[ebp+8], 176 ; 000000b0H
  013be	68 00 00 00 00	 push	 OFFSET ??_C@_1CA@GAGMPGBP@?$AAL?$AAG?$AA_?$AAT?$AAA?$AAP?$AAC?$AAN?$AAE?$AAW?$AA_?$AAN?$AAT?$AAS?$AAC?$AA?$AA@
  013c3	c6 45 fc af	 mov	 BYTE PTR __$EHRec$[ebp+8], 175 ; 000000afH
  013c7	8d 8d 74 fc ff
	ff		 lea	 ecx, DWORD PTR $T362655[ebp]
  013cd	e8 00 00 00 00	 call	 ??0CParseConstant@HCParser@@QAE@PB_WVCParseValue@1@@Z ; HCParser::CParseConstant::CParseConstant
  013d2	89 85 ec f7 ff
	ff		 mov	 DWORD PTR tv2159[ebp], eax
  013d8	8b 8d ec f7 ff
	ff		 mov	 ecx, DWORD PTR tv2159[ebp]
  013de	89 8d e8 f7 ff
	ff		 mov	 DWORD PTR tv2161[ebp], ecx
  013e4	c6 45 fc b1	 mov	 BYTE PTR __$EHRec$[ebp+8], 177 ; 000000b1H
  013e8	8b 95 e8 f7 ff
	ff		 mov	 edx, DWORD PTR tv2161[ebp]
  013ee	52		 push	 edx
  013ef	b9 c0 02 00 00	 mov	 ecx, OFFSET ?k_parseTunerConstants@@3QBVCParseConstant@HCParser@@B+704
  013f4	e8 00 00 00 00	 call	 ??0CParseConstant@HCParser@@QAE@ABV01@@Z
  013f9	c6 45 fc b3	 mov	 BYTE PTR __$EHRec$[ebp+8], 179 ; 000000b3H
  013fd	8d 8d 74 fc ff
	ff		 lea	 ecx, DWORD PTR $T362655[ebp]
  01403	e8 00 00 00 00	 call	 ??1CParseConstant@HCParser@@QAE@XZ

; 85   :     PC( _T("MT2032_PAL"),                    TUNER_MT2032_PAL                ),

  01408	83 ec 0c	 sub	 esp, 12			; 0000000cH
  0140b	8b cc		 mov	 ecx, esp
  0140d	89 a5 5c fc ff
	ff		 mov	 DWORD PTR $T362658[ebp], esp
  01413	6a 2b		 push	 43			; 0000002bH
  01415	e8 00 00 00 00	 call	 ??0CParseValue@HCParser@@QAE@H@Z ; HCParser::CParseValue::CParseValue
  0141a	89 85 e4 f7 ff
	ff		 mov	 DWORD PTR tv1237[ebp], eax
  01420	8b 85 e4 f7 ff
	ff		 mov	 eax, DWORD PTR tv1237[ebp]
  01426	89 85 e0 f7 ff
	ff		 mov	 DWORD PTR tv2164[ebp], eax
  0142c	c6 45 fc b4	 mov	 BYTE PTR __$EHRec$[ebp+8], 180 ; 000000b4H
  01430	68 00 00 00 00	 push	 OFFSET ??_C@_1BG@FEPCEPIB@?$AAM?$AAT?$AA2?$AA0?$AA3?$AA2?$AA_?$AAP?$AAA?$AAL?$AA?$AA@
  01435	c6 45 fc b3	 mov	 BYTE PTR __$EHRec$[ebp+8], 179 ; 000000b3H
  01439	8d 8d 60 fc ff
	ff		 lea	 ecx, DWORD PTR $T362657[ebp]
  0143f	e8 00 00 00 00	 call	 ??0CParseConstant@HCParser@@QAE@PB_WVCParseValue@1@@Z ; HCParser::CParseConstant::CParseConstant
  01444	89 85 dc f7 ff
	ff		 mov	 DWORD PTR tv2165[ebp], eax
  0144a	8b 8d dc f7 ff
	ff		 mov	 ecx, DWORD PTR tv2165[ebp]
  01450	89 8d d8 f7 ff
	ff		 mov	 DWORD PTR tv2167[ebp], ecx
  01456	c6 45 fc b5	 mov	 BYTE PTR __$EHRec$[ebp+8], 181 ; 000000b5H
  0145a	8b 95 d8 f7 ff
	ff		 mov	 edx, DWORD PTR tv2167[ebp]
  01460	52		 push	 edx
  01461	b9 d0 02 00 00	 mov	 ecx, OFFSET ?k_parseTunerConstants@@3QBVCParseConstant@HCParser@@B+720
  01466	e8 00 00 00 00	 call	 ??0CParseConstant@HCParser@@QAE@ABV01@@Z
  0146b	c6 45 fc b7	 mov	 BYTE PTR __$EHRec$[ebp+8], 183 ; 000000b7H
  0146f	8d 8d 60 fc ff
	ff		 lea	 ecx, DWORD PTR $T362657[ebp]
  01475	e8 00 00 00 00	 call	 ??1CParseConstant@HCParser@@QAE@XZ

; 86   :     PC( _T("PHILIPS_FI1286_NTSC_M_J"),        TUNER_PHILIPS_FI1286_NTSC_M_J    ),

  0147a	83 ec 0c	 sub	 esp, 12			; 0000000cH
  0147d	8b cc		 mov	 ecx, esp
  0147f	89 a5 48 fc ff
	ff		 mov	 DWORD PTR $T362660[ebp], esp
  01485	6a 2c		 push	 44			; 0000002cH
  01487	e8 00 00 00 00	 call	 ??0CParseValue@HCParser@@QAE@H@Z ; HCParser::CParseValue::CParseValue
  0148c	89 85 d4 f7 ff
	ff		 mov	 DWORD PTR tv1260[ebp], eax
  01492	8b 85 d4 f7 ff
	ff		 mov	 eax, DWORD PTR tv1260[ebp]
  01498	89 85 d0 f7 ff
	ff		 mov	 DWORD PTR tv2170[ebp], eax
  0149e	c6 45 fc b8	 mov	 BYTE PTR __$EHRec$[ebp+8], 184 ; 000000b8H
  014a2	68 00 00 00 00	 push	 OFFSET ??_C@_1DA@JEOOMIMC@?$AAP?$AAH?$AAI?$AAL?$AAI?$AAP?$AAS?$AA_?$AAF?$AAI?$AA1?$AA2?$AA8?$AA6?$AA_?$AAN?$AAT?$AAS?$AAC?$AA_?$AAM?$AA_?$AAJ?$AA?$AA@
  014a7	c6 45 fc b7	 mov	 BYTE PTR __$EHRec$[ebp+8], 183 ; 000000b7H
  014ab	8d 8d 4c fc ff
	ff		 lea	 ecx, DWORD PTR $T362659[ebp]
  014b1	e8 00 00 00 00	 call	 ??0CParseConstant@HCParser@@QAE@PB_WVCParseValue@1@@Z ; HCParser::CParseConstant::CParseConstant
  014b6	89 85 cc f7 ff
	ff		 mov	 DWORD PTR tv2171[ebp], eax
  014bc	8b 8d cc f7 ff
	ff		 mov	 ecx, DWORD PTR tv2171[ebp]
  014c2	89 8d c8 f7 ff
	ff		 mov	 DWORD PTR tv2173[ebp], ecx
  014c8	c6 45 fc b9	 mov	 BYTE PTR __$EHRec$[ebp+8], 185 ; 000000b9H
  014cc	8b 95 c8 f7 ff
	ff		 mov	 edx, DWORD PTR tv2173[ebp]
  014d2	52		 push	 edx
  014d3	b9 e0 02 00 00	 mov	 ecx, OFFSET ?k_parseTunerConstants@@3QBVCParseConstant@HCParser@@B+736
  014d8	e8 00 00 00 00	 call	 ??0CParseConstant@HCParser@@QAE@ABV01@@Z
  014dd	c6 45 fc bb	 mov	 BYTE PTR __$EHRec$[ebp+8], 187 ; 000000bbH
  014e1	8d 8d 4c fc ff
	ff		 lea	 ecx, DWORD PTR $T362659[ebp]
  014e7	e8 00 00 00 00	 call	 ??1CParseConstant@HCParser@@QAE@XZ

; 87   :     PC( _T("MT2050"),                        TUNER_MT2050                    ),

  014ec	83 ec 0c	 sub	 esp, 12			; 0000000cH
  014ef	8b cc		 mov	 ecx, esp
  014f1	89 a5 34 fc ff
	ff		 mov	 DWORD PTR $T362662[ebp], esp
  014f7	6a 2d		 push	 45			; 0000002dH
  014f9	e8 00 00 00 00	 call	 ??0CParseValue@HCParser@@QAE@H@Z ; HCParser::CParseValue::CParseValue
  014fe	89 85 c4 f7 ff
	ff		 mov	 DWORD PTR tv1283[ebp], eax
  01504	8b 85 c4 f7 ff
	ff		 mov	 eax, DWORD PTR tv1283[ebp]
  0150a	89 85 c0 f7 ff
	ff		 mov	 DWORD PTR tv2176[ebp], eax
  01510	c6 45 fc bc	 mov	 BYTE PTR __$EHRec$[ebp+8], 188 ; 000000bcH
  01514	68 00 00 00 00	 push	 OFFSET ??_C@_1O@KKCNAPCG@?$AAM?$AAT?$AA2?$AA0?$AA5?$AA0?$AA?$AA@
  01519	c6 45 fc bb	 mov	 BYTE PTR __$EHRec$[ebp+8], 187 ; 000000bbH
  0151d	8d 8d 38 fc ff
	ff		 lea	 ecx, DWORD PTR $T362661[ebp]
  01523	e8 00 00 00 00	 call	 ??0CParseConstant@HCParser@@QAE@PB_WVCParseValue@1@@Z ; HCParser::CParseConstant::CParseConstant
  01528	89 85 bc f7 ff
	ff		 mov	 DWORD PTR tv2177[ebp], eax
  0152e	8b 8d bc f7 ff
	ff		 mov	 ecx, DWORD PTR tv2177[ebp]
  01534	89 8d b8 f7 ff
	ff		 mov	 DWORD PTR tv2179[ebp], ecx
  0153a	c6 45 fc bd	 mov	 BYTE PTR __$EHRec$[ebp+8], 189 ; 000000bdH
  0153e	8b 95 b8 f7 ff
	ff		 mov	 edx, DWORD PTR tv2179[ebp]
  01544	52		 push	 edx
  01545	b9 f0 02 00 00	 mov	 ecx, OFFSET ?k_parseTunerConstants@@3QBVCParseConstant@HCParser@@B+752
  0154a	e8 00 00 00 00	 call	 ??0CParseConstant@HCParser@@QAE@ABV01@@Z
  0154f	c6 45 fc bf	 mov	 BYTE PTR __$EHRec$[ebp+8], 191 ; 000000bfH
  01553	8d 8d 38 fc ff
	ff		 lea	 ecx, DWORD PTR $T362661[ebp]
  01559	e8 00 00 00 00	 call	 ??1CParseConstant@HCParser@@QAE@XZ

; 88   :     PC( _T("MT2050_PAL"),                    TUNER_MT2050_PAL                ),

  0155e	83 ec 0c	 sub	 esp, 12			; 0000000cH
  01561	8b cc		 mov	 ecx, esp
  01563	89 a5 20 fc ff
	ff		 mov	 DWORD PTR $T362664[ebp], esp
  01569	6a 2e		 push	 46			; 0000002eH
  0156b	e8 00 00 00 00	 call	 ??0CParseValue@HCParser@@QAE@H@Z ; HCParser::CParseValue::CParseValue
  01570	89 85 b4 f7 ff
	ff		 mov	 DWORD PTR tv1306[ebp], eax
  01576	8b 85 b4 f7 ff
	ff		 mov	 eax, DWORD PTR tv1306[ebp]
  0157c	89 85 b0 f7 ff
	ff		 mov	 DWORD PTR tv2182[ebp], eax
  01582	c6 45 fc c0	 mov	 BYTE PTR __$EHRec$[ebp+8], 192 ; 000000c0H
  01586	68 00 00 00 00	 push	 OFFSET ??_C@_1BG@EAALJKKI@?$AAM?$AAT?$AA2?$AA0?$AA5?$AA0?$AA_?$AAP?$AAA?$AAL?$AA?$AA@
  0158b	c6 45 fc bf	 mov	 BYTE PTR __$EHRec$[ebp+8], 191 ; 000000bfH
  0158f	8d 8d 24 fc ff
	ff		 lea	 ecx, DWORD PTR $T362663[ebp]
  01595	e8 00 00 00 00	 call	 ??0CParseConstant@HCParser@@QAE@PB_WVCParseValue@1@@Z ; HCParser::CParseConstant::CParseConstant
  0159a	89 85 ac f7 ff
	ff		 mov	 DWORD PTR tv2183[ebp], eax
  015a0	8b 8d ac f7 ff
	ff		 mov	 ecx, DWORD PTR tv2183[ebp]
  015a6	89 8d a8 f7 ff
	ff		 mov	 DWORD PTR tv2185[ebp], ecx
  015ac	c6 45 fc c1	 mov	 BYTE PTR __$EHRec$[ebp+8], 193 ; 000000c1H
  015b0	8b 95 a8 f7 ff
	ff		 mov	 edx, DWORD PTR tv2185[ebp]
  015b6	52		 push	 edx
  015b7	b9 00 03 00 00	 mov	 ecx, OFFSET ?k_parseTunerConstants@@3QBVCParseConstant@HCParser@@B+768
  015bc	e8 00 00 00 00	 call	 ??0CParseConstant@HCParser@@QAE@ABV01@@Z
  015c1	c6 45 fc c3	 mov	 BYTE PTR __$EHRec$[ebp+8], 195 ; 000000c3H
  015c5	8d 8d 24 fc ff
	ff		 lea	 ecx, DWORD PTR $T362663[ebp]
  015cb	e8 00 00 00 00	 call	 ??1CParseConstant@HCParser@@QAE@XZ

; 89   :     PC( _T("PHILIPS_4IN1"),                    TUNER_PHILIPS_4IN1                ),

  015d0	83 ec 0c	 sub	 esp, 12			; 0000000cH
  015d3	8b cc		 mov	 ecx, esp
  015d5	89 a5 0c fc ff
	ff		 mov	 DWORD PTR $T362666[ebp], esp
  015db	6a 2f		 push	 47			; 0000002fH
  015dd	e8 00 00 00 00	 call	 ??0CParseValue@HCParser@@QAE@H@Z ; HCParser::CParseValue::CParseValue
  015e2	89 85 a4 f7 ff
	ff		 mov	 DWORD PTR tv1361[ebp], eax
  015e8	8b 85 a4 f7 ff
	ff		 mov	 eax, DWORD PTR tv1361[ebp]
  015ee	89 85 a0 f7 ff
	ff		 mov	 DWORD PTR tv2188[ebp], eax
  015f4	c6 45 fc c4	 mov	 BYTE PTR __$EHRec$[ebp+8], 196 ; 000000c4H
  015f8	68 00 00 00 00	 push	 OFFSET ??_C@_1BK@PNPMMDOJ@?$AAP?$AAH?$AAI?$AAL?$AAI?$AAP?$AAS?$AA_?$AA4?$AAI?$AAN?$AA1?$AA?$AA@
  015fd	c6 45 fc c3	 mov	 BYTE PTR __$EHRec$[ebp+8], 195 ; 000000c3H
  01601	8d 8d 10 fc ff
	ff		 lea	 ecx, DWORD PTR $T362665[ebp]
  01607	e8 00 00 00 00	 call	 ??0CParseConstant@HCParser@@QAE@PB_WVCParseValue@1@@Z ; HCParser::CParseConstant::CParseConstant
  0160c	89 85 9c f7 ff
	ff		 mov	 DWORD PTR tv2189[ebp], eax
  01612	8b 8d 9c f7 ff
	ff		 mov	 ecx, DWORD PTR tv2189[ebp]
  01618	89 8d 98 f7 ff
	ff		 mov	 DWORD PTR tv2191[ebp], ecx
  0161e	c6 45 fc c5	 mov	 BYTE PTR __$EHRec$[ebp+8], 197 ; 000000c5H
  01622	8b 95 98 f7 ff
	ff		 mov	 edx, DWORD PTR tv2191[ebp]
  01628	52		 push	 edx
  01629	b9 10 03 00 00	 mov	 ecx, OFFSET ?k_parseTunerConstants@@3QBVCParseConstant@HCParser@@B+784
  0162e	e8 00 00 00 00	 call	 ??0CParseConstant@HCParser@@QAE@ABV01@@Z
  01633	c6 45 fc c7	 mov	 BYTE PTR __$EHRec$[ebp+8], 199 ; 000000c7H
  01637	8d 8d 10 fc ff
	ff		 lea	 ecx, DWORD PTR $T362665[ebp]
  0163d	e8 00 00 00 00	 call	 ??1CParseConstant@HCParser@@QAE@XZ

; 90   :     PC( _T("TCL_2002N"),                    TUNER_TCL_2002N                  ),

  01642	83 ec 0c	 sub	 esp, 12			; 0000000cH
  01645	8b cc		 mov	 ecx, esp
  01647	89 a5 f8 fb ff
	ff		 mov	 DWORD PTR $T362668[ebp], esp
  0164d	6a 30		 push	 48			; 00000030H
  0164f	e8 00 00 00 00	 call	 ??0CParseValue@HCParser@@QAE@H@Z ; HCParser::CParseValue::CParseValue
  01654	89 85 94 f7 ff
	ff		 mov	 DWORD PTR tv1416[ebp], eax
  0165a	8b 85 94 f7 ff
	ff		 mov	 eax, DWORD PTR tv1416[ebp]
  01660	89 85 90 f7 ff
	ff		 mov	 DWORD PTR tv2194[ebp], eax
  01666	c6 45 fc c8	 mov	 BYTE PTR __$EHRec$[ebp+8], 200 ; 000000c8H
  0166a	68 00 00 00 00	 push	 OFFSET ??_C@_1BE@OEGEIDDF@?$AAT?$AAC?$AAL?$AA_?$AA2?$AA0?$AA0?$AA2?$AAN?$AA?$AA@
  0166f	c6 45 fc c7	 mov	 BYTE PTR __$EHRec$[ebp+8], 199 ; 000000c7H
  01673	8d 8d fc fb ff
	ff		 lea	 ecx, DWORD PTR $T362667[ebp]
  01679	e8 00 00 00 00	 call	 ??0CParseConstant@HCParser@@QAE@PB_WVCParseValue@1@@Z ; HCParser::CParseConstant::CParseConstant
  0167e	89 85 8c f7 ff
	ff		 mov	 DWORD PTR tv2195[ebp], eax
  01684	8b 8d 8c f7 ff
	ff		 mov	 ecx, DWORD PTR tv2195[ebp]
  0168a	89 8d 88 f7 ff
	ff		 mov	 DWORD PTR tv2197[ebp], ecx
  01690	c6 45 fc c9	 mov	 BYTE PTR __$EHRec$[ebp+8], 201 ; 000000c9H
  01694	8b 95 88 f7 ff
	ff		 mov	 edx, DWORD PTR tv2197[ebp]
  0169a	52		 push	 edx
  0169b	b9 20 03 00 00	 mov	 ecx, OFFSET ?k_parseTunerConstants@@3QBVCParseConstant@HCParser@@B+800
  016a0	e8 00 00 00 00	 call	 ??0CParseConstant@HCParser@@QAE@ABV01@@Z
  016a5	c6 45 fc cb	 mov	 BYTE PTR __$EHRec$[ebp+8], 203 ; 000000cbH
  016a9	8d 8d fc fb ff
	ff		 lea	 ecx, DWORD PTR $T362667[ebp]
  016af	e8 00 00 00 00	 call	 ??1CParseConstant@HCParser@@QAE@XZ

; 91   :     PC( _T("HITACHI_NTSC"),                    TUNER_HITACHI_NTSC              ),

  016b4	83 ec 0c	 sub	 esp, 12			; 0000000cH
  016b7	8b cc		 mov	 ecx, esp
  016b9	89 a5 e4 fb ff
	ff		 mov	 DWORD PTR $T362670[ebp], esp
  016bf	6a 31		 push	 49			; 00000031H
  016c1	e8 00 00 00 00	 call	 ??0CParseValue@HCParser@@QAE@H@Z ; HCParser::CParseValue::CParseValue
  016c6	89 85 84 f7 ff
	ff		 mov	 DWORD PTR tv1439[ebp], eax
  016cc	8b 85 84 f7 ff
	ff		 mov	 eax, DWORD PTR tv1439[ebp]
  016d2	89 85 80 f7 ff
	ff		 mov	 DWORD PTR tv2200[ebp], eax
  016d8	c6 45 fc cc	 mov	 BYTE PTR __$EHRec$[ebp+8], 204 ; 000000ccH
  016dc	68 00 00 00 00	 push	 OFFSET ??_C@_1BK@CFFBIHHG@?$AAH?$AAI?$AAT?$AAA?$AAC?$AAH?$AAI?$AA_?$AAN?$AAT?$AAS?$AAC?$AA?$AA@
  016e1	c6 45 fc cb	 mov	 BYTE PTR __$EHRec$[ebp+8], 203 ; 000000cbH
  016e5	8d 8d e8 fb ff
	ff		 lea	 ecx, DWORD PTR $T362669[ebp]
  016eb	e8 00 00 00 00	 call	 ??0CParseConstant@HCParser@@QAE@PB_WVCParseValue@1@@Z ; HCParser::CParseConstant::CParseConstant
  016f0	89 85 7c f7 ff
	ff		 mov	 DWORD PTR tv2201[ebp], eax
  016f6	8b 8d 7c f7 ff
	ff		 mov	 ecx, DWORD PTR tv2201[ebp]
  016fc	89 8d 78 f7 ff
	ff		 mov	 DWORD PTR tv2203[ebp], ecx
  01702	c6 45 fc cd	 mov	 BYTE PTR __$EHRec$[ebp+8], 205 ; 000000cdH
  01706	8b 95 78 f7 ff
	ff		 mov	 edx, DWORD PTR tv2203[ebp]
  0170c	52		 push	 edx
  0170d	b9 30 03 00 00	 mov	 ecx, OFFSET ?k_parseTunerConstants@@3QBVCParseConstant@HCParser@@B+816
  01712	e8 00 00 00 00	 call	 ??0CParseConstant@HCParser@@QAE@ABV01@@Z
  01717	c6 45 fc cf	 mov	 BYTE PTR __$EHRec$[ebp+8], 207 ; 000000cfH
  0171b	8d 8d e8 fb ff
	ff		 lea	 ecx, DWORD PTR $T362669[ebp]
  01721	e8 00 00 00 00	 call	 ??1CParseConstant@HCParser@@QAE@XZ

; 92   :     PC( _T("PHILIPS_PAL_MK"),                TUNER_PHILIPS_PAL_MK              ),

  01726	83 ec 0c	 sub	 esp, 12			; 0000000cH
  01729	8b cc		 mov	 ecx, esp
  0172b	89 a5 d0 fb ff
	ff		 mov	 DWORD PTR $T362672[ebp], esp
  01731	6a 32		 push	 50			; 00000032H
  01733	e8 00 00 00 00	 call	 ??0CParseValue@HCParser@@QAE@H@Z ; HCParser::CParseValue::CParseValue
  01738	89 85 74 f7 ff
	ff		 mov	 DWORD PTR tv1462[ebp], eax
  0173e	8b 85 74 f7 ff
	ff		 mov	 eax, DWORD PTR tv1462[ebp]
  01744	89 85 70 f7 ff
	ff		 mov	 DWORD PTR tv2206[ebp], eax
  0174a	c6 45 fc d0	 mov	 BYTE PTR __$EHRec$[ebp+8], 208 ; 000000d0H
  0174e	68 00 00 00 00	 push	 OFFSET ??_C@_1BO@OOKBNEEN@?$AAP?$AAH?$AAI?$AAL?$AAI?$AAP?$AAS?$AA_?$AAP?$AAA?$AAL?$AA_?$AAM?$AAK?$AA?$AA@
  01753	c6 45 fc cf	 mov	 BYTE PTR __$EHRec$[ebp+8], 207 ; 000000cfH
  01757	8d 8d d4 fb ff
	ff		 lea	 ecx, DWORD PTR $T362671[ebp]
  0175d	e8 00 00 00 00	 call	 ??0CParseConstant@HCParser@@QAE@PB_WVCParseValue@1@@Z ; HCParser::CParseConstant::CParseConstant
  01762	89 85 6c f7 ff
	ff		 mov	 DWORD PTR tv2207[ebp], eax
  01768	8b 8d 6c f7 ff
	ff		 mov	 ecx, DWORD PTR tv2207[ebp]
  0176e	89 8d 68 f7 ff
	ff		 mov	 DWORD PTR tv2209[ebp], ecx
  01774	c6 45 fc d1	 mov	 BYTE PTR __$EHRec$[ebp+8], 209 ; 000000d1H
  01778	8b 95 68 f7 ff
	ff		 mov	 edx, DWORD PTR tv2209[ebp]
  0177e	52		 push	 edx
  0177f	b9 40 03 00 00	 mov	 ecx, OFFSET ?k_parseTunerConstants@@3QBVCParseConstant@HCParser@@B+832
  01784	e8 00 00 00 00	 call	 ??0CParseConstant@HCParser@@QAE@ABV01@@Z
  01789	c6 45 fc d3	 mov	 BYTE PTR __$EHRec$[ebp+8], 211 ; 000000d3H
  0178d	8d 8d d4 fb ff
	ff		 lea	 ecx, DWORD PTR $T362671[ebp]
  01793	e8 00 00 00 00	 call	 ??1CParseConstant@HCParser@@QAE@XZ

; 93   :     PC( _T("PHILIPS_FM1236_MK3"),            TUNER_PHILIPS_FM1236_MK3          ),

  01798	83 ec 0c	 sub	 esp, 12			; 0000000cH
  0179b	8b cc		 mov	 ecx, esp
  0179d	89 a5 bc fb ff
	ff		 mov	 DWORD PTR $T362674[ebp], esp
  017a3	6a 33		 push	 51			; 00000033H
  017a5	e8 00 00 00 00	 call	 ??0CParseValue@HCParser@@QAE@H@Z ; HCParser::CParseValue::CParseValue
  017aa	89 85 64 f7 ff
	ff		 mov	 DWORD PTR tv1485[ebp], eax
  017b0	8b 85 64 f7 ff
	ff		 mov	 eax, DWORD PTR tv1485[ebp]
  017b6	89 85 60 f7 ff
	ff		 mov	 DWORD PTR tv2212[ebp], eax
  017bc	c6 45 fc d4	 mov	 BYTE PTR __$EHRec$[ebp+8], 212 ; 000000d4H
  017c0	68 00 00 00 00	 push	 OFFSET ??_C@_1CG@EMNPDDAO@?$AAP?$AAH?$AAI?$AAL?$AAI?$AAP?$AAS?$AA_?$AAF?$AAM?$AA1?$AA2?$AA3?$AA6?$AA_?$AAM?$AAK?$AA3?$AA?$AA@
  017c5	c6 45 fc d3	 mov	 BYTE PTR __$EHRec$[ebp+8], 211 ; 000000d3H
  017c9	8d 8d c0 fb ff
	ff		 lea	 ecx, DWORD PTR $T362673[ebp]
  017cf	e8 00 00 00 00	 call	 ??0CParseConstant@HCParser@@QAE@PB_WVCParseValue@1@@Z ; HCParser::CParseConstant::CParseConstant
  017d4	89 85 5c f7 ff
	ff		 mov	 DWORD PTR tv2213[ebp], eax
  017da	8b 8d 5c f7 ff
	ff		 mov	 ecx, DWORD PTR tv2213[ebp]
  017e0	89 8d 58 f7 ff
	ff		 mov	 DWORD PTR tv2215[ebp], ecx
  017e6	c6 45 fc d5	 mov	 BYTE PTR __$EHRec$[ebp+8], 213 ; 000000d5H
  017ea	8b 95 58 f7 ff
	ff		 mov	 edx, DWORD PTR tv2215[ebp]
  017f0	52		 push	 edx
  017f1	b9 50 03 00 00	 mov	 ecx, OFFSET ?k_parseTunerConstants@@3QBVCParseConstant@HCParser@@B+848
  017f6	e8 00 00 00 00	 call	 ??0CParseConstant@HCParser@@QAE@ABV01@@Z
  017fb	c6 45 fc d7	 mov	 BYTE PTR __$EHRec$[ebp+8], 215 ; 000000d7H
  017ff	8d 8d c0 fb ff
	ff		 lea	 ecx, DWORD PTR $T362673[ebp]
  01805	e8 00 00 00 00	 call	 ??1CParseConstant@HCParser@@QAE@XZ

; 94   :     PC( _T("LG_NTSC_TAPE"),                    TUNER_LG_NTSC_TAPE              ),

  0180a	83 ec 0c	 sub	 esp, 12			; 0000000cH
  0180d	8b cc		 mov	 ecx, esp
  0180f	89 a5 a8 fb ff
	ff		 mov	 DWORD PTR $T362676[ebp], esp
  01815	6a 34		 push	 52			; 00000034H
  01817	e8 00 00 00 00	 call	 ??0CParseValue@HCParser@@QAE@H@Z ; HCParser::CParseValue::CParseValue
  0181c	89 85 54 f7 ff
	ff		 mov	 DWORD PTR tv1508[ebp], eax
  01822	8b 85 54 f7 ff
	ff		 mov	 eax, DWORD PTR tv1508[ebp]
  01828	89 85 50 f7 ff
	ff		 mov	 DWORD PTR tv2218[ebp], eax
  0182e	c6 45 fc d8	 mov	 BYTE PTR __$EHRec$[ebp+8], 216 ; 000000d8H
  01832	68 00 00 00 00	 push	 OFFSET ??_C@_1BK@JHDPBOPP@?$AAL?$AAG?$AA_?$AAN?$AAT?$AAS?$AAC?$AA_?$AAT?$AAA?$AAP?$AAE?$AA?$AA@
  01837	c6 45 fc d7	 mov	 BYTE PTR __$EHRec$[ebp+8], 215 ; 000000d7H
  0183b	8d 8d ac fb ff
	ff		 lea	 ecx, DWORD PTR $T362675[ebp]
  01841	e8 00 00 00 00	 call	 ??0CParseConstant@HCParser@@QAE@PB_WVCParseValue@1@@Z ; HCParser::CParseConstant::CParseConstant
  01846	89 85 4c f7 ff
	ff		 mov	 DWORD PTR tv2219[ebp], eax
  0184c	8b 8d 4c f7 ff
	ff		 mov	 ecx, DWORD PTR tv2219[ebp]
  01852	89 8d 48 f7 ff
	ff		 mov	 DWORD PTR tv2221[ebp], ecx
  01858	c6 45 fc d9	 mov	 BYTE PTR __$EHRec$[ebp+8], 217 ; 000000d9H
  0185c	8b 95 48 f7 ff
	ff		 mov	 edx, DWORD PTR tv2221[ebp]
  01862	52		 push	 edx
  01863	b9 60 03 00 00	 mov	 ecx, OFFSET ?k_parseTunerConstants@@3QBVCParseConstant@HCParser@@B+864
  01868	e8 00 00 00 00	 call	 ??0CParseConstant@HCParser@@QAE@ABV01@@Z
  0186d	c6 45 fc db	 mov	 BYTE PTR __$EHRec$[ebp+8], 219 ; 000000dbH
  01871	8d 8d ac fb ff
	ff		 lea	 ecx, DWORD PTR $T362675[ebp]
  01877	e8 00 00 00 00	 call	 ??1CParseConstant@HCParser@@QAE@XZ

; 95   :     PC( _T("TNF_8831BGFF"),                    TUNER_TNF_8831BGFF              ),

  0187c	83 ec 0c	 sub	 esp, 12			; 0000000cH
  0187f	8b cc		 mov	 ecx, esp
  01881	89 a5 94 fb ff
	ff		 mov	 DWORD PTR $T362678[ebp], esp
  01887	6a 35		 push	 53			; 00000035H
  01889	e8 00 00 00 00	 call	 ??0CParseValue@HCParser@@QAE@H@Z ; HCParser::CParseValue::CParseValue
  0188e	89 85 44 f7 ff
	ff		 mov	 DWORD PTR tv1531[ebp], eax
  01894	8b 85 44 f7 ff
	ff		 mov	 eax, DWORD PTR tv1531[ebp]
  0189a	89 85 40 f7 ff
	ff		 mov	 DWORD PTR tv2224[ebp], eax
  018a0	c6 45 fc dc	 mov	 BYTE PTR __$EHRec$[ebp+8], 220 ; 000000dcH
  018a4	68 00 00 00 00	 push	 OFFSET ??_C@_1BK@CBBAAEDD@?$AAT?$AAN?$AAF?$AA_?$AA8?$AA8?$AA3?$AA1?$AAB?$AAG?$AAF?$AAF?$AA?$AA@
  018a9	c6 45 fc db	 mov	 BYTE PTR __$EHRec$[ebp+8], 219 ; 000000dbH
  018ad	8d 8d 98 fb ff
	ff		 lea	 ecx, DWORD PTR $T362677[ebp]
  018b3	e8 00 00 00 00	 call	 ??0CParseConstant@HCParser@@QAE@PB_WVCParseValue@1@@Z ; HCParser::CParseConstant::CParseConstant
  018b8	89 85 3c f7 ff
	ff		 mov	 DWORD PTR tv2225[ebp], eax
  018be	8b 8d 3c f7 ff
	ff		 mov	 ecx, DWORD PTR tv2225[ebp]
  018c4	89 8d 38 f7 ff
	ff		 mov	 DWORD PTR tv2227[ebp], ecx
  018ca	c6 45 fc dd	 mov	 BYTE PTR __$EHRec$[ebp+8], 221 ; 000000ddH
  018ce	8b 95 38 f7 ff
	ff		 mov	 edx, DWORD PTR tv2227[ebp]
  018d4	52		 push	 edx
  018d5	b9 70 03 00 00	 mov	 ecx, OFFSET ?k_parseTunerConstants@@3QBVCParseConstant@HCParser@@B+880
  018da	e8 00 00 00 00	 call	 ??0CParseConstant@HCParser@@QAE@ABV01@@Z
  018df	c6 45 fc df	 mov	 BYTE PTR __$EHRec$[ebp+8], 223 ; 000000dfH
  018e3	8d 8d 98 fb ff
	ff		 lea	 ecx, DWORD PTR $T362677[ebp]
  018e9	e8 00 00 00 00	 call	 ??1CParseConstant@HCParser@@QAE@XZ

; 96   :     PC( _T("PHILIPS_FM1256_IH3"),            TUNER_PHILIPS_FM1256_IH3          ),

  018ee	83 ec 0c	 sub	 esp, 12			; 0000000cH
  018f1	8b cc		 mov	 ecx, esp
  018f3	89 a5 80 fb ff
	ff		 mov	 DWORD PTR $T362680[ebp], esp
  018f9	6a 36		 push	 54			; 00000036H
  018fb	e8 00 00 00 00	 call	 ??0CParseValue@HCParser@@QAE@H@Z ; HCParser::CParseValue::CParseValue
  01900	89 85 34 f7 ff
	ff		 mov	 DWORD PTR tv1554[ebp], eax
  01906	8b 85 34 f7 ff
	ff		 mov	 eax, DWORD PTR tv1554[ebp]
  0190c	89 85 30 f7 ff
	ff		 mov	 DWORD PTR tv2230[ebp], eax
  01912	c6 45 fc e0	 mov	 BYTE PTR __$EHRec$[ebp+8], 224 ; 000000e0H
  01916	68 00 00 00 00	 push	 OFFSET ??_C@_1CG@LGMDAEOM@?$AAP?$AAH?$AAI?$AAL?$AAI?$AAP?$AAS?$AA_?$AAF?$AAM?$AA1?$AA2?$AA5?$AA6?$AA_?$AAI?$AAH?$AA3?$AA?$AA@
  0191b	c6 45 fc df	 mov	 BYTE PTR __$EHRec$[ebp+8], 223 ; 000000dfH
  0191f	8d 8d 84 fb ff
	ff		 lea	 ecx, DWORD PTR $T362679[ebp]
  01925	e8 00 00 00 00	 call	 ??0CParseConstant@HCParser@@QAE@PB_WVCParseValue@1@@Z ; HCParser::CParseConstant::CParseConstant
  0192a	89 85 2c f7 ff
	ff		 mov	 DWORD PTR tv2231[ebp], eax
  01930	8b 8d 2c f7 ff
	ff		 mov	 ecx, DWORD PTR tv2231[ebp]
  01936	89 8d 28 f7 ff
	ff		 mov	 DWORD PTR tv2233[ebp], ecx
  0193c	c6 45 fc e1	 mov	 BYTE PTR __$EHRec$[ebp+8], 225 ; 000000e1H
  01940	8b 95 28 f7 ff
	ff		 mov	 edx, DWORD PTR tv2233[ebp]
  01946	52		 push	 edx
  01947	b9 80 03 00 00	 mov	 ecx, OFFSET ?k_parseTunerConstants@@3QBVCParseConstant@HCParser@@B+896
  0194c	e8 00 00 00 00	 call	 ??0CParseConstant@HCParser@@QAE@ABV01@@Z
  01951	c6 45 fc e3	 mov	 BYTE PTR __$EHRec$[ebp+8], 227 ; 000000e3H
  01955	8d 8d 84 fb ff
	ff		 lea	 ecx, DWORD PTR $T362679[ebp]
  0195b	e8 00 00 00 00	 call	 ??1CParseConstant@HCParser@@QAE@XZ

; 97   :     PC( _T("PHILIPS_FQ1286"),                TUNER_PHILIPS_FQ1286              ),

  01960	83 ec 0c	 sub	 esp, 12			; 0000000cH
  01963	8b cc		 mov	 ecx, esp
  01965	89 a5 6c fb ff
	ff		 mov	 DWORD PTR $T362682[ebp], esp
  0196b	6a 37		 push	 55			; 00000037H
  0196d	e8 00 00 00 00	 call	 ??0CParseValue@HCParser@@QAE@H@Z ; HCParser::CParseValue::CParseValue
  01972	89 85 24 f7 ff
	ff		 mov	 DWORD PTR tv1577[ebp], eax
  01978	8b 85 24 f7 ff
	ff		 mov	 eax, DWORD PTR tv1577[ebp]
  0197e	89 85 20 f7 ff
	ff		 mov	 DWORD PTR tv2236[ebp], eax
  01984	c6 45 fc e4	 mov	 BYTE PTR __$EHRec$[ebp+8], 228 ; 000000e4H
  01988	68 00 00 00 00	 push	 OFFSET ??_C@_1BO@PGCKBBBK@?$AAP?$AAH?$AAI?$AAL?$AAI?$AAP?$AAS?$AA_?$AAF?$AAQ?$AA1?$AA2?$AA8?$AA6?$AA?$AA@
  0198d	c6 45 fc e3	 mov	 BYTE PTR __$EHRec$[ebp+8], 227 ; 000000e3H
  01991	8d 8d 70 fb ff
	ff		 lea	 ecx, DWORD PTR $T362681[ebp]
  01997	e8 00 00 00 00	 call	 ??0CParseConstant@HCParser@@QAE@PB_WVCParseValue@1@@Z ; HCParser::CParseConstant::CParseConstant
  0199c	89 85 1c f7 ff
	ff		 mov	 DWORD PTR tv2237[ebp], eax
  019a2	8b 8d 1c f7 ff
	ff		 mov	 ecx, DWORD PTR tv2237[ebp]
  019a8	89 8d 18 f7 ff
	ff		 mov	 DWORD PTR tv2239[ebp], ecx
  019ae	c6 45 fc e5	 mov	 BYTE PTR __$EHRec$[ebp+8], 229 ; 000000e5H
  019b2	8b 95 18 f7 ff
	ff		 mov	 edx, DWORD PTR tv2239[ebp]
  019b8	52		 push	 edx
  019b9	b9 90 03 00 00	 mov	 ecx, OFFSET ?k_parseTunerConstants@@3QBVCParseConstant@HCParser@@B+912
  019be	e8 00 00 00 00	 call	 ??0CParseConstant@HCParser@@QAE@ABV01@@Z
  019c3	c6 45 fc e7	 mov	 BYTE PTR __$EHRec$[ebp+8], 231 ; 000000e7H
  019c7	8d 8d 70 fb ff
	ff		 lea	 ecx, DWORD PTR $T362681[ebp]
  019cd	e8 00 00 00 00	 call	 ??1CParseConstant@HCParser@@QAE@XZ

; 98   :     PC( _T("LG_PAL_TAPE"),                    TUNER_LG_PAL_TAPE                  ),

  019d2	83 ec 0c	 sub	 esp, 12			; 0000000cH
  019d5	8b cc		 mov	 ecx, esp
  019d7	89 a5 58 fb ff
	ff		 mov	 DWORD PTR $T362684[ebp], esp
  019dd	6a 38		 push	 56			; 00000038H
  019df	e8 00 00 00 00	 call	 ??0CParseValue@HCParser@@QAE@H@Z ; HCParser::CParseValue::CParseValue
  019e4	89 85 14 f7 ff
	ff		 mov	 DWORD PTR tv1600[ebp], eax
  019ea	8b 85 14 f7 ff
	ff		 mov	 eax, DWORD PTR tv1600[ebp]
  019f0	89 85 10 f7 ff
	ff		 mov	 DWORD PTR tv2242[ebp], eax
  019f6	c6 45 fc e8	 mov	 BYTE PTR __$EHRec$[ebp+8], 232 ; 000000e8H
  019fa	68 00 00 00 00	 push	 OFFSET ??_C@_1BI@DMIKHBF@?$AAL?$AAG?$AA_?$AAP?$AAA?$AAL?$AA_?$AAT?$AAA?$AAP?$AAE?$AA?$AA@
  019ff	c6 45 fc e7	 mov	 BYTE PTR __$EHRec$[ebp+8], 231 ; 000000e7H
  01a03	8d 8d 5c fb ff
	ff		 lea	 ecx, DWORD PTR $T362683[ebp]
  01a09	e8 00 00 00 00	 call	 ??0CParseConstant@HCParser@@QAE@PB_WVCParseValue@1@@Z ; HCParser::CParseConstant::CParseConstant
  01a0e	89 85 0c f7 ff
	ff		 mov	 DWORD PTR tv2243[ebp], eax
  01a14	8b 8d 0c f7 ff
	ff		 mov	 ecx, DWORD PTR tv2243[ebp]
  01a1a	89 8d 08 f7 ff
	ff		 mov	 DWORD PTR tv2245[ebp], ecx
  01a20	c6 45 fc e9	 mov	 BYTE PTR __$EHRec$[ebp+8], 233 ; 000000e9H
  01a24	8b 95 08 f7 ff
	ff		 mov	 edx, DWORD PTR tv2245[ebp]
  01a2a	52		 push	 edx
  01a2b	b9 a0 03 00 00	 mov	 ecx, OFFSET ?k_parseTunerConstants@@3QBVCParseConstant@HCParser@@B+928
  01a30	e8 00 00 00 00	 call	 ??0CParseConstant@HCParser@@QAE@ABV01@@Z
  01a35	c6 45 fc eb	 mov	 BYTE PTR __$EHRec$[ebp+8], 235 ; 000000ebH
  01a39	8d 8d 5c fb ff
	ff		 lea	 ecx, DWORD PTR $T362683[ebp]
  01a3f	e8 00 00 00 00	 call	 ??1CParseConstant@HCParser@@QAE@XZ

; 99   :     PC( _T("TUNER_PHILIPS_FQ1216AME_MK4"),  TUNER_PHILIPS_FQ1216AME_MK4        ),

  01a44	83 ec 0c	 sub	 esp, 12			; 0000000cH
  01a47	8b cc		 mov	 ecx, esp
  01a49	89 a5 44 fb ff
	ff		 mov	 DWORD PTR $T362686[ebp], esp
  01a4f	6a 39		 push	 57			; 00000039H
  01a51	e8 00 00 00 00	 call	 ??0CParseValue@HCParser@@QAE@H@Z ; HCParser::CParseValue::CParseValue
  01a56	89 85 04 f7 ff
	ff		 mov	 DWORD PTR tv1623[ebp], eax
  01a5c	8b 85 04 f7 ff
	ff		 mov	 eax, DWORD PTR tv1623[ebp]
  01a62	89 85 00 f7 ff
	ff		 mov	 DWORD PTR tv2248[ebp], eax
  01a68	c6 45 fc ec	 mov	 BYTE PTR __$EHRec$[ebp+8], 236 ; 000000ecH
  01a6c	68 00 00 00 00	 push	 OFFSET ??_C@_1DI@EAGAPDHM@?$AAT?$AAU?$AAN?$AAE?$AAR?$AA_?$AAP?$AAH?$AAI?$AAL?$AAI?$AAP?$AAS?$AA_?$AAF?$AAQ?$AA1?$AA2?$AA1?$AA6?$AAA?$AAM?$AAE?$AA_?$AAM?$AAK?$AA4?$AA?$AA@
  01a71	c6 45 fc eb	 mov	 BYTE PTR __$EHRec$[ebp+8], 235 ; 000000ebH
  01a75	8d 8d 48 fb ff
	ff		 lea	 ecx, DWORD PTR $T362685[ebp]
  01a7b	e8 00 00 00 00	 call	 ??0CParseConstant@HCParser@@QAE@PB_WVCParseValue@1@@Z ; HCParser::CParseConstant::CParseConstant
  01a80	89 85 fc f6 ff
	ff		 mov	 DWORD PTR tv2249[ebp], eax
  01a86	8b 8d fc f6 ff
	ff		 mov	 ecx, DWORD PTR tv2249[ebp]
  01a8c	89 8d f8 f6 ff
	ff		 mov	 DWORD PTR tv2251[ebp], ecx
  01a92	c6 45 fc ed	 mov	 BYTE PTR __$EHRec$[ebp+8], 237 ; 000000edH
  01a96	8b 95 f8 f6 ff
	ff		 mov	 edx, DWORD PTR tv2251[ebp]
  01a9c	52		 push	 edx
  01a9d	b9 b0 03 00 00	 mov	 ecx, OFFSET ?k_parseTunerConstants@@3QBVCParseConstant@HCParser@@B+944
  01aa2	e8 00 00 00 00	 call	 ??0CParseConstant@HCParser@@QAE@ABV01@@Z
  01aa7	c6 45 fc ef	 mov	 BYTE PTR __$EHRec$[ebp+8], 239 ; 000000efH
  01aab	8d 8d 48 fb ff
	ff		 lea	 ecx, DWORD PTR $T362685[ebp]
  01ab1	e8 00 00 00 00	 call	 ??1CParseConstant@HCParser@@QAE@XZ

; 100  :     PC( _T("PHILIPS_FQ1236A_MK4"),            TUNER_PHILIPS_FQ1236A_MK4          ),

  01ab6	83 ec 0c	 sub	 esp, 12			; 0000000cH
  01ab9	8b cc		 mov	 ecx, esp
  01abb	89 a5 30 fb ff
	ff		 mov	 DWORD PTR $T362688[ebp], esp
  01ac1	6a 3a		 push	 58			; 0000003aH
  01ac3	e8 00 00 00 00	 call	 ??0CParseValue@HCParser@@QAE@H@Z ; HCParser::CParseValue::CParseValue
  01ac8	89 85 f4 f6 ff
	ff		 mov	 DWORD PTR tv1646[ebp], eax
  01ace	8b 85 f4 f6 ff
	ff		 mov	 eax, DWORD PTR tv1646[ebp]
  01ad4	89 85 f0 f6 ff
	ff		 mov	 DWORD PTR tv2254[ebp], eax
  01ada	c6 45 fc f0	 mov	 BYTE PTR __$EHRec$[ebp+8], 240 ; 000000f0H
  01ade	68 00 00 00 00	 push	 OFFSET ??_C@_1CI@PFGDHJOM@?$AAP?$AAH?$AAI?$AAL?$AAI?$AAP?$AAS?$AA_?$AAF?$AAQ?$AA1?$AA2?$AA3?$AA6?$AAA?$AA_?$AAM?$AAK?$AA4?$AA?$AA@
  01ae3	c6 45 fc ef	 mov	 BYTE PTR __$EHRec$[ebp+8], 239 ; 000000efH
  01ae7	8d 8d 34 fb ff
	ff		 lea	 ecx, DWORD PTR $T362687[ebp]
  01aed	e8 00 00 00 00	 call	 ??0CParseConstant@HCParser@@QAE@PB_WVCParseValue@1@@Z ; HCParser::CParseConstant::CParseConstant
  01af2	89 85 ec f6 ff
	ff		 mov	 DWORD PTR tv2255[ebp], eax
  01af8	8b 8d ec f6 ff
	ff		 mov	 ecx, DWORD PTR tv2255[ebp]
  01afe	89 8d e8 f6 ff
	ff		 mov	 DWORD PTR tv2257[ebp], ecx
  01b04	c6 45 fc f1	 mov	 BYTE PTR __$EHRec$[ebp+8], 241 ; 000000f1H
  01b08	8b 95 e8 f6 ff
	ff		 mov	 edx, DWORD PTR tv2257[ebp]
  01b0e	52		 push	 edx
  01b0f	b9 c0 03 00 00	 mov	 ecx, OFFSET ?k_parseTunerConstants@@3QBVCParseConstant@HCParser@@B+960
  01b14	e8 00 00 00 00	 call	 ??0CParseConstant@HCParser@@QAE@ABV01@@Z
  01b19	c6 45 fc f3	 mov	 BYTE PTR __$EHRec$[ebp+8], 243 ; 000000f3H
  01b1d	8d 8d 34 fb ff
	ff		 lea	 ecx, DWORD PTR $T362687[ebp]
  01b23	e8 00 00 00 00	 call	 ??1CParseConstant@HCParser@@QAE@XZ

; 101  :     PC( _T("PHILIPS_TDA8275"),                TUNER_TDA8275                      ),

  01b28	83 ec 0c	 sub	 esp, 12			; 0000000cH
  01b2b	8b cc		 mov	 ecx, esp
  01b2d	89 a5 1c fb ff
	ff		 mov	 DWORD PTR $T362690[ebp], esp
  01b33	6a 3b		 push	 59			; 0000003bH
  01b35	e8 00 00 00 00	 call	 ??0CParseValue@HCParser@@QAE@H@Z ; HCParser::CParseValue::CParseValue
  01b3a	89 85 e4 f6 ff
	ff		 mov	 DWORD PTR tv1669[ebp], eax
  01b40	8b 85 e4 f6 ff
	ff		 mov	 eax, DWORD PTR tv1669[ebp]
  01b46	89 85 e0 f6 ff
	ff		 mov	 DWORD PTR tv2260[ebp], eax
  01b4c	c6 45 fc f4	 mov	 BYTE PTR __$EHRec$[ebp+8], 244 ; 000000f4H
  01b50	68 00 00 00 00	 push	 OFFSET ??_C@_1CA@PHAKLDDM@?$AAP?$AAH?$AAI?$AAL?$AAI?$AAP?$AAS?$AA_?$AAT?$AAD?$AAA?$AA8?$AA2?$AA7?$AA5?$AA?$AA@
  01b55	c6 45 fc f3	 mov	 BYTE PTR __$EHRec$[ebp+8], 243 ; 000000f3H
  01b59	8d 8d 20 fb ff
	ff		 lea	 ecx, DWORD PTR $T362689[ebp]
  01b5f	e8 00 00 00 00	 call	 ??0CParseConstant@HCParser@@QAE@PB_WVCParseValue@1@@Z ; HCParser::CParseConstant::CParseConstant
  01b64	89 85 dc f6 ff
	ff		 mov	 DWORD PTR tv2261[ebp], eax
  01b6a	8b 8d dc f6 ff
	ff		 mov	 ecx, DWORD PTR tv2261[ebp]
  01b70	89 8d d8 f6 ff
	ff		 mov	 DWORD PTR tv2263[ebp], ecx
  01b76	c6 45 fc f5	 mov	 BYTE PTR __$EHRec$[ebp+8], 245 ; 000000f5H
  01b7a	8b 95 d8 f6 ff
	ff		 mov	 edx, DWORD PTR tv2263[ebp]
  01b80	52		 push	 edx
  01b81	b9 d0 03 00 00	 mov	 ecx, OFFSET ?k_parseTunerConstants@@3QBVCParseConstant@HCParser@@B+976
  01b86	e8 00 00 00 00	 call	 ??0CParseConstant@HCParser@@QAE@ABV01@@Z
  01b8b	c6 45 fc f7	 mov	 BYTE PTR __$EHRec$[ebp+8], 247 ; 000000f7H
  01b8f	8d 8d 20 fb ff
	ff		 lea	 ecx, DWORD PTR $T362689[ebp]
  01b95	e8 00 00 00 00	 call	 ??1CParseConstant@HCParser@@QAE@XZ

; 102  :     PC( _T("YMEC_TVF_8531MF"),              TUNER_YMEC_TVF_8531MF           ),

  01b9a	83 ec 0c	 sub	 esp, 12			; 0000000cH
  01b9d	8b cc		 mov	 ecx, esp
  01b9f	89 a5 08 fb ff
	ff		 mov	 DWORD PTR $T362692[ebp], esp
  01ba5	6a 3c		 push	 60			; 0000003cH
  01ba7	e8 00 00 00 00	 call	 ??0CParseValue@HCParser@@QAE@H@Z ; HCParser::CParseValue::CParseValue
  01bac	89 85 d4 f6 ff
	ff		 mov	 DWORD PTR tv1692[ebp], eax
  01bb2	8b 85 d4 f6 ff
	ff		 mov	 eax, DWORD PTR tv1692[ebp]
  01bb8	89 85 d0 f6 ff
	ff		 mov	 DWORD PTR tv2266[ebp], eax
  01bbe	c6 45 fc f8	 mov	 BYTE PTR __$EHRec$[ebp+8], 248 ; 000000f8H
  01bc2	68 00 00 00 00	 push	 OFFSET ??_C@_1CA@NIDJODPE@?$AAY?$AAM?$AAE?$AAC?$AA_?$AAT?$AAV?$AAF?$AA_?$AA8?$AA5?$AA3?$AA1?$AAM?$AAF?$AA?$AA@
  01bc7	c6 45 fc f7	 mov	 BYTE PTR __$EHRec$[ebp+8], 247 ; 000000f7H
  01bcb	8d 8d 0c fb ff
	ff		 lea	 ecx, DWORD PTR $T362691[ebp]
  01bd1	e8 00 00 00 00	 call	 ??0CParseConstant@HCParser@@QAE@PB_WVCParseValue@1@@Z ; HCParser::CParseConstant::CParseConstant
  01bd6	89 85 cc f6 ff
	ff		 mov	 DWORD PTR tv2267[ebp], eax
  01bdc	8b 8d cc f6 ff
	ff		 mov	 ecx, DWORD PTR tv2267[ebp]
  01be2	89 8d c8 f6 ff
	ff		 mov	 DWORD PTR tv2269[ebp], ecx
  01be8	c6 45 fc f9	 mov	 BYTE PTR __$EHRec$[ebp+8], 249 ; 000000f9H
  01bec	8b 95 c8 f6 ff
	ff		 mov	 edx, DWORD PTR tv2269[ebp]
  01bf2	52		 push	 edx
  01bf3	b9 e0 03 00 00	 mov	 ecx, OFFSET ?k_parseTunerConstants@@3QBVCParseConstant@HCParser@@B+992
  01bf8	e8 00 00 00 00	 call	 ??0CParseConstant@HCParser@@QAE@ABV01@@Z
  01bfd	c6 45 fc fb	 mov	 BYTE PTR __$EHRec$[ebp+8], 251 ; 000000fbH
  01c01	8d 8d 0c fb ff
	ff		 lea	 ecx, DWORD PTR $T362691[ebp]
  01c07	e8 00 00 00 00	 call	 ??1CParseConstant@HCParser@@QAE@XZ

; 103  :     PC( _T("YMEC_TVF_5533MF"),              TUNER_YMEC_TVF_5533MF           ),

  01c0c	83 ec 0c	 sub	 esp, 12			; 0000000cH
  01c0f	8b cc		 mov	 ecx, esp
  01c11	89 a5 f4 fa ff
	ff		 mov	 DWORD PTR $T362694[ebp], esp
  01c17	6a 3d		 push	 61			; 0000003dH
  01c19	e8 00 00 00 00	 call	 ??0CParseValue@HCParser@@QAE@H@Z ; HCParser::CParseValue::CParseValue
  01c1e	89 85 c4 f6 ff
	ff		 mov	 DWORD PTR tv1715[ebp], eax
  01c24	8b 85 c4 f6 ff
	ff		 mov	 eax, DWORD PTR tv1715[ebp]
  01c2a	89 85 c0 f6 ff
	ff		 mov	 DWORD PTR tv2272[ebp], eax
  01c30	c6 45 fc fc	 mov	 BYTE PTR __$EHRec$[ebp+8], 252 ; 000000fcH
  01c34	68 00 00 00 00	 push	 OFFSET ??_C@_1CA@CNOGJENC@?$AAY?$AAM?$AAE?$AAC?$AA_?$AAT?$AAV?$AAF?$AA_?$AA5?$AA5?$AA3?$AA3?$AAM?$AAF?$AA?$AA@
  01c39	c6 45 fc fb	 mov	 BYTE PTR __$EHRec$[ebp+8], 251 ; 000000fbH
  01c3d	8d 8d f8 fa ff
	ff		 lea	 ecx, DWORD PTR $T362693[ebp]
  01c43	e8 00 00 00 00	 call	 ??0CParseConstant@HCParser@@QAE@PB_WVCParseValue@1@@Z ; HCParser::CParseConstant::CParseConstant
  01c48	89 85 bc f6 ff
	ff		 mov	 DWORD PTR tv2273[ebp], eax
  01c4e	8b 8d bc f6 ff
	ff		 mov	 ecx, DWORD PTR tv2273[ebp]
  01c54	89 8d b8 f6 ff
	ff		 mov	 DWORD PTR tv2275[ebp], ecx
  01c5a	c6 45 fc fd	 mov	 BYTE PTR __$EHRec$[ebp+8], 253 ; 000000fdH
  01c5e	8b 95 b8 f6 ff
	ff		 mov	 edx, DWORD PTR tv2275[ebp]
  01c64	52		 push	 edx
  01c65	b9 f0 03 00 00	 mov	 ecx, OFFSET ?k_parseTunerConstants@@3QBVCParseConstant@HCParser@@B+1008
  01c6a	e8 00 00 00 00	 call	 ??0CParseConstant@HCParser@@QAE@ABV01@@Z
  01c6f	c6 45 fc ff	 mov	 BYTE PTR __$EHRec$[ebp+8], 255 ; 000000ffH
  01c73	8d 8d f8 fa ff
	ff		 lea	 ecx, DWORD PTR $T362693[ebp]
  01c79	e8 00 00 00 00	 call	 ??1CParseConstant@HCParser@@QAE@XZ

; 104  :     PC( _T("TENA_9533_DI"),                 TUNER_TENA_9533_DI              ),

  01c7e	83 ec 0c	 sub	 esp, 12			; 0000000cH
  01c81	8b cc		 mov	 ecx, esp
  01c83	89 a5 e0 fa ff
	ff		 mov	 DWORD PTR $T362696[ebp], esp
  01c89	6a 3e		 push	 62			; 0000003eH
  01c8b	e8 00 00 00 00	 call	 ??0CParseValue@HCParser@@QAE@H@Z ; HCParser::CParseValue::CParseValue
  01c90	89 85 b4 f6 ff
	ff		 mov	 DWORD PTR tv1738[ebp], eax
  01c96	8b 85 b4 f6 ff
	ff		 mov	 eax, DWORD PTR tv1738[ebp]
  01c9c	89 85 b0 f6 ff
	ff		 mov	 DWORD PTR tv2278[ebp], eax
  01ca2	c7 45 fc 00 01
	00 00		 mov	 DWORD PTR __$EHRec$[ebp+8], 256 ; 00000100H
  01ca9	68 00 00 00 00	 push	 OFFSET ??_C@_1BK@PEHEKEAO@?$AAT?$AAE?$AAN?$AAA?$AA_?$AA9?$AA5?$AA3?$AA3?$AA_?$AAD?$AAI?$AA?$AA@
  01cae	c7 45 fc ff 00
	00 00		 mov	 DWORD PTR __$EHRec$[ebp+8], 255 ; 000000ffH
  01cb5	8d 8d e4 fa ff
	ff		 lea	 ecx, DWORD PTR $T362695[ebp]
  01cbb	e8 00 00 00 00	 call	 ??0CParseConstant@HCParser@@QAE@PB_WVCParseValue@1@@Z ; HCParser::CParseConstant::CParseConstant
  01cc0	89 85 ac f6 ff
	ff		 mov	 DWORD PTR tv2279[ebp], eax
  01cc6	8b 8d ac f6 ff
	ff		 mov	 ecx, DWORD PTR tv2279[ebp]
  01ccc	89 8d a8 f6 ff
	ff		 mov	 DWORD PTR tv2281[ebp], ecx
  01cd2	c7 45 fc 01 01
	00 00		 mov	 DWORD PTR __$EHRec$[ebp+8], 257 ; 00000101H
  01cd9	8b 95 a8 f6 ff
	ff		 mov	 edx, DWORD PTR tv2281[ebp]
  01cdf	52		 push	 edx
  01ce0	b9 00 04 00 00	 mov	 ecx, OFFSET ?k_parseTunerConstants@@3QBVCParseConstant@HCParser@@B+1024
  01ce5	e8 00 00 00 00	 call	 ??0CParseConstant@HCParser@@QAE@ABV01@@Z
  01cea	c6 45 fc 03	 mov	 BYTE PTR __$EHRec$[ebp+8], 3
  01cee	8d 8d e4 fa ff
	ff		 lea	 ecx, DWORD PTR $T362695[ebp]
  01cf4	e8 00 00 00 00	 call	 ??1CParseConstant@HCParser@@QAE@XZ

; 105  :     PC( _T("PHILIPS_FMD1216ME_MK3"),        TUNER_PHILIPS_FMD1216ME_MK3     ),

  01cf9	83 ec 0c	 sub	 esp, 12			; 0000000cH
  01cfc	8b cc		 mov	 ecx, esp
  01cfe	89 a5 cc fa ff
	ff		 mov	 DWORD PTR $T362698[ebp], esp
  01d04	6a 3f		 push	 63			; 0000003fH
  01d06	e8 00 00 00 00	 call	 ??0CParseValue@HCParser@@QAE@H@Z ; HCParser::CParseValue::CParseValue
  01d0b	89 85 a4 f6 ff
	ff		 mov	 DWORD PTR tv1793[ebp], eax
  01d11	8b 85 a4 f6 ff
	ff		 mov	 eax, DWORD PTR tv1793[ebp]
  01d17	89 85 a0 f6 ff
	ff		 mov	 DWORD PTR tv2284[ebp], eax
  01d1d	c6 45 fc 04	 mov	 BYTE PTR __$EHRec$[ebp+8], 4
  01d21	68 00 00 00 00	 push	 OFFSET ??_C@_1CM@NKAGKMMA@?$AAP?$AAH?$AAI?$AAL?$AAI?$AAP?$AAS?$AA_?$AAF?$AAM?$AAD?$AA1?$AA2?$AA1?$AA6?$AAM?$AAE?$AA_?$AAM?$AAK?$AA3?$AA?$AA@
  01d26	c6 45 fc 03	 mov	 BYTE PTR __$EHRec$[ebp+8], 3
  01d2a	8d 8d d0 fa ff
	ff		 lea	 ecx, DWORD PTR $T362697[ebp]
  01d30	e8 00 00 00 00	 call	 ??0CParseConstant@HCParser@@QAE@PB_WVCParseValue@1@@Z ; HCParser::CParseConstant::CParseConstant
  01d35	89 85 9c f6 ff
	ff		 mov	 DWORD PTR tv2285[ebp], eax
  01d3b	8b 8d 9c f6 ff
	ff		 mov	 ecx, DWORD PTR tv2285[ebp]
  01d41	89 8d 98 f6 ff
	ff		 mov	 DWORD PTR tv2287[ebp], ecx
  01d47	c6 45 fc 05	 mov	 BYTE PTR __$EHRec$[ebp+8], 5
  01d4b	8b 95 98 f6 ff
	ff		 mov	 edx, DWORD PTR tv2287[ebp]
  01d51	52		 push	 edx
  01d52	b9 10 04 00 00	 mov	 ecx, OFFSET ?k_parseTunerConstants@@3QBVCParseConstant@HCParser@@B+1040
  01d57	e8 00 00 00 00	 call	 ??0CParseConstant@HCParser@@QAE@ABV01@@Z
  01d5c	c6 45 fc 07	 mov	 BYTE PTR __$EHRec$[ebp+8], 7
  01d60	8d 8d d0 fa ff
	ff		 lea	 ecx, DWORD PTR $T362697[ebp]
  01d66	e8 00 00 00 00	 call	 ??1CParseConstant@HCParser@@QAE@XZ

; 106  :     PC( NULL )
; 107  : };

  01d6b	83 ec 0c	 sub	 esp, 12			; 0000000cH
  01d6e	8b cc		 mov	 ecx, esp
  01d70	89 a5 b8 fa ff
	ff		 mov	 DWORD PTR $T362700[ebp], esp
  01d76	e8 00 00 00 00	 call	 ??0CParseValue@HCParser@@QAE@XZ ; HCParser::CParseValue::CParseValue
  01d7b	89 85 94 f6 ff
	ff		 mov	 DWORD PTR tv1816[ebp], eax
  01d81	8b 85 94 f6 ff
	ff		 mov	 eax, DWORD PTR tv1816[ebp]
  01d87	89 85 90 f6 ff
	ff		 mov	 DWORD PTR tv2290[ebp], eax
  01d8d	c6 45 fc 08	 mov	 BYTE PTR __$EHRec$[ebp+8], 8
  01d91	6a 00		 push	 0
  01d93	c6 45 fc 07	 mov	 BYTE PTR __$EHRec$[ebp+8], 7
  01d97	8d 8d bc fa ff
	ff		 lea	 ecx, DWORD PTR $T362699[ebp]
  01d9d	e8 00 00 00 00	 call	 ??0CParseConstant@HCParser@@QAE@PB_WVCParseValue@1@@Z ; HCParser::CParseConstant::CParseConstant
  01da2	89 85 8c f6 ff
	ff		 mov	 DWORD PTR tv2291[ebp], eax
  01da8	8b 8d 8c f6 ff
	ff		 mov	 ecx, DWORD PTR tv2291[ebp]
  01dae	89 8d 88 f6 ff
	ff		 mov	 DWORD PTR tv2293[ebp], ecx
  01db4	c6 45 fc 09	 mov	 BYTE PTR __$EHRec$[ebp+8], 9
  01db8	8b 95 88 f6 ff
	ff		 mov	 edx, DWORD PTR tv2293[ebp]
  01dbe	52		 push	 edx
  01dbf	b9 20 04 00 00	 mov	 ecx, OFFSET ?k_parseTunerConstants@@3QBVCParseConstant@HCParser@@B+1056
  01dc4	e8 00 00 00 00	 call	 ??0CParseConstant@HCParser@@QAE@ABV01@@Z
  01dc9	c6 45 fc 0b	 mov	 BYTE PTR __$EHRec$[ebp+8], 11 ; 0000000bH
  01dcd	8d 8d bc fa ff
	ff		 lea	 ecx, DWORD PTR $T362699[ebp]
  01dd3	e8 00 00 00 00	 call	 ??1CParseConstant@HCParser@@QAE@XZ
  01dd8	c7 45 fc ff ff
	ff ff		 mov	 DWORD PTR __$EHRec$[ebp+8], -1
  01ddf	68 00 00 00 00	 push	 OFFSET ??__Fk_parseTunerConstants@@YAXXZ ; `dynamic atexit destructor for 'k_parseTunerConstants''
  01de4	e8 00 00 00 00	 call	 _atexit
  01de9	83 c4 04	 add	 esp, 4
  01dec	8b 4d f4	 mov	 ecx, DWORD PTR __$EHRec$[ebp]
  01def	64 89 0d 00 00
	00 00		 mov	 DWORD PTR fs:0, ecx
  01df6	59		 pop	 ecx
  01df7	8b e5		 mov	 esp, ebp
  01df9	5d		 pop	 ebp
  01dfa	c3		 ret	 0
text$yc	ENDS
;	COMDAT text$x
text$x	SEGMENT
__unwindfunclet$??__Ek_parseTunerConstants@@YAXXZ$0:
  00000	8b 4d e0	 mov	 ecx, DWORD PTR $T362568[ebp]
  00003	e9 00 00 00 00	 jmp	 ??1CParseValue@HCParser@@UAE@XZ ; HCParser::CParseValue::~CParseValue
__unwindfunclet$??__Ek_parseTunerConstants@@YAXXZ$1:
  00008	8d 4d e4	 lea	 ecx, DWORD PTR $T362567[ebp]
  0000b	e9 00 00 00 00	 jmp	 ??1CParseConstant@HCParser@@QAE@XZ
__unwindfunclet$??__Ek_parseTunerConstants@@YAXXZ$2:
  00010	b9 00 00 00 00	 mov	 ecx, OFFSET ?k_parseTunerConstants@@3QBVCParseConstant@HCParser@@B ; k_parseTunerConstants
  00015	e9 00 00 00 00	 jmp	 ??1CParseConstant@HCParser@@QAE@XZ
__unwindfunclet$??__Ek_parseTunerConstants@@YAXXZ$3:
  0001a	8b 4d cc	 mov	 ecx, DWORD PTR $T362570[ebp]
  0001d	e9 00 00 00 00	 jmp	 ??1CParseValue@HCParser@@UAE@XZ ; HCParser::CParseValue::~CParseValue
__unwindfunclet$??__Ek_parseTunerConstants@@YAXXZ$4:
  00022	8d 4d d0	 lea	 ecx, DWORD PTR $T362569[ebp]
  00025	e9 00 00 00 00	 jmp	 ??1CParseConstant@HCParser@@QAE@XZ
__unwindfunclet$??__Ek_parseTunerConstants@@YAXXZ$5:
  0002a	b9 10 00 00 00	 mov	 ecx, OFFSET ?k_parseTunerConstants@@3QBVCParseConstant@HCParser@@B+16
  0002f	e9 00 00 00 00	 jmp	 ??1CParseConstant@HCParser@@QAE@XZ
__unwindfunclet$??__Ek_parseTunerConstants@@YAXXZ$6:
  00034	8b 4d b8	 mov	 ecx, DWORD PTR $T362572[ebp]
  00037	e9 00 00 00 00	 jmp	 ??1CParseValue@HCParser@@UAE@XZ ; HCParser::CParseValue::~CParseValue
__unwindfunclet$??__Ek_parseTunerConstants@@YAXXZ$7:
  0003c	8d 4d bc	 lea	 ecx, DWORD PTR $T362571[ebp]
  0003f	e9 00 00 00 00	 jmp	 ??1CParseConstant@HCParser@@QAE@XZ
__unwindfunclet$??__Ek_parseTunerConstants@@YAXXZ$8:
  00044	b9 20 00 00 00	 mov	 ecx, OFFSET ?k_parseTunerConstants@@3QBVCParseConstant@HCParser@@B+32
  00049	e9 00 00 00 00	 jmp	 ??1CParseConstant@HCParser@@QAE@XZ
__unwindfunclet$??__Ek_parseTunerConstants@@YAXXZ$9:
  0004e	8b 4d a4	 mov	 ecx, DWORD PTR $T362574[ebp]
  00051	e9 00 00 00 00	 jmp	 ??1CParseValue@HCParser@@UAE@XZ ; HCParser::CParseValue::~CParseValue
__unwindfunclet$??__Ek_parseTunerConstants@@YAXXZ$10:
  00056	8d 4d a8	 lea	 ecx, DWORD PTR $T362573[ebp]
  00059	e9 00 00 00 00	 jmp	 ??1CParseConstant@HCParser@@QAE@XZ
__unwindfunclet$??__Ek_parseTunerConstants@@YAXXZ$11:
  0005e	b9 30 00 00 00	 mov	 ecx, OFFSET ?k_parseTunerConstants@@3QBVCParseConstant@HCParser@@B+48
  00063	e9 00 00 00 00	 jmp	 ??1CParseConstant@HCParser@@QAE@XZ
__unwindfunclet$??__Ek_parseTunerConstants@@YAXXZ$12:
  00068	8b 4d 90	 mov	 ecx, DWORD PTR $T362576[ebp]
  0006b	e9 00 00 00 00	 jmp	 ??1CParseValue@HCParser@@UAE@XZ ; HCParser::CParseValue::~CParseValue
__unwindfunclet$??__Ek_parseTunerConstants@@YAXXZ$13:
  00070	8d 4d 94	 lea	 ecx, DWORD PTR $T362575[ebp]
  00073	e9 00 00 00 00	 jmp	 ??1CParseConstant@HCParser@@QAE@XZ
__unwindfunclet$??__Ek_parseTunerConstants@@YAXXZ$14:
  00078	b9 40 00 00 00	 mov	 ecx, OFFSET ?k_parseTunerConstants@@3QBVCParseConstant@HCParser@@B+64
  0007d	e9 00 00 00 00	 jmp	 ??1CParseConstant@HCParser@@QAE@XZ
__unwindfunclet$??__Ek_parseTunerConstants@@YAXXZ$15:
  00082	8b 8d 7c ff ff
	ff		 mov	 ecx, DWORD PTR $T362578[ebp]
  00088	e9 00 00 00 00	 jmp	 ??1CParseValue@HCParser@@UAE@XZ ; HCParser::CParseValue::~CParseValue
__unwindfunclet$??__Ek_parseTunerConstants@@YAXXZ$16:
  0008d	8d 4d 80	 lea	 ecx, DWORD PTR $T362577[ebp]
  00090	e9 00 00 00 00	 jmp	 ??1CParseConstant@HCParser@@QAE@XZ
__unwindfunclet$??__Ek_parseTunerConstants@@YAXXZ$17:
  00095	b9 50 00 00 00	 mov	 ecx, OFFSET ?k_parseTunerConstants@@3QBVCParseConstant@HCParser@@B+80
  0009a	e9 00 00 00 00	 jmp	 ??1CParseConstant@HCParser@@QAE@XZ
__unwindfunclet$??__Ek_parseTunerConstants@@YAXXZ$18:
  0009f	8b 8d 68 ff ff
	ff		 mov	 ecx, DWORD PTR $T362580[ebp]
  000a5	e9 00 00 00 00	 jmp	 ??1CParseValue@HCParser@@UAE@XZ ; HCParser::CParseValue::~CParseValue
__unwindfunclet$??__Ek_parseTunerConstants@@YAXXZ$19:
  000aa	8d 8d 6c ff ff
	ff		 lea	 ecx, DWORD PTR $T362579[ebp]
  000b0	e9 00 00 00 00	 jmp	 ??1CParseConstant@HCParser@@QAE@XZ
__unwindfunclet$??__Ek_parseTunerConstants@@YAXXZ$20:
  000b5	b9 60 00 00 00	 mov	 ecx, OFFSET ?k_parseTunerConstants@@3QBVCParseConstant@HCParser@@B+96
  000ba	e9 00 00 00 00	 jmp	 ??1CParseConstant@HCParser@@QAE@XZ
__unwindfunclet$??__Ek_parseTunerConstants@@YAXXZ$21:
  000bf	8b 8d 54 ff ff
	ff		 mov	 ecx, DWORD PTR $T362582[ebp]
  000c5	e9 00 00 00 00	 jmp	 ??1CParseValue@HCParser@@UAE@XZ ; HCParser::CParseValue::~CParseValue
__unwindfunclet$??__Ek_parseTunerConstants@@YAXXZ$22:
  000ca	8d 8d 58 ff ff
	ff		 lea	 ecx, DWORD PTR $T362581[ebp]
  000d0	e9 00 00 00 00	 jmp	 ??1CParseConstant@HCParser@@QAE@XZ
__unwindfunclet$??__Ek_parseTunerConstants@@YAXXZ$23:
  000d5	b9 70 00 00 00	 mov	 ecx, OFFSET ?k_parseTunerConstants@@3QBVCParseConstant@HCParser@@B+112
  000da	e9 00 00 00 00	 jmp	 ??1CParseConstant@HCParser@@QAE@XZ
__unwindfunclet$??__Ek_parseTunerConstants@@YAXXZ$24:
  000df	8b 8d 40 ff ff
	ff		 mov	 ecx, DWORD PTR $T362584[ebp]
  000e5	e9 00 00 00 00	 jmp	 ??1CParseValue@HCParser@@UAE@XZ ; HCParser::CParseValue::~CParseValue
__unwindfunclet$??__Ek_parseTunerConstants@@YAXXZ$25:
  000ea	8d 8d 44 ff ff
	ff		 lea	 ecx, DWORD PTR $T362583[ebp]
  000f0	e9 00 00 00 00	 jmp	 ??1CParseConstant@HCParser@@QAE@XZ
__unwindfunclet$??__Ek_parseTunerConstants@@YAXXZ$26:
  000f5	b9 80 00 00 00	 mov	 ecx, OFFSET ?k_parseTunerConstants@@3QBVCParseConstant@HCParser@@B+128
  000fa	e9 00 00 00 00	 jmp	 ??1CParseConstant@HCParser@@QAE@XZ
__unwindfunclet$??__Ek_parseTunerConstants@@YAXXZ$27:
  000ff	8b 8d 2c ff ff
	ff		 mov	 ecx, DWORD PTR $T362586[ebp]
  00105	e9 00 00 00 00	 jmp	 ??1CParseValue@HCParser@@UAE@XZ ; HCParser::CParseValue::~CParseValue
__unwindfunclet$??__Ek_parseTunerConstants@@YAXXZ$28:
  0010a	8d 8d 30 ff ff
	ff		 lea	 ecx, DWORD PTR $T362585[ebp]
  00110	e9 00 00 00 00	 jmp	 ??1CParseConstant@HCParser@@QAE@XZ
__unwindfunclet$??__Ek_parseTunerConstants@@YAXXZ$29:
  00115	b9 90 00 00 00	 mov	 ecx, OFFSET ?k_parseTunerConstants@@3QBVCParseConstant@HCParser@@B+144
  0011a	e9 00 00 00 00	 jmp	 ??1CParseConstant@HCParser@@QAE@XZ
__unwindfunclet$??__Ek_parseTunerConstants@@YAXXZ$30:
  0011f	8b 8d 18 ff ff
	ff		 mov	 ecx, DWORD PTR $T362588[ebp]
  00125	e9 00 00 00 00	 jmp	 ??1CParseValue@HCParser@@UAE@XZ ; HCParser::CParseValue::~CParseValue
__unwindfunclet$??__Ek_parseTunerConstants@@YAXXZ$31:
  0012a	8d 8d 1c ff ff
	ff		 lea	 ecx, DWORD PTR $T362587[ebp]
  00130	e9 00 00 00 00	 jmp	 ??1CParseConstant@HCParser@@QAE@XZ
__unwindfunclet$??__Ek_parseTunerConstants@@YAXXZ$32:
  00135	b9 a0 00 00 00	 mov	 ecx, OFFSET ?k_parseTunerConstants@@3QBVCParseConstant@HCParser@@B+160
  0013a	e9 00 00 00 00	 jmp	 ??1CParseConstant@HCParser@@QAE@XZ
__unwindfunclet$??__Ek_parseTunerConstants@@YAXXZ$33:
  0013f	8b 8d 04 ff ff
	ff		 mov	 ecx, DWORD PTR $T362590[ebp]
  00145	e9 00 00 00 00	 jmp	 ??1CParseValue@HCParser@@UAE@XZ ; HCParser::CParseValue::~CParseValue
__unwindfunclet$??__Ek_parseTunerConstants@@YAXXZ$34:
  0014a	8d 8d 08 ff ff
	ff		 lea	 ecx, DWORD PTR $T362589[ebp]
  00150	e9 00 00 00 00	 jmp	 ??1CParseConstant@HCParser@@QAE@XZ
__unwindfunclet$??__Ek_parseTunerConstants@@YAXXZ$35:
  00155	b9 b0 00 00 00	 mov	 ecx, OFFSET ?k_parseTunerConstants@@3QBVCParseConstant@HCParser@@B+176
  0015a	e9 00 00 00 00	 jmp	 ??1CParseConstant@HCParser@@QAE@XZ
__unwindfunclet$??__Ek_parseTunerConstants@@YAXXZ$36:
  0015f	8b 8d f0 fe ff
	ff		 mov	 ecx, DWORD PTR $T362592[ebp]
  00165	e9 00 00 00 00	 jmp	 ??1CParseValue@HCParser@@UAE@XZ ; HCParser::CParseValue::~CParseValue
__unwindfunclet$??__Ek_parseTunerConstants@@YAXXZ$37:
  0016a	8d 8d f4 fe ff
	ff		 lea	 ecx, DWORD PTR $T362591[ebp]
  00170	e9 00 00 00 00	 jmp	 ??1CParseConstant@HCParser@@QAE@XZ
__unwindfunclet$??__Ek_parseTunerConstants@@YAXXZ$38:
  00175	b9 c0 00 00 00	 mov	 ecx, OFFSET ?k_parseTunerConstants@@3QBVCParseConstant@HCParser@@B+192
  0017a	e9 00 00 00 00	 jmp	 ??1CParseConstant@HCParser@@QAE@XZ
__unwindfunclet$??__Ek_parseTunerConstants@@YAXXZ$39:
  0017f	8b 8d dc fe ff
	ff		 mov	 ecx, DWORD PTR $T362594[ebp]
  00185	e9 00 00 00 00	 jmp	 ??1CParseValue@HCParser@@UAE@XZ ; HCParser::CParseValue::~CParseValue
__unwindfunclet$??__Ek_parseTunerConstants@@YAXXZ$40:
  0018a	8d 8d e0 fe ff
	ff		 lea	 ecx, DWORD PTR $T362593[ebp]
  00190	e9 00 00 00 00	 jmp	 ??1CParseConstant@HCParser@@QAE@XZ
__unwindfunclet$??__Ek_parseTunerConstants@@YAXXZ$41:
  00195	b9 d0 00 00 00	 mov	 ecx, OFFSET ?k_parseTunerConstants@@3QBVCParseConstant@HCParser@@B+208
  0019a	e9 00 00 00 00	 jmp	 ??1CParseConstant@HCParser@@QAE@XZ
__unwindfunclet$??__Ek_parseTunerConstants@@YAXXZ$42:
  0019f	8b 8d c8 fe ff
	ff		 mov	 ecx, DWORD PTR $T362596[ebp]
  001a5	e9 00 00 00 00	 jmp	 ??1CParseValue@HCParser@@UAE@XZ ; HCParser::CParseValue::~CParseValue
__unwindfunclet$??__Ek_parseTunerConstants@@YAXXZ$43:
  001aa	8d 8d cc fe ff
	ff		 lea	 ecx, DWORD PTR $T362595[ebp]
  001b0	e9 00 00 00 00	 jmp	 ??1CParseConstant@HCParser@@QAE@XZ
__unwindfunclet$??__Ek_parseTunerConstants@@YAXXZ$44:
  001b5	b9 e0 00 00 00	 mov	 ecx, OFFSET ?k_parseTunerConstants@@3QBVCParseConstant@HCParser@@B+224
  001ba	e9 00 00 00 00	 jmp	 ??1CParseConstant@HCParser@@QAE@XZ
__unwindfunclet$??__Ek_parseTunerConstants@@YAXXZ$45:
  001bf	8b 8d b4 fe ff
	ff		 mov	 ecx, DWORD PTR $T362598[ebp]
  001c5	e9 00 00 00 00	 jmp	 ??1CParseValue@HCParser@@UAE@XZ ; HCParser::CParseValue::~CParseValue
__unwindfunclet$??__Ek_parseTunerConstants@@YAXXZ$46:
  001ca	8d 8d b8 fe ff
	ff		 lea	 ecx, DWORD PTR $T362597[ebp]
  001d0	e9 00 00 00 00	 jmp	 ??1CParseConstant@HCParser@@QAE@XZ
__unwindfunclet$??__Ek_parseTunerConstants@@YAXXZ$47:
  001d5	b9 f0 00 00 00	 mov	 ecx, OFFSET ?k_parseTunerConstants@@3QBVCParseConstant@HCParser@@B+240
  001da	e9 00 00 00 00	 jmp	 ??1CParseConstant@HCParser@@QAE@XZ
__unwindfunclet$??__Ek_parseTunerConstants@@YAXXZ$48:
  001df	8b 8d a0 fe ff
	ff		 mov	 ecx, DWORD PTR $T362600[ebp]
  001e5	e9 00 00 00 00	 jmp	 ??1CParseValue@HCParser@@UAE@XZ ; HCParser::CParseValue::~CParseValue
__unwindfunclet$??__Ek_parseTunerConstants@@YAXXZ$49:
  001ea	8d 8d a4 fe ff
	ff		 lea	 ecx, DWORD PTR $T362599[ebp]
  001f0	e9 00 00 00 00	 jmp	 ??1CParseConstant@HCParser@@QAE@XZ
__unwindfunclet$??__Ek_parseTunerConstants@@YAXXZ$50:
  001f5	b9 00 01 00 00	 mov	 ecx, OFFSET ?k_parseTunerConstants@@3QBVCParseConstant@HCParser@@B+256
  001fa	e9 00 00 00 00	 jmp	 ??1CParseConstant@HCParser@@QAE@XZ
__unwindfunclet$??__Ek_parseTunerConstants@@YAXXZ$51:
  001ff	8b 8d 8c fe ff
	ff		 mov	 ecx, DWORD PTR $T362602[ebp]
  00205	e9 00 00 00 00	 jmp	 ??1CParseValue@HCParser@@UAE@XZ ; HCParser::CParseValue::~CParseValue
__unwindfunclet$??__Ek_parseTunerConstants@@YAXXZ$52:
  0020a	8d 8d 90 fe ff
	ff		 lea	 ecx, DWORD PTR $T362601[ebp]
  00210	e9 00 00 00 00	 jmp	 ??1CParseConstant@HCParser@@QAE@XZ
__unwindfunclet$??__Ek_parseTunerConstants@@YAXXZ$53:
  00215	b9 10 01 00 00	 mov	 ecx, OFFSET ?k_parseTunerConstants@@3QBVCParseConstant@HCParser@@B+272
  0021a	e9 00 00 00 00	 jmp	 ??1CParseConstant@HCParser@@QAE@XZ
__unwindfunclet$??__Ek_parseTunerConstants@@YAXXZ$54:
  0021f	8b 8d 78 fe ff
	ff		 mov	 ecx, DWORD PTR $T362604[ebp]
  00225	e9 00 00 00 00	 jmp	 ??1CParseValue@HCParser@@UAE@XZ ; HCParser::CParseValue::~CParseValue
__unwindfunclet$??__Ek_parseTunerConstants@@YAXXZ$55:
  0022a	8d 8d 7c fe ff
	ff		 lea	 ecx, DWORD PTR $T362603[ebp]
  00230	e9 00 00 00 00	 jmp	 ??1CParseConstant@HCParser@@QAE@XZ
__unwindfunclet$??__Ek_parseTunerConstants@@YAXXZ$56:
  00235	b9 20 01 00 00	 mov	 ecx, OFFSET ?k_parseTunerConstants@@3QBVCParseConstant@HCParser@@B+288
  0023a	e9 00 00 00 00	 jmp	 ??1CParseConstant@HCParser@@QAE@XZ
__unwindfunclet$??__Ek_parseTunerConstants@@YAXXZ$57:
  0023f	8b 8d 64 fe ff
	ff		 mov	 ecx, DWORD PTR $T362606[ebp]
  00245	e9 00 00 00 00	 jmp	 ??1CParseValue@HCParser@@UAE@XZ ; HCParser::CParseValue::~CParseValue
__unwindfunclet$??__Ek_parseTunerConstants@@YAXXZ$58:
  0024a	8d 8d 68 fe ff
	ff		 lea	 ecx, DWORD PTR $T362605[ebp]
  00250	e9 00 00 00 00	 jmp	 ??1CParseConstant@HCParser@@QAE@XZ
__unwindfunclet$??__Ek_parseTunerConstants@@YAXXZ$59:
  00255	b9 30 01 00 00	 mov	 ecx, OFFSET ?k_parseTunerConstants@@3QBVCParseConstant@HCParser@@B+304
  0025a	e9 00 00 00 00	 jmp	 ??1CParseConstant@HCParser@@QAE@XZ
__unwindfunclet$??__Ek_parseTunerConstants@@YAXXZ$60:
  0025f	8b 8d 50 fe ff
	ff		 mov	 ecx, DWORD PTR $T362608[ebp]
  00265	e9 00 00 00 00	 jmp	 ??1CParseValue@HCParser@@UAE@XZ ; HCParser::CParseValue::~CParseValue
__unwindfunclet$??__Ek_parseTunerConstants@@YAXXZ$61:
  0026a	8d 8d 54 fe ff
	ff		 lea	 ecx, DWORD PTR $T362607[ebp]
  00270	e9 00 00 00 00	 jmp	 ??1CParseConstant@HCParser@@QAE@XZ
__unwindfunclet$??__Ek_parseTunerConstants@@YAXXZ$62:
  00275	b9 40 01 00 00	 mov	 ecx, OFFSET ?k_parseTunerConstants@@3QBVCParseConstant@HCParser@@B+320
  0027a	e9 00 00 00 00	 jmp	 ??1CParseConstant@HCParser@@QAE@XZ
__unwindfunclet$??__Ek_parseTunerConstants@@YAXXZ$63:
  0027f	8b 8d 3c fe ff
	ff		 mov	 ecx, DWORD PTR $T362610[ebp]
  00285	e9 00 00 00 00	 jmp	 ??1CParseValue@HCParser@@UAE@XZ ; HCParser::CParseValue::~CParseValue
__unwindfunclet$??__Ek_parseTunerConstants@@YAXXZ$64:
  0028a	8d 8d 40 fe ff
	ff		 lea	 ecx, DWORD PTR $T362609[ebp]
  00290	e9 00 00 00 00	 jmp	 ??1CParseConstant@HCParser@@QAE@XZ
__unwindfunclet$??__Ek_parseTunerConstants@@YAXXZ$65:
  00295	b9 50 01 00 00	 mov	 ecx, OFFSET ?k_parseTunerConstants@@3QBVCParseConstant@HCParser@@B+336
  0029a	e9 00 00 00 00	 jmp	 ??1CParseConstant@HCParser@@QAE@XZ
__unwindfunclet$??__Ek_parseTunerConstants@@YAXXZ$66:
  0029f	8b 8d 28 fe ff
	ff		 mov	 ecx, DWORD PTR $T362612[ebp]
  002a5	e9 00 00 00 00	 jmp	 ??1CParseValue@HCParser@@UAE@XZ ; HCParser::CParseValue::~CParseValue
__unwindfunclet$??__Ek_parseTunerConstants@@YAXXZ$67:
  002aa	8d 8d 2c fe ff
	ff		 lea	 ecx, DWORD PTR $T362611[ebp]
  002b0	e9 00 00 00 00	 jmp	 ??1CParseConstant@HCParser@@QAE@XZ
__unwindfunclet$??__Ek_parseTunerConstants@@YAXXZ$68:
  002b5	b9 60 01 00 00	 mov	 ecx, OFFSET ?k_parseTunerConstants@@3QBVCParseConstant@HCParser@@B+352
  002ba	e9 00 00 00 00	 jmp	 ??1CParseConstant@HCParser@@QAE@XZ
__unwindfunclet$??__Ek_parseTunerConstants@@YAXXZ$69:
  002bf	8b 8d 14 fe ff
	ff		 mov	 ecx, DWORD PTR $T362614[ebp]
  002c5	e9 00 00 00 00	 jmp	 ??1CParseValue@HCParser@@UAE@XZ ; HCParser::CParseValue::~CParseValue
__unwindfunclet$??__Ek_parseTunerConstants@@YAXXZ$70:
  002ca	8d 8d 18 fe ff
	ff		 lea	 ecx, DWORD PTR $T362613[ebp]
  002d0	e9 00 00 00 00	 jmp	 ??1CParseConstant@HCParser@@QAE@XZ
__unwindfunclet$??__Ek_parseTunerConstants@@YAXXZ$71:
  002d5	b9 70 01 00 00	 mov	 ecx, OFFSET ?k_parseTunerConstants@@3QBVCParseConstant@HCParser@@B+368
  002da	e9 00 00 00 00	 jmp	 ??1CParseConstant@HCParser@@QAE@XZ
__unwindfunclet$??__Ek_parseTunerConstants@@YAXXZ$72:
  002df	8b 8d 00 fe ff
	ff		 mov	 ecx, DWORD PTR $T362616[ebp]
  002e5	e9 00 00 00 00	 jmp	 ??1CParseValue@HCParser@@UAE@XZ ; HCParser::CParseValue::~CParseValue
__unwindfunclet$??__Ek_parseTunerConstants@@YAXXZ$73:
  002ea	8d 8d 04 fe ff
	ff		 lea	 ecx, DWORD PTR $T362615[ebp]
  002f0	e9 00 00 00 00	 jmp	 ??1CParseConstant@HCParser@@QAE@XZ
__unwindfunclet$??__Ek_parseTunerConstants@@YAXXZ$74:
  002f5	b9 80 01 00 00	 mov	 ecx, OFFSET ?k_parseTunerConstants@@3QBVCParseConstant@HCParser@@B+384
  002fa	e9 00 00 00 00	 jmp	 ??1CParseConstant@HCParser@@QAE@XZ
__unwindfunclet$??__Ek_parseTunerConstants@@YAXXZ$75:
  002ff	8b 8d ec fd ff
	ff		 mov	 ecx, DWORD PTR $T362618[ebp]
  00305	e9 00 00 00 00	 jmp	 ??1CParseValue@HCParser@@UAE@XZ ; HCParser::CParseValue::~CParseValue
__unwindfunclet$??__Ek_parseTunerConstants@@YAXXZ$76:
  0030a	8d 8d f0 fd ff
	ff		 lea	 ecx, DWORD PTR $T362617[ebp]
  00310	e9 00 00 00 00	 jmp	 ??1CParseConstant@HCParser@@QAE@XZ
__unwindfunclet$??__Ek_parseTunerConstants@@YAXXZ$77:
  00315	b9 90 01 00 00	 mov	 ecx, OFFSET ?k_parseTunerConstants@@3QBVCParseConstant@HCParser@@B+400
  0031a	e9 00 00 00 00	 jmp	 ??1CParseConstant@HCParser@@QAE@XZ
__unwindfunclet$??__Ek_parseTunerConstants@@YAXXZ$78:
  0031f	8b 8d d8 fd ff
	ff		 mov	 ecx, DWORD PTR $T362620[ebp]
  00325	e9 00 00 00 00	 jmp	 ??1CParseValue@HCParser@@UAE@XZ ; HCParser::CParseValue::~CParseValue
__unwindfunclet$??__Ek_parseTunerConstants@@YAXXZ$79:
  0032a	8d 8d dc fd ff
	ff		 lea	 ecx, DWORD PTR $T362619[ebp]
  00330	e9 00 00 00 00	 jmp	 ??1CParseConstant@HCParser@@QAE@XZ
__unwindfunclet$??__Ek_parseTunerConstants@@YAXXZ$80:
  00335	b9 a0 01 00 00	 mov	 ecx, OFFSET ?k_parseTunerConstants@@3QBVCParseConstant@HCParser@@B+416
  0033a	e9 00 00 00 00	 jmp	 ??1CParseConstant@HCParser@@QAE@XZ
__unwindfunclet$??__Ek_parseTunerConstants@@YAXXZ$81:
  0033f	8b 8d c4 fd ff
	ff		 mov	 ecx, DWORD PTR $T362622[ebp]
  00345	e9 00 00 00 00	 jmp	 ??1CParseValue@HCParser@@UAE@XZ ; HCParser::CParseValue::~CParseValue
__unwindfunclet$??__Ek_parseTunerConstants@@YAXXZ$82:
  0034a	8d 8d c8 fd ff
	ff		 lea	 ecx, DWORD PTR $T362621[ebp]
  00350	e9 00 00 00 00	 jmp	 ??1CParseConstant@HCParser@@QAE@XZ
__unwindfunclet$??__Ek_parseTunerConstants@@YAXXZ$83:
  00355	b9 b0 01 00 00	 mov	 ecx, OFFSET ?k_parseTunerConstants@@3QBVCParseConstant@HCParser@@B+432
  0035a	e9 00 00 00 00	 jmp	 ??1CParseConstant@HCParser@@QAE@XZ
__unwindfunclet$??__Ek_parseTunerConstants@@YAXXZ$84:
  0035f	8b 8d b0 fd ff
	ff		 mov	 ecx, DWORD PTR $T362624[ebp]
  00365	e9 00 00 00 00	 jmp	 ??1CParseValue@HCParser@@UAE@XZ ; HCParser::CParseValue::~CParseValue
__unwindfunclet$??__Ek_parseTunerConstants@@YAXXZ$85:
  0036a	8d 8d b4 fd ff
	ff		 lea	 ecx, DWORD PTR $T362623[ebp]
  00370	e9 00 00 00 00	 jmp	 ??1CParseConstant@HCParser@@QAE@XZ
__unwindfunclet$??__Ek_parseTunerConstants@@YAXXZ$86:
  00375	b9 c0 01 00 00	 mov	 ecx, OFFSET ?k_parseTunerConstants@@3QBVCParseConstant@HCParser@@B+448
  0037a	e9 00 00 00 00	 jmp	 ??1CParseConstant@HCParser@@QAE@XZ
__unwindfunclet$??__Ek_parseTunerConstants@@YAXXZ$87:
  0037f	8b 8d 9c fd ff
	ff		 mov	 ecx, DWORD PTR $T362626[ebp]
  00385	e9 00 00 00 00	 jmp	 ??1CParseValue@HCParser@@UAE@XZ ; HCParser::CParseValue::~CParseValue
__unwindfunclet$??__Ek_parseTunerConstants@@YAXXZ$88:
  0038a	8d 8d a0 fd ff
	ff		 lea	 ecx, DWORD PTR $T362625[ebp]
  00390	e9 00 00 00 00	 jmp	 ??1CParseConstant@HCParser@@QAE@XZ
__unwindfunclet$??__Ek_parseTunerConstants@@YAXXZ$89:
  00395	b9 d0 01 00 00	 mov	 ecx, OFFSET ?k_parseTunerConstants@@3QBVCParseConstant@HCParser@@B+464
  0039a	e9 00 00 00 00	 jmp	 ??1CParseConstant@HCParser@@QAE@XZ
__unwindfunclet$??__Ek_parseTunerConstants@@YAXXZ$90:
  0039f	8b 8d 88 fd ff
	ff		 mov	 ecx, DWORD PTR $T362628[ebp]
  003a5	e9 00 00 00 00	 jmp	 ??1CParseValue@HCParser@@UAE@XZ ; HCParser::CParseValue::~CParseValue
__unwindfunclet$??__Ek_parseTunerConstants@@YAXXZ$91:
  003aa	8d 8d 8c fd ff
	ff		 lea	 ecx, DWORD PTR $T362627[ebp]
  003b0	e9 00 00 00 00	 jmp	 ??1CParseConstant@HCParser@@QAE@XZ
__unwindfunclet$??__Ek_parseTunerConstants@@YAXXZ$92:
  003b5	b9 e0 01 00 00	 mov	 ecx, OFFSET ?k_parseTunerConstants@@3QBVCParseConstant@HCParser@@B+480
  003ba	e9 00 00 00 00	 jmp	 ??1CParseConstant@HCParser@@QAE@XZ
__unwindfunclet$??__Ek_parseTunerConstants@@YAXXZ$93:
  003bf	8b 8d 74 fd ff
	ff		 mov	 ecx, DWORD PTR $T362630[ebp]
  003c5	e9 00 00 00 00	 jmp	 ??1CParseValue@HCParser@@UAE@XZ ; HCParser::CParseValue::~CParseValue
__unwindfunclet$??__Ek_parseTunerConstants@@YAXXZ$94:
  003ca	8d 8d 78 fd ff
	ff		 lea	 ecx, DWORD PTR $T362629[ebp]
  003d0	e9 00 00 00 00	 jmp	 ??1CParseConstant@HCParser@@QAE@XZ
__unwindfunclet$??__Ek_parseTunerConstants@@YAXXZ$95:
  003d5	b9 f0 01 00 00	 mov	 ecx, OFFSET ?k_parseTunerConstants@@3QBVCParseConstant@HCParser@@B+496
  003da	e9 00 00 00 00	 jmp	 ??1CParseConstant@HCParser@@QAE@XZ
__unwindfunclet$??__Ek_parseTunerConstants@@YAXXZ$96:
  003df	8b 8d 60 fd ff
	ff		 mov	 ecx, DWORD PTR $T362632[ebp]
  003e5	e9 00 00 00 00	 jmp	 ??1CParseValue@HCParser@@UAE@XZ ; HCParser::CParseValue::~CParseValue
__unwindfunclet$??__Ek_parseTunerConstants@@YAXXZ$97:
  003ea	8d 8d 64 fd ff
	ff		 lea	 ecx, DWORD PTR $T362631[ebp]
  003f0	e9 00 00 00 00	 jmp	 ??1CParseConstant@HCParser@@QAE@XZ
__unwindfunclet$??__Ek_parseTunerConstants@@YAXXZ$98:
  003f5	b9 00 02 00 00	 mov	 ecx, OFFSET ?k_parseTunerConstants@@3QBVCParseConstant@HCParser@@B+512
  003fa	e9 00 00 00 00	 jmp	 ??1CParseConstant@HCParser@@QAE@XZ
__unwindfunclet$??__Ek_parseTunerConstants@@YAXXZ$99:
  003ff	8b 8d 4c fd ff
	ff		 mov	 ecx, DWORD PTR $T362634[ebp]
  00405	e9 00 00 00 00	 jmp	 ??1CParseValue@HCParser@@UAE@XZ ; HCParser::CParseValue::~CParseValue
__unwindfunclet$??__Ek_parseTunerConstants@@YAXXZ$100:
  0040a	8d 8d 50 fd ff
	ff		 lea	 ecx, DWORD PTR $T362633[ebp]
  00410	e9 00 00 00 00	 jmp	 ??1CParseConstant@HCParser@@QAE@XZ
__unwindfunclet$??__Ek_parseTunerConstants@@YAXXZ$101:
  00415	b9 10 02 00 00	 mov	 ecx, OFFSET ?k_parseTunerConstants@@3QBVCParseConstant@HCParser@@B+528
  0041a	e9 00 00 00 00	 jmp	 ??1CParseConstant@HCParser@@QAE@XZ
__unwindfunclet$??__Ek_parseTunerConstants@@YAXXZ$102:
  0041f	8b 8d 38 fd ff
	ff		 mov	 ecx, DWORD PTR $T362636[ebp]
  00425	e9 00 00 00 00	 jmp	 ??1CParseValue@HCParser@@UAE@XZ ; HCParser::CParseValue::~CParseValue
__unwindfunclet$??__Ek_parseTunerConstants@@YAXXZ$103:
  0042a	8d 8d 3c fd ff
	ff		 lea	 ecx, DWORD PTR $T362635[ebp]
  00430	e9 00 00 00 00	 jmp	 ??1CParseConstant@HCParser@@QAE@XZ
__unwindfunclet$??__Ek_parseTunerConstants@@YAXXZ$104:
  00435	b9 20 02 00 00	 mov	 ecx, OFFSET ?k_parseTunerConstants@@3QBVCParseConstant@HCParser@@B+544
  0043a	e9 00 00 00 00	 jmp	 ??1CParseConstant@HCParser@@QAE@XZ
__unwindfunclet$??__Ek_parseTunerConstants@@YAXXZ$105:
  0043f	8b 8d 24 fd ff
	ff		 mov	 ecx, DWORD PTR $T362638[ebp]
  00445	e9 00 00 00 00	 jmp	 ??1CParseValue@HCParser@@UAE@XZ ; HCParser::CParseValue::~CParseValue
__unwindfunclet$??__Ek_parseTunerConstants@@YAXXZ$106:
  0044a	8d 8d 28 fd ff
	ff		 lea	 ecx, DWORD PTR $T362637[ebp]
  00450	e9 00 00 00 00	 jmp	 ??1CParseConstant@HCParser@@QAE@XZ
__unwindfunclet$??__Ek_parseTunerConstants@@YAXXZ$107:
  00455	b9 30 02 00 00	 mov	 ecx, OFFSET ?k_parseTunerConstants@@3QBVCParseConstant@HCParser@@B+560
  0045a	e9 00 00 00 00	 jmp	 ??1CParseConstant@HCParser@@QAE@XZ
__unwindfunclet$??__Ek_parseTunerConstants@@YAXXZ$108:
  0045f	8b 8d 10 fd ff
	ff		 mov	 ecx, DWORD PTR $T362640[ebp]
  00465	e9 00 00 00 00	 jmp	 ??1CParseValue@HCParser@@UAE@XZ ; HCParser::CParseValue::~CParseValue
__unwindfunclet$??__Ek_parseTunerConstants@@YAXXZ$109:
  0046a	8d 8d 14 fd ff
	ff		 lea	 ecx, DWORD PTR $T362639[ebp]
  00470	e9 00 00 00 00	 jmp	 ??1CParseConstant@HCParser@@QAE@XZ
__unwindfunclet$??__Ek_parseTunerConstants@@YAXXZ$110:
  00475	b9 40 02 00 00	 mov	 ecx, OFFSET ?k_parseTunerConstants@@3QBVCParseConstant@HCParser@@B+576
  0047a	e9 00 00 00 00	 jmp	 ??1CParseConstant@HCParser@@QAE@XZ
__unwindfunclet$??__Ek_parseTunerConstants@@YAXXZ$111:
  0047f	8b 8d fc fc ff
	ff		 mov	 ecx, DWORD PTR $T362642[ebp]
  00485	e9 00 00 00 00	 jmp	 ??1CParseValue@HCParser@@UAE@XZ ; HCParser::CParseValue::~CParseValue
__unwindfunclet$??__Ek_parseTunerConstants@@YAXXZ$112:
  0048a	8d 8d 00 fd ff
	ff		 lea	 ecx, DWORD PTR $T362641[ebp]
  00490	e9 00 00 00 00	 jmp	 ??1CParseConstant@HCParser@@QAE@XZ
__unwindfunclet$??__Ek_parseTunerConstants@@YAXXZ$113:
  00495	b9 50 02 00 00	 mov	 ecx, OFFSET ?k_parseTunerConstants@@3QBVCParseConstant@HCParser@@B+592
  0049a	e9 00 00 00 00	 jmp	 ??1CParseConstant@HCParser@@QAE@XZ
__unwindfunclet$??__Ek_parseTunerConstants@@YAXXZ$114:
  0049f	8b 8d e8 fc ff
	ff		 mov	 ecx, DWORD PTR $T362644[ebp]
  004a5	e9 00 00 00 00	 jmp	 ??1CParseValue@HCParser@@UAE@XZ ; HCParser::CParseValue::~CParseValue
__unwindfunclet$??__Ek_parseTunerConstants@@YAXXZ$115:
  004aa	8d 8d ec fc ff
	ff		 lea	 ecx, DWORD PTR $T362643[ebp]
  004b0	e9 00 00 00 00	 jmp	 ??1CParseConstant@HCParser@@QAE@XZ
__unwindfunclet$??__Ek_parseTunerConstants@@YAXXZ$116:
  004b5	b9 60 02 00 00	 mov	 ecx, OFFSET ?k_parseTunerConstants@@3QBVCParseConstant@HCParser@@B+608
  004ba	e9 00 00 00 00	 jmp	 ??1CParseConstant@HCParser@@QAE@XZ
__unwindfunclet$??__Ek_parseTunerConstants@@YAXXZ$117:
  004bf	8b 8d d4 fc ff
	ff		 mov	 ecx, DWORD PTR $T362646[ebp]
  004c5	e9 00 00 00 00	 jmp	 ??1CParseValue@HCParser@@UAE@XZ ; HCParser::CParseValue::~CParseValue
__unwindfunclet$??__Ek_parseTunerConstants@@YAXXZ$118:
  004ca	8d 8d d8 fc ff
	ff		 lea	 ecx, DWORD PTR $T362645[ebp]
  004d0	e9 00 00 00 00	 jmp	 ??1CParseConstant@HCParser@@QAE@XZ
__unwindfunclet$??__Ek_parseTunerConstants@@YAXXZ$119:
  004d5	b9 70 02 00 00	 mov	 ecx, OFFSET ?k_parseTunerConstants@@3QBVCParseConstant@HCParser@@B+624
  004da	e9 00 00 00 00	 jmp	 ??1CParseConstant@HCParser@@QAE@XZ
__unwindfunclet$??__Ek_parseTunerConstants@@YAXXZ$120:
  004df	8b 8d c0 fc ff
	ff		 mov	 ecx, DWORD PTR $T362648[ebp]
  004e5	e9 00 00 00 00	 jmp	 ??1CParseValue@HCParser@@UAE@XZ ; HCParser::CParseValue::~CParseValue
__unwindfunclet$??__Ek_parseTunerConstants@@YAXXZ$121:
  004ea	8d 8d c4 fc ff
	ff		 lea	 ecx, DWORD PTR $T362647[ebp]
  004f0	e9 00 00 00 00	 jmp	 ??1CParseConstant@HCParser@@QAE@XZ
__unwindfunclet$??__Ek_parseTunerConstants@@YAXXZ$122:
  004f5	b9 80 02 00 00	 mov	 ecx, OFFSET ?k_parseTunerConstants@@3QBVCParseConstant@HCParser@@B+640
  004fa	e9 00 00 00 00	 jmp	 ??1CParseConstant@HCParser@@QAE@XZ
__unwindfunclet$??__Ek_parseTunerConstants@@YAXXZ$123:
  004ff	8b 8d ac fc ff
	ff		 mov	 ecx, DWORD PTR $T362650[ebp]
  00505	e9 00 00 00 00	 jmp	 ??1CParseValue@HCParser@@UAE@XZ ; HCParser::CParseValue::~CParseValue
__unwindfunclet$??__Ek_parseTunerConstants@@YAXXZ$124:
  0050a	8d 8d b0 fc ff
	ff		 lea	 ecx, DWORD PTR $T362649[ebp]
  00510	e9 00 00 00 00	 jmp	 ??1CParseConstant@HCParser@@QAE@XZ
__unwindfunclet$??__Ek_parseTunerConstants@@YAXXZ$125:
  00515	b9 90 02 00 00	 mov	 ecx, OFFSET ?k_parseTunerConstants@@3QBVCParseConstant@HCParser@@B+656
  0051a	e9 00 00 00 00	 jmp	 ??1CParseConstant@HCParser@@QAE@XZ
__unwindfunclet$??__Ek_parseTunerConstants@@YAXXZ$126:
  0051f	8b 8d 98 fc ff
	ff		 mov	 ecx, DWORD PTR $T362652[ebp]
  00525	e9 00 00 00 00	 jmp	 ??1CParseValue@HCParser@@UAE@XZ ; HCParser::CParseValue::~CParseValue
__unwindfunclet$??__Ek_parseTunerConstants@@YAXXZ$127:
  0052a	8d 8d 9c fc ff
	ff		 lea	 ecx, DWORD PTR $T362651[ebp]
  00530	e9 00 00 00 00	 jmp	 ??1CParseConstant@HCParser@@QAE@XZ
__unwindfunclet$??__Ek_parseTunerConstants@@YAXXZ$128:
  00535	b9 a0 02 00 00	 mov	 ecx, OFFSET ?k_parseTunerConstants@@3QBVCParseConstant@HCParser@@B+672
  0053a	e9 00 00 00 00	 jmp	 ??1CParseConstant@HCParser@@QAE@XZ
__unwindfunclet$??__Ek_parseTunerConstants@@YAXXZ$129:
  0053f	8b 8d 84 fc ff
	ff		 mov	 ecx, DWORD PTR $T362654[ebp]
  00545	e9 00 00 00 00	 jmp	 ??1CParseValue@HCParser@@UAE@XZ ; HCParser::CParseValue::~CParseValue
__unwindfunclet$??__Ek_parseTunerConstants@@YAXXZ$130:
  0054a	8d 8d 88 fc ff
	ff		 lea	 ecx, DWORD PTR $T362653[ebp]
  00550	e9 00 00 00 00	 jmp	 ??1CParseConstant@HCParser@@QAE@XZ
__unwindfunclet$??__Ek_parseTunerConstants@@YAXXZ$131:
  00555	b9 b0 02 00 00	 mov	 ecx, OFFSET ?k_parseTunerConstants@@3QBVCParseConstant@HCParser@@B+688
  0055a	e9 00 00 00 00	 jmp	 ??1CParseConstant@HCParser@@QAE@XZ
__unwindfunclet$??__Ek_parseTunerConstants@@YAXXZ$132:
  0055f	8b 8d 70 fc ff
	ff		 mov	 ecx, DWORD PTR $T362656[ebp]
  00565	e9 00 00 00 00	 jmp	 ??1CParseValue@HCParser@@UAE@XZ ; HCParser::CParseValue::~CParseValue
__unwindfunclet$??__Ek_parseTunerConstants@@YAXXZ$133:
  0056a	8d 8d 74 fc ff
	ff		 lea	 ecx, DWORD PTR $T362655[ebp]
  00570	e9 00 00 00 00	 jmp	 ??1CParseConstant@HCParser@@QAE@XZ
__unwindfunclet$??__Ek_parseTunerConstants@@YAXXZ$134:
  00575	b9 c0 02 00 00	 mov	 ecx, OFFSET ?k_parseTunerConstants@@3QBVCParseConstant@HCParser@@B+704
  0057a	e9 00 00 00 00	 jmp	 ??1CParseConstant@HCParser@@QAE@XZ
__unwindfunclet$??__Ek_parseTunerConstants@@YAXXZ$135:
  0057f	8b 8d 5c fc ff
	ff		 mov	 ecx, DWORD PTR $T362658[ebp]
  00585	e9 00 00 00 00	 jmp	 ??1CParseValue@HCParser@@UAE@XZ ; HCParser::CParseValue::~CParseValue
__unwindfunclet$??__Ek_parseTunerConstants@@YAXXZ$136:
  0058a	8d 8d 60 fc ff
	ff		 lea	 ecx, DWORD PTR $T362657[ebp]
  00590	e9 00 00 00 00	 jmp	 ??1CParseConstant@HCParser@@QAE@XZ
__unwindfunclet$??__Ek_parseTunerConstants@@YAXXZ$137:
  00595	b9 d0 02 00 00	 mov	 ecx, OFFSET ?k_parseTunerConstants@@3QBVCParseConstant@HCParser@@B+720
  0059a	e9 00 00 00 00	 jmp	 ??1CParseConstant@HCParser@@QAE@XZ
__unwindfunclet$??__Ek_parseTunerConstants@@YAXXZ$138:
  0059f	8b 8d 48 fc ff
	ff		 mov	 ecx, DWORD PTR $T362660[ebp]
  005a5	e9 00 00 00 00	 jmp	 ??1CParseValue@HCParser@@UAE@XZ ; HCParser::CParseValue::~CParseValue
__unwindfunclet$??__Ek_parseTunerConstants@@YAXXZ$139:
  005aa	8d 8d 4c fc ff
	ff		 lea	 ecx, DWORD PTR $T362659[ebp]
  005b0	e9 00 00 00 00	 jmp	 ??1CParseConstant@HCParser@@QAE@XZ
__unwindfunclet$??__Ek_parseTunerConstants@@YAXXZ$140:
  005b5	b9 e0 02 00 00	 mov	 ecx, OFFSET ?k_parseTunerConstants@@3QBVCParseConstant@HCParser@@B+736
  005ba	e9 00 00 00 00	 jmp	 ??1CParseConstant@HCParser@@QAE@XZ
__unwindfunclet$??__Ek_parseTunerConstants@@YAXXZ$141:
  005bf	8b 8d 34 fc ff
	ff		 mov	 ecx, DWORD PTR $T362662[ebp]
  005c5	e9 00 00 00 00	 jmp	 ??1CParseValue@HCParser@@UAE@XZ ; HCParser::CParseValue::~CParseValue
__unwindfunclet$??__Ek_parseTunerConstants@@YAXXZ$142:
  005ca	8d 8d 38 fc ff
	ff		 lea	 ecx, DWORD PTR $T362661[ebp]
  005d0	e9 00 00 00 00	 jmp	 ??1CParseConstant@HCParser@@QAE@XZ
__unwindfunclet$??__Ek_parseTunerConstants@@YAXXZ$143:
  005d5	b9 f0 02 00 00	 mov	 ecx, OFFSET ?k_parseTunerConstants@@3QBVCParseConstant@HCParser@@B+752
  005da	e9 00 00 00 00	 jmp	 ??1CParseConstant@HCParser@@QAE@XZ
__unwindfunclet$??__Ek_parseTunerConstants@@YAXXZ$144:
  005df	8b 8d 20 fc ff
	ff		 mov	 ecx, DWORD PTR $T362664[ebp]
  005e5	e9 00 00 00 00	 jmp	 ??1CParseValue@HCParser@@UAE@XZ ; HCParser::CParseValue::~CParseValue
__unwindfunclet$??__Ek_parseTunerConstants@@YAXXZ$145:
  005ea	8d 8d 24 fc ff
	ff		 lea	 ecx, DWORD PTR $T362663[ebp]
  005f0	e9 00 00 00 00	 jmp	 ??1CParseConstant@HCParser@@QAE@XZ
__unwindfunclet$??__Ek_parseTunerConstants@@YAXXZ$146:
  005f5	b9 00 03 00 00	 mov	 ecx, OFFSET ?k_parseTunerConstants@@3QBVCParseConstant@HCParser@@B+768
  005fa	e9 00 00 00 00	 jmp	 ??1CParseConstant@HCParser@@QAE@XZ
__unwindfunclet$??__Ek_parseTunerConstants@@YAXXZ$147:
  005ff	8b 8d 0c fc ff
	ff		 mov	 ecx, DWORD PTR $T362666[ebp]
  00605	e9 00 00 00 00	 jmp	 ??1CParseValue@HCParser@@UAE@XZ ; HCParser::CParseValue::~CParseValue
__unwindfunclet$??__Ek_parseTunerConstants@@YAXXZ$148:
  0060a	8d 8d 10 fc ff
	ff		 lea	 ecx, DWORD PTR $T362665[ebp]
  00610	e9 00 00 00 00	 jmp	 ??1CParseConstant@HCParser@@QAE@XZ
__unwindfunclet$??__Ek_parseTunerConstants@@YAXXZ$149:
  00615	b9 10 03 00 00	 mov	 ecx, OFFSET ?k_parseTunerConstants@@3QBVCParseConstant@HCParser@@B+784
  0061a	e9 00 00 00 00	 jmp	 ??1CParseConstant@HCParser@@QAE@XZ
__unwindfunclet$??__Ek_parseTunerConstants@@YAXXZ$150:
  0061f	8b 8d f8 fb ff
	ff		 mov	 ecx, DWORD PTR $T362668[ebp]
  00625	e9 00 00 00 00	 jmp	 ??1CParseValue@HCParser@@UAE@XZ ; HCParser::CParseValue::~CParseValue
__unwindfunclet$??__Ek_parseTunerConstants@@YAXXZ$151:
  0062a	8d 8d fc fb ff
	ff		 lea	 ecx, DWORD PTR $T362667[ebp]
  00630	e9 00 00 00 00	 jmp	 ??1CParseConstant@HCParser@@QAE@XZ
__unwindfunclet$??__Ek_parseTunerConstants@@YAXXZ$152:
  00635	b9 20 03 00 00	 mov	 ecx, OFFSET ?k_parseTunerConstants@@3QBVCParseConstant@HCParser@@B+800
  0063a	e9 00 00 00 00	 jmp	 ??1CParseConstant@HCParser@@QAE@XZ
__unwindfunclet$??__Ek_parseTunerConstants@@YAXXZ$153:
  0063f	8b 8d e4 fb ff
	ff		 mov	 ecx, DWORD PTR $T362670[ebp]
  00645	e9 00 00 00 00	 jmp	 ??1CParseValue@HCParser@@UAE@XZ ; HCParser::CParseValue::~CParseValue
__unwindfunclet$??__Ek_parseTunerConstants@@YAXXZ$154:
  0064a	8d 8d e8 fb ff
	ff		 lea	 ecx, DWORD PTR $T362669[ebp]
  00650	e9 00 00 00 00	 jmp	 ??1CParseConstant@HCParser@@QAE@XZ
__unwindfunclet$??__Ek_parseTunerConstants@@YAXXZ$155:
  00655	b9 30 03 00 00	 mov	 ecx, OFFSET ?k_parseTunerConstants@@3QBVCParseConstant@HCParser@@B+816
  0065a	e9 00 00 00 00	 jmp	 ??1CParseConstant@HCParser@@QAE@XZ
__unwindfunclet$??__Ek_parseTunerConstants@@YAXXZ$156:
  0065f	8b 8d d0 fb ff
	ff		 mov	 ecx, DWORD PTR $T362672[ebp]
  00665	e9 00 00 00 00	 jmp	 ??1CParseValue@HCParser@@UAE@XZ ; HCParser::CParseValue::~CParseValue
__unwindfunclet$??__Ek_parseTunerConstants@@YAXXZ$157:
  0066a	8d 8d d4 fb ff
	ff		 lea	 ecx, DWORD PTR $T362671[ebp]
  00670	e9 00 00 00 00	 jmp	 ??1CParseConstant@HCParser@@QAE@XZ
__unwindfunclet$??__Ek_parseTunerConstants@@YAXXZ$158:
  00675	b9 40 03 00 00	 mov	 ecx, OFFSET ?k_parseTunerConstants@@3QBVCParseConstant@HCParser@@B+832
  0067a	e9 00 00 00 00	 jmp	 ??1CParseConstant@HCParser@@QAE@XZ
__unwindfunclet$??__Ek_parseTunerConstants@@YAXXZ$159:
  0067f	8b 8d bc fb ff
	ff		 mov	 ecx, DWORD PTR $T362674[ebp]
  00685	e9 00 00 00 00	 jmp	 ??1CParseValue@HCParser@@UAE@XZ ; HCParser::CParseValue::~CParseValue
__unwindfunclet$??__Ek_parseTunerConstants@@YAXXZ$160:
  0068a	8d 8d c0 fb ff
	ff		 lea	 ecx, DWORD PTR $T362673[ebp]
  00690	e9 00 00 00 00	 jmp	 ??1CParseConstant@HCParser@@QAE@XZ
__unwindfunclet$??__Ek_parseTunerConstants@@YAXXZ$161:
  00695	b9 50 03 00 00	 mov	 ecx, OFFSET ?k_parseTunerConstants@@3QBVCParseConstant@HCParser@@B+848
  0069a	e9 00 00 00 00	 jmp	 ??1CParseConstant@HCParser@@QAE@XZ
__unwindfunclet$??__Ek_parseTunerConstants@@YAXXZ$162:
  0069f	8b 8d a8 fb ff
	ff		 mov	 ecx, DWORD PTR $T362676[ebp]
  006a5	e9 00 00 00 00	 jmp	 ??1CParseValue@HCParser@@UAE@XZ ; HCParser::CParseValue::~CParseValue
__unwindfunclet$??__Ek_parseTunerConstants@@YAXXZ$163:
  006aa	8d 8d ac fb ff
	ff		 lea	 ecx, DWORD PTR $T362675[ebp]
  006b0	e9 00 00 00 00	 jmp	 ??1CParseConstant@HCParser@@QAE@XZ
__unwindfunclet$??__Ek_parseTunerConstants@@YAXXZ$164:
  006b5	b9 60 03 00 00	 mov	 ecx, OFFSET ?k_parseTunerConstants@@3QBVCParseConstant@HCParser@@B+864
  006ba	e9 00 00 00 00	 jmp	 ??1CParseConstant@HCParser@@QAE@XZ
__unwindfunclet$??__Ek_parseTunerConstants@@YAXXZ$165:
  006bf	8b 8d 94 fb ff
	ff		 mov	 ecx, DWORD PTR $T362678[ebp]
  006c5	e9 00 00 00 00	 jmp	 ??1CParseValue@HCParser@@UAE@XZ ; HCParser::CParseValue::~CParseValue
__unwindfunclet$??__Ek_parseTunerConstants@@YAXXZ$166:
  006ca	8d 8d 98 fb ff
	ff		 lea	 ecx, DWORD PTR $T362677[ebp]
  006d0	e9 00 00 00 00	 jmp	 ??1CParseConstant@HCParser@@QAE@XZ
__unwindfunclet$??__Ek_parseTunerConstants@@YAXXZ$167:
  006d5	b9 70 03 00 00	 mov	 ecx, OFFSET ?k_parseTunerConstants@@3QBVCParseConstant@HCParser@@B+880
  006da	e9 00 00 00 00	 jmp	 ??1CParseConstant@HCParser@@QAE@XZ
__unwindfunclet$??__Ek_parseTunerConstants@@YAXXZ$168:
  006df	8b 8d 80 fb ff
	ff		 mov	 ecx, DWORD PTR $T362680[ebp]
  006e5	e9 00 00 00 00	 jmp	 ??1CParseValue@HCParser@@UAE@XZ ; HCParser::CParseValue::~CParseValue
__unwindfunclet$??__Ek_parseTunerConstants@@YAXXZ$169:
  006ea	8d 8d 84 fb ff
	ff		 lea	 ecx, DWORD PTR $T362679[ebp]
  006f0	e9 00 00 00 00	 jmp	 ??1CParseConstant@HCParser@@QAE@XZ
__unwindfunclet$??__Ek_parseTunerConstants@@YAXXZ$170:
  006f5	b9 80 03 00 00	 mov	 ecx, OFFSET ?k_parseTunerConstants@@3QBVCParseConstant@HCParser@@B+896
  006fa	e9 00 00 00 00	 jmp	 ??1CParseConstant@HCParser@@QAE@XZ
__unwindfunclet$??__Ek_parseTunerConstants@@YAXXZ$171:
  006ff	8b 8d 6c fb ff
	ff		 mov	 ecx, DWORD PTR $T362682[ebp]
  00705	e9 00 00 00 00	 jmp	 ??1CParseValue@HCParser@@UAE@XZ ; HCParser::CParseValue::~CParseValue
__unwindfunclet$??__Ek_parseTunerConstants@@YAXXZ$172:
  0070a	8d 8d 70 fb ff
	ff		 lea	 ecx, DWORD PTR $T362681[ebp]
  00710	e9 00 00 00 00	 jmp	 ??1CParseConstant@HCParser@@QAE@XZ
__unwindfunclet$??__Ek_parseTunerConstants@@YAXXZ$173:
  00715	b9 90 03 00 00	 mov	 ecx, OFFSET ?k_parseTunerConstants@@3QBVCParseConstant@HCParser@@B+912
  0071a	e9 00 00 00 00	 jmp	 ??1CParseConstant@HCParser@@QAE@XZ
__unwindfunclet$??__Ek_parseTunerConstants@@YAXXZ$174:
  0071f	8b 8d 58 fb ff
	ff		 mov	 ecx, DWORD PTR $T362684[ebp]
  00725	e9 00 00 00 00	 jmp	 ??1CParseValue@HCParser@@UAE@XZ ; HCParser::CParseValue::~CParseValue
__unwindfunclet$??__Ek_parseTunerConstants@@YAXXZ$175:
  0072a	8d 8d 5c fb ff
	ff		 lea	 ecx, DWORD PTR $T362683[ebp]
  00730	e9 00 00 00 00	 jmp	 ??1CParseConstant@HCParser@@QAE@XZ
__unwindfunclet$??__Ek_parseTunerConstants@@YAXXZ$176:
  00735	b9 a0 03 00 00	 mov	 ecx, OFFSET ?k_parseTunerConstants@@3QBVCParseConstant@HCParser@@B+928
  0073a	e9 00 00 00 00	 jmp	 ??1CParseConstant@HCParser@@QAE@XZ
__unwindfunclet$??__Ek_parseTunerConstants@@YAXXZ$177:
  0073f	8b 8d 44 fb ff
	ff		 mov	 ecx, DWORD PTR $T362686[ebp]
  00745	e9 00 00 00 00	 jmp	 ??1CParseValue@HCParser@@UAE@XZ ; HCParser::CParseValue::~CParseValue
__unwindfunclet$??__Ek_parseTunerConstants@@YAXXZ$178:
  0074a	8d 8d 48 fb ff
	ff		 lea	 ecx, DWORD PTR $T362685[ebp]
  00750	e9 00 00 00 00	 jmp	 ??1CParseConstant@HCParser@@QAE@XZ
__unwindfunclet$??__Ek_parseTunerConstants@@YAXXZ$179:
  00755	b9 b0 03 00 00	 mov	 ecx, OFFSET ?k_parseTunerConstants@@3QBVCParseConstant@HCParser@@B+944
  0075a	e9 00 00 00 00	 jmp	 ??1CParseConstant@HCParser@@QAE@XZ
__unwindfunclet$??__Ek_parseTunerConstants@@YAXXZ$180:
  0075f	8b 8d 30 fb ff
	ff		 mov	 ecx, DWORD PTR $T362688[ebp]
  00765	e9 00 00 00 00	 jmp	 ??1CParseValue@HCParser@@UAE@XZ ; HCParser::CParseValue::~CParseValue
__unwindfunclet$??__Ek_parseTunerConstants@@YAXXZ$181:
  0076a	8d 8d 34 fb ff
	ff		 lea	 ecx, DWORD PTR $T362687[ebp]
  00770	e9 00 00 00 00	 jmp	 ??1CParseConstant@HCParser@@QAE@XZ
__unwindfunclet$??__Ek_parseTunerConstants@@YAXXZ$182:
  00775	b9 c0 03 00 00	 mov	 ecx, OFFSET ?k_parseTunerConstants@@3QBVCParseConstant@HCParser@@B+960
  0077a	e9 00 00 00 00	 jmp	 ??1CParseConstant@HCParser@@QAE@XZ
__unwindfunclet$??__Ek_parseTunerConstants@@YAXXZ$183:
  0077f	8b 8d 1c fb ff
	ff		 mov	 ecx, DWORD PTR $T362690[ebp]
  00785	e9 00 00 00 00	 jmp	 ??1CParseValue@HCParser@@UAE@XZ ; HCParser::CParseValue::~CParseValue
__unwindfunclet$??__Ek_parseTunerConstants@@YAXXZ$184:
  0078a	8d 8d 20 fb ff
	ff		 lea	 ecx, DWORD PTR $T362689[ebp]
  00790	e9 00 00 00 00	 jmp	 ??1CParseConstant@HCParser@@QAE@XZ
__unwindfunclet$??__Ek_parseTunerConstants@@YAXXZ$185:
  00795	b9 d0 03 00 00	 mov	 ecx, OFFSET ?k_parseTunerConstants@@3QBVCParseConstant@HCParser@@B+976
  0079a	e9 00 00 00 00	 jmp	 ??1CParseConstant@HCParser@@QAE@XZ
__unwindfunclet$??__Ek_parseTunerConstants@@YAXXZ$186:
  0079f	8b 8d 08 fb ff
	ff		 mov	 ecx, DWORD PTR $T362692[ebp]
  007a5	e9 00 00 00 00	 jmp	 ??1CParseValue@HCParser@@UAE@XZ ; HCParser::CParseValue::~CParseValue
__unwindfunclet$??__Ek_parseTunerConstants@@YAXXZ$187:
  007aa	8d 8d 0c fb ff
	ff		 lea	 ecx, DWORD PTR $T362691[ebp]
  007b0	e9 00 00 00 00	 jmp	 ??1CParseConstant@HCParser@@QAE@XZ
__unwindfunclet$??__Ek_parseTunerConstants@@YAXXZ$188:
  007b5	b9 e0 03 00 00	 mov	 ecx, OFFSET ?k_parseTunerConstants@@3QBVCParseConstant@HCParser@@B+992
  007ba	e9 00 00 00 00	 jmp	 ??1CParseConstant@HCParser@@QAE@XZ
__unwindfunclet$??__Ek_parseTunerConstants@@YAXXZ$189:
  007bf	8b 8d f4 fa ff
	ff		 mov	 ecx, DWORD PTR $T362694[ebp]
  007c5	e9 00 00 00 00	 jmp	 ??1CParseValue@HCParser@@UAE@XZ ; HCParser::CParseValue::~CParseValue
__unwindfunclet$??__Ek_parseTunerConstants@@YAXXZ$190:
  007ca	8d 8d f8 fa ff
	ff		 lea	 ecx, DWORD PTR $T362693[ebp]
  007d0	e9 00 00 00 00	 jmp	 ??1CParseConstant@HCParser@@QAE@XZ
__unwindfunclet$??__Ek_parseTunerConstants@@YAXXZ$191:
  007d5	b9 f0 03 00 00	 mov	 ecx, OFFSET ?k_parseTunerConstants@@3QBVCParseConstant@HCParser@@B+1008
  007da	e9 00 00 00 00	 jmp	 ??1CParseConstant@HCParser@@QAE@XZ
__unwindfunclet$??__Ek_parseTunerConstants@@YAXXZ$192:
  007df	8b 8d e0 fa ff
	ff		 mov	 ecx, DWORD PTR $T362696[ebp]
  007e5	e9 00 00 00 00	 jmp	 ??1CParseValue@HCParser@@UAE@XZ ; HCParser::CParseValue::~CParseValue
__unwindfunclet$??__Ek_parseTunerConstants@@YAXXZ$193:
  007ea	8d 8d e4 fa ff
	ff		 lea	 ecx, DWORD PTR $T362695[ebp]
  007f0	e9 00 00 00 00	 jmp	 ??1CParseConstant@HCParser@@QAE@XZ
__unwindfunclet$??__Ek_parseTunerConstants@@YAXXZ$194:
  007f5	b9 00 04 00 00	 mov	 ecx, OFFSET ?k_parseTunerConstants@@3QBVCParseConstant@HCParser@@B+1024
  007fa	e9 00 00 00 00	 jmp	 ??1CParseConstant@HCParser@@QAE@XZ
__unwindfunclet$??__Ek_parseTunerConstants@@YAXXZ$195:
  007ff	8b 8d cc fa ff
	ff		 mov	 ecx, DWORD PTR $T362698[ebp]
  00805	e9 00 00 00 00	 jmp	 ??1CParseValue@HCParser@@UAE@XZ ; HCParser::CParseValue::~CParseValue
__unwindfunclet$??__Ek_parseTunerConstants@@YAXXZ$196:
  0080a	8d 8d d0 fa ff
	ff		 lea	 ecx, DWORD PTR $T362697[ebp]
  00810	e9 00 00 00 00	 jmp	 ??1CParseConstant@HCParser@@QAE@XZ
__unwindfunclet$??__Ek_parseTunerConstants@@YAXXZ$197:
  00815	b9 10 04 00 00	 mov	 ecx, OFFSET ?k_parseTunerConstants@@3QBVCParseConstant@HCParser@@B+1040
  0081a	e9 00 00 00 00	 jmp	 ??1CParseConstant@HCParser@@QAE@XZ
__unwindfunclet$??__Ek_parseTunerConstants@@YAXXZ$198:
  0081f	8b 8d b8 fa ff
	ff		 mov	 ecx, DWORD PTR $T362700[ebp]
  00825	e9 00 00 00 00	 jmp	 ??1CParseValue@HCParser@@UAE@XZ ; HCParser::CParseValue::~CParseValue
__unwindfunclet$??__Ek_parseTunerConstants@@YAXXZ$199:
  0082a	8d 8d bc fa ff
	ff		 lea	 ecx, DWORD PTR $T362699[ebp]
  00830	e9 00 00 00 00	 jmp	 ??1CParseConstant@HCParser@@QAE@XZ
__unwindfunclet$??__Ek_parseTunerConstants@@YAXXZ$200:
  00835	b9 20 04 00 00	 mov	 ecx, OFFSET ?k_parseTunerConstants@@3QBVCParseConstant@HCParser@@B+1056
  0083a	e9 00 00 00 00	 jmp	 ??1CParseConstant@HCParser@@QAE@XZ
__ehhandler$??__Ek_parseTunerConstants@@YAXXZ:
  0083f	8b 54 24 08	 mov	 edx, DWORD PTR [esp+8]
  00843	8d 42 0c	 lea	 eax, DWORD PTR [edx+12]
  00846	8b 8a 90 f6 ff
	ff		 mov	 ecx, DWORD PTR [edx-2416]
  0084c	33 c8		 xor	 ecx, eax
  0084e	e8 00 00 00 00	 call	 @__security_check_cookie@4
  00853	b8 00 00 00 00	 mov	 eax, OFFSET __ehfuncinfo$??__Ek_parseTunerConstants@@YAXXZ
  00858	e9 00 00 00 00	 jmp	 ___CxxFrameHandler3
text$x	ENDS
??__Ek_parseTunerConstants@@YAXXZ ENDP			; `dynamic initializer for 'k_parseTunerConstants''
;	COMDAT xdata$x
xdata$x	SEGMENT
__unwindtable$??__Ek_parseTDAFormatConstants@@YAXXZ DD 0ffffffffH
	DD	FLAT:__unwindfunclet$??__Ek_parseTDAFormatConstants@@YAXXZ$0
	DD	0ffffffffH
	DD	FLAT:__unwindfunclet$??__Ek_parseTDAFormatConstants@@YAXXZ$1
	DD	01H
	DD	FLAT:__unwindfunclet$??__Ek_parseTDAFormatConstants@@YAXXZ$2
	DD	0ffffffffH
	DD	FLAT:__unwindfunclet$??__Ek_parseTDAFormatConstants@@YAXXZ$2
	DD	03H
	DD	FLAT:__unwindfunclet$??__Ek_parseTDAFormatConstants@@YAXXZ$3
	DD	03H
	DD	FLAT:__unwindfunclet$??__Ek_parseTDAFormatConstants@@YAXXZ$4
	DD	05H
	DD	FLAT:__unwindfunclet$??__Ek_parseTDAFormatConstants@@YAXXZ$5
	DD	03H
	DD	FLAT:__unwindfunclet$??__Ek_parseTDAFormatConstants@@YAXXZ$5
	DD	07H
	DD	FLAT:__unwindfunclet$??__Ek_parseTDAFormatConstants@@YAXXZ$6
	DD	07H
	DD	FLAT:__unwindfunclet$??__Ek_parseTDAFormatConstants@@YAXXZ$7
	DD	09H
	DD	FLAT:__unwindfunclet$??__Ek_parseTDAFormatConstants@@YAXXZ$8
	DD	07H
	DD	FLAT:__unwindfunclet$??__Ek_parseTDAFormatConstants@@YAXXZ$8
	DD	0bH
	DD	FLAT:__unwindfunclet$??__Ek_parseTDAFormatConstants@@YAXXZ$9
	DD	0bH
	DD	FLAT:__unwindfunclet$??__Ek_parseTDAFormatConstants@@YAXXZ$10
	DD	0dH
	DD	FLAT:__unwindfunclet$??__Ek_parseTDAFormatConstants@@YAXXZ$11
	DD	0bH
	DD	FLAT:__unwindfunclet$??__Ek_parseTDAFormatConstants@@YAXXZ$11
	DD	0fH
	DD	FLAT:__unwindfunclet$??__Ek_parseTDAFormatConstants@@YAXXZ$12
	DD	0fH
	DD	FLAT:__unwindfunclet$??__Ek_parseTDAFormatConstants@@YAXXZ$13
	DD	011H
	DD	FLAT:__unwindfunclet$??__Ek_parseTDAFormatConstants@@YAXXZ$14
	DD	0fH
	DD	FLAT:__unwindfunclet$??__Ek_parseTDAFormatConstants@@YAXXZ$14
	DD	013H
	DD	FLAT:__unwindfunclet$??__Ek_parseTDAFormatConstants@@YAXXZ$15
	DD	013H
	DD	FLAT:__unwindfunclet$??__Ek_parseTDAFormatConstants@@YAXXZ$16
	DD	015H
	DD	FLAT:__unwindfunclet$??__Ek_parseTDAFormatConstants@@YAXXZ$17
	DD	013H
	DD	FLAT:__unwindfunclet$??__Ek_parseTDAFormatConstants@@YAXXZ$17
	DD	017H
	DD	FLAT:__unwindfunclet$??__Ek_parseTDAFormatConstants@@YAXXZ$18
	DD	017H
	DD	FLAT:__unwindfunclet$??__Ek_parseTDAFormatConstants@@YAXXZ$19
	DD	019H
	DD	FLAT:__unwindfunclet$??__Ek_parseTDAFormatConstants@@YAXXZ$20
	DD	017H
	DD	FLAT:__unwindfunclet$??__Ek_parseTDAFormatConstants@@YAXXZ$20
	DD	01bH
	DD	FLAT:__unwindfunclet$??__Ek_parseTDAFormatConstants@@YAXXZ$21
	DD	01bH
	DD	FLAT:__unwindfunclet$??__Ek_parseTDAFormatConstants@@YAXXZ$22
	DD	01dH
	DD	FLAT:__unwindfunclet$??__Ek_parseTDAFormatConstants@@YAXXZ$23
	DD	01bH
	DD	FLAT:__unwindfunclet$??__Ek_parseTDAFormatConstants@@YAXXZ$23
	DD	01fH
	DD	FLAT:__unwindfunclet$??__Ek_parseTDAFormatConstants@@YAXXZ$24
	DD	01fH
	DD	FLAT:__unwindfunclet$??__Ek_parseTDAFormatConstants@@YAXXZ$25
	DD	021H
	DD	FLAT:__unwindfunclet$??__Ek_parseTDAFormatConstants@@YAXXZ$26
	DD	01fH
	DD	FLAT:__unwindfunclet$??__Ek_parseTDAFormatConstants@@YAXXZ$26
	DD	023H
	DD	FLAT:__unwindfunclet$??__Ek_parseTDAFormatConstants@@YAXXZ$27
	DD	023H
	DD	FLAT:__unwindfunclet$??__Ek_parseTDAFormatConstants@@YAXXZ$28
	DD	025H
	DD	FLAT:__unwindfunclet$??__Ek_parseTDAFormatConstants@@YAXXZ$29
	DD	023H
	DD	FLAT:__unwindfunclet$??__Ek_parseTDAFormatConstants@@YAXXZ$29
	DD	027H
	DD	FLAT:__unwindfunclet$??__Ek_parseTDAFormatConstants@@YAXXZ$30
	DD	027H
	DD	FLAT:__unwindfunclet$??__Ek_parseTDAFormatConstants@@YAXXZ$31
	DD	029H
	DD	FLAT:__unwindfunclet$??__Ek_parseTDAFormatConstants@@YAXXZ$32
	DD	027H
	DD	FLAT:__unwindfunclet$??__Ek_parseTDAFormatConstants@@YAXXZ$32
__ehfuncinfo$??__Ek_parseTDAFormatConstants@@YAXXZ DD 019930522H
	DD	02cH
	DD	FLAT:__unwindtable$??__Ek_parseTDAFormatConstants@@YAXXZ
	DD	2 DUP(00H)
	DD	2 DUP(00H)
	DD	00H
	DD	00H
; Function compile flags: /Odtp
xdata$x	ENDS
;	COMDAT ??__Ek_parseTDAFormatConstants@@YAXXZ
text$yc	SEGMENT
tv413 = -408						; size = 4
tv411 = -404						; size = 4
tv410 = -400						; size = 4
tv304 = -396						; size = 4
tv407 = -392						; size = 4
tv405 = -388						; size = 4
tv404 = -384						; size = 4
tv281 = -380						; size = 4
tv401 = -376						; size = 4
tv399 = -372						; size = 4
tv398 = -368						; size = 4
tv258 = -364						; size = 4
tv395 = -360						; size = 4
tv393 = -356						; size = 4
tv392 = -352						; size = 4
tv235 = -348						; size = 4
tv389 = -344						; size = 4
tv387 = -340						; size = 4
tv386 = -336						; size = 4
tv212 = -332						; size = 4
tv383 = -328						; size = 4
tv381 = -324						; size = 4
tv380 = -320						; size = 4
tv189 = -316						; size = 4
tv377 = -312						; size = 4
tv375 = -308						; size = 4
tv374 = -304						; size = 4
tv166 = -300						; size = 4
tv371 = -296						; size = 4
tv369 = -292						; size = 4
tv368 = -288						; size = 4
tv143 = -284						; size = 4
tv365 = -280						; size = 4
tv363 = -276						; size = 4
tv362 = -272						; size = 4
tv88 = -268						; size = 4
tv359 = -264						; size = 4
tv357 = -260						; size = 4
tv356 = -256						; size = 4
tv65 = -252						; size = 4
tv353 = -248						; size = 4
tv351 = -244						; size = 4
tv350 = -240						; size = 4
tv415 = -236						; size = 4
$T362931 = -232						; size = 4
$T362930 = -228						; size = 16
$T362929 = -212						; size = 4
$T362928 = -208						; size = 16
$T362927 = -192						; size = 4
$T362926 = -188						; size = 16
$T362925 = -172						; size = 4
$T362924 = -168						; size = 16
$T362923 = -152						; size = 4
$T362922 = -148						; size = 16
$T362921 = -132						; size = 4
$T362920 = -128						; size = 16
$T362919 = -112						; size = 4
$T362918 = -108						; size = 16
$T362917 = -92						; size = 4
$T362916 = -88						; size = 16
$T362915 = -72						; size = 4
$T362914 = -68						; size = 16
$T362913 = -52						; size = 4
$T362912 = -48						; size = 16
$T362911 = -32						; size = 4
$T362910 = -28						; size = 16
__$EHRec$ = -12						; size = 12
??__Ek_parseTDAFormatConstants@@YAXXZ PROC		; `dynamic initializer for 'k_parseTDAFormatConstants'', COMDAT

; 110  : {

  00000	55		 push	 ebp
  00001	8b ec		 mov	 ebp, esp
  00003	6a ff		 push	 -1
  00005	68 00 00 00 00	 push	 __ehhandler$??__Ek_parseTDAFormatConstants@@YAXXZ
  0000a	64 a1 00 00 00
	00		 mov	 eax, DWORD PTR fs:0
  00010	50		 push	 eax
  00011	81 ec 8c 01 00
	00		 sub	 esp, 396		; 0000018cH
  00017	a1 00 00 00 00	 mov	 eax, DWORD PTR ___security_cookie
  0001c	33 c5		 xor	 eax, ebp
  0001e	50		 push	 eax
  0001f	8d 45 f4	 lea	 eax, DWORD PTR __$EHRec$[ebp]
  00022	64 a3 00 00 00
	00		 mov	 DWORD PTR fs:0, eax

; 111  :     PC( _T("GLOBAL"),                        TDA9887_FORMAT_NONE            ),

  00028	83 ec 0c	 sub	 esp, 12			; 0000000cH
  0002b	8b cc		 mov	 ecx, esp
  0002d	89 65 e0	 mov	 DWORD PTR $T362911[ebp], esp
  00030	6a ff		 push	 -1
  00032	e8 00 00 00 00	 call	 ??0CParseValue@HCParser@@QAE@H@Z ; HCParser::CParseValue::CParseValue
  00037	89 85 14 ff ff
	ff		 mov	 DWORD PTR tv415[ebp], eax
  0003d	8b 85 14 ff ff
	ff		 mov	 eax, DWORD PTR tv415[ebp]
  00043	89 85 10 ff ff
	ff		 mov	 DWORD PTR tv350[ebp], eax
  00049	c7 45 fc 00 00
	00 00		 mov	 DWORD PTR __$EHRec$[ebp+8], 0
  00050	68 00 00 00 00	 push	 OFFSET ??_C@_1O@COJGIGIJ@?$AAG?$AAL?$AAO?$AAB?$AAA?$AAL?$AA?$AA@
  00055	c7 45 fc ff ff
	ff ff		 mov	 DWORD PTR __$EHRec$[ebp+8], -1
  0005c	8d 4d e4	 lea	 ecx, DWORD PTR $T362910[ebp]
  0005f	e8 00 00 00 00	 call	 ??0CParseConstant@HCParser@@QAE@PB_WVCParseValue@1@@Z ; HCParser::CParseConstant::CParseConstant
  00064	89 85 0c ff ff
	ff		 mov	 DWORD PTR tv351[ebp], eax
  0006a	8b 8d 0c ff ff
	ff		 mov	 ecx, DWORD PTR tv351[ebp]
  00070	89 8d 08 ff ff
	ff		 mov	 DWORD PTR tv353[ebp], ecx
  00076	c7 45 fc 01 00
	00 00		 mov	 DWORD PTR __$EHRec$[ebp+8], 1
  0007d	8b 95 08 ff ff
	ff		 mov	 edx, DWORD PTR tv353[ebp]
  00083	52		 push	 edx
  00084	b9 00 00 00 00	 mov	 ecx, OFFSET _k_parseTDAFormatConstants
  00089	e8 00 00 00 00	 call	 ??0CParseConstant@HCParser@@QAE@ABV01@@Z
  0008e	c6 45 fc 03	 mov	 BYTE PTR __$EHRec$[ebp+8], 3
  00092	8d 4d e4	 lea	 ecx, DWORD PTR $T362910[ebp]
  00095	e8 00 00 00 00	 call	 ??1CParseConstant@HCParser@@QAE@XZ

; 112  :     PC( _T("PAL-BG"),                        TDA9887_FORMAT_PAL_BG        ),

  0009a	83 ec 0c	 sub	 esp, 12			; 0000000cH
  0009d	8b cc		 mov	 ecx, esp
  0009f	89 65 cc	 mov	 DWORD PTR $T362913[ebp], esp
  000a2	6a 00		 push	 0
  000a4	e8 00 00 00 00	 call	 ??0CParseValue@HCParser@@QAE@H@Z ; HCParser::CParseValue::CParseValue
  000a9	89 85 04 ff ff
	ff		 mov	 DWORD PTR tv65[ebp], eax
  000af	8b 85 04 ff ff
	ff		 mov	 eax, DWORD PTR tv65[ebp]
  000b5	89 85 00 ff ff
	ff		 mov	 DWORD PTR tv356[ebp], eax
  000bb	c6 45 fc 04	 mov	 BYTE PTR __$EHRec$[ebp+8], 4
  000bf	68 00 00 00 00	 push	 OFFSET ??_C@_1O@CPONHA@?$AAP?$AAA?$AAL?$AA?9?$AAB?$AAG?$AA?$AA@
  000c4	c6 45 fc 03	 mov	 BYTE PTR __$EHRec$[ebp+8], 3
  000c8	8d 4d d0	 lea	 ecx, DWORD PTR $T362912[ebp]
  000cb	e8 00 00 00 00	 call	 ??0CParseConstant@HCParser@@QAE@PB_WVCParseValue@1@@Z ; HCParser::CParseConstant::CParseConstant
  000d0	89 85 fc fe ff
	ff		 mov	 DWORD PTR tv357[ebp], eax
  000d6	8b 8d fc fe ff
	ff		 mov	 ecx, DWORD PTR tv357[ebp]
  000dc	89 8d f8 fe ff
	ff		 mov	 DWORD PTR tv359[ebp], ecx
  000e2	c6 45 fc 05	 mov	 BYTE PTR __$EHRec$[ebp+8], 5
  000e6	8b 95 f8 fe ff
	ff		 mov	 edx, DWORD PTR tv359[ebp]
  000ec	52		 push	 edx
  000ed	b9 10 00 00 00	 mov	 ecx, OFFSET _k_parseTDAFormatConstants+16
  000f2	e8 00 00 00 00	 call	 ??0CParseConstant@HCParser@@QAE@ABV01@@Z
  000f7	c6 45 fc 07	 mov	 BYTE PTR __$EHRec$[ebp+8], 7
  000fb	8d 4d d0	 lea	 ecx, DWORD PTR $T362912[ebp]
  000fe	e8 00 00 00 00	 call	 ??1CParseConstant@HCParser@@QAE@XZ

; 113  :     PC( _T("PAL-I"),                        TDA9887_FORMAT_PAL_I        ),

  00103	83 ec 0c	 sub	 esp, 12			; 0000000cH
  00106	8b cc		 mov	 ecx, esp
  00108	89 65 b8	 mov	 DWORD PTR $T362915[ebp], esp
  0010b	6a 01		 push	 1
  0010d	e8 00 00 00 00	 call	 ??0CParseValue@HCParser@@QAE@H@Z ; HCParser::CParseValue::CParseValue
  00112	89 85 f4 fe ff
	ff		 mov	 DWORD PTR tv88[ebp], eax
  00118	8b 85 f4 fe ff
	ff		 mov	 eax, DWORD PTR tv88[ebp]
  0011e	89 85 f0 fe ff
	ff		 mov	 DWORD PTR tv362[ebp], eax
  00124	c6 45 fc 08	 mov	 BYTE PTR __$EHRec$[ebp+8], 8
  00128	68 00 00 00 00	 push	 OFFSET ??_C@_1M@OKDFNJPP@?$AAP?$AAA?$AAL?$AA?9?$AAI?$AA?$AA@
  0012d	c6 45 fc 07	 mov	 BYTE PTR __$EHRec$[ebp+8], 7
  00131	8d 4d bc	 lea	 ecx, DWORD PTR $T362914[ebp]
  00134	e8 00 00 00 00	 call	 ??0CParseConstant@HCParser@@QAE@PB_WVCParseValue@1@@Z ; HCParser::CParseConstant::CParseConstant
  00139	89 85 ec fe ff
	ff		 mov	 DWORD PTR tv363[ebp], eax
  0013f	8b 8d ec fe ff
	ff		 mov	 ecx, DWORD PTR tv363[ebp]
  00145	89 8d e8 fe ff
	ff		 mov	 DWORD PTR tv365[ebp], ecx
  0014b	c6 45 fc 09	 mov	 BYTE PTR __$EHRec$[ebp+8], 9
  0014f	8b 95 e8 fe ff
	ff		 mov	 edx, DWORD PTR tv365[ebp]
  00155	52		 push	 edx
  00156	b9 20 00 00 00	 mov	 ecx, OFFSET _k_parseTDAFormatConstants+32
  0015b	e8 00 00 00 00	 call	 ??0CParseConstant@HCParser@@QAE@ABV01@@Z
  00160	c6 45 fc 0b	 mov	 BYTE PTR __$EHRec$[ebp+8], 11 ; 0000000bH
  00164	8d 4d bc	 lea	 ecx, DWORD PTR $T362914[ebp]
  00167	e8 00 00 00 00	 call	 ??1CParseConstant@HCParser@@QAE@XZ

; 114  :     PC( _T("PAL-DK"),                        TDA9887_FORMAT_PAL_DK        ),

  0016c	83 ec 0c	 sub	 esp, 12			; 0000000cH
  0016f	8b cc		 mov	 ecx, esp
  00171	89 65 a4	 mov	 DWORD PTR $T362917[ebp], esp
  00174	6a 02		 push	 2
  00176	e8 00 00 00 00	 call	 ??0CParseValue@HCParser@@QAE@H@Z ; HCParser::CParseValue::CParseValue
  0017b	89 85 e4 fe ff
	ff		 mov	 DWORD PTR tv143[ebp], eax
  00181	8b 85 e4 fe ff
	ff		 mov	 eax, DWORD PTR tv143[ebp]
  00187	89 85 e0 fe ff
	ff		 mov	 DWORD PTR tv368[ebp], eax
  0018d	c6 45 fc 0c	 mov	 BYTE PTR __$EHRec$[ebp+8], 12 ; 0000000cH
  00191	68 00 00 00 00	 push	 OFFSET ??_C@_1O@JMKALBNF@?$AAP?$AAA?$AAL?$AA?9?$AAD?$AAK?$AA?$AA@
  00196	c6 45 fc 0b	 mov	 BYTE PTR __$EHRec$[ebp+8], 11 ; 0000000bH
  0019a	8d 4d a8	 lea	 ecx, DWORD PTR $T362916[ebp]
  0019d	e8 00 00 00 00	 call	 ??0CParseConstant@HCParser@@QAE@PB_WVCParseValue@1@@Z ; HCParser::CParseConstant::CParseConstant
  001a2	89 85 dc fe ff
	ff		 mov	 DWORD PTR tv369[ebp], eax
  001a8	8b 8d dc fe ff
	ff		 mov	 ecx, DWORD PTR tv369[ebp]
  001ae	89 8d d8 fe ff
	ff		 mov	 DWORD PTR tv371[ebp], ecx
  001b4	c6 45 fc 0d	 mov	 BYTE PTR __$EHRec$[ebp+8], 13 ; 0000000dH
  001b8	8b 95 d8 fe ff
	ff		 mov	 edx, DWORD PTR tv371[ebp]
  001be	52		 push	 edx
  001bf	b9 30 00 00 00	 mov	 ecx, OFFSET _k_parseTDAFormatConstants+48
  001c4	e8 00 00 00 00	 call	 ??0CParseConstant@HCParser@@QAE@ABV01@@Z
  001c9	c6 45 fc 0f	 mov	 BYTE PTR __$EHRec$[ebp+8], 15 ; 0000000fH
  001cd	8d 4d a8	 lea	 ecx, DWORD PTR $T362916[ebp]
  001d0	e8 00 00 00 00	 call	 ??1CParseConstant@HCParser@@QAE@XZ

; 115  :     PC( _T("PAL-MN"),                        TDA9887_FORMAT_PAL_MN        ),

  001d5	83 ec 0c	 sub	 esp, 12			; 0000000cH
  001d8	8b cc		 mov	 ecx, esp
  001da	89 65 90	 mov	 DWORD PTR $T362919[ebp], esp
  001dd	6a 03		 push	 3
  001df	e8 00 00 00 00	 call	 ??0CParseValue@HCParser@@QAE@H@Z ; HCParser::CParseValue::CParseValue
  001e4	89 85 d4 fe ff
	ff		 mov	 DWORD PTR tv166[ebp], eax
  001ea	8b 85 d4 fe ff
	ff		 mov	 eax, DWORD PTR tv166[ebp]
  001f0	89 85 d0 fe ff
	ff		 mov	 DWORD PTR tv374[ebp], eax
  001f6	c6 45 fc 10	 mov	 BYTE PTR __$EHRec$[ebp+8], 16 ; 00000010H
  001fa	68 00 00 00 00	 push	 OFFSET ??_C@_1O@IMHBBACP@?$AAP?$AAA?$AAL?$AA?9?$AAM?$AAN?$AA?$AA@
  001ff	c6 45 fc 0f	 mov	 BYTE PTR __$EHRec$[ebp+8], 15 ; 0000000fH
  00203	8d 4d 94	 lea	 ecx, DWORD PTR $T362918[ebp]
  00206	e8 00 00 00 00	 call	 ??0CParseConstant@HCParser@@QAE@PB_WVCParseValue@1@@Z ; HCParser::CParseConstant::CParseConstant
  0020b	89 85 cc fe ff
	ff		 mov	 DWORD PTR tv375[ebp], eax
  00211	8b 8d cc fe ff
	ff		 mov	 ecx, DWORD PTR tv375[ebp]
  00217	89 8d c8 fe ff
	ff		 mov	 DWORD PTR tv377[ebp], ecx
  0021d	c6 45 fc 11	 mov	 BYTE PTR __$EHRec$[ebp+8], 17 ; 00000011H
  00221	8b 95 c8 fe ff
	ff		 mov	 edx, DWORD PTR tv377[ebp]
  00227	52		 push	 edx
  00228	b9 40 00 00 00	 mov	 ecx, OFFSET _k_parseTDAFormatConstants+64
  0022d	e8 00 00 00 00	 call	 ??0CParseConstant@HCParser@@QAE@ABV01@@Z
  00232	c6 45 fc 13	 mov	 BYTE PTR __$EHRec$[ebp+8], 19 ; 00000013H
  00236	8d 4d 94	 lea	 ecx, DWORD PTR $T362918[ebp]
  00239	e8 00 00 00 00	 call	 ??1CParseConstant@HCParser@@QAE@XZ

; 116  :     PC( _T("SECAM-L"),                        TDA9887_FORMAT_SECAM_L        ),

  0023e	83 ec 0c	 sub	 esp, 12			; 0000000cH
  00241	8b cc		 mov	 ecx, esp
  00243	89 a5 7c ff ff
	ff		 mov	 DWORD PTR $T362921[ebp], esp
  00249	6a 04		 push	 4
  0024b	e8 00 00 00 00	 call	 ??0CParseValue@HCParser@@QAE@H@Z ; HCParser::CParseValue::CParseValue
  00250	89 85 c4 fe ff
	ff		 mov	 DWORD PTR tv189[ebp], eax
  00256	8b 85 c4 fe ff
	ff		 mov	 eax, DWORD PTR tv189[ebp]
  0025c	89 85 c0 fe ff
	ff		 mov	 DWORD PTR tv380[ebp], eax
  00262	c6 45 fc 14	 mov	 BYTE PTR __$EHRec$[ebp+8], 20 ; 00000014H
  00266	68 00 00 00 00	 push	 OFFSET ??_C@_1BA@NJCCHOGP@?$AAS?$AAE?$AAC?$AAA?$AAM?$AA?9?$AAL?$AA?$AA@
  0026b	c6 45 fc 13	 mov	 BYTE PTR __$EHRec$[ebp+8], 19 ; 00000013H
  0026f	8d 4d 80	 lea	 ecx, DWORD PTR $T362920[ebp]
  00272	e8 00 00 00 00	 call	 ??0CParseConstant@HCParser@@QAE@PB_WVCParseValue@1@@Z ; HCParser::CParseConstant::CParseConstant
  00277	89 85 bc fe ff
	ff		 mov	 DWORD PTR tv381[ebp], eax
  0027d	8b 8d bc fe ff
	ff		 mov	 ecx, DWORD PTR tv381[ebp]
  00283	89 8d b8 fe ff
	ff		 mov	 DWORD PTR tv383[ebp], ecx
  00289	c6 45 fc 15	 mov	 BYTE PTR __$EHRec$[ebp+8], 21 ; 00000015H
  0028d	8b 95 b8 fe ff
	ff		 mov	 edx, DWORD PTR tv383[ebp]
  00293	52		 push	 edx
  00294	b9 50 00 00 00	 mov	 ecx, OFFSET _k_parseTDAFormatConstants+80
  00299	e8 00 00 00 00	 call	 ??0CParseConstant@HCParser@@QAE@ABV01@@Z
  0029e	c6 45 fc 17	 mov	 BYTE PTR __$EHRec$[ebp+8], 23 ; 00000017H
  002a2	8d 4d 80	 lea	 ecx, DWORD PTR $T362920[ebp]
  002a5	e8 00 00 00 00	 call	 ??1CParseConstant@HCParser@@QAE@XZ

; 117  :     PC( _T("SECAM-DK"),                        TDA9887_FORMAT_SECAM_DK        ),

  002aa	83 ec 0c	 sub	 esp, 12			; 0000000cH
  002ad	8b cc		 mov	 ecx, esp
  002af	89 a5 68 ff ff
	ff		 mov	 DWORD PTR $T362923[ebp], esp
  002b5	6a 05		 push	 5
  002b7	e8 00 00 00 00	 call	 ??0CParseValue@HCParser@@QAE@H@Z ; HCParser::CParseValue::CParseValue
  002bc	89 85 b4 fe ff
	ff		 mov	 DWORD PTR tv212[ebp], eax
  002c2	8b 85 b4 fe ff
	ff		 mov	 eax, DWORD PTR tv212[ebp]
  002c8	89 85 b0 fe ff
	ff		 mov	 DWORD PTR tv386[ebp], eax
  002ce	c6 45 fc 18	 mov	 BYTE PTR __$EHRec$[ebp+8], 24 ; 00000018H
  002d2	68 00 00 00 00	 push	 OFFSET ??_C@_1BC@PFJOKPCA@?$AAS?$AAE?$AAC?$AAA?$AAM?$AA?9?$AAD?$AAK?$AA?$AA@
  002d7	c6 45 fc 17	 mov	 BYTE PTR __$EHRec$[ebp+8], 23 ; 00000017H
  002db	8d 8d 6c ff ff
	ff		 lea	 ecx, DWORD PTR $T362922[ebp]
  002e1	e8 00 00 00 00	 call	 ??0CParseConstant@HCParser@@QAE@PB_WVCParseValue@1@@Z ; HCParser::CParseConstant::CParseConstant
  002e6	89 85 ac fe ff
	ff		 mov	 DWORD PTR tv387[ebp], eax
  002ec	8b 8d ac fe ff
	ff		 mov	 ecx, DWORD PTR tv387[ebp]
  002f2	89 8d a8 fe ff
	ff		 mov	 DWORD PTR tv389[ebp], ecx
  002f8	c6 45 fc 19	 mov	 BYTE PTR __$EHRec$[ebp+8], 25 ; 00000019H
  002fc	8b 95 a8 fe ff
	ff		 mov	 edx, DWORD PTR tv389[ebp]
  00302	52		 push	 edx
  00303	b9 60 00 00 00	 mov	 ecx, OFFSET _k_parseTDAFormatConstants+96
  00308	e8 00 00 00 00	 call	 ??0CParseConstant@HCParser@@QAE@ABV01@@Z
  0030d	c6 45 fc 1b	 mov	 BYTE PTR __$EHRec$[ebp+8], 27 ; 0000001bH
  00311	8d 8d 6c ff ff
	ff		 lea	 ecx, DWORD PTR $T362922[ebp]
  00317	e8 00 00 00 00	 call	 ??1CParseConstant@HCParser@@QAE@XZ

; 118  :     PC( _T("NTSC-M"),                        TDA9887_FORMAT_NTSC_M        ),

  0031c	83 ec 0c	 sub	 esp, 12			; 0000000cH
  0031f	8b cc		 mov	 ecx, esp
  00321	89 a5 54 ff ff
	ff		 mov	 DWORD PTR $T362925[ebp], esp
  00327	6a 06		 push	 6
  00329	e8 00 00 00 00	 call	 ??0CParseValue@HCParser@@QAE@H@Z ; HCParser::CParseValue::CParseValue
  0032e	89 85 a4 fe ff
	ff		 mov	 DWORD PTR tv235[ebp], eax
  00334	8b 85 a4 fe ff
	ff		 mov	 eax, DWORD PTR tv235[ebp]
  0033a	89 85 a0 fe ff
	ff		 mov	 DWORD PTR tv392[ebp], eax
  00340	c6 45 fc 1c	 mov	 BYTE PTR __$EHRec$[ebp+8], 28 ; 0000001cH
  00344	68 00 00 00 00	 push	 OFFSET ??_C@_1O@LMGGCLHH@?$AAN?$AAT?$AAS?$AAC?$AA?9?$AAM?$AA?$AA@
  00349	c6 45 fc 1b	 mov	 BYTE PTR __$EHRec$[ebp+8], 27 ; 0000001bH
  0034d	8d 8d 58 ff ff
	ff		 lea	 ecx, DWORD PTR $T362924[ebp]
  00353	e8 00 00 00 00	 call	 ??0CParseConstant@HCParser@@QAE@PB_WVCParseValue@1@@Z ; HCParser::CParseConstant::CParseConstant
  00358	89 85 9c fe ff
	ff		 mov	 DWORD PTR tv393[ebp], eax
  0035e	8b 8d 9c fe ff
	ff		 mov	 ecx, DWORD PTR tv393[ebp]
  00364	89 8d 98 fe ff
	ff		 mov	 DWORD PTR tv395[ebp], ecx
  0036a	c6 45 fc 1d	 mov	 BYTE PTR __$EHRec$[ebp+8], 29 ; 0000001dH
  0036e	8b 95 98 fe ff
	ff		 mov	 edx, DWORD PTR tv395[ebp]
  00374	52		 push	 edx
  00375	b9 70 00 00 00	 mov	 ecx, OFFSET _k_parseTDAFormatConstants+112
  0037a	e8 00 00 00 00	 call	 ??0CParseConstant@HCParser@@QAE@ABV01@@Z
  0037f	c6 45 fc 1f	 mov	 BYTE PTR __$EHRec$[ebp+8], 31 ; 0000001fH
  00383	8d 8d 58 ff ff
	ff		 lea	 ecx, DWORD PTR $T362924[ebp]
  00389	e8 00 00 00 00	 call	 ??1CParseConstant@HCParser@@QAE@XZ

; 119  :     PC( _T("NTSC-JP"),                        TDA9887_FORMAT_NTSC_JP        ),

  0038e	83 ec 0c	 sub	 esp, 12			; 0000000cH
  00391	8b cc		 mov	 ecx, esp
  00393	89 a5 40 ff ff
	ff		 mov	 DWORD PTR $T362927[ebp], esp
  00399	6a 07		 push	 7
  0039b	e8 00 00 00 00	 call	 ??0CParseValue@HCParser@@QAE@H@Z ; HCParser::CParseValue::CParseValue
  003a0	89 85 94 fe ff
	ff		 mov	 DWORD PTR tv258[ebp], eax
  003a6	8b 85 94 fe ff
	ff		 mov	 eax, DWORD PTR tv258[ebp]
  003ac	89 85 90 fe ff
	ff		 mov	 DWORD PTR tv398[ebp], eax
  003b2	c6 45 fc 20	 mov	 BYTE PTR __$EHRec$[ebp+8], 32 ; 00000020H
  003b6	68 00 00 00 00	 push	 OFFSET ??_C@_1BA@BKMKJFAN@?$AAN?$AAT?$AAS?$AAC?$AA?9?$AAJ?$AAP?$AA?$AA@
  003bb	c6 45 fc 1f	 mov	 BYTE PTR __$EHRec$[ebp+8], 31 ; 0000001fH
  003bf	8d 8d 44 ff ff
	ff		 lea	 ecx, DWORD PTR $T362926[ebp]
  003c5	e8 00 00 00 00	 call	 ??0CParseConstant@HCParser@@QAE@PB_WVCParseValue@1@@Z ; HCParser::CParseConstant::CParseConstant
  003ca	89 85 8c fe ff
	ff		 mov	 DWORD PTR tv399[ebp], eax
  003d0	8b 8d 8c fe ff
	ff		 mov	 ecx, DWORD PTR tv399[ebp]
  003d6	89 8d 88 fe ff
	ff		 mov	 DWORD PTR tv401[ebp], ecx
  003dc	c6 45 fc 21	 mov	 BYTE PTR __$EHRec$[ebp+8], 33 ; 00000021H
  003e0	8b 95 88 fe ff
	ff		 mov	 edx, DWORD PTR tv401[ebp]
  003e6	52		 push	 edx
  003e7	b9 80 00 00 00	 mov	 ecx, OFFSET _k_parseTDAFormatConstants+128
  003ec	e8 00 00 00 00	 call	 ??0CParseConstant@HCParser@@QAE@ABV01@@Z
  003f1	c6 45 fc 23	 mov	 BYTE PTR __$EHRec$[ebp+8], 35 ; 00000023H
  003f5	8d 8d 44 ff ff
	ff		 lea	 ecx, DWORD PTR $T362926[ebp]
  003fb	e8 00 00 00 00	 call	 ??1CParseConstant@HCParser@@QAE@XZ

; 120  :     PC( _T("Radio"),                        TDA9887_FORMAT_RADIO        ),

  00400	83 ec 0c	 sub	 esp, 12			; 0000000cH
  00403	8b cc		 mov	 ecx, esp
  00405	89 a5 2c ff ff
	ff		 mov	 DWORD PTR $T362929[ebp], esp
  0040b	6a 08		 push	 8
  0040d	e8 00 00 00 00	 call	 ??0CParseValue@HCParser@@QAE@H@Z ; HCParser::CParseValue::CParseValue
  00412	89 85 84 fe ff
	ff		 mov	 DWORD PTR tv281[ebp], eax
  00418	8b 85 84 fe ff
	ff		 mov	 eax, DWORD PTR tv281[ebp]
  0041e	89 85 80 fe ff
	ff		 mov	 DWORD PTR tv404[ebp], eax
  00424	c6 45 fc 24	 mov	 BYTE PTR __$EHRec$[ebp+8], 36 ; 00000024H
  00428	68 00 00 00 00	 push	 OFFSET ??_C@_1M@HCFAIFML@?$AAR?$AAa?$AAd?$AAi?$AAo?$AA?$AA@
  0042d	c6 45 fc 23	 mov	 BYTE PTR __$EHRec$[ebp+8], 35 ; 00000023H
  00431	8d 8d 30 ff ff
	ff		 lea	 ecx, DWORD PTR $T362928[ebp]
  00437	e8 00 00 00 00	 call	 ??0CParseConstant@HCParser@@QAE@PB_WVCParseValue@1@@Z ; HCParser::CParseConstant::CParseConstant
  0043c	89 85 7c fe ff
	ff		 mov	 DWORD PTR tv405[ebp], eax
  00442	8b 8d 7c fe ff
	ff		 mov	 ecx, DWORD PTR tv405[ebp]
  00448	89 8d 78 fe ff
	ff		 mov	 DWORD PTR tv407[ebp], ecx
  0044e	c6 45 fc 25	 mov	 BYTE PTR __$EHRec$[ebp+8], 37 ; 00000025H
  00452	8b 95 78 fe ff
	ff		 mov	 edx, DWORD PTR tv407[ebp]
  00458	52		 push	 edx
  00459	b9 90 00 00 00	 mov	 ecx, OFFSET _k_parseTDAFormatConstants+144
  0045e	e8 00 00 00 00	 call	 ??0CParseConstant@HCParser@@QAE@ABV01@@Z
  00463	c6 45 fc 27	 mov	 BYTE PTR __$EHRec$[ebp+8], 39 ; 00000027H
  00467	8d 8d 30 ff ff
	ff		 lea	 ecx, DWORD PTR $T362928[ebp]
  0046d	e8 00 00 00 00	 call	 ??1CParseConstant@HCParser@@QAE@XZ

; 121  :     PC( NULL )
; 122  : };

  00472	83 ec 0c	 sub	 esp, 12			; 0000000cH
  00475	8b cc		 mov	 ecx, esp
  00477	89 a5 18 ff ff
	ff		 mov	 DWORD PTR $T362931[ebp], esp
  0047d	e8 00 00 00 00	 call	 ??0CParseValue@HCParser@@QAE@XZ ; HCParser::CParseValue::CParseValue
  00482	89 85 74 fe ff
	ff		 mov	 DWORD PTR tv304[ebp], eax
  00488	8b 85 74 fe ff
	ff		 mov	 eax, DWORD PTR tv304[ebp]
  0048e	89 85 70 fe ff
	ff		 mov	 DWORD PTR tv410[ebp], eax
  00494	c6 45 fc 28	 mov	 BYTE PTR __$EHRec$[ebp+8], 40 ; 00000028H
  00498	6a 00		 push	 0
  0049a	c6 45 fc 27	 mov	 BYTE PTR __$EHRec$[ebp+8], 39 ; 00000027H
  0049e	8d 8d 1c ff ff
	ff		 lea	 ecx, DWORD PTR $T362930[ebp]
  004a4	e8 00 00 00 00	 call	 ??0CParseConstant@HCParser@@QAE@PB_WVCParseValue@1@@Z ; HCParser::CParseConstant::CParseConstant
  004a9	89 85 6c fe ff
	ff		 mov	 DWORD PTR tv411[ebp], eax
  004af	8b 8d 6c fe ff
	ff		 mov	 ecx, DWORD PTR tv411[ebp]
  004b5	89 8d 68 fe ff
	ff		 mov	 DWORD PTR tv413[ebp], ecx
  004bb	c6 45 fc 29	 mov	 BYTE PTR __$EHRec$[ebp+8], 41 ; 00000029H
  004bf	8b 95 68 fe ff
	ff		 mov	 edx, DWORD PTR tv413[ebp]
  004c5	52		 push	 edx
  004c6	b9 a0 00 00 00	 mov	 ecx, OFFSET _k_parseTDAFormatConstants+160
  004cb	e8 00 00 00 00	 call	 ??0CParseConstant@HCParser@@QAE@ABV01@@Z
  004d0	c6 45 fc 2b	 mov	 BYTE PTR __$EHRec$[ebp+8], 43 ; 0000002bH
  004d4	8d 8d 1c ff ff
	ff		 lea	 ecx, DWORD PTR $T362930[ebp]
  004da	e8 00 00 00 00	 call	 ??1CParseConstant@HCParser@@QAE@XZ
  004df	c7 45 fc ff ff
	ff ff		 mov	 DWORD PTR __$EHRec$[ebp+8], -1
  004e6	68 00 00 00 00	 push	 OFFSET ??__Fk_parseTDAFormatConstants@@YAXXZ ; `dynamic atexit destructor for 'k_parseTDAFormatConstants''
  004eb	e8 00 00 00 00	 call	 _atexit
  004f0	83 c4 04	 add	 esp, 4
  004f3	8b 4d f4	 mov	 ecx, DWORD PTR __$EHRec$[ebp]
  004f6	64 89 0d 00 00
	00 00		 mov	 DWORD PTR fs:0, ecx
  004fd	59		 pop	 ecx
  004fe	8b e5		 mov	 esp, ebp
  00500	5d		 pop	 ebp
  00501	c3		 ret	 0
text$yc	ENDS
;	COMDAT text$x
text$x	SEGMENT
__unwindfunclet$??__Ek_parseTDAFormatConstants@@YAXXZ$0:
  00000	8b 4d e0	 mov	 ecx, DWORD PTR $T362911[ebp]
  00003	e9 00 00 00 00	 jmp	 ??1CParseValue@HCParser@@UAE@XZ ; HCParser::CParseValue::~CParseValue
__unwindfunclet$??__Ek_parseTDAFormatConstants@@YAXXZ$1:
  00008	8d 4d e4	 lea	 ecx, DWORD PTR $T362910[ebp]
  0000b	e9 00 00 00 00	 jmp	 ??1CParseConstant@HCParser@@QAE@XZ
__unwindfunclet$??__Ek_parseTDAFormatConstants@@YAXXZ$2:
  00010	b9 00 00 00 00	 mov	 ecx, OFFSET _k_parseTDAFormatConstants
  00015	e9 00 00 00 00	 jmp	 ??1CParseConstant@HCParser@@QAE@XZ
__unwindfunclet$??__Ek_parseTDAFormatConstants@@YAXXZ$3:
  0001a	8b 4d cc	 mov	 ecx, DWORD PTR $T362913[ebp]
  0001d	e9 00 00 00 00	 jmp	 ??1CParseValue@HCParser@@UAE@XZ ; HCParser::CParseValue::~CParseValue
__unwindfunclet$??__Ek_parseTDAFormatConstants@@YAXXZ$4:
  00022	8d 4d d0	 lea	 ecx, DWORD PTR $T362912[ebp]
  00025	e9 00 00 00 00	 jmp	 ??1CParseConstant@HCParser@@QAE@XZ
__unwindfunclet$??__Ek_parseTDAFormatConstants@@YAXXZ$5:
  0002a	b9 10 00 00 00	 mov	 ecx, OFFSET _k_parseTDAFormatConstants+16
  0002f	e9 00 00 00 00	 jmp	 ??1CParseConstant@HCParser@@QAE@XZ
__unwindfunclet$??__Ek_parseTDAFormatConstants@@YAXXZ$6:
  00034	8b 4d b8	 mov	 ecx, DWORD PTR $T362915[ebp]
  00037	e9 00 00 00 00	 jmp	 ??1CParseValue@HCParser@@UAE@XZ ; HCParser::CParseValue::~CParseValue
__unwindfunclet$??__Ek_parseTDAFormatConstants@@YAXXZ$7:
  0003c	8d 4d bc	 lea	 ecx, DWORD PTR $T362914[ebp]
  0003f	e9 00 00 00 00	 jmp	 ??1CParseConstant@HCParser@@QAE@XZ
__unwindfunclet$??__Ek_parseTDAFormatConstants@@YAXXZ$8:
  00044	b9 20 00 00 00	 mov	 ecx, OFFSET _k_parseTDAFormatConstants+32
  00049	e9 00 00 00 00	 jmp	 ??1CParseConstant@HCParser@@QAE@XZ
__unwindfunclet$??__Ek_parseTDAFormatConstants@@YAXXZ$9:
  0004e	8b 4d a4	 mov	 ecx, DWORD PTR $T362917[ebp]
  00051	e9 00 00 00 00	 jmp	 ??1CParseValue@HCParser@@UAE@XZ ; HCParser::CParseValue::~CParseValue
__unwindfunclet$??__Ek_parseTDAFormatConstants@@YAXXZ$10:
  00056	8d 4d a8	 lea	 ecx, DWORD PTR $T362916[ebp]
  00059	e9 00 00 00 00	 jmp	 ??1CParseConstant@HCParser@@QAE@XZ
__unwindfunclet$??__Ek_parseTDAFormatConstants@@YAXXZ$11:
  0005e	b9 30 00 00 00	 mov	 ecx, OFFSET _k_parseTDAFormatConstants+48
  00063	e9 00 00 00 00	 jmp	 ??1CParseConstant@HCParser@@QAE@XZ
__unwindfunclet$??__Ek_parseTDAFormatConstants@@YAXXZ$12:
  00068	8b 4d 90	 mov	 ecx, DWORD PTR $T362919[ebp]
  0006b	e9 00 00 00 00	 jmp	 ??1CParseValue@HCParser@@UAE@XZ ; HCParser::CParseValue::~CParseValue
__unwindfunclet$??__Ek_parseTDAFormatConstants@@YAXXZ$13:
  00070	8d 4d 94	 lea	 ecx, DWORD PTR $T362918[ebp]
  00073	e9 00 00 00 00	 jmp	 ??1CParseConstant@HCParser@@QAE@XZ
__unwindfunclet$??__Ek_parseTDAFormatConstants@@YAXXZ$14:
  00078	b9 40 00 00 00	 mov	 ecx, OFFSET _k_parseTDAFormatConstants+64
  0007d	e9 00 00 00 00	 jmp	 ??1CParseConstant@HCParser@@QAE@XZ
__unwindfunclet$??__Ek_parseTDAFormatConstants@@YAXXZ$15:
  00082	8b 8d 7c ff ff
	ff		 mov	 ecx, DWORD PTR $T362921[ebp]
  00088	e9 00 00 00 00	 jmp	 ??1CParseValue@HCParser@@UAE@XZ ; HCParser::CParseValue::~CParseValue
__unwindfunclet$??__Ek_parseTDAFormatConstants@@YAXXZ$16:
  0008d	8d 4d 80	 lea	 ecx, DWORD PTR $T362920[ebp]
  00090	e9 00 00 00 00	 jmp	 ??1CParseConstant@HCParser@@QAE@XZ
__unwindfunclet$??__Ek_parseTDAFormatConstants@@YAXXZ$17:
  00095	b9 50 00 00 00	 mov	 ecx, OFFSET _k_parseTDAFormatConstants+80
  0009a	e9 00 00 00 00	 jmp	 ??1CParseConstant@HCParser@@QAE@XZ
__unwindfunclet$??__Ek_parseTDAFormatConstants@@YAXXZ$18:
  0009f	8b 8d 68 ff ff
	ff		 mov	 ecx, DWORD PTR $T362923[ebp]
  000a5	e9 00 00 00 00	 jmp	 ??1CParseValue@HCParser@@UAE@XZ ; HCParser::CParseValue::~CParseValue
__unwindfunclet$??__Ek_parseTDAFormatConstants@@YAXXZ$19:
  000aa	8d 8d 6c ff ff
	ff		 lea	 ecx, DWORD PTR $T362922[ebp]
  000b0	e9 00 00 00 00	 jmp	 ??1CParseConstant@HCParser@@QAE@XZ
__unwindfunclet$??__Ek_parseTDAFormatConstants@@YAXXZ$20:
  000b5	b9 60 00 00 00	 mov	 ecx, OFFSET _k_parseTDAFormatConstants+96
  000ba	e9 00 00 00 00	 jmp	 ??1CParseConstant@HCParser@@QAE@XZ
__unwindfunclet$??__Ek_parseTDAFormatConstants@@YAXXZ$21:
  000bf	8b 8d 54 ff ff
	ff		 mov	 ecx, DWORD PTR $T362925[ebp]
  000c5	e9 00 00 00 00	 jmp	 ??1CParseValue@HCParser@@UAE@XZ ; HCParser::CParseValue::~CParseValue
__unwindfunclet$??__Ek_parseTDAFormatConstants@@YAXXZ$22:
  000ca	8d 8d 58 ff ff
	ff		 lea	 ecx, DWORD PTR $T362924[ebp]
  000d0	e9 00 00 00 00	 jmp	 ??1CParseConstant@HCParser@@QAE@XZ
__unwindfunclet$??__Ek_parseTDAFormatConstants@@YAXXZ$23:
  000d5	b9 70 00 00 00	 mov	 ecx, OFFSET _k_parseTDAFormatConstants+112
  000da	e9 00 00 00 00	 jmp	 ??1CParseConstant@HCParser@@QAE@XZ
__unwindfunclet$??__Ek_parseTDAFormatConstants@@YAXXZ$24:
  000df	8b 8d 40 ff ff
	ff		 mov	 ecx, DWORD PTR $T362927[ebp]
  000e5	e9 00 00 00 00	 jmp	 ??1CParseValue@HCParser@@UAE@XZ ; HCParser::CParseValue::~CParseValue
__unwindfunclet$??__Ek_parseTDAFormatConstants@@YAXXZ$25:
  000ea	8d 8d 44 ff ff
	ff		 lea	 ecx, DWORD PTR $T362926[ebp]
  000f0	e9 00 00 00 00	 jmp	 ??1CParseConstant@HCParser@@QAE@XZ
__unwindfunclet$??__Ek_parseTDAFormatConstants@@YAXXZ$26:
  000f5	b9 80 00 00 00	 mov	 ecx, OFFSET _k_parseTDAFormatConstants+128
  000fa	e9 00 00 00 00	 jmp	 ??1CParseConstant@HCParser@@QAE@XZ
__unwindfunclet$??__Ek_parseTDAFormatConstants@@YAXXZ$27:
  000ff	8b 8d 2c ff ff
	ff		 mov	 ecx, DWORD PTR $T362929[ebp]
  00105	e9 00 00 00 00	 jmp	 ??1CParseValue@HCParser@@UAE@XZ ; HCParser::CParseValue::~CParseValue
__unwindfunclet$??__Ek_parseTDAFormatConstants@@YAXXZ$28:
  0010a	8d 8d 30 ff ff
	ff		 lea	 ecx, DWORD PTR $T362928[ebp]
  00110	e9 00 00 00 00	 jmp	 ??1CParseConstant@HCParser@@QAE@XZ
__unwindfunclet$??__Ek_parseTDAFormatConstants@@YAXXZ$29:
  00115	b9 90 00 00 00	 mov	 ecx, OFFSET _k_parseTDAFormatConstants+144
  0011a	e9 00 00 00 00	 jmp	 ??1CParseConstant@HCParser@@QAE@XZ
__unwindfunclet$??__Ek_parseTDAFormatConstants@@YAXXZ$30:
  0011f	8b 8d 18 ff ff
	ff		 mov	 ecx, DWORD PTR $T362931[ebp]
  00125	e9 00 00 00 00	 jmp	 ??1CParseValue@HCParser@@UAE@XZ ; HCParser::CParseValue::~CParseValue
__unwindfunclet$??__Ek_parseTDAFormatConstants@@YAXXZ$31:
  0012a	8d 8d 1c ff ff
	ff		 lea	 ecx, DWORD PTR $T362930[ebp]
  00130	e9 00 00 00 00	 jmp	 ??1CParseConstant@HCParser@@QAE@XZ
__unwindfunclet$??__Ek_parseTDAFormatConstants@@YAXXZ$32:
  00135	b9 a0 00 00 00	 mov	 ecx, OFFSET _k_parseTDAFormatConstants+160
  0013a	e9 00 00 00 00	 jmp	 ??1CParseConstant@HCParser@@QAE@XZ
__ehhandler$??__Ek_parseTDAFormatConstants@@YAXXZ:
  0013f	8b 54 24 08	 mov	 edx, DWORD PTR [esp+8]
  00143	8d 42 0c	 lea	 eax, DWORD PTR [edx+12]
  00146	8b 8a 70 fe ff
	ff		 mov	 ecx, DWORD PTR [edx-400]
  0014c	33 c8		 xor	 ecx, eax
  0014e	e8 00 00 00 00	 call	 @__security_check_cookie@4
  00153	b8 00 00 00 00	 mov	 eax, OFFSET __ehfuncinfo$??__Ek_parseTDAFormatConstants@@YAXXZ
  00158	e9 00 00 00 00	 jmp	 ___CxxFrameHandler3
text$x	ENDS
??__Ek_parseTDAFormatConstants@@YAXXZ ENDP		; `dynamic initializer for 'k_parseTDAFormatConstants''
;	COMDAT xdata$x
xdata$x	SEGMENT
__unwindtable$??__Ek_parseCarrierConstants@@YAXXZ DD 0ffffffffH
	DD	FLAT:__unwindfunclet$??__Ek_parseCarrierConstants@@YAXXZ$0
	DD	0ffffffffH
	DD	FLAT:__unwindfunclet$??__Ek_parseCarrierConstants@@YAXXZ$1
	DD	01H
	DD	FLAT:__unwindfunclet$??__Ek_parseCarrierConstants@@YAXXZ$2
	DD	0ffffffffH
	DD	FLAT:__unwindfunclet$??__Ek_parseCarrierConstants@@YAXXZ$2
	DD	03H
	DD	FLAT:__unwindfunclet$??__Ek_parseCarrierConstants@@YAXXZ$3
	DD	03H
	DD	FLAT:__unwindfunclet$??__Ek_parseCarrierConstants@@YAXXZ$4
	DD	05H
	DD	FLAT:__unwindfunclet$??__Ek_parseCarrierConstants@@YAXXZ$5
	DD	03H
	DD	FLAT:__unwindfunclet$??__Ek_parseCarrierConstants@@YAXXZ$5
	DD	07H
	DD	FLAT:__unwindfunclet$??__Ek_parseCarrierConstants@@YAXXZ$6
	DD	07H
	DD	FLAT:__unwindfunclet$??__Ek_parseCarrierConstants@@YAXXZ$7
	DD	09H
	DD	FLAT:__unwindfunclet$??__Ek_parseCarrierConstants@@YAXXZ$8
	DD	07H
	DD	FLAT:__unwindfunclet$??__Ek_parseCarrierConstants@@YAXXZ$8
__ehfuncinfo$??__Ek_parseCarrierConstants@@YAXXZ DD 019930522H
	DD	0cH
	DD	FLAT:__unwindtable$??__Ek_parseCarrierConstants@@YAXXZ
	DD	2 DUP(00H)
	DD	2 DUP(00H)
	DD	00H
	DD	00H
; Function compile flags: /Odtp
xdata$x	ENDS
;	COMDAT ??__Ek_parseCarrierConstants@@YAXXZ
text$yc	SEGMENT
tv181 = -120						; size = 4
tv179 = -116						; size = 4
tv178 = -112						; size = 4
tv88 = -108						; size = 4
tv175 = -104						; size = 4
tv173 = -100						; size = 4
tv172 = -96						; size = 4
tv65 = -92						; size = 4
tv169 = -88						; size = 4
tv167 = -84						; size = 4
tv166 = -80						; size = 4
tv183 = -76						; size = 4
$T362978 = -72						; size = 4
$T362977 = -68						; size = 16
$T362976 = -52						; size = 4
$T362975 = -48						; size = 16
$T362974 = -32						; size = 4
$T362973 = -28						; size = 16
__$EHRec$ = -12						; size = 12
??__Ek_parseCarrierConstants@@YAXXZ PROC		; `dynamic initializer for 'k_parseCarrierConstants'', COMDAT

; 125  : {

  00000	55		 push	 ebp
  00001	8b ec		 mov	 ebp, esp
  00003	6a ff		 push	 -1
  00005	68 00 00 00 00	 push	 __ehhandler$??__Ek_parseCarrierConstants@@YAXXZ
  0000a	64 a1 00 00 00
	00		 mov	 eax, DWORD PTR fs:0
  00010	50		 push	 eax
  00011	83 ec 6c	 sub	 esp, 108		; 0000006cH
  00014	a1 00 00 00 00	 mov	 eax, DWORD PTR ___security_cookie
  00019	33 c5		 xor	 eax, ebp
  0001b	50		 push	 eax
  0001c	8d 45 f4	 lea	 eax, DWORD PTR __$EHRec$[ebp]
  0001f	64 a3 00 00 00
	00		 mov	 DWORD PTR fs:0, eax

; 126  :     PC( _T("intercarrier"),                0 ),

  00025	83 ec 0c	 sub	 esp, 12			; 0000000cH
  00028	8b cc		 mov	 ecx, esp
  0002a	89 65 e0	 mov	 DWORD PTR $T362974[ebp], esp
  0002d	6a 00		 push	 0
  0002f	e8 00 00 00 00	 call	 ??0CParseValue@HCParser@@QAE@H@Z ; HCParser::CParseValue::CParseValue
  00034	89 45 b4	 mov	 DWORD PTR tv183[ebp], eax
  00037	8b 45 b4	 mov	 eax, DWORD PTR tv183[ebp]
  0003a	89 45 b0	 mov	 DWORD PTR tv166[ebp], eax
  0003d	c7 45 fc 00 00
	00 00		 mov	 DWORD PTR __$EHRec$[ebp+8], 0
  00044	68 00 00 00 00	 push	 OFFSET ??_C@_1BK@BJKJAFD@?$AAi?$AAn?$AAt?$AAe?$AAr?$AAc?$AAa?$AAr?$AAr?$AAi?$AAe?$AAr?$AA?$AA@
  00049	c7 45 fc ff ff
	ff ff		 mov	 DWORD PTR __$EHRec$[ebp+8], -1
  00050	8d 4d e4	 lea	 ecx, DWORD PTR $T362973[ebp]
  00053	e8 00 00 00 00	 call	 ??0CParseConstant@HCParser@@QAE@PB_WVCParseValue@1@@Z ; HCParser::CParseConstant::CParseConstant
  00058	89 45 ac	 mov	 DWORD PTR tv167[ebp], eax
  0005b	8b 4d ac	 mov	 ecx, DWORD PTR tv167[ebp]
  0005e	89 4d a8	 mov	 DWORD PTR tv169[ebp], ecx
  00061	c7 45 fc 01 00
	00 00		 mov	 DWORD PTR __$EHRec$[ebp+8], 1
  00068	8b 55 a8	 mov	 edx, DWORD PTR tv169[ebp]
  0006b	52		 push	 edx
  0006c	b9 00 00 00 00	 mov	 ecx, OFFSET _k_parseCarrierConstants
  00071	e8 00 00 00 00	 call	 ??0CParseConstant@HCParser@@QAE@ABV01@@Z
  00076	c6 45 fc 03	 mov	 BYTE PTR __$EHRec$[ebp+8], 3
  0007a	8d 4d e4	 lea	 ecx, DWORD PTR $T362973[ebp]
  0007d	e8 00 00 00 00	 call	 ??1CParseConstant@HCParser@@QAE@XZ

; 127  :     PC( _T("qss"),                        1 ),

  00082	83 ec 0c	 sub	 esp, 12			; 0000000cH
  00085	8b cc		 mov	 ecx, esp
  00087	89 65 cc	 mov	 DWORD PTR $T362976[ebp], esp
  0008a	6a 01		 push	 1
  0008c	e8 00 00 00 00	 call	 ??0CParseValue@HCParser@@QAE@H@Z ; HCParser::CParseValue::CParseValue
  00091	89 45 a4	 mov	 DWORD PTR tv65[ebp], eax
  00094	8b 45 a4	 mov	 eax, DWORD PTR tv65[ebp]
  00097	89 45 a0	 mov	 DWORD PTR tv172[ebp], eax
  0009a	c6 45 fc 04	 mov	 BYTE PTR __$EHRec$[ebp+8], 4
  0009e	68 00 00 00 00	 push	 OFFSET ??_C@_17OBLMBIF@?$AAq?$AAs?$AAs?$AA?$AA@
  000a3	c6 45 fc 03	 mov	 BYTE PTR __$EHRec$[ebp+8], 3
  000a7	8d 4d d0	 lea	 ecx, DWORD PTR $T362975[ebp]
  000aa	e8 00 00 00 00	 call	 ??0CParseConstant@HCParser@@QAE@PB_WVCParseValue@1@@Z ; HCParser::CParseConstant::CParseConstant
  000af	89 45 9c	 mov	 DWORD PTR tv173[ebp], eax
  000b2	8b 4d 9c	 mov	 ecx, DWORD PTR tv173[ebp]
  000b5	89 4d 98	 mov	 DWORD PTR tv175[ebp], ecx
  000b8	c6 45 fc 05	 mov	 BYTE PTR __$EHRec$[ebp+8], 5
  000bc	8b 55 98	 mov	 edx, DWORD PTR tv175[ebp]
  000bf	52		 push	 edx
  000c0	b9 10 00 00 00	 mov	 ecx, OFFSET _k_parseCarrierConstants+16
  000c5	e8 00 00 00 00	 call	 ??0CParseConstant@HCParser@@QAE@ABV01@@Z
  000ca	c6 45 fc 07	 mov	 BYTE PTR __$EHRec$[ebp+8], 7
  000ce	8d 4d d0	 lea	 ecx, DWORD PTR $T362975[ebp]
  000d1	e8 00 00 00 00	 call	 ??1CParseConstant@HCParser@@QAE@XZ

; 128  :     PC( NULL )
; 129  : };

  000d6	83 ec 0c	 sub	 esp, 12			; 0000000cH
  000d9	8b cc		 mov	 ecx, esp
  000db	89 65 b8	 mov	 DWORD PTR $T362978[ebp], esp
  000de	e8 00 00 00 00	 call	 ??0CParseValue@HCParser@@QAE@XZ ; HCParser::CParseValue::CParseValue
  000e3	89 45 94	 mov	 DWORD PTR tv88[ebp], eax
  000e6	8b 45 94	 mov	 eax, DWORD PTR tv88[ebp]
  000e9	89 45 90	 mov	 DWORD PTR tv178[ebp], eax
  000ec	c6 45 fc 08	 mov	 BYTE PTR __$EHRec$[ebp+8], 8
  000f0	6a 00		 push	 0
  000f2	c6 45 fc 07	 mov	 BYTE PTR __$EHRec$[ebp+8], 7
  000f6	8d 4d bc	 lea	 ecx, DWORD PTR $T362977[ebp]
  000f9	e8 00 00 00 00	 call	 ??0CParseConstant@HCParser@@QAE@PB_WVCParseValue@1@@Z ; HCParser::CParseConstant::CParseConstant
  000fe	89 45 8c	 mov	 DWORD PTR tv179[ebp], eax
  00101	8b 4d 8c	 mov	 ecx, DWORD PTR tv179[ebp]
  00104	89 4d 88	 mov	 DWORD PTR tv181[ebp], ecx
  00107	c6 45 fc 09	 mov	 BYTE PTR __$EHRec$[ebp+8], 9
  0010b	8b 55 88	 mov	 edx, DWORD PTR tv181[ebp]
  0010e	52		 push	 edx
  0010f	b9 20 00 00 00	 mov	 ecx, OFFSET _k_parseCarrierConstants+32
  00114	e8 00 00 00 00	 call	 ??0CParseConstant@HCParser@@QAE@ABV01@@Z
  00119	c6 45 fc 0b	 mov	 BYTE PTR __$EHRec$[ebp+8], 11 ; 0000000bH
  0011d	8d 4d bc	 lea	 ecx, DWORD PTR $T362977[ebp]
  00120	e8 00 00 00 00	 call	 ??1CParseConstant@HCParser@@QAE@XZ
  00125	c7 45 fc ff ff
	ff ff		 mov	 DWORD PTR __$EHRec$[ebp+8], -1
  0012c	68 00 00 00 00	 push	 OFFSET ??__Fk_parseCarrierConstants@@YAXXZ ; `dynamic atexit destructor for 'k_parseCarrierConstants''
  00131	e8 00 00 00 00	 call	 _atexit
  00136	83 c4 04	 add	 esp, 4
  00139	8b 4d f4	 mov	 ecx, DWORD PTR __$EHRec$[ebp]
  0013c	64 89 0d 00 00
	00 00		 mov	 DWORD PTR fs:0, ecx
  00143	59		 pop	 ecx
  00144	8b e5		 mov	 esp, ebp
  00146	5d		 pop	 ebp
  00147	c3		 ret	 0
text$yc	ENDS
;	COMDAT text$x
text$x	SEGMENT
__unwindfunclet$??__Ek_parseCarrierConstants@@YAXXZ$0:
  00000	8b 4d e0	 mov	 ecx, DWORD PTR $T362974[ebp]
  00003	e9 00 00 00 00	 jmp	 ??1CParseValue@HCParser@@UAE@XZ ; HCParser::CParseValue::~CParseValue
__unwindfunclet$??__Ek_parseCarrierConstants@@YAXXZ$1:
  00008	8d 4d e4	 lea	 ecx, DWORD PTR $T362973[ebp]
  0000b	e9 00 00 00 00	 jmp	 ??1CParseConstant@HCParser@@QAE@XZ
__unwindfunclet$??__Ek_parseCarrierConstants@@YAXXZ$2:
  00010	b9 00 00 00 00	 mov	 ecx, OFFSET _k_parseCarrierConstants
  00015	e9 00 00 00 00	 jmp	 ??1CParseConstant@HCParser@@QAE@XZ
__unwindfunclet$??__Ek_parseCarrierConstants@@YAXXZ$3:
  0001a	8b 4d cc	 mov	 ecx, DWORD PTR $T362976[ebp]
  0001d	e9 00 00 00 00	 jmp	 ??1CParseValue@HCParser@@UAE@XZ ; HCParser::CParseValue::~CParseValue
__unwindfunclet$??__Ek_parseCarrierConstants@@YAXXZ$4:
  00022	8d 4d d0	 lea	 ecx, DWORD PTR $T362975[ebp]
  00025	e9 00 00 00 00	 jmp	 ??1CParseConstant@HCParser@@QAE@XZ
__unwindfunclet$??__Ek_parseCarrierConstants@@YAXXZ$5:
  0002a	b9 10 00 00 00	 mov	 ecx, OFFSET _k_parseCarrierConstants+16
  0002f	e9 00 00 00 00	 jmp	 ??1CParseConstant@HCParser@@QAE@XZ
__unwindfunclet$??__Ek_parseCarrierConstants@@YAXXZ$6:
  00034	8b 4d b8	 mov	 ecx, DWORD PTR $T362978[ebp]
  00037	e9 00 00 00 00	 jmp	 ??1CParseValue@HCParser@@UAE@XZ ; HCParser::CParseValue::~CParseValue
__unwindfunclet$??__Ek_parseCarrierConstants@@YAXXZ$7:
  0003c	8d 4d bc	 lea	 ecx, DWORD PTR $T362977[ebp]
  0003f	e9 00 00 00 00	 jmp	 ??1CParseConstant@HCParser@@QAE@XZ
__unwindfunclet$??__Ek_parseCarrierConstants@@YAXXZ$8:
  00044	b9 20 00 00 00	 mov	 ecx, OFFSET _k_parseCarrierConstants+32
  00049	e9 00 00 00 00	 jmp	 ??1CParseConstant@HCParser@@QAE@XZ
__ehhandler$??__Ek_parseCarrierConstants@@YAXXZ:
  0004e	8b 54 24 08	 mov	 edx, DWORD PTR [esp+8]
  00052	8d 42 0c	 lea	 eax, DWORD PTR [edx+12]
  00055	8b 4a 90	 mov	 ecx, DWORD PTR [edx-112]
  00058	33 c8		 xor	 ecx, eax
  0005a	e8 00 00 00 00	 call	 @__security_check_cookie@4
  0005f	b8 00 00 00 00	 mov	 eax, OFFSET __ehfuncinfo$??__Ek_parseCarrierConstants@@YAXXZ
  00064	e9 00 00 00 00	 jmp	 ___CxxFrameHandler3
text$x	ENDS
??__Ek_parseCarrierConstants@@YAXXZ ENDP		; `dynamic initializer for 'k_parseCarrierConstants''
;	COMDAT xdata$x
xdata$x	SEGMENT
__unwindtable$??__Ek_parseYesNoConstants@@YAXXZ DD 0ffffffffH
	DD	FLAT:__unwindfunclet$??__Ek_parseYesNoConstants@@YAXXZ$0
	DD	0ffffffffH
	DD	FLAT:__unwindfunclet$??__Ek_parseYesNoConstants@@YAXXZ$1
	DD	01H
	DD	FLAT:__unwindfunclet$??__Ek_parseYesNoConstants@@YAXXZ$2
	DD	0ffffffffH
	DD	FLAT:__unwindfunclet$??__Ek_parseYesNoConstants@@YAXXZ$2
	DD	03H
	DD	FLAT:__unwindfunclet$??__Ek_parseYesNoConstants@@YAXXZ$3
	DD	03H
	DD	FLAT:__unwindfunclet$??__Ek_parseYesNoConstants@@YAXXZ$4
	DD	05H
	DD	FLAT:__unwindfunclet$??__Ek_parseYesNoConstants@@YAXXZ$5
	DD	03H
	DD	FLAT:__unwindfunclet$??__Ek_parseYesNoConstants@@YAXXZ$5
	DD	07H
	DD	FLAT:__unwindfunclet$??__Ek_parseYesNoConstants@@YAXXZ$6
	DD	07H
	DD	FLAT:__unwindfunclet$??__Ek_parseYesNoConstants@@YAXXZ$7
	DD	09H
	DD	FLAT:__unwindfunclet$??__Ek_parseYesNoConstants@@YAXXZ$8
	DD	07H
	DD	FLAT:__unwindfunclet$??__Ek_parseYesNoConstants@@YAXXZ$8
	DD	0bH
	DD	FLAT:__unwindfunclet$??__Ek_parseYesNoConstants@@YAXXZ$9
	DD	0bH
	DD	FLAT:__unwindfunclet$??__Ek_parseYesNoConstants@@YAXXZ$10
	DD	0dH
	DD	FLAT:__unwindfunclet$??__Ek_parseYesNoConstants@@YAXXZ$11
	DD	0bH
	DD	FLAT:__unwindfunclet$??__Ek_parseYesNoConstants@@YAXXZ$11
	DD	0fH
	DD	FLAT:__unwindfunclet$??__Ek_parseYesNoConstants@@YAXXZ$12
	DD	0fH
	DD	FLAT:__unwindfunclet$??__Ek_parseYesNoConstants@@YAXXZ$13
	DD	011H
	DD	FLAT:__unwindfunclet$??__Ek_parseYesNoConstants@@YAXXZ$14
	DD	0fH
	DD	FLAT:__unwindfunclet$??__Ek_parseYesNoConstants@@YAXXZ$14
	DD	013H
	DD	FLAT:__unwindfunclet$??__Ek_parseYesNoConstants@@YAXXZ$15
	DD	013H
	DD	FLAT:__unwindfunclet$??__Ek_parseYesNoConstants@@YAXXZ$16
	DD	015H
	DD	FLAT:__unwindfunclet$??__Ek_parseYesNoConstants@@YAXXZ$17
	DD	013H
	DD	FLAT:__unwindfunclet$??__Ek_parseYesNoConstants@@YAXXZ$17
	DD	017H
	DD	FLAT:__unwindfunclet$??__Ek_parseYesNoConstants@@YAXXZ$18
	DD	017H
	DD	FLAT:__unwindfunclet$??__Ek_parseYesNoConstants@@YAXXZ$19
	DD	019H
	DD	FLAT:__unwindfunclet$??__Ek_parseYesNoConstants@@YAXXZ$20
	DD	017H
	DD	FLAT:__unwindfunclet$??__Ek_parseYesNoConstants@@YAXXZ$20
	DD	01bH
	DD	FLAT:__unwindfunclet$??__Ek_parseYesNoConstants@@YAXXZ$21
	DD	01bH
	DD	FLAT:__unwindfunclet$??__Ek_parseYesNoConstants@@YAXXZ$22
	DD	01dH
	DD	FLAT:__unwindfunclet$??__Ek_parseYesNoConstants@@YAXXZ$23
	DD	01bH
	DD	FLAT:__unwindfunclet$??__Ek_parseYesNoConstants@@YAXXZ$23
	DD	01fH
	DD	FLAT:__unwindfunclet$??__Ek_parseYesNoConstants@@YAXXZ$24
	DD	01fH
	DD	FLAT:__unwindfunclet$??__Ek_parseYesNoConstants@@YAXXZ$25
	DD	021H
	DD	FLAT:__unwindfunclet$??__Ek_parseYesNoConstants@@YAXXZ$26
	DD	01fH
	DD	FLAT:__unwindfunclet$??__Ek_parseYesNoConstants@@YAXXZ$26
__ehfuncinfo$??__Ek_parseYesNoConstants@@YAXXZ DD 019930522H
	DD	024H
	DD	FLAT:__unwindtable$??__Ek_parseYesNoConstants@@YAXXZ
	DD	2 DUP(00H)
	DD	2 DUP(00H)
	DD	00H
	DD	00H
; Function compile flags: /Odtp
xdata$x	ENDS
;	COMDAT ??__Ek_parseYesNoConstants@@YAXXZ
text$yc	SEGMENT
tv355 = -336						; size = 4
tv353 = -332						; size = 4
tv352 = -328						; size = 4
tv258 = -324						; size = 4
tv349 = -320						; size = 4
tv347 = -316						; size = 4
tv346 = -312						; size = 4
tv235 = -308						; size = 4
tv343 = -304						; size = 4
tv341 = -300						; size = 4
tv340 = -296						; size = 4
tv212 = -292						; size = 4
tv337 = -288						; size = 4
tv335 = -284						; size = 4
tv334 = -280						; size = 4
tv189 = -276						; size = 4
tv331 = -272						; size = 4
tv329 = -268						; size = 4
tv328 = -264						; size = 4
tv166 = -260						; size = 4
tv325 = -256						; size = 4
tv323 = -252						; size = 4
tv322 = -248						; size = 4
tv143 = -244						; size = 4
tv319 = -240						; size = 4
tv317 = -236						; size = 4
tv316 = -232						; size = 4
tv88 = -228						; size = 4
tv313 = -224						; size = 4
tv311 = -220						; size = 4
tv310 = -216						; size = 4
tv65 = -212						; size = 4
tv307 = -208						; size = 4
tv305 = -204						; size = 4
tv304 = -200						; size = 4
tv357 = -196						; size = 4
$T363013 = -192						; size = 4
$T363012 = -188						; size = 16
$T363011 = -172						; size = 4
$T363010 = -168						; size = 16
$T363009 = -152						; size = 4
$T363008 = -148						; size = 16
$T363007 = -132						; size = 4
$T363006 = -128						; size = 16
$T363005 = -112						; size = 4
$T363004 = -108						; size = 16
$T363003 = -92						; size = 4
$T363002 = -88						; size = 16
$T363001 = -72						; size = 4
$T363000 = -68						; size = 16
$T362999 = -52						; size = 4
$T362998 = -48						; size = 16
$T362997 = -32						; size = 4
$T362996 = -28						; size = 16
__$EHRec$ = -12						; size = 12
??__Ek_parseYesNoConstants@@YAXXZ PROC			; `dynamic initializer for 'k_parseYesNoConstants'', COMDAT

; 132  : {

  00000	55		 push	 ebp
  00001	8b ec		 mov	 ebp, esp
  00003	6a ff		 push	 -1
  00005	68 00 00 00 00	 push	 __ehhandler$??__Ek_parseYesNoConstants@@YAXXZ
  0000a	64 a1 00 00 00
	00		 mov	 eax, DWORD PTR fs:0
  00010	50		 push	 eax
  00011	81 ec 44 01 00
	00		 sub	 esp, 324		; 00000144H
  00017	a1 00 00 00 00	 mov	 eax, DWORD PTR ___security_cookie
  0001c	33 c5		 xor	 eax, ebp
  0001e	50		 push	 eax
  0001f	8d 45 f4	 lea	 eax, DWORD PTR __$EHRec$[ebp]
  00022	64 a3 00 00 00
	00		 mov	 DWORD PTR fs:0, eax

; 133  :     PC( _T("yes"),                        1 ),

  00028	83 ec 0c	 sub	 esp, 12			; 0000000cH
  0002b	8b cc		 mov	 ecx, esp
  0002d	89 65 e0	 mov	 DWORD PTR $T362997[ebp], esp
  00030	6a 01		 push	 1
  00032	e8 00 00 00 00	 call	 ??0CParseValue@HCParser@@QAE@H@Z ; HCParser::CParseValue::CParseValue
  00037	89 85 3c ff ff
	ff		 mov	 DWORD PTR tv357[ebp], eax
  0003d	8b 85 3c ff ff
	ff		 mov	 eax, DWORD PTR tv357[ebp]
  00043	89 85 38 ff ff
	ff		 mov	 DWORD PTR tv304[ebp], eax
  00049	c7 45 fc 00 00
	00 00		 mov	 DWORD PTR __$EHRec$[ebp+8], 0
  00050	68 00 00 00 00	 push	 OFFSET ??_C@_17IHBDLLG@?$AAy?$AAe?$AAs?$AA?$AA@
  00055	c7 45 fc ff ff
	ff ff		 mov	 DWORD PTR __$EHRec$[ebp+8], -1
  0005c	8d 4d e4	 lea	 ecx, DWORD PTR $T362996[ebp]
  0005f	e8 00 00 00 00	 call	 ??0CParseConstant@HCParser@@QAE@PB_WVCParseValue@1@@Z ; HCParser::CParseConstant::CParseConstant
  00064	89 85 34 ff ff
	ff		 mov	 DWORD PTR tv305[ebp], eax
  0006a	8b 8d 34 ff ff
	ff		 mov	 ecx, DWORD PTR tv305[ebp]
  00070	89 8d 30 ff ff
	ff		 mov	 DWORD PTR tv307[ebp], ecx
  00076	c7 45 fc 01 00
	00 00		 mov	 DWORD PTR __$EHRec$[ebp+8], 1
  0007d	8b 95 30 ff ff
	ff		 mov	 edx, DWORD PTR tv307[ebp]
  00083	52		 push	 edx
  00084	b9 00 00 00 00	 mov	 ecx, OFFSET _k_parseYesNoConstants
  00089	e8 00 00 00 00	 call	 ??0CParseConstant@HCParser@@QAE@ABV01@@Z
  0008e	c6 45 fc 03	 mov	 BYTE PTR __$EHRec$[ebp+8], 3
  00092	8d 4d e4	 lea	 ecx, DWORD PTR $T362996[ebp]
  00095	e8 00 00 00 00	 call	 ??1CParseConstant@HCParser@@QAE@XZ

; 134  :     PC( _T("no"),                        0 ),

  0009a	83 ec 0c	 sub	 esp, 12			; 0000000cH
  0009d	8b cc		 mov	 ecx, esp
  0009f	89 65 cc	 mov	 DWORD PTR $T362999[ebp], esp
  000a2	6a 00		 push	 0
  000a4	e8 00 00 00 00	 call	 ??0CParseValue@HCParser@@QAE@H@Z ; HCParser::CParseValue::CParseValue
  000a9	89 85 2c ff ff
	ff		 mov	 DWORD PTR tv65[ebp], eax
  000af	8b 85 2c ff ff
	ff		 mov	 eax, DWORD PTR tv65[ebp]
  000b5	89 85 28 ff ff
	ff		 mov	 DWORD PTR tv310[ebp], eax
  000bb	c6 45 fc 04	 mov	 BYTE PTR __$EHRec$[ebp+8], 4
  000bf	68 00 00 00 00	 push	 OFFSET ??_C@_15BPIGNHCD@?$AAn?$AAo?$AA?$AA@
  000c4	c6 45 fc 03	 mov	 BYTE PTR __$EHRec$[ebp+8], 3
  000c8	8d 4d d0	 lea	 ecx, DWORD PTR $T362998[ebp]
  000cb	e8 00 00 00 00	 call	 ??0CParseConstant@HCParser@@QAE@PB_WVCParseValue@1@@Z ; HCParser::CParseConstant::CParseConstant
  000d0	89 85 24 ff ff
	ff		 mov	 DWORD PTR tv311[ebp], eax
  000d6	8b 8d 24 ff ff
	ff		 mov	 ecx, DWORD PTR tv311[ebp]
  000dc	89 8d 20 ff ff
	ff		 mov	 DWORD PTR tv313[ebp], ecx
  000e2	c6 45 fc 05	 mov	 BYTE PTR __$EHRec$[ebp+8], 5
  000e6	8b 95 20 ff ff
	ff		 mov	 edx, DWORD PTR tv313[ebp]
  000ec	52		 push	 edx
  000ed	b9 10 00 00 00	 mov	 ecx, OFFSET _k_parseYesNoConstants+16
  000f2	e8 00 00 00 00	 call	 ??0CParseConstant@HCParser@@QAE@ABV01@@Z
  000f7	c6 45 fc 07	 mov	 BYTE PTR __$EHRec$[ebp+8], 7
  000fb	8d 4d d0	 lea	 ecx, DWORD PTR $T362998[ebp]
  000fe	e8 00 00 00 00	 call	 ??1CParseConstant@HCParser@@QAE@XZ

; 135  :     PC( _T("TRUE"),                        1 ),

  00103	83 ec 0c	 sub	 esp, 12			; 0000000cH
  00106	8b cc		 mov	 ecx, esp
  00108	89 65 b8	 mov	 DWORD PTR $T363001[ebp], esp
  0010b	6a 01		 push	 1
  0010d	e8 00 00 00 00	 call	 ??0CParseValue@HCParser@@QAE@H@Z ; HCParser::CParseValue::CParseValue
  00112	89 85 1c ff ff
	ff		 mov	 DWORD PTR tv88[ebp], eax
  00118	8b 85 1c ff ff
	ff		 mov	 eax, DWORD PTR tv88[ebp]
  0011e	89 85 18 ff ff
	ff		 mov	 DWORD PTR tv316[ebp], eax
  00124	c6 45 fc 08	 mov	 BYTE PTR __$EHRec$[ebp+8], 8
  00128	68 00 00 00 00	 push	 OFFSET ??_C@_19ELAAHEEL@?$AAT?$AAR?$AAU?$AAE?$AA?$AA@
  0012d	c6 45 fc 07	 mov	 BYTE PTR __$EHRec$[ebp+8], 7
  00131	8d 4d bc	 lea	 ecx, DWORD PTR $T363000[ebp]
  00134	e8 00 00 00 00	 call	 ??0CParseConstant@HCParser@@QAE@PB_WVCParseValue@1@@Z ; HCParser::CParseConstant::CParseConstant
  00139	89 85 14 ff ff
	ff		 mov	 DWORD PTR tv317[ebp], eax
  0013f	8b 8d 14 ff ff
	ff		 mov	 ecx, DWORD PTR tv317[ebp]
  00145	89 8d 10 ff ff
	ff		 mov	 DWORD PTR tv319[ebp], ecx
  0014b	c6 45 fc 09	 mov	 BYTE PTR __$EHRec$[ebp+8], 9
  0014f	8b 95 10 ff ff
	ff		 mov	 edx, DWORD PTR tv319[ebp]
  00155	52		 push	 edx
  00156	b9 20 00 00 00	 mov	 ecx, OFFSET _k_parseYesNoConstants+32
  0015b	e8 00 00 00 00	 call	 ??0CParseConstant@HCParser@@QAE@ABV01@@Z
  00160	c6 45 fc 0b	 mov	 BYTE PTR __$EHRec$[ebp+8], 11 ; 0000000bH
  00164	8d 4d bc	 lea	 ecx, DWORD PTR $T363000[ebp]
  00167	e8 00 00 00 00	 call	 ??1CParseConstant@HCParser@@QAE@XZ

; 136  :     PC( _T("FALSE"),                    0 ),

  0016c	83 ec 0c	 sub	 esp, 12			; 0000000cH
  0016f	8b cc		 mov	 ecx, esp
  00171	89 65 a4	 mov	 DWORD PTR $T363003[ebp], esp
  00174	6a 00		 push	 0
  00176	e8 00 00 00 00	 call	 ??0CParseValue@HCParser@@QAE@H@Z ; HCParser::CParseValue::CParseValue
  0017b	89 85 0c ff ff
	ff		 mov	 DWORD PTR tv143[ebp], eax
  00181	8b 85 0c ff ff
	ff		 mov	 eax, DWORD PTR tv143[ebp]
  00187	89 85 08 ff ff
	ff		 mov	 DWORD PTR tv322[ebp], eax
  0018d	c6 45 fc 0c	 mov	 BYTE PTR __$EHRec$[ebp+8], 12 ; 0000000cH
  00191	68 00 00 00 00	 push	 OFFSET ??_C@_1M@HCOOECOK@?$AAF?$AAA?$AAL?$AAS?$AAE?$AA?$AA@
  00196	c6 45 fc 0b	 mov	 BYTE PTR __$EHRec$[ebp+8], 11 ; 0000000bH
  0019a	8d 4d a8	 lea	 ecx, DWORD PTR $T363002[ebp]
  0019d	e8 00 00 00 00	 call	 ??0CParseConstant@HCParser@@QAE@PB_WVCParseValue@1@@Z ; HCParser::CParseConstant::CParseConstant
  001a2	89 85 04 ff ff
	ff		 mov	 DWORD PTR tv323[ebp], eax
  001a8	8b 8d 04 ff ff
	ff		 mov	 ecx, DWORD PTR tv323[ebp]
  001ae	89 8d 00 ff ff
	ff		 mov	 DWORD PTR tv325[ebp], ecx
  001b4	c6 45 fc 0d	 mov	 BYTE PTR __$EHRec$[ebp+8], 13 ; 0000000dH
  001b8	8b 95 00 ff ff
	ff		 mov	 edx, DWORD PTR tv325[ebp]
  001be	52		 push	 edx
  001bf	b9 30 00 00 00	 mov	 ecx, OFFSET _k_parseYesNoConstants+48
  001c4	e8 00 00 00 00	 call	 ??0CParseConstant@HCParser@@QAE@ABV01@@Z
  001c9	c6 45 fc 0f	 mov	 BYTE PTR __$EHRec$[ebp+8], 15 ; 0000000fH
  001cd	8d 4d a8	 lea	 ecx, DWORD PTR $T363002[ebp]
  001d0	e8 00 00 00 00	 call	 ??1CParseConstant@HCParser@@QAE@XZ

; 137  :     PC( _T("active"),                    1 ),

  001d5	83 ec 0c	 sub	 esp, 12			; 0000000cH
  001d8	8b cc		 mov	 ecx, esp
  001da	89 65 90	 mov	 DWORD PTR $T363005[ebp], esp
  001dd	6a 01		 push	 1
  001df	e8 00 00 00 00	 call	 ??0CParseValue@HCParser@@QAE@H@Z ; HCParser::CParseValue::CParseValue
  001e4	89 85 fc fe ff
	ff		 mov	 DWORD PTR tv166[ebp], eax
  001ea	8b 85 fc fe ff
	ff		 mov	 eax, DWORD PTR tv166[ebp]
  001f0	89 85 f8 fe ff
	ff		 mov	 DWORD PTR tv328[ebp], eax
  001f6	c6 45 fc 10	 mov	 BYTE PTR __$EHRec$[ebp+8], 16 ; 00000010H
  001fa	68 00 00 00 00	 push	 OFFSET ??_C@_1O@IBNPCBAA@?$AAa?$AAc?$AAt?$AAi?$AAv?$AAe?$AA?$AA@
  001ff	c6 45 fc 0f	 mov	 BYTE PTR __$EHRec$[ebp+8], 15 ; 0000000fH
  00203	8d 4d 94	 lea	 ecx, DWORD PTR $T363004[ebp]
  00206	e8 00 00 00 00	 call	 ??0CParseConstant@HCParser@@QAE@PB_WVCParseValue@1@@Z ; HCParser::CParseConstant::CParseConstant
  0020b	89 85 f4 fe ff
	ff		 mov	 DWORD PTR tv329[ebp], eax
  00211	8b 8d f4 fe ff
	ff		 mov	 ecx, DWORD PTR tv329[ebp]
  00217	89 8d f0 fe ff
	ff		 mov	 DWORD PTR tv331[ebp], ecx
  0021d	c6 45 fc 11	 mov	 BYTE PTR __$EHRec$[ebp+8], 17 ; 00000011H
  00221	8b 95 f0 fe ff
	ff		 mov	 edx, DWORD PTR tv331[ebp]
  00227	52		 push	 edx
  00228	b9 40 00 00 00	 mov	 ecx, OFFSET _k_parseYesNoConstants+64
  0022d	e8 00 00 00 00	 call	 ??0CParseConstant@HCParser@@QAE@ABV01@@Z
  00232	c6 45 fc 13	 mov	 BYTE PTR __$EHRec$[ebp+8], 19 ; 00000013H
  00236	8d 4d 94	 lea	 ecx, DWORD PTR $T363004[ebp]
  00239	e8 00 00 00 00	 call	 ??1CParseConstant@HCParser@@QAE@XZ

; 138  :     PC( _T("inactive"),                    0 ),

  0023e	83 ec 0c	 sub	 esp, 12			; 0000000cH
  00241	8b cc		 mov	 ecx, esp
  00243	89 a5 7c ff ff
	ff		 mov	 DWORD PTR $T363007[ebp], esp
  00249	6a 00		 push	 0
  0024b	e8 00 00 00 00	 call	 ??0CParseValue@HCParser@@QAE@H@Z ; HCParser::CParseValue::CParseValue
  00250	89 85 ec fe ff
	ff		 mov	 DWORD PTR tv189[ebp], eax
  00256	8b 85 ec fe ff
	ff		 mov	 eax, DWORD PTR tv189[ebp]
  0025c	89 85 e8 fe ff
	ff		 mov	 DWORD PTR tv334[ebp], eax
  00262	c6 45 fc 14	 mov	 BYTE PTR __$EHRec$[ebp+8], 20 ; 00000014H
  00266	68 00 00 00 00	 push	 OFFSET ??_C@_1BC@DBHEDMBL@?$AAi?$AAn?$AAa?$AAc?$AAt?$AAi?$AAv?$AAe?$AA?$AA@
  0026b	c6 45 fc 13	 mov	 BYTE PTR __$EHRec$[ebp+8], 19 ; 00000013H
  0026f	8d 4d 80	 lea	 ecx, DWORD PTR $T363006[ebp]
  00272	e8 00 00 00 00	 call	 ??0CParseConstant@HCParser@@QAE@PB_WVCParseValue@1@@Z ; HCParser::CParseConstant::CParseConstant
  00277	89 85 e4 fe ff
	ff		 mov	 DWORD PTR tv335[ebp], eax
  0027d	8b 8d e4 fe ff
	ff		 mov	 ecx, DWORD PTR tv335[ebp]
  00283	89 8d e0 fe ff
	ff		 mov	 DWORD PTR tv337[ebp], ecx
  00289	c6 45 fc 15	 mov	 BYTE PTR __$EHRec$[ebp+8], 21 ; 00000015H
  0028d	8b 95 e0 fe ff
	ff		 mov	 edx, DWORD PTR tv337[ebp]
  00293	52		 push	 edx
  00294	b9 50 00 00 00	 mov	 ecx, OFFSET _k_parseYesNoConstants+80
  00299	e8 00 00 00 00	 call	 ??0CParseConstant@HCParser@@QAE@ABV01@@Z
  0029e	c6 45 fc 17	 mov	 BYTE PTR __$EHRec$[ebp+8], 23 ; 00000017H
  002a2	8d 4d 80	 lea	 ecx, DWORD PTR $T363006[ebp]
  002a5	e8 00 00 00 00	 call	 ??1CParseConstant@HCParser@@QAE@XZ

; 139  :     PC( _T("1"),                        1 ),

  002aa	83 ec 0c	 sub	 esp, 12			; 0000000cH
  002ad	8b cc		 mov	 ecx, esp
  002af	89 a5 68 ff ff
	ff		 mov	 DWORD PTR $T363009[ebp], esp
  002b5	6a 01		 push	 1
  002b7	e8 00 00 00 00	 call	 ??0CParseValue@HCParser@@QAE@H@Z ; HCParser::CParseValue::CParseValue
  002bc	89 85 dc fe ff
	ff		 mov	 DWORD PTR tv212[ebp], eax
  002c2	8b 85 dc fe ff
	ff		 mov	 eax, DWORD PTR tv212[ebp]
  002c8	89 85 d8 fe ff
	ff		 mov	 DWORD PTR tv340[ebp], eax
  002ce	c6 45 fc 18	 mov	 BYTE PTR __$EHRec$[ebp+8], 24 ; 00000018H
  002d2	68 00 00 00 00	 push	 OFFSET ??_C@_13JGCMLPCH@?$AA1?$AA?$AA@
  002d7	c6 45 fc 17	 mov	 BYTE PTR __$EHRec$[ebp+8], 23 ; 00000017H
  002db	8d 8d 6c ff ff
	ff		 lea	 ecx, DWORD PTR $T363008[ebp]
  002e1	e8 00 00 00 00	 call	 ??0CParseConstant@HCParser@@QAE@PB_WVCParseValue@1@@Z ; HCParser::CParseConstant::CParseConstant
  002e6	89 85 d4 fe ff
	ff		 mov	 DWORD PTR tv341[ebp], eax
  002ec	8b 8d d4 fe ff
	ff		 mov	 ecx, DWORD PTR tv341[ebp]
  002f2	89 8d d0 fe ff
	ff		 mov	 DWORD PTR tv343[ebp], ecx
  002f8	c6 45 fc 19	 mov	 BYTE PTR __$EHRec$[ebp+8], 25 ; 00000019H
  002fc	8b 95 d0 fe ff
	ff		 mov	 edx, DWORD PTR tv343[ebp]
  00302	52		 push	 edx
  00303	b9 60 00 00 00	 mov	 ecx, OFFSET _k_parseYesNoConstants+96
  00308	e8 00 00 00 00	 call	 ??0CParseConstant@HCParser@@QAE@ABV01@@Z
  0030d	c6 45 fc 1b	 mov	 BYTE PTR __$EHRec$[ebp+8], 27 ; 0000001bH
  00311	8d 8d 6c ff ff
	ff		 lea	 ecx, DWORD PTR $T363008[ebp]
  00317	e8 00 00 00 00	 call	 ??1CParseConstant@HCParser@@QAE@XZ

; 140  :     PC( _T("0"),                        0 ),

  0031c	83 ec 0c	 sub	 esp, 12			; 0000000cH
  0031f	8b cc		 mov	 ecx, esp
  00321	89 a5 54 ff ff
	ff		 mov	 DWORD PTR $T363011[ebp], esp
  00327	6a 00		 push	 0
  00329	e8 00 00 00 00	 call	 ??0CParseValue@HCParser@@QAE@H@Z ; HCParser::CParseValue::CParseValue
  0032e	89 85 cc fe ff
	ff		 mov	 DWORD PTR tv235[ebp], eax
  00334	8b 85 cc fe ff
	ff		 mov	 eax, DWORD PTR tv235[ebp]
  0033a	89 85 c8 fe ff
	ff		 mov	 DWORD PTR tv346[ebp], eax
  00340	c6 45 fc 1c	 mov	 BYTE PTR __$EHRec$[ebp+8], 28 ; 0000001cH
  00344	68 00 00 00 00	 push	 OFFSET ??_C@_13COJANIEC@?$AA0?$AA?$AA@
  00349	c6 45 fc 1b	 mov	 BYTE PTR __$EHRec$[ebp+8], 27 ; 0000001bH
  0034d	8d 8d 58 ff ff
	ff		 lea	 ecx, DWORD PTR $T363010[ebp]
  00353	e8 00 00 00 00	 call	 ??0CParseConstant@HCParser@@QAE@PB_WVCParseValue@1@@Z ; HCParser::CParseConstant::CParseConstant
  00358	89 85 c4 fe ff
	ff		 mov	 DWORD PTR tv347[ebp], eax
  0035e	8b 8d c4 fe ff
	ff		 mov	 ecx, DWORD PTR tv347[ebp]
  00364	89 8d c0 fe ff
	ff		 mov	 DWORD PTR tv349[ebp], ecx
  0036a	c6 45 fc 1d	 mov	 BYTE PTR __$EHRec$[ebp+8], 29 ; 0000001dH
  0036e	8b 95 c0 fe ff
	ff		 mov	 edx, DWORD PTR tv349[ebp]
  00374	52		 push	 edx
  00375	b9 70 00 00 00	 mov	 ecx, OFFSET _k_parseYesNoConstants+112
  0037a	e8 00 00 00 00	 call	 ??0CParseConstant@HCParser@@QAE@ABV01@@Z
  0037f	c6 45 fc 1f	 mov	 BYTE PTR __$EHRec$[ebp+8], 31 ; 0000001fH
  00383	8d 8d 58 ff ff
	ff		 lea	 ecx, DWORD PTR $T363010[ebp]
  00389	e8 00 00 00 00	 call	 ??1CParseConstant@HCParser@@QAE@XZ

; 141  :     PC( NULL )
; 142  : };

  0038e	83 ec 0c	 sub	 esp, 12			; 0000000cH
  00391	8b cc		 mov	 ecx, esp
  00393	89 a5 40 ff ff
	ff		 mov	 DWORD PTR $T363013[ebp], esp
  00399	e8 00 00 00 00	 call	 ??0CParseValue@HCParser@@QAE@XZ ; HCParser::CParseValue::CParseValue
  0039e	89 85 bc fe ff
	ff		 mov	 DWORD PTR tv258[ebp], eax
  003a4	8b 85 bc fe ff
	ff		 mov	 eax, DWORD PTR tv258[ebp]
  003aa	89 85 b8 fe ff
	ff		 mov	 DWORD PTR tv352[ebp], eax
  003b0	c6 45 fc 20	 mov	 BYTE PTR __$EHRec$[ebp+8], 32 ; 00000020H
  003b4	6a 00		 push	 0
  003b6	c6 45 fc 1f	 mov	 BYTE PTR __$EHRec$[ebp+8], 31 ; 0000001fH
  003ba	8d 8d 44 ff ff
	ff		 lea	 ecx, DWORD PTR $T363012[ebp]
  003c0	e8 00 00 00 00	 call	 ??0CParseConstant@HCParser@@QAE@PB_WVCParseValue@1@@Z ; HCParser::CParseConstant::CParseConstant
  003c5	89 85 b4 fe ff
	ff		 mov	 DWORD PTR tv353[ebp], eax
  003cb	8b 8d b4 fe ff
	ff		 mov	 ecx, DWORD PTR tv353[ebp]
  003d1	89 8d b0 fe ff
	ff		 mov	 DWORD PTR tv355[ebp], ecx
  003d7	c6 45 fc 21	 mov	 BYTE PTR __$EHRec$[ebp+8], 33 ; 00000021H
  003db	8b 95 b0 fe ff
	ff		 mov	 edx, DWORD PTR tv355[ebp]
  003e1	52		 push	 edx
  003e2	b9 80 00 00 00	 mov	 ecx, OFFSET _k_parseYesNoConstants+128
  003e7	e8 00 00 00 00	 call	 ??0CParseConstant@HCParser@@QAE@ABV01@@Z
  003ec	c6 45 fc 23	 mov	 BYTE PTR __$EHRec$[ebp+8], 35 ; 00000023H
  003f0	8d 8d 44 ff ff
	ff		 lea	 ecx, DWORD PTR $T363012[ebp]
  003f6	e8 00 00 00 00	 call	 ??1CParseConstant@HCParser@@QAE@XZ
  003fb	c7 45 fc ff ff
	ff ff		 mov	 DWORD PTR __$EHRec$[ebp+8], -1
  00402	68 00 00 00 00	 push	 OFFSET ??__Fk_parseYesNoConstants@@YAXXZ ; `dynamic atexit destructor for 'k_parseYesNoConstants''
  00407	e8 00 00 00 00	 call	 _atexit
  0040c	83 c4 04	 add	 esp, 4
  0040f	8b 4d f4	 mov	 ecx, DWORD PTR __$EHRec$[ebp]
  00412	64 89 0d 00 00
	00 00		 mov	 DWORD PTR fs:0, ecx
  00419	59		 pop	 ecx
  0041a	8b e5		 mov	 esp, ebp
  0041c	5d		 pop	 ebp
  0041d	c3		 ret	 0
text$yc	ENDS
;	COMDAT text$x
text$x	SEGMENT
__unwindfunclet$??__Ek_parseYesNoConstants@@YAXXZ$0:
  00000	8b 4d e0	 mov	 ecx, DWORD PTR $T362997[ebp]
  00003	e9 00 00 00 00	 jmp	 ??1CParseValue@HCParser@@UAE@XZ ; HCParser::CParseValue::~CParseValue
__unwindfunclet$??__Ek_parseYesNoConstants@@YAXXZ$1:
  00008	8d 4d e4	 lea	 ecx, DWORD PTR $T362996[ebp]
  0000b	e9 00 00 00 00	 jmp	 ??1CParseConstant@HCParser@@QAE@XZ
__unwindfunclet$??__Ek_parseYesNoConstants@@YAXXZ$2:
  00010	b9 00 00 00 00	 mov	 ecx, OFFSET _k_parseYesNoConstants
  00015	e9 00 00 00 00	 jmp	 ??1CParseConstant@HCParser@@QAE@XZ
__unwindfunclet$??__Ek_parseYesNoConstants@@YAXXZ$3:
  0001a	8b 4d cc	 mov	 ecx, DWORD PTR $T362999[ebp]
  0001d	e9 00 00 00 00	 jmp	 ??1CParseValue@HCParser@@UAE@XZ ; HCParser::CParseValue::~CParseValue
__unwindfunclet$??__Ek_parseYesNoConstants@@YAXXZ$4:
  00022	8d 4d d0	 lea	 ecx, DWORD PTR $T362998[ebp]
  00025	e9 00 00 00 00	 jmp	 ??1CParseConstant@HCParser@@QAE@XZ
__unwindfunclet$??__Ek_parseYesNoConstants@@YAXXZ$5:
  0002a	b9 10 00 00 00	 mov	 ecx, OFFSET _k_parseYesNoConstants+16
  0002f	e9 00 00 00 00	 jmp	 ??1CParseConstant@HCParser@@QAE@XZ
__unwindfunclet$??__Ek_parseYesNoConstants@@YAXXZ$6:
  00034	8b 4d b8	 mov	 ecx, DWORD PTR $T363001[ebp]
  00037	e9 00 00 00 00	 jmp	 ??1CParseValue@HCParser@@UAE@XZ ; HCParser::CParseValue::~CParseValue
__unwindfunclet$??__Ek_parseYesNoConstants@@YAXXZ$7:
  0003c	8d 4d bc	 lea	 ecx, DWORD PTR $T363000[ebp]
  0003f	e9 00 00 00 00	 jmp	 ??1CParseConstant@HCParser@@QAE@XZ
__unwindfunclet$??__Ek_parseYesNoConstants@@YAXXZ$8:
  00044	b9 20 00 00 00	 mov	 ecx, OFFSET _k_parseYesNoConstants+32
  00049	e9 00 00 00 00	 jmp	 ??1CParseConstant@HCParser@@QAE@XZ
__unwindfunclet$??__Ek_parseYesNoConstants@@YAXXZ$9:
  0004e	8b 4d a4	 mov	 ecx, DWORD PTR $T363003[ebp]
  00051	e9 00 00 00 00	 jmp	 ??1CParseValue@HCParser@@UAE@XZ ; HCParser::CParseValue::~CParseValue
__unwindfunclet$??__Ek_parseYesNoConstants@@YAXXZ$10:
  00056	8d 4d a8	 lea	 ecx, DWORD PTR $T363002[ebp]
  00059	e9 00 00 00 00	 jmp	 ??1CParseConstant@HCParser@@QAE@XZ
__unwindfunclet$??__Ek_parseYesNoConstants@@YAXXZ$11:
  0005e	b9 30 00 00 00	 mov	 ecx, OFFSET _k_parseYesNoConstants+48
  00063	e9 00 00 00 00	 jmp	 ??1CParseConstant@HCParser@@QAE@XZ
__unwindfunclet$??__Ek_parseYesNoConstants@@YAXXZ$12:
  00068	8b 4d 90	 mov	 ecx, DWORD PTR $T363005[ebp]
  0006b	e9 00 00 00 00	 jmp	 ??1CParseValue@HCParser@@UAE@XZ ; HCParser::CParseValue::~CParseValue
__unwindfunclet$??__Ek_parseYesNoConstants@@YAXXZ$13:
  00070	8d 4d 94	 lea	 ecx, DWORD PTR $T363004[ebp]
  00073	e9 00 00 00 00	 jmp	 ??1CParseConstant@HCParser@@QAE@XZ
__unwindfunclet$??__Ek_parseYesNoConstants@@YAXXZ$14:
  00078	b9 40 00 00 00	 mov	 ecx, OFFSET _k_parseYesNoConstants+64
  0007d	e9 00 00 00 00	 jmp	 ??1CParseConstant@HCParser@@QAE@XZ
__unwindfunclet$??__Ek_parseYesNoConstants@@YAXXZ$15:
  00082	8b 8d 7c ff ff
	ff		 mov	 ecx, DWORD PTR $T363007[ebp]
  00088	e9 00 00 00 00	 jmp	 ??1CParseValue@HCParser@@UAE@XZ ; HCParser::CParseValue::~CParseValue
__unwindfunclet$??__Ek_parseYesNoConstants@@YAXXZ$16:
  0008d	8d 4d 80	 lea	 ecx, DWORD PTR $T363006[ebp]
  00090	e9 00 00 00 00	 jmp	 ??1CParseConstant@HCParser@@QAE@XZ
__unwindfunclet$??__Ek_parseYesNoConstants@@YAXXZ$17:
  00095	b9 50 00 00 00	 mov	 ecx, OFFSET _k_parseYesNoConstants+80
  0009a	e9 00 00 00 00	 jmp	 ??1CParseConstant@HCParser@@QAE@XZ
__unwindfunclet$??__Ek_parseYesNoConstants@@YAXXZ$18:
  0009f	8b 8d 68 ff ff
	ff		 mov	 ecx, DWORD PTR $T363009[ebp]
  000a5	e9 00 00 00 00	 jmp	 ??1CParseValue@HCParser@@UAE@XZ ; HCParser::CParseValue::~CParseValue
__unwindfunclet$??__Ek_parseYesNoConstants@@YAXXZ$19:
  000aa	8d 8d 6c ff ff
	ff		 lea	 ecx, DWORD PTR $T363008[ebp]
  000b0	e9 00 00 00 00	 jmp	 ??1CParseConstant@HCParser@@QAE@XZ
__unwindfunclet$??__Ek_parseYesNoConstants@@YAXXZ$20:
  000b5	b9 60 00 00 00	 mov	 ecx, OFFSET _k_parseYesNoConstants+96
  000ba	e9 00 00 00 00	 jmp	 ??1CParseConstant@HCParser@@QAE@XZ
__unwindfunclet$??__Ek_parseYesNoConstants@@YAXXZ$21:
  000bf	8b 8d 54 ff ff
	ff		 mov	 ecx, DWORD PTR $T363011[ebp]
  000c5	e9 00 00 00 00	 jmp	 ??1CParseValue@HCParser@@UAE@XZ ; HCParser::CParseValue::~CParseValue
__unwindfunclet$??__Ek_parseYesNoConstants@@YAXXZ$22:
  000ca	8d 8d 58 ff ff
	ff		 lea	 ecx, DWORD PTR $T363010[ebp]
  000d0	e9 00 00 00 00	 jmp	 ??1CParseConstant@HCParser@@QAE@XZ
__unwindfunclet$??__Ek_parseYesNoConstants@@YAXXZ$23:
  000d5	b9 70 00 00 00	 mov	 ecx, OFFSET _k_parseYesNoConstants+112
  000da	e9 00 00 00 00	 jmp	 ??1CParseConstant@HCParser@@QAE@XZ
__unwindfunclet$??__Ek_parseYesNoConstants@@YAXXZ$24:
  000df	8b 8d 40 ff ff
	ff		 mov	 ecx, DWORD PTR $T363013[ebp]
  000e5	e9 00 00 00 00	 jmp	 ??1CParseValue@HCParser@@UAE@XZ ; HCParser::CParseValue::~CParseValue
__unwindfunclet$??__Ek_parseYesNoConstants@@YAXXZ$25:
  000ea	8d 8d 44 ff ff
	ff		 lea	 ecx, DWORD PTR $T363012[ebp]
  000f0	e9 00 00 00 00	 jmp	 ??1CParseConstant@HCParser@@QAE@XZ
__unwindfunclet$??__Ek_parseYesNoConstants@@YAXXZ$26:
  000f5	b9 80 00 00 00	 mov	 ecx, OFFSET _k_parseYesNoConstants+128
  000fa	e9 00 00 00 00	 jmp	 ??1CParseConstant@HCParser@@QAE@XZ
__ehhandler$??__Ek_parseYesNoConstants@@YAXXZ:
  000ff	8b 54 24 08	 mov	 edx, DWORD PTR [esp+8]
  00103	8d 42 0c	 lea	 eax, DWORD PTR [edx+12]
  00106	8b 8a b8 fe ff
	ff		 mov	 ecx, DWORD PTR [edx-328]
  0010c	33 c8		 xor	 ecx, eax
  0010e	e8 00 00 00 00	 call	 @__security_check_cookie@4
  00113	b8 00 00 00 00	 mov	 eax, OFFSET __ehfuncinfo$??__Ek_parseYesNoConstants@@YAXXZ
  00118	e9 00 00 00 00	 jmp	 ___CxxFrameHandler3
text$x	ENDS
??__Ek_parseYesNoConstants@@YAXXZ ENDP			; `dynamic initializer for 'k_parseYesNoConstants''
;	COMDAT xdata$x
xdata$x	SEGMENT
__unwindtable$??__Ek_parseTakeoverPointConstants@@YAXXZ DD 0ffffffffH
	DD	FLAT:__unwindfunclet$??__Ek_parseTakeoverPointConstants@@YAXXZ$0
	DD	0ffffffffH
	DD	FLAT:__unwindfunclet$??__Ek_parseTakeoverPointConstants@@YAXXZ$1
	DD	01H
	DD	FLAT:__unwindfunclet$??__Ek_parseTakeoverPointConstants@@YAXXZ$2
	DD	0ffffffffH
	DD	FLAT:__unwindfunclet$??__Ek_parseTakeoverPointConstants@@YAXXZ$2
	DD	03H
	DD	FLAT:__unwindfunclet$??__Ek_parseTakeoverPointConstants@@YAXXZ$3
	DD	03H
	DD	FLAT:__unwindfunclet$??__Ek_parseTakeoverPointConstants@@YAXXZ$4
	DD	05H
	DD	FLAT:__unwindfunclet$??__Ek_parseTakeoverPointConstants@@YAXXZ$5
	DD	03H
	DD	FLAT:__unwindfunclet$??__Ek_parseTakeoverPointConstants@@YAXXZ$5
	DD	07H
	DD	FLAT:__unwindfunclet$??__Ek_parseTakeoverPointConstants@@YAXXZ$6
	DD	07H
	DD	FLAT:__unwindfunclet$??__Ek_parseTakeoverPointConstants@@YAXXZ$7
	DD	09H
	DD	FLAT:__unwindfunclet$??__Ek_parseTakeoverPointConstants@@YAXXZ$8
	DD	07H
	DD	FLAT:__unwindfunclet$??__Ek_parseTakeoverPointConstants@@YAXXZ$8
	DD	0bH
	DD	FLAT:__unwindfunclet$??__Ek_parseTakeoverPointConstants@@YAXXZ$9
	DD	0bH
	DD	FLAT:__unwindfunclet$??__Ek_parseTakeoverPointConstants@@YAXXZ$10
	DD	0dH
	DD	FLAT:__unwindfunclet$??__Ek_parseTakeoverPointConstants@@YAXXZ$11
	DD	0bH
	DD	FLAT:__unwindfunclet$??__Ek_parseTakeoverPointConstants@@YAXXZ$11
__ehfuncinfo$??__Ek_parseTakeoverPointConstants@@YAXXZ DD 019930522H
	DD	010H
	DD	FLAT:__unwindtable$??__Ek_parseTakeoverPointConstants@@YAXXZ
	DD	2 DUP(00H)
	DD	2 DUP(00H)
	DD	00H
	DD	00H
; Function compile flags: /Odtp
xdata$x	ENDS
;	COMDAT ??__Ek_parseTakeoverPointConstants@@YAXXZ
text$yc	SEGMENT
tv210 = -156						; size = 4
tv208 = -152						; size = 4
tv207 = -148						; size = 4
tv143 = -144						; size = 4
tv204 = -140						; size = 4
tv202 = -136						; size = 4
tv201 = -132						; size = 4
tv88 = -128						; size = 4
tv198 = -124						; size = 4
tv196 = -120						; size = 4
tv195 = -116						; size = 4
tv65 = -112						; size = 4
tv192 = -108						; size = 4
tv190 = -104						; size = 4
tv189 = -100						; size = 4
tv212 = -96						; size = 4
$T363056 = -92						; size = 4
$T363055 = -88						; size = 16
$T363054 = -72						; size = 4
$T363053 = -68						; size = 16
$T363052 = -52						; size = 4
$T363051 = -48						; size = 16
$T363050 = -32						; size = 4
$T363049 = -28						; size = 16
__$EHRec$ = -12						; size = 12
??__Ek_parseTakeoverPointConstants@@YAXXZ PROC		; `dynamic initializer for 'k_parseTakeoverPointConstants'', COMDAT

; 145  : {

  00000	55		 push	 ebp
  00001	8b ec		 mov	 ebp, esp
  00003	6a ff		 push	 -1
  00005	68 00 00 00 00	 push	 __ehhandler$??__Ek_parseTakeoverPointConstants@@YAXXZ
  0000a	64 a1 00 00 00
	00		 mov	 eax, DWORD PTR fs:0
  00010	50		 push	 eax
  00011	81 ec 90 00 00
	00		 sub	 esp, 144		; 00000090H
  00017	a1 00 00 00 00	 mov	 eax, DWORD PTR ___security_cookie
  0001c	33 c5		 xor	 eax, ebp
  0001e	50		 push	 eax
  0001f	8d 45 f4	 lea	 eax, DWORD PTR __$EHRec$[ebp]
  00022	64 a3 00 00 00
	00		 mov	 DWORD PTR fs:0, eax

; 146  :     PC( _T("min"),                        TDA9887_SM_TAKEOVERPOINT_MIN        ),

  00028	83 ec 0c	 sub	 esp, 12			; 0000000cH
  0002b	8b cc		 mov	 ecx, esp
  0002d	89 65 e0	 mov	 DWORD PTR $T363050[ebp], esp
  00030	6a 00		 push	 0
  00032	e8 00 00 00 00	 call	 ??0CParseValue@HCParser@@QAE@H@Z ; HCParser::CParseValue::CParseValue
  00037	89 45 a0	 mov	 DWORD PTR tv212[ebp], eax
  0003a	8b 45 a0	 mov	 eax, DWORD PTR tv212[ebp]
  0003d	89 45 9c	 mov	 DWORD PTR tv189[ebp], eax
  00040	c7 45 fc 00 00
	00 00		 mov	 DWORD PTR __$EHRec$[ebp+8], 0
  00047	68 00 00 00 00	 push	 OFFSET ??_C@_17CFDBELFO@?$AAm?$AAi?$AAn?$AA?$AA@
  0004c	c7 45 fc ff ff
	ff ff		 mov	 DWORD PTR __$EHRec$[ebp+8], -1
  00053	8d 4d e4	 lea	 ecx, DWORD PTR $T363049[ebp]
  00056	e8 00 00 00 00	 call	 ??0CParseConstant@HCParser@@QAE@PB_WVCParseValue@1@@Z ; HCParser::CParseConstant::CParseConstant
  0005b	89 45 98	 mov	 DWORD PTR tv190[ebp], eax
  0005e	8b 4d 98	 mov	 ecx, DWORD PTR tv190[ebp]
  00061	89 4d 94	 mov	 DWORD PTR tv192[ebp], ecx
  00064	c7 45 fc 01 00
	00 00		 mov	 DWORD PTR __$EHRec$[ebp+8], 1
  0006b	8b 55 94	 mov	 edx, DWORD PTR tv192[ebp]
  0006e	52		 push	 edx
  0006f	b9 00 00 00 00	 mov	 ecx, OFFSET _k_parseTakeoverPointConstants
  00074	e8 00 00 00 00	 call	 ??0CParseConstant@HCParser@@QAE@ABV01@@Z
  00079	c6 45 fc 03	 mov	 BYTE PTR __$EHRec$[ebp+8], 3
  0007d	8d 4d e4	 lea	 ecx, DWORD PTR $T363049[ebp]
  00080	e8 00 00 00 00	 call	 ??1CParseConstant@HCParser@@QAE@XZ

; 147  :     PC( _T("max"),                        TDA9887_SM_TAKEOVERPOINT_MAX        ),

  00085	83 ec 0c	 sub	 esp, 12			; 0000000cH
  00088	8b cc		 mov	 ecx, esp
  0008a	89 65 cc	 mov	 DWORD PTR $T363052[ebp], esp
  0008d	6a 1f		 push	 31			; 0000001fH
  0008f	e8 00 00 00 00	 call	 ??0CParseValue@HCParser@@QAE@H@Z ; HCParser::CParseValue::CParseValue
  00094	89 45 90	 mov	 DWORD PTR tv65[ebp], eax
  00097	8b 45 90	 mov	 eax, DWORD PTR tv65[ebp]
  0009a	89 45 8c	 mov	 DWORD PTR tv195[ebp], eax
  0009d	c6 45 fc 04	 mov	 BYTE PTR __$EHRec$[ebp+8], 4
  000a1	68 00 00 00 00	 push	 OFFSET ??_C@_17LMBAMBHA@?$AAm?$AAa?$AAx?$AA?$AA@
  000a6	c6 45 fc 03	 mov	 BYTE PTR __$EHRec$[ebp+8], 3
  000aa	8d 4d d0	 lea	 ecx, DWORD PTR $T363051[ebp]
  000ad	e8 00 00 00 00	 call	 ??0CParseConstant@HCParser@@QAE@PB_WVCParseValue@1@@Z ; HCParser::CParseConstant::CParseConstant
  000b2	89 45 88	 mov	 DWORD PTR tv196[ebp], eax
  000b5	8b 4d 88	 mov	 ecx, DWORD PTR tv196[ebp]
  000b8	89 4d 84	 mov	 DWORD PTR tv198[ebp], ecx
  000bb	c6 45 fc 05	 mov	 BYTE PTR __$EHRec$[ebp+8], 5
  000bf	8b 55 84	 mov	 edx, DWORD PTR tv198[ebp]
  000c2	52		 push	 edx
  000c3	b9 10 00 00 00	 mov	 ecx, OFFSET _k_parseTakeoverPointConstants+16
  000c8	e8 00 00 00 00	 call	 ??0CParseConstant@HCParser@@QAE@ABV01@@Z
  000cd	c6 45 fc 07	 mov	 BYTE PTR __$EHRec$[ebp+8], 7
  000d1	8d 4d d0	 lea	 ecx, DWORD PTR $T363051[ebp]
  000d4	e8 00 00 00 00	 call	 ??1CParseConstant@HCParser@@QAE@XZ

; 148  :     PC( _T("default"),                    TDA9887_SM_TAKEOVERPOINT_DEFAULT    ),

  000d9	83 ec 0c	 sub	 esp, 12			; 0000000cH
  000dc	8b cc		 mov	 ecx, esp
  000de	89 65 b8	 mov	 DWORD PTR $T363054[ebp], esp
  000e1	6a 10		 push	 16			; 00000010H
  000e3	e8 00 00 00 00	 call	 ??0CParseValue@HCParser@@QAE@H@Z ; HCParser::CParseValue::CParseValue
  000e8	89 45 80	 mov	 DWORD PTR tv88[ebp], eax
  000eb	8b 45 80	 mov	 eax, DWORD PTR tv88[ebp]
  000ee	89 85 7c ff ff
	ff		 mov	 DWORD PTR tv201[ebp], eax
  000f4	c6 45 fc 08	 mov	 BYTE PTR __$EHRec$[ebp+8], 8
  000f8	68 00 00 00 00	 push	 OFFSET ??_C@_1BA@HANLFFFG@?$AAd?$AAe?$AAf?$AAa?$AAu?$AAl?$AAt?$AA?$AA@
  000fd	c6 45 fc 07	 mov	 BYTE PTR __$EHRec$[ebp+8], 7
  00101	8d 4d bc	 lea	 ecx, DWORD PTR $T363053[ebp]
  00104	e8 00 00 00 00	 call	 ??0CParseConstant@HCParser@@QAE@PB_WVCParseValue@1@@Z ; HCParser::CParseConstant::CParseConstant
  00109	89 85 78 ff ff
	ff		 mov	 DWORD PTR tv202[ebp], eax
  0010f	8b 8d 78 ff ff
	ff		 mov	 ecx, DWORD PTR tv202[ebp]
  00115	89 8d 74 ff ff
	ff		 mov	 DWORD PTR tv204[ebp], ecx
  0011b	c6 45 fc 09	 mov	 BYTE PTR __$EHRec$[ebp+8], 9
  0011f	8b 95 74 ff ff
	ff		 mov	 edx, DWORD PTR tv204[ebp]
  00125	52		 push	 edx
  00126	b9 20 00 00 00	 mov	 ecx, OFFSET _k_parseTakeoverPointConstants+32
  0012b	e8 00 00 00 00	 call	 ??0CParseConstant@HCParser@@QAE@ABV01@@Z
  00130	c6 45 fc 0b	 mov	 BYTE PTR __$EHRec$[ebp+8], 11 ; 0000000bH
  00134	8d 4d bc	 lea	 ecx, DWORD PTR $T363053[ebp]
  00137	e8 00 00 00 00	 call	 ??1CParseConstant@HCParser@@QAE@XZ

; 149  :     PC( NULL )
; 150  : };

  0013c	83 ec 0c	 sub	 esp, 12			; 0000000cH
  0013f	8b cc		 mov	 ecx, esp
  00141	89 65 a4	 mov	 DWORD PTR $T363056[ebp], esp
  00144	e8 00 00 00 00	 call	 ??0CParseValue@HCParser@@QAE@XZ ; HCParser::CParseValue::CParseValue
  00149	89 85 70 ff ff
	ff		 mov	 DWORD PTR tv143[ebp], eax
  0014f	8b 85 70 ff ff
	ff		 mov	 eax, DWORD PTR tv143[ebp]
  00155	89 85 6c ff ff
	ff		 mov	 DWORD PTR tv207[ebp], eax
  0015b	c6 45 fc 0c	 mov	 BYTE PTR __$EHRec$[ebp+8], 12 ; 0000000cH
  0015f	6a 00		 push	 0
  00161	c6 45 fc 0b	 mov	 BYTE PTR __$EHRec$[ebp+8], 11 ; 0000000bH
  00165	8d 4d a8	 lea	 ecx, DWORD PTR $T363055[ebp]
  00168	e8 00 00 00 00	 call	 ??0CParseConstant@HCParser@@QAE@PB_WVCParseValue@1@@Z ; HCParser::CParseConstant::CParseConstant
  0016d	89 85 68 ff ff
	ff		 mov	 DWORD PTR tv208[ebp], eax
  00173	8b 8d 68 ff ff
	ff		 mov	 ecx, DWORD PTR tv208[ebp]
  00179	89 8d 64 ff ff
	ff		 mov	 DWORD PTR tv210[ebp], ecx
  0017f	c6 45 fc 0d	 mov	 BYTE PTR __$EHRec$[ebp+8], 13 ; 0000000dH
  00183	8b 95 64 ff ff
	ff		 mov	 edx, DWORD PTR tv210[ebp]
  00189	52		 push	 edx
  0018a	b9 30 00 00 00	 mov	 ecx, OFFSET _k_parseTakeoverPointConstants+48
  0018f	e8 00 00 00 00	 call	 ??0CParseConstant@HCParser@@QAE@ABV01@@Z
  00194	c6 45 fc 0f	 mov	 BYTE PTR __$EHRec$[ebp+8], 15 ; 0000000fH
  00198	8d 4d a8	 lea	 ecx, DWORD PTR $T363055[ebp]
  0019b	e8 00 00 00 00	 call	 ??1CParseConstant@HCParser@@QAE@XZ
  001a0	c7 45 fc ff ff
	ff ff		 mov	 DWORD PTR __$EHRec$[ebp+8], -1
  001a7	68 00 00 00 00	 push	 OFFSET ??__Fk_parseTakeoverPointConstants@@YAXXZ ; `dynamic atexit destructor for 'k_parseTakeoverPointConstants''
  001ac	e8 00 00 00 00	 call	 _atexit
  001b1	83 c4 04	 add	 esp, 4
  001b4	8b 4d f4	 mov	 ecx, DWORD PTR __$EHRec$[ebp]
  001b7	64 89 0d 00 00
	00 00		 mov	 DWORD PTR fs:0, ecx
  001be	59		 pop	 ecx
  001bf	8b e5		 mov	 esp, ebp
  001c1	5d		 pop	 ebp
  001c2	c3		 ret	 0
text$yc	ENDS
;	COMDAT text$x
text$x	SEGMENT
__unwindfunclet$??__Ek_parseTakeoverPointConstants@@YAXXZ$0:
  00000	8b 4d e0	 mov	 ecx, DWORD PTR $T363050[ebp]
  00003	e9 00 00 00 00	 jmp	 ??1CParseValue@HCParser@@UAE@XZ ; HCParser::CParseValue::~CParseValue
__unwindfunclet$??__Ek_parseTakeoverPointConstants@@YAXXZ$1:
  00008	8d 4d e4	 lea	 ecx, DWORD PTR $T363049[ebp]
  0000b	e9 00 00 00 00	 jmp	 ??1CParseConstant@HCParser@@QAE@XZ
__unwindfunclet$??__Ek_parseTakeoverPointConstants@@YAXXZ$2:
  00010	b9 00 00 00 00	 mov	 ecx, OFFSET _k_parseTakeoverPointConstants
  00015	e9 00 00 00 00	 jmp	 ??1CParseConstant@HCParser@@QAE@XZ
__unwindfunclet$??__Ek_parseTakeoverPointConstants@@YAXXZ$3:
  0001a	8b 4d cc	 mov	 ecx, DWORD PTR $T363052[ebp]
  0001d	e9 00 00 00 00	 jmp	 ??1CParseValue@HCParser@@UAE@XZ ; HCParser::CParseValue::~CParseValue
__unwindfunclet$??__Ek_parseTakeoverPointConstants@@YAXXZ$4:
  00022	8d 4d d0	 lea	 ecx, DWORD PTR $T363051[ebp]
  00025	e9 00 00 00 00	 jmp	 ??1CParseConstant@HCParser@@QAE@XZ
__unwindfunclet$??__Ek_parseTakeoverPointConstants@@YAXXZ$5:
  0002a	b9 10 00 00 00	 mov	 ecx, OFFSET _k_parseTakeoverPointConstants+16
  0002f	e9 00 00 00 00	 jmp	 ??1CParseConstant@HCParser@@QAE@XZ
__unwindfunclet$??__Ek_parseTakeoverPointConstants@@YAXXZ$6:
  00034	8b 4d b8	 mov	 ecx, DWORD PTR $T363054[ebp]
  00037	e9 00 00 00 00	 jmp	 ??1CParseValue@HCParser@@UAE@XZ ; HCParser::CParseValue::~CParseValue
__unwindfunclet$??__Ek_parseTakeoverPointConstants@@YAXXZ$7:
  0003c	8d 4d bc	 lea	 ecx, DWORD PTR $T363053[ebp]
  0003f	e9 00 00 00 00	 jmp	 ??1CParseConstant@HCParser@@QAE@XZ
__unwindfunclet$??__Ek_parseTakeoverPointConstants@@YAXXZ$8:
  00044	b9 20 00 00 00	 mov	 ecx, OFFSET _k_parseTakeoverPointConstants+32
  00049	e9 00 00 00 00	 jmp	 ??1CParseConstant@HCParser@@QAE@XZ
__unwindfunclet$??__Ek_parseTakeoverPointConstants@@YAXXZ$9:
  0004e	8b 4d a4	 mov	 ecx, DWORD PTR $T363056[ebp]
  00051	e9 00 00 00 00	 jmp	 ??1CParseValue@HCParser@@UAE@XZ ; HCParser::CParseValue::~CParseValue
__unwindfunclet$??__Ek_parseTakeoverPointConstants@@YAXXZ$10:
  00056	8d 4d a8	 lea	 ecx, DWORD PTR $T363055[ebp]
  00059	e9 00 00 00 00	 jmp	 ??1CParseConstant@HCParser@@QAE@XZ
__unwindfunclet$??__Ek_parseTakeoverPointConstants@@YAXXZ$11:
  0005e	b9 30 00 00 00	 mov	 ecx, OFFSET _k_parseTakeoverPointConstants+48
  00063	e9 00 00 00 00	 jmp	 ??1CParseConstant@HCParser@@QAE@XZ
__ehhandler$??__Ek_parseTakeoverPointConstants@@YAXXZ:
  00068	8b 54 24 08	 mov	 edx, DWORD PTR [esp+8]
  0006c	8d 42 0c	 lea	 eax, DWORD PTR [edx+12]
  0006f	8b 8a 6c ff ff
	ff		 mov	 ecx, DWORD PTR [edx-148]
  00075	33 c8		 xor	 ecx, eax
  00077	e8 00 00 00 00	 call	 @__security_check_cookie@4
  0007c	b8 00 00 00 00	 mov	 eax, OFFSET __ehfuncinfo$??__Ek_parseTakeoverPointConstants@@YAXXZ
  00081	e9 00 00 00 00	 jmp	 ___CxxFrameHandler3
text$x	ENDS
??__Ek_parseTakeoverPointConstants@@YAXXZ ENDP		; `dynamic initializer for 'k_parseTakeoverPointConstants''
; Function compile flags: /Odtp
;	COMDAT ??__Ek_parseUseTDA9887SetOverride@@YAXXZ
text$yc	SEGMENT
$T363084 = -36						; size = 8
??__Ek_parseUseTDA9887SetOverride@@YAXXZ PROC		; `dynamic initializer for 'k_parseUseTDA9887SetOverride'', COMDAT

; 153  : {

  00000	55		 push	 ebp
  00001	8b ec		 mov	 ebp, esp
  00003	83 ec 24	 sub	 esp, 36			; 00000024H

; 154  :     PT( _T("Format"),            PARSE_CONSTANT,        0, 8,    k_parseTDAFormatConstants,        PASS_TO_PARENT    ),

  00006	68 00 00 00 00	 push	 OFFSET ?PASS_TO_PARENT@HCParser@@YAXHPBVCParseTag@1@EPBVCParseValue@1@PAX@Z ; HCParser::PASS_TO_PARENT
  0000b	83 ec 08	 sub	 esp, 8
  0000e	8b cc		 mov	 ecx, esp
  00010	68 00 00 00 00	 push	 OFFSET _k_parseTDAFormatConstants
  00015	e8 00 00 00 00	 call	 ??0CAttributes@CParseTag@HCParser@@QAE@PBVCParseConstant@2@@Z ; HCParser::CParseTag::CAttributes::CAttributes
  0001a	6a 08		 push	 8
  0001c	6a 00		 push	 0
  0001e	6a 04		 push	 4
  00020	68 00 00 00 00	 push	 OFFSET ??_C@_1O@FDFOMCPN@?$AAF?$AAo?$AAr?$AAm?$AAa?$AAt?$AA?$AA@
  00025	b9 00 00 00 00	 mov	 ecx, OFFSET _k_parseUseTDA9887SetOverride
  0002a	e8 00 00 00 00	 call	 ??0CParseTag@HCParser@@QAE@PB_WEEKVCAttributes@01@P6AXHPBV01@EPBVCParseValue@1@PAX@Z@Z ; HCParser::CParseTag::CParseTag

; 155  :     PT( _T("Intercarrier"),        0,                    0, 0,    NULL,                            PASS_TO_PARENT    ),

  0002f	68 00 00 00 00	 push	 OFFSET ?PASS_TO_PARENT@HCParser@@YAXHPBVCParseTag@1@EPBVCParseValue@1@PAX@Z ; HCParser::PASS_TO_PARENT
  00034	83 ec 08	 sub	 esp, 8
  00037	8b cc		 mov	 ecx, esp
  00039	6a 00		 push	 0
  0003b	e8 00 00 00 00	 call	 ??0CAttributes@CParseTag@HCParser@@QAE@H@Z ; HCParser::CParseTag::CAttributes::CAttributes
  00040	6a 00		 push	 0
  00042	6a 00		 push	 0
  00044	6a 00		 push	 0
  00046	68 00 00 00 00	 push	 OFFSET ??_C@_1BK@IOEPCAOC@?$AAI?$AAn?$AAt?$AAe?$AAr?$AAc?$AAa?$AAr?$AAr?$AAi?$AAe?$AAr?$AA?$AA@
  0004b	b9 1c 00 00 00	 mov	 ecx, OFFSET _k_parseUseTDA9887SetOverride+28
  00050	e8 00 00 00 00	 call	 ??0CParseTag@HCParser@@QAE@PB_WEEKVCAttributes@01@P6AXHPBV01@EPBVCParseValue@1@PAX@Z@Z ; HCParser::CParseTag::CParseTag

; 156  :     PT( _T("QSS"),                0,                    0, 0,    NULL,                            PASS_TO_PARENT    ),

  00055	68 00 00 00 00	 push	 OFFSET ?PASS_TO_PARENT@HCParser@@YAXHPBVCParseTag@1@EPBVCParseValue@1@PAX@Z ; HCParser::PASS_TO_PARENT
  0005a	83 ec 08	 sub	 esp, 8
  0005d	8b cc		 mov	 ecx, esp
  0005f	6a 00		 push	 0
  00061	e8 00 00 00 00	 call	 ??0CAttributes@CParseTag@HCParser@@QAE@H@Z ; HCParser::CParseTag::CAttributes::CAttributes
  00066	6a 00		 push	 0
  00068	6a 00		 push	 0
  0006a	6a 00		 push	 0
  0006c	68 00 00 00 00	 push	 OFFSET ??_C@_17FAPDAJNL@?$AAQ?$AAS?$AAS?$AA?$AA@
  00071	b9 38 00 00 00	 mov	 ecx, OFFSET _k_parseUseTDA9887SetOverride+56
  00076	e8 00 00 00 00	 call	 ??0CParseTag@HCParser@@QAE@PB_WEEKVCAttributes@01@P6AXHPBV01@EPBVCParseValue@1@PAX@Z@Z ; HCParser::CParseTag::CParseTag

; 157  :     PT( _T("Carrier"),            PARSE_CONSTANT,        0, 16,    k_parseCarrierConstants,        PASS_TO_PARENT    ),

  0007b	68 00 00 00 00	 push	 OFFSET ?PASS_TO_PARENT@HCParser@@YAXHPBVCParseTag@1@EPBVCParseValue@1@PAX@Z ; HCParser::PASS_TO_PARENT
  00080	83 ec 08	 sub	 esp, 8
  00083	8b cc		 mov	 ecx, esp
  00085	68 00 00 00 00	 push	 OFFSET _k_parseCarrierConstants
  0008a	e8 00 00 00 00	 call	 ??0CAttributes@CParseTag@HCParser@@QAE@PBVCParseConstant@2@@Z ; HCParser::CParseTag::CAttributes::CAttributes
  0008f	6a 10		 push	 16			; 00000010H
  00091	6a 00		 push	 0
  00093	6a 04		 push	 4
  00095	68 00 00 00 00	 push	 OFFSET ??_C@_1BA@GJEGJPFN@?$AAC?$AAa?$AAr?$AAr?$AAi?$AAe?$AAr?$AA?$AA@
  0009a	b9 54 00 00 00	 mov	 ecx, OFFSET _k_parseUseTDA9887SetOverride+84
  0009f	e8 00 00 00 00	 call	 ??0CParseTag@HCParser@@QAE@PB_WEEKVCAttributes@01@P6AXHPBV01@EPBVCParseValue@1@PAX@Z@Z ; HCParser::CParseTag::CParseTag

; 158  :     PT( _T("OutputPort1"),        PARSE_CONSTANT,        0, 8,    k_parseYesNoConstants,            PASS_TO_PARENT    ),

  000a4	68 00 00 00 00	 push	 OFFSET ?PASS_TO_PARENT@HCParser@@YAXHPBVCParseTag@1@EPBVCParseValue@1@PAX@Z ; HCParser::PASS_TO_PARENT
  000a9	83 ec 08	 sub	 esp, 8
  000ac	8b cc		 mov	 ecx, esp
  000ae	68 00 00 00 00	 push	 OFFSET _k_parseYesNoConstants
  000b3	e8 00 00 00 00	 call	 ??0CAttributes@CParseTag@HCParser@@QAE@PBVCParseConstant@2@@Z ; HCParser::CParseTag::CAttributes::CAttributes
  000b8	6a 08		 push	 8
  000ba	6a 00		 push	 0
  000bc	6a 04		 push	 4
  000be	68 00 00 00 00	 push	 OFFSET ??_C@_1BI@NCFPNFB@?$AAO?$AAu?$AAt?$AAp?$AAu?$AAt?$AAP?$AAo?$AAr?$AAt?$AA1?$AA?$AA@
  000c3	b9 70 00 00 00	 mov	 ecx, OFFSET _k_parseUseTDA9887SetOverride+112
  000c8	e8 00 00 00 00	 call	 ??0CParseTag@HCParser@@QAE@PB_WEEKVCAttributes@01@P6AXHPBV01@EPBVCParseValue@1@PAX@Z@Z ; HCParser::CParseTag::CParseTag

; 159  :     PT( _T("OutputPort2"),        PARSE_CONSTANT,        0, 8,    k_parseYesNoConstants,            PASS_TO_PARENT    ),

  000cd	68 00 00 00 00	 push	 OFFSET ?PASS_TO_PARENT@HCParser@@YAXHPBVCParseTag@1@EPBVCParseValue@1@PAX@Z ; HCParser::PASS_TO_PARENT
  000d2	83 ec 08	 sub	 esp, 8
  000d5	8b cc		 mov	 ecx, esp
  000d7	68 00 00 00 00	 push	 OFFSET _k_parseYesNoConstants
  000dc	e8 00 00 00 00	 call	 ??0CAttributes@CParseTag@HCParser@@QAE@PBVCParseConstant@2@@Z ; HCParser::CParseTag::CAttributes::CAttributes
  000e1	6a 08		 push	 8
  000e3	6a 00		 push	 0
  000e5	6a 04		 push	 4
  000e7	68 00 00 00 00	 push	 OFFSET ??_C@_1BI@BPJAFCLP@?$AAO?$AAu?$AAt?$AAp?$AAu?$AAt?$AAP?$AAo?$AAr?$AAt?$AA2?$AA?$AA@
  000ec	b9 8c 00 00 00	 mov	 ecx, OFFSET _k_parseUseTDA9887SetOverride+140
  000f1	e8 00 00 00 00	 call	 ??0CParseTag@HCParser@@QAE@PB_WEEKVCAttributes@01@P6AXHPBV01@EPBVCParseValue@1@PAX@Z@Z ; HCParser::CParseTag::CParseTag

; 160  :     PT( _T("TakeOverPoint"),    PARSE_NUM_OR_CONST,    0, 8,    k_parseTakeoverPointConstants,    PASS_TO_PARENT    ),

  000f6	68 00 00 00 00	 push	 OFFSET ?PASS_TO_PARENT@HCParser@@YAXHPBVCParseTag@1@EPBVCParseValue@1@PAX@Z ; HCParser::PASS_TO_PARENT
  000fb	83 ec 08	 sub	 esp, 8
  000fe	8b cc		 mov	 ecx, esp
  00100	68 00 00 00 00	 push	 OFFSET _k_parseTakeoverPointConstants
  00105	e8 00 00 00 00	 call	 ??0CAttributes@CParseTag@HCParser@@QAE@PBVCParseConstant@2@@Z ; HCParser::CParseTag::CAttributes::CAttributes
  0010a	6a 08		 push	 8
  0010c	6a 00		 push	 0
  0010e	6a 06		 push	 6
  00110	68 00 00 00 00	 push	 OFFSET ??_C@_1BM@DLNBHEGJ@?$AAT?$AAa?$AAk?$AAe?$AAO?$AAv?$AAe?$AAr?$AAP?$AAo?$AAi?$AAn?$AAt?$AA?$AA@
  00115	b9 a8 00 00 00	 mov	 ecx, OFFSET _k_parseUseTDA9887SetOverride+168
  0011a	e8 00 00 00 00	 call	 ??0CParseTag@HCParser@@QAE@PB_WEEKVCAttributes@01@P6AXHPBV01@EPBVCParseValue@1@PAX@Z@Z ; HCParser::CParseTag::CParseTag

; 161  :     PT( NULL )
; 162  : };

  0011f	6a 00		 push	 0
  00121	6a 00		 push	 0
  00123	8d 4d dc	 lea	 ecx, DWORD PTR $T363084[ebp]
  00126	e8 00 00 00 00	 call	 ??0CAttributes@CParseTag@HCParser@@QAE@H@Z ; HCParser::CParseTag::CAttributes::CAttributes
  0012b	8b 48 04	 mov	 ecx, DWORD PTR [eax+4]
  0012e	51		 push	 ecx
  0012f	8b 10		 mov	 edx, DWORD PTR [eax]
  00131	52		 push	 edx
  00132	6a 00		 push	 0
  00134	6a 00		 push	 0
  00136	6a 00		 push	 0
  00138	6a 00		 push	 0
  0013a	b9 c4 00 00 00	 mov	 ecx, OFFSET _k_parseUseTDA9887SetOverride+196
  0013f	e8 00 00 00 00	 call	 ??0CParseTag@HCParser@@QAE@PB_WEEKVCAttributes@01@P6AXHPBV01@EPBVCParseValue@1@PAX@Z@Z ; HCParser::CParseTag::CParseTag
  00144	8b e5		 mov	 esp, ebp
  00146	5d		 pop	 ebp
  00147	c3		 ret	 0
??__Ek_parseUseTDA9887SetOverride@@YAXXZ ENDP		; `dynamic initializer for 'k_parseUseTDA9887SetOverride''
; Function compile flags: /Odtp
text$yc	ENDS
;	COMDAT ??__Ek_parseUseTDA9887@@YAXXZ
text$yc	SEGMENT
$T363089 = -16						; size = 8
??__Ek_parseUseTDA9887@@YAXXZ PROC			; `dynamic initializer for 'k_parseUseTDA9887'', COMDAT

; 165  : {

  00000	55		 push	 ebp
  00001	8b ec		 mov	 ebp, esp
  00003	83 ec 10	 sub	 esp, 16			; 00000010H

; 166  :     PT( _T("Use"),                PARSE_CONSTANT,        0, 8,    k_parseYesNoConstants,            PASS_TO_PARENT    ),

  00006	68 00 00 00 00	 push	 OFFSET ?PASS_TO_PARENT@HCParser@@YAXHPBVCParseTag@1@EPBVCParseValue@1@PAX@Z ; HCParser::PASS_TO_PARENT
  0000b	83 ec 08	 sub	 esp, 8
  0000e	8b cc		 mov	 ecx, esp
  00010	68 00 00 00 00	 push	 OFFSET _k_parseYesNoConstants
  00015	e8 00 00 00 00	 call	 ??0CAttributes@CParseTag@HCParser@@QAE@PBVCParseConstant@2@@Z ; HCParser::CParseTag::CAttributes::CAttributes
  0001a	6a 08		 push	 8
  0001c	6a 00		 push	 0
  0001e	6a 04		 push	 4
  00020	68 00 00 00 00	 push	 OFFSET ??_C@_17GFFKFGK@?$AAU?$AAs?$AAe?$AA?$AA@
  00025	b9 00 00 00 00	 mov	 ecx, OFFSET ?k_parseUseTDA9887@@3QBVCParseTag@HCParser@@B ; k_parseUseTDA9887
  0002a	e8 00 00 00 00	 call	 ??0CParseTag@HCParser@@QAE@PB_WEEKVCAttributes@01@P6AXHPBV01@EPBVCParseValue@1@PAX@Z@Z ; HCParser::CParseTag::CParseTag

; 167  :     PT( _T("SetModes"),            PARSE_CHILDREN,        0, 9,    k_parseUseTDA9887SetOverride,    PASS_TO_PARENT    ),

  0002f	68 00 00 00 00	 push	 OFFSET ?PASS_TO_PARENT@HCParser@@YAXHPBVCParseTag@1@EPBVCParseValue@1@PAX@Z ; HCParser::PASS_TO_PARENT
  00034	83 ec 08	 sub	 esp, 8
  00037	8b cc		 mov	 ecx, esp
  00039	68 00 00 00 00	 push	 OFFSET _k_parseUseTDA9887SetOverride
  0003e	e8 00 00 00 00	 call	 ??0CAttributes@CParseTag@HCParser@@QAE@PBV12@@Z ; HCParser::CParseTag::CAttributes::CAttributes
  00043	6a 09		 push	 9
  00045	6a 00		 push	 0
  00047	6a 08		 push	 8
  00049	68 00 00 00 00	 push	 OFFSET ??_C@_1BC@KNKFHLFO@?$AAS?$AAe?$AAt?$AAM?$AAo?$AAd?$AAe?$AAs?$AA?$AA@
  0004e	b9 1c 00 00 00	 mov	 ecx, OFFSET ?k_parseUseTDA9887@@3QBVCParseTag@HCParser@@B+28
  00053	e8 00 00 00 00	 call	 ??0CParseTag@HCParser@@QAE@PB_WEEKVCAttributes@01@P6AXHPBV01@EPBVCParseValue@1@PAX@Z@Z ; HCParser::CParseTag::CParseTag

; 168  :     PT( NULL )
; 169  : };

  00058	6a 00		 push	 0
  0005a	6a 00		 push	 0
  0005c	8d 4d f0	 lea	 ecx, DWORD PTR $T363089[ebp]
  0005f	e8 00 00 00 00	 call	 ??0CAttributes@CParseTag@HCParser@@QAE@H@Z ; HCParser::CParseTag::CAttributes::CAttributes
  00064	8b 48 04	 mov	 ecx, DWORD PTR [eax+4]
  00067	51		 push	 ecx
  00068	8b 10		 mov	 edx, DWORD PTR [eax]
  0006a	52		 push	 edx
  0006b	6a 00		 push	 0
  0006d	6a 00		 push	 0
  0006f	6a 00		 push	 0
  00071	6a 00		 push	 0
  00073	b9 38 00 00 00	 mov	 ecx, OFFSET ?k_parseUseTDA9887@@3QBVCParseTag@HCParser@@B+56
  00078	e8 00 00 00 00	 call	 ??0CParseTag@HCParser@@QAE@PB_WEEKVCAttributes@01@P6AXHPBV01@EPBVCParseValue@1@PAX@Z@Z ; HCParser::CParseTag::CParseTag
  0007d	8b e5		 mov	 esp, ebp
  0007f	5d		 pop	 ebp
  00080	c3		 ret	 0
??__Ek_parseUseTDA9887@@YAXXZ ENDP			; `dynamic initializer for 'k_parseUseTDA9887''
; Function compile flags: /Odtp
;	COMDAT ??__Fk_parseTakeoverPointConstants@@YAXXZ
text$yd	SEGMENT
??__Fk_parseTakeoverPointConstants@@YAXXZ PROC		; `dynamic atexit destructor for 'k_parseTakeoverPointConstants'', COMDAT
  00000	55		 push	 ebp
  00001	8b ec		 mov	 ebp, esp
  00003	68 00 00 00 00	 push	 OFFSET ??1CParseConstant@HCParser@@QAE@XZ
  00008	6a 04		 push	 4
  0000a	6a 10		 push	 16			; 00000010H
  0000c	68 00 00 00 00	 push	 OFFSET _k_parseTakeoverPointConstants
  00011	e8 00 00 00 00	 call	 ??_M@YGXPAXIHP6EX0@Z@Z
  00016	5d		 pop	 ebp
  00017	c3		 ret	 0
??__Fk_parseTakeoverPointConstants@@YAXXZ ENDP		; `dynamic atexit destructor for 'k_parseTakeoverPointConstants''
; Function compile flags: /Odtp
text$yd	ENDS
;	COMDAT ??__Fk_parseYesNoConstants@@YAXXZ
text$yd	SEGMENT
??__Fk_parseYesNoConstants@@YAXXZ PROC			; `dynamic atexit destructor for 'k_parseYesNoConstants'', COMDAT
  00000	55		 push	 ebp
  00001	8b ec		 mov	 ebp, esp
  00003	68 00 00 00 00	 push	 OFFSET ??1CParseConstant@HCParser@@QAE@XZ
  00008	6a 09		 push	 9
  0000a	6a 10		 push	 16			; 00000010H
  0000c	68 00 00 00 00	 push	 OFFSET _k_parseYesNoConstants
  00011	e8 00 00 00 00	 call	 ??_M@YGXPAXIHP6EX0@Z@Z
  00016	5d		 pop	 ebp
  00017	c3		 ret	 0
??__Fk_parseYesNoConstants@@YAXXZ ENDP			; `dynamic atexit destructor for 'k_parseYesNoConstants''
; Function compile flags: /Odtp
text$yd	ENDS
;	COMDAT ??__Fk_parseCarrierConstants@@YAXXZ
text$yd	SEGMENT
??__Fk_parseCarrierConstants@@YAXXZ PROC		; `dynamic atexit destructor for 'k_parseCarrierConstants'', COMDAT
  00000	55		 push	 ebp
  00001	8b ec		 mov	 ebp, esp
  00003	68 00 00 00 00	 push	 OFFSET ??1CParseConstant@HCParser@@QAE@XZ
  00008	6a 03		 push	 3
  0000a	6a 10		 push	 16			; 00000010H
  0000c	68 00 00 00 00	 push	 OFFSET _k_parseCarrierConstants
  00011	e8 00 00 00 00	 call	 ??_M@YGXPAXIHP6EX0@Z@Z
  00016	5d		 pop	 ebp
  00017	c3		 ret	 0
??__Fk_parseCarrierConstants@@YAXXZ ENDP		; `dynamic atexit destructor for 'k_parseCarrierConstants''
; Function compile flags: /Odtp
text$yd	ENDS
;	COMDAT ??__Fk_parseTDAFormatConstants@@YAXXZ
text$yd	SEGMENT
??__Fk_parseTDAFormatConstants@@YAXXZ PROC		; `dynamic atexit destructor for 'k_parseTDAFormatConstants'', COMDAT
  00000	55		 push	 ebp
  00001	8b ec		 mov	 ebp, esp
  00003	68 00 00 00 00	 push	 OFFSET ??1CParseConstant@HCParser@@QAE@XZ
  00008	6a 0b		 push	 11			; 0000000bH
  0000a	6a 10		 push	 16			; 00000010H
  0000c	68 00 00 00 00	 push	 OFFSET _k_parseTDAFormatConstants
  00011	e8 00 00 00 00	 call	 ??_M@YGXPAXIHP6EX0@Z@Z
  00016	5d		 pop	 ebp
  00017	c3		 ret	 0
??__Fk_parseTDAFormatConstants@@YAXXZ ENDP		; `dynamic atexit destructor for 'k_parseTDAFormatConstants''
; Function compile flags: /Odtp
text$yd	ENDS
;	COMDAT ??__Fk_parseTunerConstants@@YAXXZ
text$yd	SEGMENT
??__Fk_parseTunerConstants@@YAXXZ PROC			; `dynamic atexit destructor for 'k_parseTunerConstants'', COMDAT
  00000	55		 push	 ebp
  00001	8b ec		 mov	 ebp, esp
  00003	68 00 00 00 00	 push	 OFFSET ??1CParseConstant@HCParser@@QAE@XZ
  00008	6a 43		 push	 67			; 00000043H
  0000a	6a 10		 push	 16			; 00000010H
  0000c	68 00 00 00 00	 push	 OFFSET ?k_parseTunerConstants@@3QBVCParseConstant@HCParser@@B ; k_parseTunerConstants
  00011	e8 00 00 00 00	 call	 ??_M@YGXPAXIHP6EX0@Z@Z
  00016	5d		 pop	 ebp
  00017	c3		 ret	 0
??__Fk_parseTunerConstants@@YAXXZ ENDP			; `dynamic atexit destructor for 'k_parseTunerConstants''
PUBLIC	?k_parseUseTDA9887@@3QBVCParseTag@HCParser@@B	; k_parseUseTDA9887
PUBLIC	?k_parseTunerConstants@@3QBVCParseConstant@HCParser@@B ; k_parseTunerConstants
?k_parseUseTDA9887@@3QBVCParseTag@HCParser@@B DB 054H DUP (?) ; k_parseUseTDA9887
_k_parseUseTDA9887SetOverride DB 0e0H DUP (?)
_k_parseTakeoverPointConstants DB 040H DUP (?)
_k_parseYesNoConstants DB 090H DUP (?)
_k_parseCarrierConstants DB 030H DUP (?)
_k_parseTDAFormatConstants DB 0b0H DUP (?)
?k_parseTunerConstants@@3QBVCParseConstant@HCParser@@B DB 0430H DUP (?) ; k_parseTunerConstants
_k_parseTunerConstants$initializer$ DD FLAT:??__Ek_parseTunerConstants@@YAXXZ
_k_parseTDAFormatConstants$initializer$ DD FLAT:??__Ek_parseTDAFormatConstants@@YAXXZ
_k_parseCarrierConstants$initializer$ DD FLAT:??__Ek_parseCarrierConstants@@YAXXZ
_k_parseYesNoConstants$initializer$ DD FLAT:??__Ek_parseYesNoConstants@@YAXXZ
_k_parseTakeoverPointConstants$initializer$ DD FLAT:??__Ek_parseTakeoverPointConstants@@YAXXZ
_k_parseUseTDA9887SetOverride$initializer$ DD FLAT:??__Ek_parseUseTDA9887SetOverride@@YAXXZ
_k_parseUseTDA9887$initializer$ DD FLAT:??__Ek_parseUseTDA9887@@YAXXZ
END
